** EXPERIMENTAL (HLL) ** Open Watcom Linker Version 1.6beta1 Limited Availability
Portions Copyright (c) 1985-2002 Sybase, Inc. All Rights Reserved.
Created on:       12/12/23 14:30:19
Executable Image: .libs/php5.dll
creating an OS/2 EMX dynamic link library


                        +------------+
                        |   Groups   |
                        +------------+

Group                           Address              Size
=====                           =======              ====

CGROUP                          0001:00000000        008bce00
DGROUP                          0002:00000000        00022380



                        +--------------+
                        |   Segments   |
                        +--------------+

Segment                Class          Group          Address         Size
=======                =====          =====          =======         ====

TEXT32                 CODE           CGROUP         0001:00000000   008bcdf8
________TEXT           CODE           CGROUP         0001:008bce00   00000000
DATA32                 DATA           DGROUP         0002:00000000   00008d10
SET1__os2dll           DATA           DGROUP         0002:00008d10   00000004
SET2__os2dll           DATA           DGROUP         0002:00008d14   00000000
SET3__os2dll           DATA           DGROUP         0002:00008d14   00000004
SET1___CTOR_LIST__     DATA           DGROUP         0002:00008d18   00000004
SET2___CTOR_LIST__     DATA           DGROUP         0002:00008d1c   00000000
SET3___CTOR_LIST__     DATA           DGROUP         0002:00008d1c   00000004
SET1___DTOR_LIST__     DATA           DGROUP         0002:00008d20   00000004
SET2___DTOR_LIST__     DATA           DGROUP         0002:00008d24   00000000
SET3___DTOR_LIST__     DATA           DGROUP         0002:00008d24   00000004
SET1___crtinit1__      DATA           DGROUP         0002:00008d28   00000004
SET2___crtinit1__      DATA           DGROUP         0002:00008d2c   00000000
SET3___crtinit1__      DATA           DGROUP         0002:00008d2c   00000004
SET1___crtexit1__      DATA           DGROUP         0002:00008d30   00000004
SET2___crtexit1__      DATA           DGROUP         0002:00008d34   00000000
SET3___crtexit1__      DATA           DGROUP         0002:00008d34   00000004
SET1___eh_frame__      DATA           DGROUP         0002:00008d38   00000004
SET2___eh_frame__      DATA           DGROUP         0002:00008d3c   0000002c
SET3___eh_frame__      DATA           DGROUP         0002:00008d68   00000004
SET1___eh_init__       DATA           DGROUP         0002:00008d6c   00000004
SET2___eh_init__       DATA           DGROUP         0002:00008d70   00000004
SET3___eh_init__       DATA           DGROUP         0002:00008d74   00000004
SET1___eh_term__       DATA           DGROUP         0002:00008d78   00000004
SET2___eh_term__       DATA           DGROUP         0002:00008d7c   00000004
SET3___eh_term__       DATA           DGROUP         0002:00008d80   00000004
SET1___fork_parent1__  DATA           DGROUP         0002:00008d84   00000004
SET2___fork_parent1__  DATA           DGROUP         0002:00008d88   00000000
SET3___fork_parent1__  DATA           DGROUP         0002:00008d88   00000004
SET1___fork_child1__   DATA           DGROUP         0002:00008d8c   00000004
SET2___fork_child1__   DATA           DGROUP         0002:00008d90   00000000
SET3___fork_child1__   DATA           DGROUP         0002:00008d90   00000004
________DATA           DATA           DGROUP         0002:00008da0   00000000
BSS32                  BSS            DGROUP         0002:00008da0   00017300
c_common               BSS            DGROUP         0002:000200a0   000022e0
________BSS            BSS            DGROUP         0002:00022380   00000000


                        +----------------+
                        |   Memory Map   |
                        +----------------+

* = unreferenced symbol
+ = symbol only referenced locally

Address        Symbol
=======        ======

Module: U:\usr\lib\dll0hi.obj({standard input})
0001:00000000* __text
0002:00000000* __data
0002:00000000* ___data_start
0002:00008da0* ___bss_start
0002:00008d10+ __os2dll
0002:00008d18  ___CTOR_LIST__
0002:00008d20  ___DTOR_LIST__
0002:00008d28* ___crtinit1__
0002:00008d30* ___crtexit1__
0002:00008d38  ___eh_frame__
0002:00008d6c  ___eh_init__
0002:00008d78  ___eh_term__
0002:00008d84+ ___fork_parent1__
0002:00008d8c+ ___fork_child1__
Module: U:\dev\php-5.3.20\ext\date\php_date.obj(php_date.obj)
0002:000200a0  _date_ce_date
0002:000200b0  _date_ce_timezone
0002:000200c0  _date_globals_id
0002:000200d0  _php_date_global_timezone_db
0002:000200e0  _date_ce_interval
0002:000200f0  _php_date_global_timezone_db_enabled
0002:00020100  _date_ce_period
0001:000000a0  _php_date_get_date_ce
0001:000000aa  _php_date_get_timezone_ce
0001:00000248  _zm_activate_date
0001:000002a9  _zif_timezone_version_get
0001:00000310  _zif_date_default_timezone_set
0001:0000041c  _zif_timezone_abbreviations_list
0001:000006ad  _zif_timezone_identifiers_list
0001:00000b4d  _zim_DatePeriod___construct
0001:00000fe2  _zif_date_timestamp_get
0001:0000111e  _zif_date_interval_format
0001:00001762  _php_parse_date
0001:00004bc3  _php_date_parse_tzfile_wrapper
0001:00001995  _zim_DateInterval___wakeup
0001:000019f4  _zim_DateInterval___construct
0001:00001c2f  _zif_timezone_location_get
0001:00001d73  _zif_timezone_offset_get
0001:00001ed6  _zif_date_offset_get
0001:00002002  _zif_timezone_name_from_abbr
0001:000020be  _zif_timezone_name_get
0001:00002469  _zim_DateTimeZone___construct
0001:00002530  _php_date_short_day_name
0001:00002578  _php_date_full_day_name
0001:000038ee  _zif_date_format
0001:00003bf5  _php_date_do_return_parsed_time
0001:0000429a  _zif_date_parse_from_format
0001:00004367  _zif_date_parse
0001:0000441f  _zif_date_get_last_errors
0001:0000447d  _zif_time
0001:0000449f  _php_date_instantiate
0001:0000458a  _zif_date_interval_create_from_date_string
0001:0000467a  _zim_DateInterval___set_state
0001:00004723  _zif_timezone_open
0001:000047c5  _zif_date_diff
0001:00004914  _zif_date_timezone_get
0001:00004a7d  _date_object_period_get_iterator
0001:00004aed  _zif_checkdate
0001:00004b8a  _php_date_set_tzdb
0001:00004ed3  _get_timezone_info
0001:00004ff2  _zif_date_sun_info
0001:00005afa  _zif_date_sunset
0001:00005b29  _zif_date_sunrise
0001:00005b58  _zif_date_default_timezone_get
0001:00005bd9  _php_date_initialize
0001:0000616e  _zim_DateTime___wakeup
0001:000061af  _zim_DateTime___set_state
0001:0000625d  _zim_DateTime___construct
0001:0000633b  _zif_date_create_from_format
0001:0000642e  _zif_date_create
0001:0000652c  _zif_getdate
0001:00006803  _zif_localtime
0001:00006b1a  _php_strftime
0001:00006da7  _zif_gmstrftime
0001:00006de5  _zif_strftime
0001:00006e7f  _php_mktime
0001:0000714d  _zif_gmmktime
0001:0000718b  _zif_mktime
0001:000071d5  _zif_strtotime
0001:0000746d  _php_idate
0001:00007a60  _zif_idate
0001:00007b2f  _php_format_date
0001:00007bd9  _zif_timezone_transitions_get
0001:0000852f  _zif_gmdate
0001:0000855e  _zif_date
0001:000085ff  _zm_info_date
0001:000086c4  _zm_shutdown_date
0001:0000c4c0  _date_funcs_date
0001:0000c690  _date_funcs_timezone
0001:0000c750  _date_funcs_interval
0001:0000a76b  _date_interval_read_property
0001:0000b873  _date_interval_write_property
0001:0000c7d0  _date_funcs_period
0001:00009333  _zm_startup_date
0001:0000a1ee  _zm_deactivate_date
0001:0000a2a2  _zif_date_isodate_set
0001:0000a421  _zif_date_timestamp_set
0001:0000a52b  _zif_date_date_set
0001:0000a647  _zif_date_time_set
0001:0000aa09  _zif_date_modify
0001:0000acfe  _zif_date_add
0001:0000b028  _zif_date_sub
0001:0000b387  _zif_date_timezone_set
0001:0000c060  _date_functions
0002:000000b0  _date_period_it_funcs
0002:00000050  _date_module_entry
Module: U:\dev\php-5.3.20\ext\date\lib\astro.obj(astro.obj)
0001:0000df90  _timelib_ts_to_juliandate
0001:0000dfaa  _timelib_astro_rise_set_altitude
Module: U:\dev\php-5.3.20\ext\date\lib\dow.obj(dow.obj)
0001:0000e83c  _timelib_day_of_week
0001:0000e876  _timelib_iso_day_of_week
0001:0000e8b0  _timelib_day_of_year
0001:0000e94a  _timelib_days_in_month
0001:0000e9c1  _timelib_isoweek_from_date
0001:0000eca5  _timelib_daynr_from_weeknr
0001:0000ed57  _timelib_valid_time
0001:0000edb2  _timelib_valid_date
Module: U:\dev\php-5.3.20\ext\date\lib\parse_date.obj(parse_date.obj)
0001:0000efc0  _timelib_timezone_abbreviations_list
0001:0000f12a  _timelib_timezone_id_from_abbr
0001:0000f14b  _timelib_fill_holes
0001:0001080b  _timelib_parse_from_format
0001:00011a9b  _timelib_strtotime
Module: U:\dev\php-5.3.20\ext\date\lib\parse_tz.obj(parse_tz.obj)
0001:00036010  _timelib_builtin_db
0001:0003601a  _timelib_timezone_builtin_identifiers_list
0001:00039020  _timezonedb_idx_builtin
0001:0003617d  _timelib_timestamp_is_in_dst
0001:000361ab  _timelib_get_time_zone_info
0001:000362e9  _timelib_get_current_offset
0001:0003646c  _timelib_timezone_id_is_valid
0001:00036482  _timelib_parse_tzfile
0001:00036bda  _timelib_dump_tzinfo
0001:0003a220  _timelib_timezone_db_data_builtin
0001:000795c0  _timezonedb_builtin
Module: U:\dev\php-5.3.20\ext\date\lib\timelib.obj(timelib.obj)
0001:000795e0  _timelib_date_to_int
0001:00079696  _timelib_dump_rel_time
0001:00079838  _timelib_dump_date
0001:00079bb9  _timelib_decimal_hour_to_hms
0001:00079c47  _timelib_error_container_dtor
0001:00079cc0  _timelib_tzinfo_dtor
0001:00079d6f  _timelib_time_offset_dtor
0001:00079d9c  _timelib_rel_time_dtor
0001:00079db1  _timelib_time_dtor
0001:00079dde  _timelib_get_tz_abbr_ptr
0001:00079e0b  _timelib_time_offset_ctor
0001:00079e27  _timelib_rel_time_ctor
0001:00079e43  _timelib_rel_time_clone
0001:00079e5d  _timelib_time_ctor
0001:00079e79  _timelib_tzinfo_ctor
0001:00079eab  _timelib_tzinfo_clone
0001:00079fc5  _timelib_time_clone
0001:0007a00d  _timelib_time_tz_abbr_update
Module: U:\dev\php-5.3.20\ext\date\lib\tm2unixtime.obj(tm2unixtime.obj)
0001:0007a1f4  _timelib_do_rel_normalize
0001:0007a579  _timelib_do_normalize
0001:0007a919  _timelib_update_ts
Module: U:\dev\php-5.3.20\ext\date\lib\unixtime2tm.obj(unixtime2tm.obj)
0001:0007b530  _timelib_unixtime2gmt
0001:0007bb8b  _timelib_set_timezone
0001:0007bc07  _timelib_update_from_sse
0001:0007bd25  _timelib_unixtime2local
0001:0007be58  _timelib_apply_localtime
Module: U:\dev\php-5.3.20\ext\date\lib\parse_iso_intervals.obj(parse_iso_intervals.obj)
0001:0007c170  _timelib_strtointerval
Module: U:\dev\php-5.3.20\ext\date\lib\interval.obj(interval.obj)
0001:0007d320  _timelib_diff
Module: U:\dev\php-5.3.20\ext\ereg\ereg.obj(ereg.obj)
0002:00020110  _ereg_globals_id
0001:0007d712  _zm_shutdown_ereg
0001:0007d71b  _zif_sql_regcase
0001:0007dde5  _zif_spliti
0001:0007de14  _zif_split
0001:0007de43  _php_ereg_replace
0001:0007e5df  _zif_eregi_replace
0001:0007e60e  _zif_ereg_replace
0001:0007ea89  _zif_eregi
0001:0007eab8  _zif_ereg
0001:0007eb0d  _zm_info_ereg
0001:0007eb3a  _zm_startup_ereg
0001:0007ec00  _ereg_functions
0002:00000130  _ereg_module_entry
Module: U:\dev\php-5.3.20\ext\ereg\regex\regcomp.obj(regcomp.obj)
0001:00080e9c  _php_regcomp
Module: U:\dev\php-5.3.20\ext\ereg\regex\regexec.obj(regexec.obj)
0001:00083e0b  _php_regexec
Module: U:\dev\php-5.3.20\ext\ereg\regex\regerror.obj(regerror.obj)
0001:00084e9e  _php_regerror
Module: U:\dev\php-5.3.20\ext\ereg\regex\regfree.obj(regfree.obj)
0001:00085380  _php_regfree
Module: U:\dev\php-5.3.20\ext\libxml\libxml.obj(libxml.obj)
0001:00085423  _php_libxml_switch_context
0001:0008543e  _php_libxml_xmlCheckUTF8
0001:00085883  _php_libxml_increment_doc_ref
0001:00085d19  _php_libxml_decrement_node_ptr
0001:00085d6d  _php_libxml_increment_node_ptr
0001:00087295  _php_libxml_structured_error_handler
0001:0008723e  _php_libxml_error_handler
0001:000863d3  _php_libxml_decrement_doc_ref
0001:000865cc  _php_libxml_node_free_resource
0001:00086694  _php_libxml_node_decrement_resource
0001:00086706  _php_libxml_import_node
0001:0008676e  _php_libxml_shutdown
0001:000867b0  _php_libxml_initialize
0001:00086e53  _php_libxml_register_export
0001:00087259  _php_libxml_ctx_warning
0001:00087277  _php_libxml_ctx_error
0001:000872a6  _php_libxml_issue_error
0002:00000190  _libxml_module_entry
Module: U:\dev\php-5.3.20\ext\pcre\pcrelib\pcre_chartables.obj(pcre_chartables.obj)
0001:00087550  _php__pcre_default_tables
Module: U:\dev\php-5.3.20\ext\pcre\pcrelib\pcre_ucd.obj(pcre_ucd.obj)
0001:00087990  _php__pcre_ucd_records
0001:00088b50  _php__pcre_ucd_stage1
0001:0008ad50  _php__pcre_ucd_stage2
Module: U:\dev\php-5.3.20\ext\pcre\pcrelib\pcre_compile.obj(pcre_compile.obj)
0001:00097f4c  __pcre_find_bracket
0001:000a0f49  _php_pcre_compile2
0001:000a1a15  _php_pcre_compile
Module: U:\dev\php-5.3.20\ext\pcre\pcrelib\pcre_config.obj(pcre_config.obj)
0001:000a2ae0  _php_pcre_config
Module: U:\dev\php-5.3.20\ext\pcre\pcrelib\pcre_exec.obj(pcre_exec.obj)
0001:000b3cdb  _php_pcre_exec
Module: U:\dev\php-5.3.20\ext\pcre\pcrelib\pcre_fullinfo.obj(pcre_fullinfo.obj)
0001:000b4e10  _php_pcre_fullinfo
Module: U:\dev\php-5.3.20\ext\pcre\pcrelib\pcre_get.obj(pcre_get.obj)
0001:000b5030  _php_pcre_free_substring_list
0001:000b503e  _php_pcre_free_substring
0001:000b504c  _php_pcre_get_substring
0001:000b50b7  _php_pcre_get_substring_list
0001:000b516b  _php_pcre_copy_substring
0001:000b51c3  _php_pcre_get_stringtable_entries
0001:000b5360  _php_pcre_get_stringnumber
0001:000b54f8  _php_pcre_get_named_substring
0001:000b5547  _php_pcre_copy_named_substring
Module: U:\dev\php-5.3.20\ext\pcre\pcrelib\pcre_globals.obj(pcre_globals.obj)
0002:000001f0  _php_pcre_malloc
0002:000001f4  _php_pcre_free
0002:000001f8  _php_pcre_stack_malloc
0002:000001fc  _php_pcre_stack_free
0002:00008fe0  _php_pcre_callout
Module: U:\dev\php-5.3.20\ext\pcre\pcrelib\pcre_maketables.obj(pcre_maketables.obj)
0001:000b55bd  _php_pcre_maketables
Module: U:\dev\php-5.3.20\ext\pcre\pcrelib\pcre_newline.obj(pcre_newline.obj)
0001:000b5950  _php__pcre_is_newline
0001:000b5aff  _php__pcre_was_newline
Module: U:\dev\php-5.3.20\ext\pcre\pcrelib\pcre_ord2utf8.obj(pcre_ord2utf8.obj)
0001:000b5cf0  __pcre_ord2utf
Module: U:\dev\php-5.3.20\ext\pcre\pcrelib\pcre_refcount.obj(pcre_refcount.obj)
0001:000b5d90  _php_pcre_refcount
Module: U:\dev\php-5.3.20\ext\pcre\pcrelib\pcre_study.obj(pcre_study.obj)
0001:000b5e00  _pcre_free_study
0001:000b711b  _php_pcre_study
Module: U:\dev\php-5.3.20\ext\pcre\pcrelib\pcre_tables.obj(pcre_tables.obj)
0001:000b7390  _php__pcre_OP_lengths
0001:000b7430  _php__pcre_utf8_table1
0001:000b7448  _php__pcre_utf8_table1_size
0001:000b7450  _php__pcre_utf8_table2
0001:000b7470  _php__pcre_utf8_table3
0001:000b7490  _php__pcre_utf8_table4
0001:000b74d0  _php__pcre_ucp_gentype
0001:000b7550  _php__pcre_utt_names
0001:000b7970  _php__pcre_utt
0001:000b7cd8  _php__pcre_utt_size
Module: U:\dev\php-5.3.20\ext\pcre\pcrelib\pcre_valid_utf8.obj(pcre_valid_utf8.obj)
0001:000b7ce0  __pcre_valid_utf
Module: U:\dev\php-5.3.20\ext\pcre\pcrelib\pcre_version.obj(pcre_version.obj)
0001:000b80e0  _php_pcre_version
Module: U:\dev\php-5.3.20\ext\pcre\pcrelib\pcre_xclass.obj(pcre_xclass.obj)
0001:000b80f0  _php__pcre_xclass
Module: U:\dev\php-5.3.20\ext\pcre\php_pcre.obj(php_pcre.obj)
0002:00020120  _pcre_globals_id
0001:000b9534  _pcre_get_compiled_regex_cache
0001:000b9c7f  _pcre_get_compiled_regex_ex
0001:000b9cf9  _pcre_get_compiled_regex
0001:000b9d81  _php_pcre_grep_impl
0001:000ba23b  _php_pcre_replace_impl
0001:000bb040  _php_pcre_replace
0001:000bbc8f  _php_pcre_split_impl
0001:000bc3e9  _php_pcre_match_impl
0002:00000200  _pcre_module_entry
Module: U:\dev\php-5.3.20\ext\sqlite3\sqlite3.obj(sqlite3.obj)
0002:00020130  _php_sqlite3_sc_entry
0002:00020140  _php_sqlite3_stmt_entry
0002:00020150  _php_sqlite3_result_entry
0002:00020160  _sqlite3_globals_id
0001:000bd8f8  _zm_info_sqlite3
0001:000bd96e  _zm_shutdown_sqlite3
0001:000bdab0  _zm_startup_sqlite3
0001:000be5b6  _zim_sqlite3result___construct
0001:000be5e7  _zim_sqlite3stmt_close
0001:000be656  _zim_sqlite3_enableExceptions
0001:000be7a4  _zim_sqlite3result_finalize
0001:000be855  _zim_sqlite3result_reset
0001:000be91b  _zim_sqlite3stmt_reset
0001:000be9b6  _zim_sqlite3result_columnType
0001:000bea6b  _zim_sqlite3result_columnName
0001:000beb6e  _zim_sqlite3_lastErrorMsg
0001:000bed8c  _zim_sqlite3result_fetchArray
0001:000bef40  _zim_sqlite3result_numColumns
0001:000beff0  _zim_sqlite3stmt___construct
0001:000bf1fe  _zim_sqlite3stmt_execute
0001:000bf5f5  _zim_sqlite3_prepare
0001:000bf8f2  _zim_sqlite3stmt_bindValue
0001:000bfa12  _zim_sqlite3stmt_bindParam
0001:000bfb28  _zim_sqlite3stmt_readOnly
0001:000bfbb5  _zim_sqlite3stmt_clear
0001:000bfc4e  _zim_sqlite3stmt_paramCount
0001:000bfcc9  _zim_sqlite3_openBlob
0001:000bff15  _zim_sqlite3_createCollation
0001:000c00e1  _zim_sqlite3_createAggregate
0001:000c036d  _zim_sqlite3_createFunction
0001:000c0eb6  _zim_sqlite3_querySingle
0001:000c11a5  _zim_sqlite3_query
0001:000c145d  _zim_sqlite3_exec
0001:000c1547  _zim_sqlite3_escapeString
0001:000c15fe  _zim_sqlite3_changes
0001:000c175c  _zim_sqlite3_loadExtension
0001:000c1aab  _zim_sqlite3_busyTimeout
0001:000c1b70  _zim_sqlite3_lastErrorCode
0001:000c1bee  _zim_sqlite3_lastInsertRowID
0001:000c1c88  _zim_sqlite3_version
0001:000c1d35  _zim_sqlite3_close
0001:000c1f16  _zim_sqlite3_open
0002:00000260  _sqlite3_module_entry
Module: U:\dev\php-5.3.20\ext\sqlite3\libsqlite\sqlite3.obj(sqlite3.obj)
0002:00020170  _doclist
0001:000c29d8  _sqlite3_compileoption_used
0001:000c2b8d  _sqlite3_compileoption_get
0001:000c3061  _sqlite3_mutex_free
0001:000c3078  _sqlite3_mutex_enter
0001:000c308f  _sqlite3_mutex_try
0001:000c30a9  _sqlite3_mutex_leave
0001:000c30c0  _sqlite3_vfs_unregister
0001:000c3161  _sqlite3_release_memory
0001:000c3202  _sqlite3_memory_alarm
0001:000c360b  _sqlite3_free
0001:000c3ac2  _sqlite3_strnicmp
0001:000c5eb3  _sqlite3_enable_shared_cache
0001:000c6407  _sqlite3_backup_remaining
0001:000c6412  _sqlite3_backup_pagecount
0001:000c66be  _sqlite3_sql
0001:000c6cee  _sqlite3_expired
0001:000c6d08  _sqlite3_value_double
0001:000c6d17  _sqlite3_value_int
0001:000c6d24  _sqlite3_value_int64
0001:000c6d30  _sqlite3_value_type
0001:000c6d3c  _sqlite3_result_null
0001:000c6d4e  _sqlite3_result_error_nomem
0001:000c6d74  _sqlite3_user_data
0001:000c6d81  _sqlite3_context_db_handle
0001:000c6d8c  _sqlite3_get_auxdata
0001:000c6db1  _sqlite3_aggregate_count
0001:000c6dbf  _sqlite3_column_count
0001:000c6dd1  _sqlite3_data_count
0001:000c6e64  _sqlite3_column_name
0001:000c6e82  _sqlite3_column_name16
0001:000c6ea0  _sqlite3_column_decltype
0001:000c6ebe  _sqlite3_column_decltype16
0001:000c6edc  _sqlite3_column_database_name
0001:000c6efa  _sqlite3_column_database_name16
0001:000c6f18  _sqlite3_column_table_name
0001:000c6f36  _sqlite3_column_table_name16
0001:000c6f54  _sqlite3_column_origin_name
0001:000c6f72  _sqlite3_column_origin_name16
0001:000c6f90  _sqlite3_bind_parameter_count
0001:000c6fa2  _sqlite3_bind_parameter_name
0001:000c6fcb  _sqlite3_db_handle
0001:000c6fdb  _sqlite3_stmt_readonly
0001:000c6ff0  _sqlite3_next_stmt
0001:000c702c  _sqlite3_stmt_status
0001:000c70f4  _sqlite3_value_numeric_type
0001:000c712a  _sqlite3_blob_bytes
0001:000c7d33  _sqlite3_set_authorizer
0001:000c8c82  _sqlite3_enable_load_extension
0001:000c90a1  _sqlite3_free_table
0001:000c94e3  _sqlite3_vtab_on_conflict
0001:000ca2ff  _sqlite3_complete
0001:000cabdd  _sqlite3_libversion
0001:000cac25  _sqlite3_sourceid
0001:000cac2f  _sqlite3_libversion_number
0001:000cac39  _sqlite3_threadsafe
0001:000cadb2  _sqlite3_db_mutex
0001:000cae6f  _sqlite3_last_insert_rowid
0001:000cae7d  _sqlite3_changes
0001:000cae88  _sqlite3_total_changes
0001:000caf66  _sqlite3_busy_handler
0001:000cafaa  _sqlite3_progress_handler
0001:000cb018  _sqlite3_busy_timeout
0001:000cb062  _sqlite3_interrupt
0001:000cb074  _sqlite3_trace
0001:000cb0b6  _sqlite3_profile
0001:000cb0f8  _sqlite3_commit_hook
0001:000cb13a  _sqlite3_update_hook
0001:000cb17c  _sqlite3_rollback_hook
0001:000cb1be  _sqlite3_wal_hook
0001:000cb200  _sqlite3_wal_autocheckpoint
0001:000cb244  _sqlite3_limit
0001:000cb27c  _sqlite3_collation_needed
0001:000cb2c0  _sqlite3_collation_needed16
0001:000cb304  _sqlite3_global_recover
0001:000cb30b  _sqlite3_get_autocommit
0001:000cb317  _sqlite3_thread_cleanup
0001:000cb31c  _sqlite3_extended_result_codes
0001:000cc2c4  _sqlite3_uri_parameter
0001:000cc376  _sqlite3_file_control
0001:000cc4b1  _sqlite3_db_config
0001:000ce9eb  _sqlite3_result_int64
0001:000cea38  _sqlite3_result_int
0001:000cecea  _sqlite3_db_status
0001:000cefc8  _sqlite3_result_zeroblob
0001:000cf058  _sqlite3_result_double
0001:000cf0e9  _sqlite3_clear_bindings
0001:000e46f5  _sqlite3_value_text
0001:000e45ea  _sqlite3_value_text16
0001:001343cf  _sqlite3_version
0001:000d2b1a  _sqlite3_transfer_bindings
0001:000d346c  _sqlite3_bind_parameter_index
0001:000d35ce  _sqlite3_os_end
0001:000d452c  _sqlite3_os_init
0001:000ec5de  _sqlite3_vfs_register
0001:000d454f  _sqlite3_initialize
0001:000daf2a  _sqlite3_malloc
0001:000e1901  _sqlite3_config
0001:000d4a34  _sqlite3_reset_auto_extension
0001:000d4a84  _sqlite3_shutdown
0001:000d4b36  _sqlite3_realloc
0001:000d55ec  _sqlite3_result_value
0001:000d58dc  _sqlite3_result_error_toobig
0001:000d59bc  _sqlite3_result_error_code
0001:000d5a48  _sqlite3_result_text16le
0001:000d5a67  _sqlite3_result_text16be
0001:000d5a86  _sqlite3_result_text16
0001:000d5aa8  _sqlite3_result_text
0001:000d5c5b  _sqlite3_result_blob
0001:000d5c7d  _sqlite3_result_error16
0001:000d5caa  _sqlite3_result_error
0001:000d6008  _sqlite3_aggregate_context
0001:000d8446  _sqlite3_set_auxdata
0001:000dae81  _sqlite3_auto_extension
0001:000dc22a  _sqlite3_create_module_v2
0001:000dc24b  _sqlite3_create_module
0001:000dc31d  _sqlite3_column_type
0001:000dc340  _sqlite3_column_value
0001:000dc374  _sqlite3_column_int64
0001:000dc3a6  _sqlite3_column_int
0001:000dc3cc  _sqlite3_column_double
0001:000e0336  _sqlite3_log
0001:000e1394  _sqlite3_create_collation_v2
0001:000e13f3  _sqlite3_create_collation
0001:000e16f3  _sqlite3_overload_function
0001:000e17b3  _sqlite3_create_function_v2
0001:000e18b5  _sqlite3_create_function
0001:000e1b25  _sqlite3_vtab_config
0001:000e1ba0  _sqlite3_status
0001:000e1be9  _sqlite3_memory_highwater
0001:000e1c16  _sqlite3_memory_used
0001:000e1cbe  _sqlite3_extended_errcode
0001:000e1d00  _sqlite3_errcode
0001:000e20d2  _sqlite3_bind_zeroblob
0001:000e2207  _sqlite3_bind_text16
0001:000e2234  _sqlite3_bind_text
0001:000e2261  _sqlite3_bind_blob
0001:000e228e  _sqlite3_bind_null
0001:000e22bf  _sqlite3_bind_int64
0001:000e2325  _sqlite3_bind_int
0001:000e234b  _sqlite3_bind_double
0001:000e239b  _sqlite3_bind_value
0001:000e247f  _sqlite3_vsnprintf
0001:000e24dc  _sqlite3_snprintf
0001:000e45c2  _sqlite3_value_text16le
0001:000e45d6  _sqlite3_value_text16be
0001:000e45fe  _sqlite3_errmsg16
0001:000e46c6  _sqlite3_column_text16
0001:000e4717  _sqlite3_errmsg
0001:000e5a2d  _sqlite3_column_text
0001:000e5a5c  _sqlite3_value_blob
0001:000e5aa2  _sqlite3_column_blob
0001:000e5ad1  _sqlite3_value_bytes16
0001:000e5b17  _sqlite3_column_bytes16
0001:000e5b46  _sqlite3_value_bytes
0001:000e6aad  _sqlite3_column_bytes
0001:000e9951  _sqlite3_wal_checkpoint_v2
0001:000e9a27  _sqlite3_wal_checkpoint
0001:000eb3d2  _sqlite3_complete16
0001:000eb44b  _sqlite3_vmprintf
0001:000eb4b9  _sqlite3_mprintf
0001:000ebda4  _sqlite3_load_extension
0001:000ec0aa  _sqlite3_soft_heap_limit64
0001:000ec132  _sqlite3_soft_heap_limit
0001:000ec153  _sqlite3_mutex_alloc
0001:000ec68e  _sqlite3_vfs_find
0001:000ec6fe  _sqlite3_sleep
0001:000ecde7  _sqlite3_randomness
0001:000ecf59  _sqlite3_test_control
0001:000f355f  _sqlite3_close
0001:000f3ce5  _sqlite3_backup_finish
0001:000f8873  _sqlite3_backup_step
0001:000f9cee  _sqlite3_blob_write
0001:000f9d10  _sqlite3_blob_read
0001:000f9d6e  _sqlite3_finalize
0001:000f9e88  _sqlite3_blob_close
0001:000fac26  _sqlite3_reset
0001:000fae62  _convertCpPathToUtf8
0001:000fb0f9  _sqlite3_create_function16
0001:000fb187  _sqlite3_create_collation16
0001:000fc994  _sqlite3_backup_init
0001:000fd31d  _sqlite3_open16
0001:000fd3c0  _sqlite3_open_v2
0001:000fd3db  _sqlite3_open
0001:0010fc85  _sqlite3_declare_vtab
0001:001120b4  _sqlite3_prepare16_v2
0001:001120e1  _sqlite3_prepare16
0001:0011210e  _sqlite3_prepare_v2
0001:001122dd  _sqlite3_prepare
0001:001124d6  _sqlite3_step
0001:00114a1e  _sqlite3_exec
0001:00115522  _sqlite3_table_column_metadata
0001:001220b0  _sqlite3_get_table
0001:0012464d  _sqlite3_blob_reopen
0001:0012478a  _sqlite3_blob_open
0002:00009140  _sqlite3_temp_directory
Module: U:\dev\php-5.3.20\ext\zlib\zlib.obj(zlib.obj)
0002:00020190  _zlib_globals_id
0001:0013af52  _php_ob_gzhandler_check
0002:00001090  _php_zlib_module_entry
Module: U:\dev\php-5.3.20\ext\zlib\zlib_fopen_wrapper.obj(zlib_fopen_wrapper.obj)
0001:0013bdc9  _php_stream_gzopen
0002:000010f0  _php_stream_gzip_wrapper
Module: U:\dev\php-5.3.20\ext\zlib\zlib_filter.obj(zlib_filter.obj)
0002:00001170  _php_zlib_filter_factory
Module: U:\dev\php-5.3.20\ext\bcmath\bcmath.obj(bcmath.obj)
0002:000201a0  _bcmath_globals_id
0001:0013d122  _zif_bcscale
0001:0013d184  _zif_bccomp
0001:0013d337  _zif_bcsqrt
0001:0013d441  _zif_bcpow
0001:0013d5a3  _zif_bcpowmod
0001:0013d758  _zif_bcmod
0001:0013d8b8  _zif_bcdiv
0001:0013da3c  _zif_bcmul
0001:0013db98  _zif_bcsub
0001:0013dcf0  _zif_bcadd
0001:0013de5f  _zm_info_bcmath
0001:0013de9c  _zm_shutdown_bcmath
0001:0013deb8  _zm_startup_bcmath
0001:0013df20  _bcmath_functions
0002:00001190  _bcmath_module_entry
Module: U:\dev\php-5.3.20\ext\bcmath\libbcmath\src\add.obj(add.obj)
0001:0013e480  _bc_add
Module: U:\dev\php-5.3.20\ext\bcmath\libbcmath\src\div.obj(div.obj)
0001:0013e63d  _bc_divide
Module: U:\dev\php-5.3.20\ext\bcmath\libbcmath\src\init.obj(init.obj)
0001:0013ec70  _bc_copy_num
0001:0013ec7c  _bc_init_num
0001:0013ec9b  __bc_free_num_ex
0001:0013ed02  __bc_new_num_ex
0001:0013edda  _bc_init_numbers
Module: U:\dev\php-5.3.20\ext\bcmath\libbcmath\src\neg.obj(neg.obj)
0001:0013eea0  _bc_is_neg
Module: U:\dev\php-5.3.20\ext\bcmath\libbcmath\src\outofmem.obj(outofmem.obj)
0001:0013eec8  _bc_out_of_memory
Module: U:\dev\php-5.3.20\ext\bcmath\libbcmath\src\raisemod.obj(raisemod.obj)
0001:0013ef4c  _bc_raisemod
Module: U:\dev\php-5.3.20\ext\bcmath\libbcmath\src\rt.obj(rt.obj)
0001:0013f1d3  _bc_rt_error
0001:0013f238  _bc_rt_warn
Module: U:\dev\php-5.3.20\ext\bcmath\libbcmath\src\sub.obj(sub.obj)
0001:0013f290  _bc_sub
Module: U:\dev\php-5.3.20\ext\bcmath\libbcmath\src\compare.obj(compare.obj)
0001:0013f3b0  __bc_do_compare
0001:0013f4b4  _bc_compare
Module: U:\dev\php-5.3.20\ext\bcmath\libbcmath\src\divmod.obj(divmod.obj)
0001:0013f4e0  _bc_divmod
0001:0013f63f  _bc_modulo
Module: U:\dev\php-5.3.20\ext\bcmath\libbcmath\src\int2num.obj(int2num.obj)
0001:0013f680  _bc_int2num
Module: U:\dev\php-5.3.20\ext\bcmath\libbcmath\src\num2long.obj(num2long.obj)
0001:0013f770  _bc_num2long
Module: U:\dev\php-5.3.20\ext\bcmath\libbcmath\src\output.obj(output.obj)
0001:0013f7c4  _bc_out_long
0001:0013f866  _bc_out_num
Module: U:\dev\php-5.3.20\ext\bcmath\libbcmath\src\recmul.obj(recmul.obj)
0001:001404a3  _bc_multiply
0002:000011f0  _mul_base_digits
Module: U:\dev\php-5.3.20\ext\bcmath\libbcmath\src\sqrt.obj(sqrt.obj)
0001:00140580  _bc_sqrt
Module: U:\dev\php-5.3.20\ext\bcmath\libbcmath\src\zero.obj(zero.obj)
0001:00140910  _bc_is_zero
Module: U:\dev\php-5.3.20\ext\bcmath\libbcmath\src\debug.obj(debug.obj)
0001:00140964  _pv
0001:001409c1  _pn
Module: U:\dev\php-5.3.20\ext\bcmath\libbcmath\src\doaddsub.obj(doaddsub.obj)
0001:00140a00  __bc_do_sub
0001:00140c13  __bc_do_add
Module: U:\dev\php-5.3.20\ext\bcmath\libbcmath\src\nearzero.obj(nearzero.obj)
0001:00140e30  _bc_is_near_zero
Module: U:\dev\php-5.3.20\ext\bcmath\libbcmath\src\num2str.obj(num2str.obj)
0001:00140e90  _bc_num2str
Module: U:\dev\php-5.3.20\ext\bcmath\libbcmath\src\raise.obj(raise.obj)
0001:00140fb7  _bc_raise
Module: U:\dev\php-5.3.20\ext\bcmath\libbcmath\src\rmzero.obj(rmzero.obj)
0001:00141200  __bc_rm_leading_zeros
Module: U:\dev\php-5.3.20\ext\bcmath\libbcmath\src\str2num.obj(str2num.obj)
0001:00141240  _bc_str2num
Module: U:\dev\php-5.3.20\ext\calendar\calendar.obj(calendar.obj)
0001:00141493  _zif_jdmonthname
0001:0014164d  _zif_jddayofweek
0001:00141731  _zif_frenchtojd
0001:001417af  _zif_jdtofrench
0001:00141870  _zif_jdtojulian
0001:00141931  _zif_jdtogregorian
0001:001419f2  _zif_jewishtojd
0001:00141a83  _zif_cal_to_jd
0001:00141b3d  _zif_cal_days_in_month
0001:00141e88  _zif_jdtojewish
0001:00142011  _zif_juliantojd
0001:00142084  _zif_gregoriantojd
0001:00142153  _zif_cal_from_jd
0001:00142599  _zif_cal_info
0001:001426a5  _zm_info_calendar
0001:0014285f  _zm_startup_calendar
0001:00142cf0  _calendar_functions
0002:00001200  _calendar_module_entry
Module: U:\dev\php-5.3.20\ext\calendar\dow.obj(dow.obj)
0001:00143480  _DayOfWeek
0002:000012e0  _DayNameShort
0002:00001300  _DayNameLong
Module: U:\dev\php-5.3.20\ext\calendar\french.obj(french.obj)
0001:00143510  _SdnToFrench
0001:001435ad  _FrenchToSdn
0002:00001320  _FrenchMonthName
Module: U:\dev\php-5.3.20\ext\calendar\gregor.obj(gregor.obj)
0001:00143680  _SdnToGregorian
0001:001437a2  _GregorianToSdn
0002:00001360  _MonthNameShort
0002:000013a0  _MonthNameLong
Module: U:\dev\php-5.3.20\ext\calendar\jewish.obj(jewish.obj)
0001:00143c75  _SdnToJewish
0001:0014400e  _JewishToSdn
0002:000013e0  _JewishMonthName
0002:00001420  _JewishMonthHebName
Module: U:\dev\php-5.3.20\ext\calendar\julian.obj(julian.obj)
0001:001443c0  _SdnToJulian
0001:001444ae  _JulianToSdn
Module: U:\dev\php-5.3.20\ext\calendar\easter.obj(easter.obj)
0001:00144967  _zif_easter_days
0001:00144996  _zif_easter_date
Module: U:\dev\php-5.3.20\ext\calendar\cal_unix.obj(cal_unix.obj)
0001:001449d2  _zif_jdtounix
0001:00144a36  _zif_unixtojd
Module: U:\dev\php-5.3.20\ext\ctype\ctype.obj(ctype.obj)
0002:00001460  _ctype_module_entry
Module: U:\dev\php-5.3.20\ext\dom\php_dom.obj(php_dom.obj)
0002:000201b0  _dom_domimplementation_class_entry
0002:000201c0  _dom_nodelist_class_entry
0002:000201d0  _dom_namednodemap_class_entry
0002:000201e0  _dom_object_handlers
0002:00020250  _dom_namespace_node_class_entry
0002:00020260  _dom_entity_class_entry
0002:00020270  _dom_notation_class_entry
0002:00020280  _dom_documentfragment_class_entry
0002:00020290  _dom_documenttype_class_entry
0002:000202a0  _dom_document_class_entry
0002:000202b0  _dom_comment_class_entry
0002:000202c0  _dom_processinginstruction_class_entry
0002:000202d0  _dom_entityreference_class_entry
0002:000202e0  _dom_cdatasection_class_entry
0002:000202f0  _dom_text_class_entry
0002:00020300  _dom_attr_class_entry
0002:00020310  _dom_element_class_entry
0002:00020320  _dom_xpath_class_entry
0002:00020330  _dom_node_class_entry
0002:00020340  _dom_domexception_class_entry
0002:00020350  _dom_domstringlist_class_entry
0002:00020360  _dom_namelist_class_entry
0002:00020370  _dom_domimplementationlist_class_entry
0002:00020380  _dom_domimplementationsource_class_entry
0002:00020390  _dom_characterdata_class_entry
0002:000203a0  _dom_typeinfo_class_entry
0002:000203b0  _dom_userdatahandler_class_entry
0002:000203c0  _dom_domerror_class_entry
0002:000203d0  _dom_domerrorhandler_class_entry
0002:000203e0  _dom_domlocator_class_entry
0002:000203f0  _dom_domconfiguration_class_entry
0002:00020400  _dom_string_extend_class_entry
0001:00146080  _dom_node_is_read_only
0001:001460e1  _dom_node_children_valid
0001:001460fd  _dom_object_get_node
0001:00146116  _php_dom_object_get_data
0001:00146131  _dom_hierarchy
0001:0014616e  _dom_get_nsdecl
0001:001461f5  _dom_get_elements_by_tag_name_ns_raw
0001:00146381  _dom_get_ns
0001:0014645a  _dom_check_qname
0001:001464dc  _dom_set_old_ns
0001:0014655b  _node_list_unlink
0001:00146618  _dom_normalize
0001:0014670a  _dom_has_feature
0001:00146794  _php_dom_create_implementation
0001:001467b9  _php_dom_create_interator
0001:001467f5  _dom_get_doc_props
0001:00146938  _dom_namednode_iter
0001:001469ad  _dom_get_doc_classmap
0001:00146a1f  _php_dom_create_object
0001:00146d1e  _dom_nnodemap_objects_new
0001:00146f54  _dom_objects_clone
0001:00146e85  _dom_nnodemap_objects_free_storage
0001:00146da5  _dom_objects_new
0001:001470cc  _dom_objects_free_storage
0001:00146e51  _dom_get_strict_error
0001:00146eb9  _dom_xpath_objects_new
0001:0014713b  _dom_xpath_objects_free_storage
0001:001471b9  _zm_shutdown_dom
0001:0014734c  _zm_info_dom
0001:00147ce6  _zm_startup_dom
0001:0014c271  _dom_read_property
0001:0014c018  _dom_write_property
0001:0014c3fe  _dom_objects_store_clone_obj
0001:0014bc98  _php_dom_export_node
0001:0014c509  _zif_dom_import_simplexml
0001:0014c5ed  _dom_set_doc_classmap
0002:000014c0  _dom_module_entry
Module: U:\dev\php-5.3.20\ext\dom\attr.obj(attr.obj)
0001:0014c7f4  _zif_dom_attr_is_id
0001:0014c8bc  _dom_attr_schema_type_info_read
0001:0014c905  _dom_attr_specified_read
0001:0014c956  _dom_attr_owner_element_read
0001:0014ca1f  _dom_attr_value_write
0001:0014cb09  _dom_attr_value_read
0001:0014cbe1  _dom_attr_name_read
0001:0014cc70  _zim_domattr___construct
0001:0014ce00  _php_dom_attr_class_functions
Module: U:\dev\php-5.3.20\ext\dom\document.obj(document.obj)
0001:0014ced4  _zif_dom_document_rename_node
0001:0014cefb  _zif_dom_document_adopt_node
0001:0014cfbd  _zim_domdocument_registerNodeClass
0001:0014d289  _zif_dom_document_save_html
0001:0014d54e  _zif_dom_document_save_html_file
0001:0014d90e  _zim_domdocument_loadHTML
0001:0014d93d  _zim_domdocument_loadHTMLFile
0001:0014d96e  _zif_dom_document_validate
0001:0014dae9  _zif_dom_document_xinclude
0001:0014dbf0  _zif_dom_document_savexml
0001:0014df21  _zif_dom_document_save
0001:0014e0c5  __dom_get_valid_file_path
0001:0014e4a2  _zif_dom_document_relaxNG_validate_xml
0001:0014e4d1  _zif_dom_document_relaxNG_validate_file
0001:0014e7ed  _zif_dom_document_schema_validate_xml
0001:0014e81c  _zif_dom_document_schema_validate_file
0001:0014ed3b  _zim_domdocument_loadXML
0001:0014ed6a  _zim_domdocument_load
0001:0014ed9e  _zim_domdocument___construct
0001:0014ef39  _zif_dom_document_normalize_document
0001:0014efda  _zif_dom_document_get_element_by_id
0001:0014f102  _zif_dom_document_get_elements_by_tag_name_ns
0001:0014f239  _zif_dom_document_get_elements_by_tag_name
0001:0014f344  _zif_dom_document_create_attribute
0001:0014f4dd  _zif_dom_document_create_attribute_ns
0001:0014f79b  _zif_dom_document_create_element
0001:0014f934  _zif_dom_document_create_element_ns
0001:0014fc1b  _zif_dom_document_import_node
0001:0014fea4  _zif_dom_document_create_entity_reference
0001:0015000a  _zif_dom_document_create_processing_instruction
0001:0015019a  _zif_dom_document_create_cdatasection
0001:001502bc  _zif_dom_document_create_comment
0001:001503d7  _zif_dom_document_create_text_node
0001:001504f2  _zif_dom_document_create_document_fragment
0001:001505f8  _dom_document_config_read
0001:0015061e  _dom_document_document_uri_read
0001:001506ba  _dom_document_substitue_entities_read
0001:0015071a  _dom_document_recover_read
0001:0015077a  _dom_document_preserve_whitespace_read
0001:001507da  _dom_document_resolve_externals_read
0001:0015083a  _dom_document_validate_on_parse_read
0001:0015089a  _dom_document_format_output_read
0001:001508f9  _dom_document_strict_error_checking_read
0001:00150959  _dom_document_version_read
0001:001509f6  _dom_document_standalone_read
0001:00150a61  _dom_document_encoding_read
0001:00150afe  _dom_document_document_element_read
0001:00150bd0  _dom_document_implementation_read
0001:00150c06  _dom_document_doctype_read
0001:00150cd8  _dom_document_format_output_write
0001:00150d6c  _dom_document_encoding_write
0001:00150e7e  _dom_document_strict_error_checking_write
0001:00150ef7  _dom_document_standalone_write
0001:00150fbb  _dom_document_document_uri_write
0001:0015108b  _dom_document_version_write
0001:0015115b  _dom_document_substitue_entities_write
0001:001511d7  _dom_document_recover_write
0001:00151252  _dom_document_preserve_whitespace_write
0001:001512cc  _dom_document_resolve_externals_write
0001:00151347  _dom_document_validate_on_parse_write
0001:001515b0  _php_dom_document_class_functions
Module: U:\dev\php-5.3.20\ext\dom\domerrorhandler.obj(domerrorhandler.obj)
0001:001520d4  _zif_dom_domerrorhandler_handle_error
0001:00152110  _php_dom_domerrorhandler_class_functions
Module: U:\dev\php-5.3.20\ext\dom\domstringlist.obj(domstringlist.obj)
0001:00152194  _zif_dom_domstringlist_item
0001:001521c0  _dom_domstringlist_length_read
0001:00152220  _php_dom_domstringlist_class_functions
Module: U:\dev\php-5.3.20\ext\dom\domexception.obj(domexception.obj)
0001:00152280  _php_dom_throw_error_with_message
0001:001522c9  _php_dom_throw_error
0001:00152310  _php_dom_domexception_class_functions
Module: U:\dev\php-5.3.20\ext\dom\namelist.obj(namelist.obj)
0001:001524c4  _zif_dom_namelist_get_namespace_uri
0001:001524eb  _zif_dom_namelist_get_name
0001:00152517  _dom_namelist_length_read
0001:00152580  _php_dom_namelist_class_functions
Module: U:\dev\php-5.3.20\ext\dom\processinginstruction.obj(processinginstruction.obj)
0001:00152630  _dom_processinginstruction_data_write
0001:00152707  _dom_processinginstruction_data_read
0001:001527df  _dom_processinginstruction_target_read
0001:0015286e  _zim_domprocessinginstruction___construct
0001:00152a00  _php_dom_processinginstruction_class_functions
Module: U:\dev\php-5.3.20\ext\dom\cdatasection.obj(cdatasection.obj)
0001:00152a93  _zim_domcdatasection___construct
0001:00152bd0  _php_dom_cdatasection_class_functions
Module: U:\dev\php-5.3.20\ext\dom\documentfragment.obj(documentfragment.obj)
0001:00152caf  _zim_domdocumentfragment_appendXML
0001:00152e25  _zim_domdocumentfragment___construct
0001:00152f40  _php_dom_documentfragment_class_functions
Module: U:\dev\php-5.3.20\ext\dom\domimplementation.obj(domimplementation.obj)
0001:00152fe4  _zim_domimplementation_getFeature
0001:00153072  _zim_domimplementation_createDocument
0001:0015342c  _zim_domimplementation_createDocumentType
0001:00153625  _zim_domimplementation_hasFeature
0001:001536e0  _php_dom_domimplementation_class_functions
Module: U:\dev\php-5.3.20\ext\dom\element.obj(element.obj)
0001:00153980  _zif_dom_element_set_id_attribute_node
0001:00153ae2  _zif_dom_element_set_id_attribute_ns
0001:00153c3b  _zif_dom_element_set_id_attribute
0001:00153da6  _zif_dom_element_has_attribute_ns
0001:0015401d  _zif_dom_element_has_attribute
0001:001540eb  _zif_dom_element_get_elements_by_tag_name_ns
0001:00154222  _zif_dom_element_get_elements_by_tag_name
0001:0015436e  _zif_dom_element_set_attribute_node_ns
0001:0015466d  _zif_dom_element_get_attribute_node_ns
0001:0015479f  _zif_dom_element_remove_attribute_node
0001:00154970  _zif_dom_element_set_attribute_node
0001:00154c20  _zif_dom_element_remove_attribute_ns
0001:00154df0  _zif_dom_element_remove_attribute
0001:00154f8f  _zif_dom_element_set_attribute
0001:0015524b  _zif_dom_element_set_attribute_ns
0001:001558c2  _zif_dom_element_get_attribute_ns
0001:00155a4e  _zif_dom_element_get_attribute
0001:00155bbf  _zif_dom_element_get_attribute_node
0001:00155d72  _dom_element_schema_type_info_read
0001:00155d9a  _dom_element_tag_name_read
0001:00155eac  _zim_domelement___construct
0001:00156300  _php_dom_element_class_functions
Module: U:\dev\php-5.3.20\ext\dom\node.obj(node.obj)
0001:00156a30  _dom_node_text_content_write
0001:00156a4b  _zif_dom_node_get_user_data
0001:00156a72  _zif_dom_node_set_user_data
0001:00156a99  _zif_dom_node_get_feature
0001:00156ac0  _zif_dom_node_is_equal_node
0001:00156ae7  _zif_dom_node_compare_document_position
0001:00156b3b  _zim_domnode_getLineNo
0001:00156bfd  _zim_domnode_getNodePath
0001:00156cea  _zif_dom_node_is_same_node
0001:00156dc8  _zif_dom_node_has_attributes
0001:00157574  _zim_domnode_C14NFile
0001:001575a3  _zim_domnode_C14N
0001:001575d6  _zif_dom_node_lookup_namespace_uri
0001:001576f9  _zif_dom_node_is_default_namespace
0001:0015780f  _zif_dom_node_lookup_prefix
0001:0015798b  _zif_dom_node_is_supported
0001:00157a1d  _zif_dom_node_normalize
0001:00157ae6  _zif_dom_node_clone_node
0001:00157cf7  _zif_dom_node_has_child_nodes
0001:00157dc2  _zif_dom_node_remove_child
0001:0015818e  _zif_dom_node_append_child
0001:00158595  _zif_dom_node_replace_child
0001:001589a0  _zif_dom_node_insert_before
0001:00159088  _dom_node_text_content_read
0001:0015915b  _dom_node_local_name_read
0001:00159208  _dom_node_prefix_read
0001:001592f2  _dom_node_namespace_uri_read
0001:001593cf  _dom_node_owner_document_read
0001:001594bc  _dom_node_next_sibling_read
0001:0015957a  _dom_node_previous_sibling_read
0001:00159643  _dom_node_last_child_read
0001:00159733  _dom_node_first_child_read
0001:00159823  _dom_node_parent_node_read
0001:001598ec  _dom_node_node_type_read
0001:00159967  _dom_node_node_value_read
0001:00159a85  _dom_node_base_uri_read
0001:00159b8d  _dom_node_prefix_write
0001:00159e1b  _dom_node_attributes_read
0001:00159ee9  _dom_node_child_nodes_read
0001:00159fbf  _dom_node_node_value_write
0001:0015a13e  _dom_node_node_name_read
0001:0015a480  _php_dom_node_class_functions
Module: U:\dev\php-5.3.20\ext\dom\string_extend.obj(string_extend.obj)
0001:0015ac44  _zif_dom_string_extend_find_offset32
0001:0015ac6b  _zif_dom_string_extend_find_offset16
0001:0015acb0  _php_dom_string_extend_class_functions
Module: U:\dev\php-5.3.20\ext\dom\characterdata.obj(characterdata.obj)
0001:0015ad87  _zif_dom_characterdata_replace_data
0001:0015afec  _zif_dom_characterdata_delete_data
0001:0015b1e2  _zif_dom_characterdata_insert_data
0001:0015b398  _zif_dom_characterdata_append_data
0001:0015b45f  _zif_dom_characterdata_substring_data
0001:0015b625  _dom_characterdata_length_read
0001:0015b6b0  _dom_characterdata_data_read
0001:0015b788  _dom_characterdata_data_write
0001:0015b8a0  _php_dom_characterdata_class_functions
Module: U:\dev\php-5.3.20\ext\dom\documenttype.obj(documenttype.obj)
0001:0015bab1  _dom_documenttype_internal_subset_read
0001:0015bbd9  _dom_documenttype_system_id_read
0001:0015bc7f  _dom_documenttype_public_id_read
0001:0015bd25  _dom_documenttype_name_read
0001:0015bdaf  _dom_documenttype_notations_read
0001:0015be70  _dom_documenttype_entities_read
0001:0015bf40  _php_dom_documenttype_class_functions
Module: U:\dev\php-5.3.20\ext\dom\domimplementationlist.obj(domimplementationlist.obj)
0001:0015bf74  _zif_dom_domimplementationlist_item
0001:0015bfa0  _dom_domimplementationlist_length_read
0001:0015c000  _php_dom_domimplementationlist_class_functions
Module: U:\dev\php-5.3.20\ext\dom\entity.obj(entity.obj)
0001:0015c060  _dom_entity_actual_encoding_write
0001:0015c067  _dom_entity_encoding_write
0001:0015c06e  _dom_entity_version_write
0001:0015c075  _dom_entity_version_read
0001:0015c09b  _dom_entity_encoding_read
0001:0015c0c1  _dom_entity_actual_encoding_read
0001:0015c0e7  _dom_entity_notation_name_read
0001:0015c19a  _dom_entity_system_id_read
0001:0015c238  _dom_entity_public_id_read
0001:0015c2e0  _php_dom_entity_class_functions
Module: U:\dev\php-5.3.20\ext\dom\nodelist.obj(nodelist.obj)
0001:0015c326  _zif_dom_nodelist_item
0001:0015c560  _dom_nodelist_length_read
0001:0015c6a0  _php_dom_nodelist_class_functions
Module: U:\dev\php-5.3.20\ext\dom\text.obj(text.obj)
0001:0015c714  _zif_dom_text_replace_whole_text
0001:0015c74f  _zif_dom_text_is_whitespace_in_element_content
0001:0015c811  _zif_dom_text_split_text
0001:0015c9fc  _dom_text_whole_text_read
0001:0015cb2f  _zim_domtext___construct
0001:0015ccb0  _php_dom_text_class_functions
Module: U:\dev\php-5.3.20\ext\dom\comment.obj(comment.obj)
0001:0015cdf4  _zim_domcomment___construct
0001:0015cf20  _php_dom_comment_class_functions
Module: U:\dev\php-5.3.20\ext\dom\domconfiguration.obj(domconfiguration.obj)
0001:0015cf94  _zif_dom_domconfiguration_can_set_parameter
0001:0015cfbb  _zif_dom_domconfiguration_get_parameter
0001:0015cfe2  _zif_dom_domconfiguration_set_parameter
0001:0015d040  _php_dom_domconfiguration_class_functions
Module: U:\dev\php-5.3.20\ext\dom\domimplementationsource.obj(domimplementationsource.obj)
0001:0015d184  _zif_dom_domimplementationsource_get_domimplementations
0001:0015d1ab  _zif_dom_domimplementationsource_get_domimplementation
0001:0015d200  _php_dom_domimplementationsource_class_functions
Module: U:\dev\php-5.3.20\ext\dom\entityreference.obj(entityreference.obj)
0001:0015d2b3  _zim_domentityreference___construct
0001:0015d430  _php_dom_entityreference_class_functions
Module: U:\dev\php-5.3.20\ext\dom\notation.obj(notation.obj)
0001:0015d491  _dom_notation_system_id_read
0001:0015d537  _dom_notation_public_id_read
0001:0015d5e0  _php_dom_notation_class_functions
Module: U:\dev\php-5.3.20\ext\dom\xpath.obj(xpath.obj)
0001:0015d61e  _zif_dom_xpath_register_php_functions
0001:0015de72  _zif_dom_xpath_evaluate
0001:0015dea1  _zif_dom_xpath_query
0001:0015ded4  _zif_dom_xpath_register_ns
0001:0015dfd2  _dom_xpath_document_read
0001:0015e0e3  _zim_domxpath___construct
0001:0015ed80  _php_dom_xpath_class_functions
Module: U:\dev\php-5.3.20\ext\dom\dom_iterators.obj(dom_iterators.obj)
0001:0015f0b9  _php_dom_libxml_hash_iter
0001:0015f127  _create_notation
0001:0015f1c8  _php_dom_libxml_notation_iter
0001:0015f481  _php_dom_get_iterator
0002:00001520  _php_dom_iterator_funcs
Module: U:\dev\php-5.3.20\ext\dom\typeinfo.obj(typeinfo.obj)
0001:0015f690  _dom_typeinfo_type_namespace_read
0001:0015f6b6  _dom_typeinfo_type_name_read
0001:0015f6e0  _php_dom_typeinfo_class_functions
Module: U:\dev\php-5.3.20\ext\dom\domerror.obj(domerror.obj)
0001:0015f705  _dom_domerror_location_read
0001:0015f753  _dom_domerror_related_data_read
0001:0015f7a1  _dom_domerror_related_exception_read
0001:0015f7ef  _dom_domerror_type_read
0001:0015f83d  _dom_domerror_message_read
0001:0015f88b  _dom_domerror_severity_read
0001:0015f8e0  _php_dom_domerror_class_functions
Module: U:\dev\php-5.3.20\ext\dom\domlocator.obj(domlocator.obj)
0001:0015f905  _dom_domlocator_uri_read
0001:0015f953  _dom_domlocator_related_node_read
0001:0015f9a1  _dom_domlocator_offset_read
0001:0015f9ef  _dom_domlocator_column_number_read
0001:0015fa3d  _dom_domlocator_line_number_read
0001:0015fa90  _php_dom_domlocator_class_functions
Module: U:\dev\php-5.3.20\ext\dom\namednodemap.obj(namednodemap.obj)
0001:0015fac4  _zif_dom_namednodemap_remove_named_item_ns
0001:0015faeb  _zif_dom_namednodemap_set_named_item_ns
0001:0015fb12  _zif_dom_namednodemap_remove_named_item
0001:0015fb39  _zif_dom_namednodemap_set_named_item
0001:0015fb8a  _zif_dom_namednodemap_get_named_item_ns
0001:0015fd09  _zif_dom_namednodemap_item
0001:0015fe68  _zif_dom_namednodemap_get_named_item
0001:0015ffca  _dom_namednodemap_length_read
0001:001600d0  _php_dom_namednodemap_class_functions
Module: U:\dev\php-5.3.20\ext\dom\userdatahandler.obj(userdatahandler.obj)
0001:00160364  _zif_dom_userdatahandler_handle
0001:001603a0  _php_dom_userdatahandler_class_functions
Module: U:\dev\php-5.3.20\ext\fileinfo\fileinfo.obj(fileinfo.obj)
0002:00020410  _finfo_class_entry
0001:0016041d  _zif_finfo_set_flags
0001:00160cac  _zif_mime_content_type
0001:00160cea  _zif_finfo_buffer
0001:00160d28  _zif_finfo_file
0001:00160d68  _zif_finfo_close
0001:00160e08  _finfo_resource_destructor
0001:00160e7b  _zif_finfo_open
0001:0016111c  _zm_info_fileinfo
0001:0016120a  _zm_startup_finfo
0001:00161506  _finfo_objects_new
0002:00001540  _finfo_class_functions
0002:000015b0  _fileinfo_functions
0002:00001640  _fileinfo_module_entry
Module: U:\dev\php-5.3.20\ext\fileinfo\libmagic\apprentice.obj(apprentice.obj)
0002:00020420  _file_formats
0002:000204d0  _file_names
0001:00161a69  _file_pstring_length_size
0001:00161ac1  _file_pstring_get_length
0001:00161b85  _file_showstr
0001:00162044  _file_signextend
0001:001624bc  _file_delmagic
0001:00166300  _php_magic_database
0001:00166194  _file_apprentice
0001:001662f4  _file_nformats
0001:001662f8  _file_nnames
Module: U:\dev\php-5.3.20\ext\fileinfo\libmagic\ascmagic.obj(ascmagic.obj)
0001:00393396  _file_ascmagic_with_encoding
0001:00393b09  _file_ascmagic
Module: U:\dev\php-5.3.20\ext\fileinfo\libmagic\cdf.obj(cdf.obj)
0001:00393c7c  _cdf_tole2
0001:00393cad  _cdf_tole4
0001:00393ce8  _cdf_tole8
0001:00393d05  _cdf_swap_header
0001:00393f60  _cdf_swap_dir
0001:003940da  _cdf_swap_class
0001:0039416d  _cdf_print_elapsed_time
0001:0039434c  _cdf_print_property_name
0001:003943e5  _cdf_print_classid
0001:00394460  _cdf_count_chain
0001:00394542  _cdf_read_short_sector
0001:00394591  _cdf_unpack_dir
0001:00394621  _cdf_unpack_header
0001:003946e4  _cdf_read_property_info
0001:00394dfa  _cdf_unpack_summary_info
0001:00395035  _cdf_read_short_sector_chain
0001:00395276  _cdf_read_sector
0001:003952ac  _cdf_read_ssat
0001:0039540e  _cdf_read_dir
0001:00395632  _cdf_read_long_sector_chain
0001:003957a9  _cdf_read_short_stream
0001:00395842  _cdf_read_sector_chain
0001:003958b5  _cdf_read_summary_info
0001:003959e0  _cdf_read_sat
0001:00395ce6  _cdf_read_header
Module: U:\dev\php-5.3.20\ext\fileinfo\libmagic\cdf_time.obj(cdf_time.obj)
0001:00395f90  _cdf_timespec_to_timestamp
0001:00395faa  _cdf_ctime
0001:00395ff8  _cdf_timestamp_to_timespec
Module: U:\dev\php-5.3.20\ext\fileinfo\libmagic\compress.obj(compress.obj)
0001:003963dd  _sread
0001:003964ef  _file_pipe2file
Module: U:\dev\php-5.3.20\ext\fileinfo\libmagic\encoding.obj(encoding.obj)
0001:003966b0  _file_looks_utf8
0001:00396921  _file_encoding
Module: U:\dev\php-5.3.20\ext\fileinfo\libmagic\fsmagic.obj(fsmagic.obj)
0001:0039710e  _file_fsmagic
Module: U:\dev\php-5.3.20\ext\fileinfo\libmagic\funcs.obj(funcs.obj)
0001:003974d0  _file_printedlen
0001:003974ef  _file_replace
0001:00397732  _file_check_mem
0001:003977a5  _file_getbuffer
0001:00397889  _file_printf
0001:003979cd  _file_buffer
0001:00397eaa  _file_magerror
0001:00397ecc  _file_error
0001:00397f06  _file_reset
0001:00397f82  _file_badread
0001:00397fb6  _file_badseek
0001:00397ff6  _file_oomem
Module: U:\dev\php-5.3.20\ext\fileinfo\libmagic\is_tar.obj(is_tar.obj)
0001:00398093  _file_is_tar
Module: U:\dev\php-5.3.20\ext\fileinfo\libmagic\magic.obj(magic.obj)
0001:003982e0  _magic_error
0001:003982f3  _magic_errno
0001:00398306  _magic_setflags
0001:00398316  _magic_buffer
0001:00398761  _magic_stream
0001:00398775  _magic_file
0001:00398789  _magic_descriptor
0001:003987eb  _magic_list
0001:0039881e  _magic_compile
0001:00398851  _magic_load
0001:00398890  _magic_close
0001:003988e7  _magic_open
Module: U:\dev\php-5.3.20\ext\fileinfo\libmagic\print.obj(print.obj)
0001:003989b1  _file_fmttime
0001:00398a26  _file_magwarn
Module: U:\dev\php-5.3.20\ext\fileinfo\libmagic\readcdf.obj(readcdf.obj)
0001:00399257  _file_trycdf
Module: U:\dev\php-5.3.20\ext\fileinfo\libmagic\softmagic.obj(softmagic.obj)
0001:00399c1c  _convert_libmagic_pattern
0001:0039cadf  _file_softmagic
Module: U:\dev\php-5.3.20\ext\filter\filter.obj(filter.obj)
0002:00020580  _filter_globals_id
0001:0039d129  _zif_filter_id
0001:0039d1bd  _zif_filter_list
0001:0039d418  _zif_filter_has_var
0001:0039d565  _zm_info_filter
0001:0039d5be  _zm_deactivate_filter
0001:0039d6b5  _zm_shutdown_filter
0001:0039db68  _zm_startup_filter
0001:0039f4a5  _zif_filter_var
0001:0039f589  _zif_filter_input
0001:0039fbe3  _zif_filter_var_array
0001:0039fc95  _zif_filter_input_array
0002:000016a0  _filter_module_entry
Module: U:\dev\php-5.3.20\ext\filter\sanitizing_filters.obj(sanitizing_filters.obj)
0001:003a0490  _php_filter_magic_quotes
0001:003a05a2  _php_filter_number_float
0001:003a064e  _php_filter_number_int
0001:003a0707  _php_filter_url
0001:003a07dd  _php_filter_email
0001:003a0976  _php_filter_encoded
0001:003a0d83  _php_filter_special_chars
0001:003a0e1a  _php_filter_unsafe_raw
0001:003a0eec  _php_filter_full_special_chars
0001:003a0f68  _php_filter_string
Module: U:\dev\php-5.3.20\ext\filter\logical_filters.obj(logical_filters.obj)
0001:003a1216  _php_filter_validate_url
0001:003a1825  _php_filter_validate_email
0001:003a199e  _php_filter_validate_regexp
0001:003a1bff  _php_filter_int
0001:003a21a9  _php_filter_validate_ip
0001:003a27cd  _php_filter_float
0001:003a2e6e  _php_filter_boolean
Module: U:\dev\php-5.3.20\ext\filter\callback_filter.obj(callback_filter.obj)
0001:003a3082  _php_filter_callback
Module: U:\dev\php-5.3.20\ext\ftp\php_ftp.obj(php_ftp.obj)
0001:003a3273  _zif_ftp_get_option
0001:003a33f0  _zif_ftp_set_option
0001:003a3579  _zif_ftp_close
0001:003a362b  _zif_ftp_site
0001:003a3707  _zif_ftp_delete
0001:003a37e7  _zif_ftp_rename
0001:003a38d8  _zif_ftp_mdtm
0001:003a3980  _zif_ftp_size
0001:003a3a5b  _zif_ftp_nb_put
0001:003a3cc1  _zif_ftp_put
0001:003a3f35  _zif_ftp_nb_fput
0001:003a41ad  _zif_ftp_fput
0001:003a4426  _zif_ftp_nb_continue
0001:003a459b  _zif_ftp_nb_fget
0001:003a4824  _zif_ftp_nb_get
0001:003a4b8c  _zif_ftp_get
0001:003a4edb  _zif_ftp_fget
0001:003a5122  _zif_ftp_pasv
0001:003a51d1  _zif_ftp_systype
0001:003a52ba  _zif_ftp_rawlist
0001:003a53ba  _zif_ftp_nlist
0001:003a54ac  _zif_ftp_alloc
0001:003a55c1  _zif_ftp_chmod
0001:003a56b5  _zif_ftp_rmdir
0001:003a5791  _zif_ftp_mkdir
0001:003a587e  _zif_ftp_raw
0001:003a5924  _zif_ftp_exec
0001:003a5a00  _zif_ftp_chdir
0001:003a5adc  _zif_ftp_cdup
0001:003a5ba3  _zif_ftp_pwd
0001:003a5c87  _zif_ftp_login
0001:003a5d81  _zif_ftp_ssl_connect
0001:003a5e6e  _zif_ftp_connect
0001:003a5f6f  _zm_info_ftp
0001:003a6015  _zm_startup_ftp
0001:003a6390  _php_ftp_functions
0002:00001700  _php_ftp_module_entry
Module: U:\dev\php-5.3.20\ext\ftp\ftp.obj(ftp.obj)
0001:003a742b  _ftp_gc
0001:003a7477  _ftp_close
0001:003a7a03  _data_writeable
0001:003a7a62  _data_available
0001:003a7dcb  _ftp_nb_continue_write
0001:003a7f9b  _ftp_site
0001:003a7ff7  _ftp_rename
0001:003a806b  _ftp_delete
0001:003a80b8  _ftp_rmdir
0001:003a8106  _ftp_cdup
0001:003a816e  _ftp_chdir
0001:003a81dd  _ftp_exec
0001:003a822b  _ftp_reinit
0001:003a828a  _ftp_quit
0001:003a8375  _ftp_login
0001:003a8621  _ftp_mdtm
0001:003a875d  _ftp_size
0001:003a87dc  _ftp_pasv
0001:003a8db1  _ftp_nb_put
0001:003a8ec9  _ftp_put
0001:003a90e0  _ftp_alloc
0001:003a9178  _ftp_chmod
0001:003a9214  _ftp_syst
0001:003a92be  _ftp_mkdir
0001:003a9357  _ftp_pwd
0001:003a940b  _ftp_open
0001:003a9568  _ftp_raw
0001:003a9669  _ftp_nb_continue_read
0001:003a9851  _ftp_nb_get
0001:003a9969  _ftp_get
0001:003a9f25  _ftp_list
0001:003a9f57  _ftp_nlist
Module: U:\dev\php-5.3.20\ext\hash\hash.obj(hash.obj)
0002:00020590  _php_hash_hashtable
0001:003a9fa9  _zm_info_hash
0001:003aa086  _zm_shutdown_hash
0001:003aa11a  _zif_hash_algos
0001:003aa1c9  _zif_hash_update
0001:003aa27f  _php_hash_copy
0001:003aa2a7  _zif_hash_copy
0001:003aa3dc  _zif_hash_final
0001:003aa638  _zif_hash_update_file
0001:003aa80b  _zif_hash_update_stream
0001:003aa9b7  _php_hash_register_algo
0001:003aabc3  _zm_startup_hash
0001:003aaf9d  _php_hash_fetch_ops
0001:003ab040  _zif_hash_init
0001:003ab62e  _zif_hash_hmac
0001:003ab64a  _zif_hash_hmac_file
0001:003ab90e  _zif_hash
0001:003ab92a  _zif_hash_file
0001:003ab9d0  _hash_functions
0002:00001760  _hash_module_entry
Module: U:\dev\php-5.3.20\ext\hash\hash_md.obj(hash_md.obj)
0001:003ac3ff  _PHP_MD4Init
0001:003ac4a3  _PHP_MD2Init
0001:003ac4ea  _PHP_MD2Final
0001:003ac54b  _PHP_MD2Update
0001:003ac64f  _PHP_MD4Update
0001:003ac724  _PHP_MD4Final
0001:003ac7f0  _php_hash_md5_ops
0001:003ac810  _php_hash_md4_ops
0001:003ac830  _php_hash_md2_ops
Module: U:\dev\php-5.3.20\ext\hash\hash_sha.obj(hash_sha.obj)
0001:003ac990  _PHP_SHA256Init
0001:003ac9dd  _PHP_SHA224Init
0001:003acabb  _PHP_SHA384Init
0001:003acb4e  _PHP_SHA512Init
0001:003ad5f4  _PHP_SHA512Update
0001:003ad6eb  _PHP_SHA512Final
0001:003ad823  _PHP_SHA384Update
0001:003ad91a  _PHP_SHA384Final
0001:003ada52  _PHP_SHA256Update
0001:003adb27  _PHP_SHA256Final
0001:003adbf3  _PHP_SHA224Update
0001:003adcc8  _PHP_SHA224Final
0001:003adda0  _php_hash_sha1_ops
0001:003addc0  _php_hash_sha256_ops
0001:003adde0  _php_hash_sha224_ops
0001:003ade00  _php_hash_sha384_ops
0001:003ade20  _php_hash_sha512_ops
Module: U:\dev\php-5.3.20\ext\hash\hash_ripemd.obj(hash_ripemd.obj)
0001:003ae3c0  _PHP_RIPEMD128Init
0001:003ae3f1  _PHP_RIPEMD256Init
0001:003ae43e  _PHP_RIPEMD160Init
0001:003ae476  _PHP_RIPEMD320Init
0001:003af3ce  _PHP_RIPEMD320Update
0001:003af4a3  _PHP_RIPEMD320Final
0001:003af54f  _PHP_RIPEMD160Update
0001:003af624  _PHP_RIPEMD160Final
0001:003af6d0  _PHP_RIPEMD256Update
0001:003af7a5  _PHP_RIPEMD256Final
0001:003af851  _PHP_RIPEMD128Update
0001:003af926  _PHP_RIPEMD128Final
0001:003af9e0  _php_hash_ripemd128_ops
0001:003afa00  _php_hash_ripemd160_ops
0001:003afa20  _php_hash_ripemd256_ops
0001:003afa40  _php_hash_ripemd320_ops
Module: U:\dev\php-5.3.20\ext\hash\hash_haval.obj(hash_haval.obj)
0001:003afc1a  _PHP_3HAVAL128Init
0001:003afc5e  _PHP_3HAVAL160Init
0001:003afca2  _PHP_3HAVAL192Init
0001:003afce6  _PHP_3HAVAL224Init
0001:003afd2a  _PHP_3HAVAL256Init
0001:003afd6e  _PHP_4HAVAL128Init
0001:003afdb2  _PHP_4HAVAL160Init
0001:003afdf6  _PHP_4HAVAL192Init
0001:003afe3a  _PHP_4HAVAL224Init
0001:003afe7e  _PHP_4HAVAL256Init
0001:003afec2  _PHP_5HAVAL128Init
0001:003aff06  _PHP_5HAVAL160Init
0001:003aff4a  _PHP_5HAVAL192Init
0001:003aff8e  _PHP_5HAVAL224Init
0001:003affd2  _PHP_5HAVAL256Init
0001:003b0d17  _PHP_HAVALUpdate
0001:003b0df3  _PHP_HAVAL256Final
0001:003b0e98  _PHP_HAVAL224Final
0001:003b0f84  _PHP_HAVAL192Final
0001:003b10b1  _PHP_HAVAL160Final
0001:003b11f5  _PHP_HAVAL128Final
0001:003b1350  _php_hash_3haval128_ops
0001:003b1370  _php_hash_3haval160_ops
0001:003b1390  _php_hash_3haval192_ops
0001:003b13b0  _php_hash_3haval224_ops
0001:003b13d0  _php_hash_3haval256_ops
0001:003b13f0  _php_hash_4haval128_ops
0001:003b1410  _php_hash_4haval160_ops
0001:003b1430  _php_hash_4haval192_ops
0001:003b1450  _php_hash_4haval224_ops
0001:003b1470  _php_hash_4haval256_ops
0001:003b1490  _php_hash_5haval128_ops
0001:003b14b0  _php_hash_5haval160_ops
0001:003b14d0  _php_hash_5haval192_ops
0001:003b14f0  _php_hash_5haval224_ops
0001:003b1510  _php_hash_5haval256_ops
Module: U:\dev\php-5.3.20\ext\hash\hash_tiger.obj(hash_tiger.obj)
0001:003b1ad0  _PHP_4TIGERInit
0001:003b1b12  _PHP_3TIGERInit
0001:003b6f18  _PHP_TIGER192Final
0001:003b7035  _PHP_TIGER160Final
0001:003b711c  _PHP_TIGER128Final
0001:003b71e6  _PHP_TIGERUpdate
0001:003bd1e0  _php_hash_3tiger128_ops
0001:003bd200  _php_hash_3tiger160_ops
0001:003bd220  _php_hash_3tiger192_ops
0001:003bd240  _php_hash_4tiger128_ops
0001:003bd260  _php_hash_4tiger160_ops
0001:003bd280  _php_hash_4tiger192_ops
Module: U:\dev\php-5.3.20\ext\hash\hash_gost.obj(hash_gost.obj)
0001:003c04fa  _PHP_GOSTInit
0001:003c050f  _PHP_GOSTUpdate
0001:003c0723  _PHP_GOSTFinal
0001:003c0830  _php_hash_gost_ops
Module: U:\dev\php-5.3.20\ext\hash\hash_snefru.obj(hash_snefru.obj)
0001:003c1850  _PHP_SNEFRUInit
0001:003c1865  _PHP_SNEFRUUpdate
0001:003c22c8  _PHP_SNEFRUFinal
0001:003c2b00  _php_hash_snefru_ops
Module: U:\dev\php-5.3.20\ext\hash\hash_whirlpool.obj(hash_whirlpool.obj)
0001:003c8475  _PHP_WHIRLPOOLUpdate
0001:003c8698  _PHP_WHIRLPOOLInit
0001:003c86ad  _PHP_WHIRLPOOLFinal
0001:003c8800  _php_hash_whirlpool_ops
Module: U:\dev\php-5.3.20\ext\hash\hash_adler32.obj(hash_adler32.obj)
0001:003cc880  _PHP_ADLER32Init
0001:003cc88e  _PHP_ADLER32Update
0001:003cc90b  _PHP_ADLER32Final
0001:003cc936  _PHP_ADLER32Copy
0001:003cc950  _php_hash_adler32_ops
Module: U:\dev\php-5.3.20\ext\hash\hash_crc32.obj(hash_crc32.obj)
0001:003cc970  _PHP_CRC32Init
0001:003cc97e  _PHP_CRC32Update
0001:003cc9bb  _PHP_CRC32BUpdate
0001:003cc9f4  _PHP_CRC32Final
0001:003cca24  _PHP_CRC32BFinal
0001:003cca54  _PHP_CRC32Copy
0001:003cca70  _php_hash_crc32_ops
0001:003cca90  _php_hash_crc32b_ops
Module: U:\dev\php-5.3.20\ext\hash\hash_salsa.obj(hash_salsa.obj)
0001:003cd81f  _PHP_SALSA20Init
0001:003cd83e  _PHP_SALSA10Init
0001:003cd85d  _PHP_SALSAUpdate
0001:003cda98  _PHP_SALSAFinal
0001:003cdb60  _php_hash_salsa10_ops
0001:003cdb80  _php_hash_salsa20_ops
Module: U:\dev\php-5.3.20\ext\json\json.obj(json.obj)
0002:000205c0  _json_globals_id
0001:003cf951  _php_json_encode
0001:003d0b20  _php_json_decode
0002:000017c0  _json_module_entry
Module: U:\dev\php-5.3.20\ext\json\utf8_to_utf16.obj(utf8_to_utf16.obj)
0001:003d12c0  _utf8_to_utf16
Module: U:\dev\php-5.3.20\ext\json\utf8_decode.obj(utf8_decode.obj)
0001:003d1350  _utf8_decode_init
0001:003d1378  _utf8_decode_at_byte
0001:003d1383  _utf8_decode_at_character
0001:003d1397  _utf8_decode_next
Module: U:\dev\php-5.3.20\ext\json\JSON_parser.obj(JSON_parser.obj)
0001:003d15f0  _free_JSON_parser
0001:003d1e42  _parse_JSON
0001:003d2e94  _new_JSON_parser
Module: U:\dev\php-5.3.20\ext\pdo\pdo.obj(pdo.obj)
0002:000205d0  _pdo_dbh_ce
0002:000205e0  _pdo_exception_ce
0002:000205f0  _pdo_driver_hash
0002:00020620  _pdo_globals_id
0002:00020630  _pdo_dbstmt_ce
0002:00020640  _pdo_row_ce
0001:003d3fe0  _php_pdo_list_entry
0001:003d3fea  _php_pdo_get_dbh_ce
0001:003d3ff4  _php_pdo_get_exception
0001:003d400c  _php_pdo_int64_to_str
0001:003d41ef  _zm_info_pdo
0001:003d42fb  _zm_shutdown_pdo
0001:003d4316  _php_pdo_parse_data_source
0001:003d4533  _pdo_find_driver
0001:003d4572  _php_pdo_unregister_driver
0001:003d4641  _php_pdo_register_driver
0001:003d46fa  _zif_pdo_drivers
0001:003d47b0  _php_pdo_get_exception_base
0001:003d484e  _zm_startup_pdo
0001:003d4a1b  _php_pdo_str_tolower_dup
0001:003d4a60  _pdo_functions
0002:00001820  _pdo_module_entry
Module: U:\dev\php-5.3.20\ext\pdo\pdo_dbh.obj(pdo_dbh.obj)
0001:003d4afa  _php_pdo_dbh_addref
0001:003d4fab  _php_pdo_pdbh_dtor
0001:003d5054  _php_pdo_dbh_delref
0001:003d5066  _pdo_dbh_new
0001:003d5567  _pdo_dbh_init
0001:003d9c00  _pdo_dbh_functions
0001:003d6242  _pdo_handle_error
0001:003d6573  _pdo_raise_impl_error
0001:003d9790  _pdo_hash_methods
Module: U:\dev\php-5.3.20\ext\pdo\pdo_stmt.obj(pdo_stmt.obj)
0002:00020650  _pdo_dbstmt_object_handlers
0001:003da00a  _php_pdo_stmt_addref
0001:003dbb1b  _pdo_row_new
0001:003dcb53  _pdo_row_free_storage
0001:003dcbc1  _php_pdo_stmt_delref
0001:003dcbe2  _pdo_dbstmt_free_storage
0001:003dcbeb  _pdo_stmt_describe_columns
0001:003dcfa6  _pdo_dbstmt_new
0001:003dd1ae  _pdo_stmt_init
0001:003e0240  _pdo_dbstmt_functions
0001:003df075  _pdo_stmt_iter_get
0001:003e0400  _pdo_row_functions
0001:003dd6e9  _pdo_stmt_setup_fetch_mode
0002:00001880  _pdo_row_object_handlers
Module: U:\dev\php-5.3.20\ext\pdo\pdo_sql_parser.obj(pdo_sql_parser.obj)
0001:003e09c2  _pdo_parse_params
Module: U:\dev\php-5.3.20\ext\pdo\pdo_sqlstate.obj(pdo_sqlstate.obj)
0001:003e1a10  _pdo_sqlstate_state_to_description
0001:003e1a4a  _pdo_sqlstate_init_error_table
0001:003e1aeb  _pdo_sqlstate_fini_error_table
Module: U:\dev\php-5.3.20\ext\phar\util.obj(util.obj)
0001:003e4458  _phar_compress_filter
0001:003e44b1  _phar_decompress_filter
0001:003e44f7  _phar_free_alias
0001:003e4588  _phar_copy_on_write
0001:003e4ab4  _phar_add_virtual_dirs
0001:003e4c1c  _phar_create_writeable_entry
0001:003e4d0c  _phar_open_archive_fp
0001:003e4e4b  _phar_mount_entry
0001:003e5349  _phar_get_entry_info_dir
0001:003e58eb  _phar_get_entry_info
0001:003e592f  _phar_get_link_source
0001:003e5a58  _phar_get_efp
0001:003e5c20  _phar_seek_efp
0001:003e61bb  _phar_create_signature
0001:003e6644  _phar_verify_signature
0001:003e6d0b  _phar_get_archive
0001:003e779f  _phar_find_in_include_path
0001:003e7d7d  _phar_open_entry_fp
0001:003e85bb  _phar_open_jit
0001:003e86cf  _phar_separate_entry_fp
0001:003e889a  _phar_copy_entry_fp
0001:003e8bf5  _phar_get_entry_data
0001:003e9296  _phar_get_or_create_entry_data
Module: U:\dev\php-5.3.20\ext\phar\tar.obj(tar.obj)
0001:003ea0ed  _phar_tar_setmetadata
0001:003ea66b  _phar_tar_flush
0001:003ec01f  _phar_parse_tarfile
0001:003ed8c6  _phar_open_or_create_tar
0001:003ed99e  _phar_is_tar
Module: U:\dev\php-5.3.20\ext\phar\zip.obj(zip.obj)
0001:003ef4b0  _phar_zip_flush
0001:003f08ef  _phar_open_or_create_zip
0001:003f13b7  _phar_parse_zipfile
Module: U:\dev\php-5.3.20\ext\phar\stream.obj(stream.obj)
0001:003f541e  _phar_dostat
0001:003f56c0  _phar_parse_url
0002:00001910  _phar_ops
0002:00001940  _phar_stream_wops
0002:00001970  _php_stream_phar_wrapper
Module: U:\dev\php-5.3.20\ext\phar\func_interceptors.obj(func_interceptors.obj)
0001:003f7e50  _phar_intercept_functions
0001:003f7e89  _phar_release_functions
0001:003f7ea4  _phar_save_orig_functions
0001:003f7fbf  _phar_restore_orig_functions
0001:003f81a8  _phar_intercept_functions_shutdown
0001:003f8b8d  _phar_intercept_functions_init
0001:003fc65e  _phar_is_dir
0001:003fc728  _phar_file_exists
0001:003fd0a0  _phar_fileperms
0001:003fcfd6  _phar_fileinode
0001:003fcf0c  _phar_filesize
0001:003fce42  _phar_fileowner
0001:003fcd78  _phar_filegroup
0001:003fccae  _phar_fileatime
0001:003fcbe4  _phar_filemtime
0001:003fcb1a  _phar_filectime
0001:003fca50  _phar_filetype
0001:003fc986  _phar_is_writable
0001:003fc8bc  _phar_is_readable
0001:003fc7f2  _phar_is_executable
0001:003fc594  _phar_lstat
0001:003fc4ca  _phar_stat
Module: U:\dev\php-5.3.20\ext\phar\dirstream.obj(dirstream.obj)
0001:003fd564  _phar_wrapper_rmdir
0001:003fdd89  _phar_wrapper_mkdir
0001:003fe8d1  _phar_wrapper_open_dir
0002:00001990  _phar_dir_ops
Module: U:\dev\php-5.3.20\ext\phar\phar.obj(phar.obj)
0002:000206c0  _phar_globals_id
0002:000206d0  _cached_phars
0002:00020700  _cached_alias
0002:00020730  _phar_orig_compile_file
0002:00020740  _phar_save_resolve_path
0001:003fed9f  _zm_globals_dtor_phar
0001:003fedfe  _zm_deactivate_phar
0001:003fefea  _phar_request_initialize
0001:003ff485  _zm_info_phar
0001:003ff751  _zm_shutdown_phar
0001:003ff8b3  _phar_create_default_stub
0001:003ffa86  _zm_startup_phar
0001:003ffcd2  _zm_globals_ctor_phar
0001:00400d65  _phar_flush
0001:00402e8f  _phar_postprocess_file
0001:004033c5  _phar_fix_filepath
0001:00403acb  _phar_detect_phar_fname_ext
0001:004040d7  _phar_split_fname
0001:00404220  _phar_parse_metadata
0001:004043e6  _phar_open_parsed_phar
0001:0040454d  _destroy_phar_manifest_entry
0001:004046a5  _phar_destroy_phar_data
0001:004083fd  _phar_open_executed_filename
0001:004086b3  _phar_open_from_filename
0001:00408ce2  _phar_create_or_parse_filename
0001:004093f1  _phar_open_or_create_filename
0001:004097da  _phar_archive_delref
0001:0040991b  _phar_entry_delref
0001:004099c2  _phar_entry_remove
0001:00409aa0  _phar_ini_cache_list
0001:00409fd2  _phar_ini_modify_handler
0002:000019c0  _phar_module_entry
0002:00009bc0  _phar_functions
Module: U:\dev\php-5.3.20\ext\phar\phar_object.obj(phar_object.obj)
0001:0040c297  _phar_object_init
0001:0040c96f  _zim_Phar_hasMetadata
0001:0040ca14  _zim_PharFileInfo_hasMetadata
0001:0040ca9e  _zim_PharFileInfo_getPharFlags
0001:0040cb25  _zim_PharFileInfo_isCRCChecked
0001:0040cbfb  _zim_PharFileInfo_getCRC32
0001:0040ccc7  _zim_PharFileInfo_isCompressed
0001:0040cdb9  _zim_PharFileInfo_getCompressedSize
0001:0040ce3b  _zim_Phar_getModified
0001:0040cec6  _zim_Phar_isBuffering
0001:0040cf52  _zim_Phar_startBuffering
0001:0040cfc9  _zim_Phar_isCompressed
0001:0040d0a4  _zim_Phar_isFileFormat
0001:0040d1c6  _zim_Phar_canWrite
0001:0040d3ab  _zim_PharFileInfo_decompress
0001:0040d726  _zim_PharFileInfo_chmod
0001:0040d9d2  _zim_PharFileInfo___destruct
0001:0040da5d  _zim_Phar_stopBuffering
0001:0040dea9  _zim_PharFileInfo_compress
0001:0040e366  _zim_PharFileInfo_getContent
0001:0040e588  _zim_Phar_getPath
0001:0040e61b  _zim_Phar_getAlias
0001:0040e6bd  _zim_Phar_apiVersion
0001:0040e7b1  _zim_PharFileInfo_delMetadata
0001:0040e9af  _zim_Phar_delMetadata
0001:0040ebeb  _zim_PharFileInfo___construct
0001:0040ef1a  _zim_Phar_isWritable
0001:0040f00f  _zim_Phar_count
0001:0040fc79  _zim_Phar_extractTo
0001:00410243  _zim_Phar_getStub
0001:004109c0  _zim_Phar_addFromString
0001:00410b16  _zim_Phar_addEmptyDir
0001:00410e40  _zim_Phar_addFile
0001:0041104f  _zim_Phar_offsetUnset
0001:0041125e  _zim_Phar_offsetExists
0001:004113b6  _zim_Phar_delete
0001:004116c7  _zim_Phar_offsetSet
0001:00411942  _zim_Phar_setSignatureAlgorithm
0001:00411c05  _zim_Phar_setStub
0001:00411fe1  _zim_Phar_offsetGet
0001:0041230a  _zim_Phar_getVersion
0001:00412558  _zim_Phar_copy
0001:00412bd5  _zim_Phar_decompressFiles
0001:00412f8f  _zim_Phar_compressFiles
0001:004131f0  _zim_Phar_isValidPharFilename
0001:004132be  _zim_Phar_getSignature
0001:004135c4  _zim_Phar_setDefaultStub
0001:004138e2  _zim_Phar_createDefaultStub
0001:004139b9  _zim_Phar___destruct
0001:00413b03  _zim_Phar_setAlias
0001:00414170  _zim_Phar_buildFromIterator
0001:00414468  _zim_Phar_buildFromDirectory
0001:0041579a  _zim_Phar_running
0001:00415a51  _zim_Phar_unlinkArchive
0001:00415d47  _zim_Phar_canCompress
0001:00415e17  _zim_Phar_loadPhar
0001:00415f04  _zim_Phar_getSupportedCompression
0001:00415fd0  _zim_Phar_getSupportedSignatures
0001:004161a2  _zim_Phar___construct
0001:004166ac  _zim_Phar_mapPhar
0001:00416771  _zim_Phar_interceptFileFuncs
0001:004169bc  _zim_Phar_mungServer
0001:00417ede  _zim_Phar_webPhar
0001:0041902f  _zim_Phar_mount
0001:0041a8bd  _zim_Phar_setMetadata
0001:0041ab72  _zim_PharFileInfo_setMetadata
0001:0041addf  _zim_PharFileInfo_getMetadata
0001:0041af1b  _zim_Phar_getMetadata
0001:0041b0e0  _zim_Phar_decompress
0001:0041b387  _zim_Phar_compress
0001:0041b6e3  _zim_Phar_convertToExecutable
0001:0041ba41  _zim_Phar_convertToData
0002:00001a20  _php_archive_methods
0002:00001ea0  _php_entry_methods
0002:00009be0  _phar_exception_methods
Module: U:\dev\php-5.3.20\ext\phar\phar_path_check.obj(phar_path_check.obj)
0001:0041cb35  _phar_path_check
Module: U:\dev\php-5.3.20\ext\posix\posix.obj(posix.obj)
0002:00020750  _posix_globals_id
0001:0041cfad  _zif_posix_get_last_error
0001:0041cff5  _zif_posix_initgroups
0001:0041d072  _zif_posix_strerror
0001:0041d107  _zif_posix_getrlimit
0001:0041d346  _php_posix_passwd_to_array
0001:0041d4a7  _zif_posix_getpwuid
0001:0041d5ce  _zif_posix_getpwnam
0001:0041d704  _zif_posix_access
0001:0041d880  _php_posix_group_to_array
0001:0041d9ea  _zif_posix_getgrgid
0001:0041db37  _zif_posix_getgrnam
0001:0041dd02  _zif_posix_mknod
0001:0041de96  _zif_posix_mkfifo
0001:0041df87  _zif_posix_getcwd
0001:0041e1ec  _zif_posix_isatty
0001:0041e2fe  _zif_posix_ttyname
0001:0041e469  _zif_posix_times
0001:0041e5ae  _zif_posix_uname
0001:0041e6ef  _zif_posix_getsid
0001:0041e765  _zif_posix_getpgid
0001:0041e7de  _zif_posix_setpgid
0001:0041e863  _zif_posix_setsid
0001:0041e89d  _zif_posix_getpgrp
0001:0041e8d7  _zif_posix_getlogin
0001:0041e95b  _zif_posix_getgroups
0001:0041ea0c  _zif_posix_setegid
0001:0041ea83  _zif_posix_seteuid
0001:0041eafa  _zif_posix_setgid
0001:0041eb71  _zif_posix_setuid
0001:0041ebe8  _zif_posix_getegid
0001:0041ec22  _zif_posix_geteuid
0001:0041ec5c  _zif_posix_getgid
0001:0041ec96  _zif_posix_getuid
0001:0041ecd0  _zif_posix_getppid
0001:0041ed0a  _zif_posix_getpid
0001:0041ed44  _zif_posix_kill
0001:0041efc0  _posix_functions
0002:00002050  _limits
0002:00001ff0  _posix_module_entry
Module: U:\dev\php-5.3.20\ext\reflection\php_reflection.obj(php_reflection.obj)
0002:00020760  _reflection_exception_ptr
0002:00020770  _reflection_ptr
0002:00020780  _reflector_ptr
0002:00020790  _reflection_function_abstract_ptr
0002:000207a0  _reflection_function_ptr
0002:000207b0  _reflection_parameter_ptr
0002:000207c0  _reflection_method_ptr
0002:000207d0  _reflection_class_ptr
0002:000207e0  _reflection_object_ptr
0002:000207f0  _reflection_property_ptr
0002:00020800  _reflection_extension_ptr
0001:0041fa04  _zm_info_reflection
0001:0041fbce  _zm_startup_reflection
0001:00420de3  _zim_reflection_property_setAccessible
0001:00420e3c  _zim_reflection_method_setAccessible
0001:00420ed1  _zim_reflection_property_getModifiers
0001:00421024  _zim_reflection_property_isDefault
0001:00421053  _zim_reflection_property_isStatic
0001:00421082  _zim_reflection_property_isProtected
0001:004210b1  _zim_reflection_property_isPrivate
0001:004210e0  _zim_reflection_property_isPublic
0001:0042110f  _zim_reflection_class_getModifiers
0001:00421262  _zim_reflection_class_isAbstract
0001:00421291  _zim_reflection_class_isFinal
0001:004212c0  _zim_reflection_class_isInterface
0001:004212ef  _zim_reflection_class_isInstantiable
0001:004213d8  _zim_reflection_class_getEndLine
0001:0042149e  _zim_reflection_class_getStartLine
0001:00421564  _zim_reflection_class_isUserDefined
0001:00421611  _zim_reflection_class_isInternal
0001:004216be  _zim_reflection_method_getModifiers
0001:00421765  _zim_reflection_method_isDestructor
0001:00421812  _zim_reflection_method_isConstructor
0001:00421994  _zim_reflection_function_isDeprecated
0001:004219c3  _zim_reflection_method_isStatic
0001:004219f2  _zim_reflection_method_isProtected
0001:00421a21  _zim_reflection_method_isPrivate
0001:00421a50  _zim_reflection_method_isPublic
0001:00421a7f  _zim_reflection_method_isAbstract
0001:00421aae  _zim_reflection_method_isFinal
0001:00421add  _zim_reflection_parameter_isDefaultValueAvailable
0001:00421bf0  _zim_reflection_parameter_isOptional
0001:00421c9f  _zim_reflection_parameter_getPosition
0001:00421d45  _zim_reflection_parameter_isPassedByReference
0001:00421df6  _zim_reflection_parameter_allowsNull
0001:00421ea7  _zim_reflection_parameter_isArray
0001:00421f58  _zim_reflection_function_getEndLine
0001:0042201b  _zim_reflection_function_getStartLine
0001:004220de  _zim_reflection_function_isUserDefined
0001:0042218b  _zim_reflection_function_isInternal
0001:00422238  _zim_reflection_function_isClosure
0001:004222e5  _zim_reflection_extension_info
0001:004223a2  _zim_reflection_extension_getDependencies
0001:00422536  _zim_reflection_extension_getClassNames
0001:0042262b  _zim_reflection_extension_getClasses
0001:00422720  _zim_reflection_extension_getINIEntries
0001:00422812  _zim_reflection_extension_getConstants
0001:00422932  _zim_reflection_class_getInterfaceNames
0001:00422a5a  _zim_reflection_getModifierNames
0001:00422cb7  _zim_reflection_class_inNamespace
0001:00422d66  _zim_reflection_function_inNamespace
0001:00422e16  _zim_reflection_extension_getVersion
0001:00422ef7  _zim_reflection_property_getDocComment
0001:00422fd1  _zim_reflection_class_getNamespaceName
0001:004230be  _zim_reflection_class_getDocComment
0001:004231a4  _zim_reflection_class_getFileName
0001:00423281  _zim_reflection_function_getNamespaceName
0001:0042336e  _zim_reflection_function_getDocComment
0001:0042344b  _zim_reflection_function_getFileName
0001:004236bf  _zim_reflection_extension_getFunctions
0001:00423a08  _zim_reflection_class_getConstructor
0001:00423add  _zend_reflection_class_factory
0001:00423c6a  _zim_reflection_class_getParentClass
0001:00423d35  _zim_reflection_class_getInterfaces
0001:00423e78  _zim_reflection_parameter_getDeclaringClass
0001:0042401d  _zim_reflection_parameter_getDefaultValue
0001:0042445f  _zim_reflection_class_getConstants
0001:00424565  _zim_reflection_function_getStaticVariables
0001:00424825  _zim_reflection_property___toString
0001:004248ff  _zim_reflection_property_getDeclaringClass
0001:00424cdf  _zim_reflection_extension___construct
0001:0042506c  _zim_reflection___clone
0001:0042544d  _zim_reflection_extension_export
0001:0042548d  _zim_reflection_property_export
0001:004254cd  _zim_reflection_object_export
0001:0042550d  _zim_reflection_class_export
0001:0042554d  _zim_reflection_method_export
0001:0042558d  _zim_reflection_parameter_export
0001:004255cd  _zim_reflection_function_export
0001:00425631  _zim_reflection_class_getExtensionName
0001:00425779  _zim_reflection_class_getExtension
0001:00425897  _zim_reflection_class_isIterateable
0001:00425a57  _zim_reflection_class_newInstance
0001:00425d32  _zim_reflection_class_isInstance
0001:00425e79  _zim_reflection_class_hasConstant
0001:00425fcb  _zim_reflection_class_getProperties
0001:00426198  _zim_reflection_class_hasProperty
0001:004263ab  _zim_reflection_class_getMethod
0001:004266b4  _zim_reflection_class_hasMethod
0001:0042688c  _zim_reflection_method_getPrototype
0001:004269e4  _zim_reflection_method_getDeclaringClass
0001:00426bf5  _zim_reflection_method_invoke
0001:00426fbb  _zim_reflection_function_getExtensionName
0001:004270df  _zim_reflection_function_getExtension
0001:004271e3  _zim_reflection_function_getNumberOfRequiredParameters
0001:004272cd  _zim_reflection_function_getNumberOfParameters
0001:004273b7  _zim_reflection_function_returnsReference
0001:004274cb  _zim_reflection_function_invoke
0001:00427741  _zim_reflection_function_isDisabled
0001:004278c0  _zim_reflection_property___construct
0001:00427e7a  _zim_reflection_class_implementsInterface
0001:004280bf  _zim_reflection_class_isSubclassOf
0001:004282fa  _zim_reflection_class_newInstanceArgs
0001:00428615  _zim_reflection_function_invokeArgs
0001:00428abb  _zim_reflection_class_getMethods
0001:00428d60  _zim_reflection_class_getProperty
0001:00429123  _zim_reflection_method___construct
0001:0042962a  _zim_reflection_method_invokeArgs
0001:00429a52  _zim_reflection_parameter_getDeclaringFunction
0001:00429b4b  _zim_reflection_function_getParameters
0001:00429eac  _zim_reflection_parameter_getClass
0001:0042a1b7  _zim_reflection_parameter___construct
0001:0042a965  _zim_reflection_function___construct
0001:0042ac70  _zim_reflection_class_getDefaultProperties
0001:0042aeec  _zim_reflection_class_getStaticProperties
0001:0042b1cf  _zim_reflection_class_setStaticPropertyValue
0001:0042b348  _zim_reflection_class_getShortName
0001:0042b456  _zim_reflection_function_getShortName
0001:0042b646  _zim_reflection_property_setValue
0001:0042ba2a  _zim_reflection_function_getName
0001:0042ba72  _zim_reflection_parameter_getName
0001:0042baba  _zim_reflection_class_getName
0001:0042bb02  _zim_reflection_property_getName
0001:0042bb4a  _zim_reflection_extension_getName
0001:0042bbfb  _zim_reflection_export
0001:0042be7d  _zim_reflection_class_getStaticPropertyValue
0001:0042c000  _zim_reflection_property_getValue
0001:0042c351  _zim_reflection_class_getConstant
0001:0042cfc4  _zim_reflection_method___toString
0001:0042d0a9  _zim_reflection_function___toString
0001:0042dec5  _zim_reflection_class___toString
0001:0042e0a2  _zim_reflection_extension___toString
0001:0042e666  _zim_reflection_parameter___toString
0001:0042ea49  _zim_reflection_object___construct
0001:0042ea78  _zim_reflection_class___construct
0001:0042eab0  _reflection_ext_functions
0002:000020b0  _reflection_module_entry
Module: U:\dev\php-5.3.20\ext\session\session.obj(session.obj)
0002:00020810  _ps_globals_id
0001:00430580  _php_session_register_serializer
0001:004305da  _php_session_register_module
0001:0043076e  _php_get_session_var
0001:00432d02  _session_adapt_url
0001:00432d57  __php_find_ps_serializer
0001:00432e88  __php_find_ps_module
0001:00432fbf  _ps_srlzr_encode_php
0001:004334de  _ps_srlzr_encode_php_binary
0001:004339ed  _php_session_create_id
0001:00434381  _php_session_start
0001:00435b33  _php_set_session_var
0001:00436bbc  _php_add_session_var
0001:004372b6  _ps_srlzr_decode_php
0001:00437485  _ps_srlzr_decode_php_binary
0002:00002110  _session_module_entry
Module: U:\dev\php-5.3.20\ext\session\mod_files.obj(mod_files.obj)
0001:004388e3  _ps_gc_files
0001:0043890c  _ps_close_files
0001:004389c9  _ps_open_files
0001:00439092  _ps_write_files
0001:004391c4  _ps_read_files
0001:0043931b  _ps_delete_files
0002:00002260  _ps_mod_files
Module: U:\dev\php-5.3.20\ext\session\mod_user.obj(mod_user.obj)
0001:00439463  _ps_gc_user
0001:004394fa  _ps_close_user
0001:0043955b  _ps_delete_user
0001:00439621  _ps_write_user
0001:00439728  _ps_read_user
0001:00439837  _ps_open_user
0002:00002280  _ps_mod_user
Module: U:\dev\php-5.3.20\ext\simplexml\simplexml.obj(simplexml.obj)
0001:00439990  _sxe_get_element_class_entry
0001:004399be  _zm_shutdown_simplexml
0001:00439bba  _sxe_object_new
0001:00439e9d  _php_sxe_get_iterator
0001:0043a064  _zm_info_simplexml
0001:0043a0da  _zm_startup_simplexml
0001:0043ac46  _simplexml_export_node
0001:0043a2d7  _zif_simplexml_import_dom
0001:0043a421  _zif_simplexml_load_file
0001:0043a55f  _zif_simplexml_load_string
0001:0043a6d6  _zim_simplexml_element___construct
0001:0043a87f  _zim_simplexml_element_registerXPathNamespace
0001:0043acac  _zim_simplexml_element_getName
0001:0043ad67  _zim_simplexml_element_attributes
0001:0043ae41  _zim_simplexml_element_children
0001:0043af9f  _zim_simplexml_element_addChild
0001:0043b2a1  _zim_simplexml_element_addAttribute
0001:0043b52d  _zim_simplexml_element_asXML
0001:0043b7c4  _zim_simplexml_element_xpath
0001:0043bc5c  _zim_simplexml_element_count
0001:0043bcbc  _php_sxe_move_forward_iterator
0001:0043d052  _zim_simplexml_element_getDocNamespaces
0001:0043da6f  _zim_simplexml_element___toString
0001:0043dd4d  _zim_simplexml_element_getNamespaces
0001:0043ee50  _simplexml_functions
0002:000022a0  _php_sxe_iterator_funcs
0002:000022c0  _simplexml_module_entry
0002:00009cd0  _sxe_class_entry
Module: U:\dev\php-5.3.20\ext\simplexml\sxe.obj(sxe.obj)
0002:00020820  _ce_SimpleXMLElement
0001:0043f533  _zm_startup_sxe
0001:0043f707  _zim_ce_SimpleXMLIterator_next
0001:0043f75d  _zim_ce_SimpleXMLIterator_valid
0001:0043f7b0  _zim_ce_SimpleXMLIterator_rewind
0001:0043f806  _zim_ce_SimpleXMLIterator_getChildren
0001:0043f892  _zim_ce_SimpleXMLIterator_current
0001:0043f92b  _zim_ce_SimpleXMLIterator_hasChildren
0001:0043f9f0  _zim_ce_SimpleXMLIterator_key
0002:00009ce0  _ce_SimpleXMLIterator
Module: U:\dev\php-5.3.20\ext\soap\soap.obj(soap.obj)
0002:00020830  _soap_globals_id
0002:00020840  _soap_var_class_entry
0001:0043fbfc  _zm_activate_soap
0001:00440148  _add_soap_fault
0001:004401e6  _zif_use_soap_error_handler
0001:0044026c  _zim_SoapClient___getLastResponseHeaders
0001:00440314  _zim_SoapClient___getLastRequestHeaders
0001:004403b5  _zim_SoapClient___getLastResponse
0001:00440455  _zim_SoapClient___getLastRequest
0001:004404f2  _zim_SoapClient___setLocation
0001:00440618  _zif_is_soap_fault
0001:004406c6  _zim_SoapParam_SoapParam
0001:00440866  _zim_SoapClient___setSoapHeaders
0001:00440a67  _zim_SoapClient___setCookie
0001:00440c73  _zim_SoapClient___doRequest
0001:00440e60  _zim_SoapServer_setPersistence
0001:00443749  _zim_SoapClient___getTypes
0001:00443b48  _zim_SoapClient___getFunctions
0001:00444b15  _zim_SoapFault_SoapFault
0001:00446551  _zim_SoapHeader_SoapHeader
0001:00446f06  _zim_SoapServer_SoapServer
0001:00449486  _zim_SoapServer_fault
0001:00449a73  _zim_SoapServer_addFunction
0001:00449fb0  _zim_SoapServer_getFunctions
0001:0044a257  _zim_SoapServer_setClass
0001:0044a4d6  _zim_SoapVar_SoapVar
0001:0044a79f  _zim_SoapFault___toString
0001:0044a990  _zm_info_soap
0001:0044b01a  _zm_startup_soap
0001:0044d198  _zm_shutdown_soap
0001:0044d23d  _OnUpdateCacheMode
0001:0044d2cf  _zim_SoapServer_addSoapHeader
0001:0044d4b2  _zim_SoapServer_setObject
0001:0044db25  _zim_SoapServer_handle
0001:00451b25  _zim_SoapClient___call
0001:004521da  _zim_SoapClient_SoapClient
0002:00002390  _soap_module_entry
0002:00009cf0  _le_url
Module: U:\dev\php-5.3.20\ext\soap\php_encoding.obj(php_encoding.obj)
0001:00454270  _whiteSpace_replace
0001:00454298  _whiteSpace_collapse
0001:0045505e  _delete_encoder
0001:00455a47  _get_conversion
0001:004560b9  _master_to_zval
0001:00457c9d  _delete_encoder_persistent
0001:00457cd4  _encode_finish
0001:00457d56  _encode_reset_ns
0001:00457df8  _encode_add_ns
0001:0045af55  _master_to_xml
0001:0045e955  _sdl_guess_convert_xml
0001:0045eac2  _to_zval_user
0001:0045ecdc  _to_xml_user
0001:0045f94d  _sdl_guess_convert_zval
0002:000023f0  _defaultEncoding
0002:00002c40  _numDefaultEncodings
Module: U:\dev\php-5.3.20\ext\soap\php_http.obj(php_http.obj)
0001:004602c9  _proxy_authentication
0001:004607b2  _http_context_headers
0001:00460bfb  _basic_authentication
0001:00461dbf  _make_http_soap_request
Module: U:\dev\php-5.3.20\ext\soap\php_packet_soap.obj(php_packet_soap.obj)
0001:00469933  _parse_packet_soap
Module: U:\dev\php-5.3.20\ext\soap\php_schema.obj(php_schema.obj)
0001:0046aa10  _delete_restriction_var_char_persistent
0001:0046aa41  _delete_restriction_var_int_persistent
0001:0046aa5b  _delete_extra_attribute_persistent
0001:0046aa91  _delete_restriction_var_char
0001:0046aac2  _delete_restriction_var_int
0001:0046aadc  _delete_extra_attribute
0001:0046ab12  _delete_attribute_persistent
0001:0046ab8f  _delete_attribute
0001:0046ac0c  _delete_model_persistent
0001:0046ac64  _delete_type_persistent
0001:0046adca  _delete_model
0001:0046ae22  _delete_type
0001:0046b794  _schema_pass2
0001:0046bb7b  _schema_min_max
0001:004725f6  _load_schema
Module: U:\dev\php-5.3.20\ext\soap\php_sdl.obj(php_sdl.obj)
0001:00473030  _delete_sdl_impl
0001:00473109  _delete_sdl
0001:00474958  _get_binding_from_name
0001:00474b9c  _sdl_restore_uri_credentials
0001:00476a8c  _get_binding_from_type
0001:0047b24d  _sdl_set_uri_credentials
0001:0047c0fa  _get_encoder_ex
0001:0047d01f  _get_encoder
0001:0047d327  _get_encoder_from_prefix
0001:00480360  _get_sdl
Module: U:\dev\php-5.3.20\ext\soap\php_xml.obj(php_xml.obj)
0001:00484e6a  _parse_namespace
0001:00484eda  _node_find_ns
0001:00484f05  _node_is_equal_ex
0001:00484f69  _get_node_recurisve_ex
0001:00484fcd  _get_node_ex
0001:0048500a  _attr_find_ns
0001:0048503f  _attr_is_equal_ex
0001:004850a3  _get_attribute_ex
0001:004850e0  _get_node_with_attribute_recursive_ex
0001:00485196  _get_node_with_attribute_ex
0001:00485217  _soap_xmlParseMemory
0001:0048535c  _soap_xmlParseFile
Module: U:\dev\php-5.3.20\ext\sockets\sockets.obj(sockets.obj)
0002:00020850  _sockets_globals_id
0001:00485450  _php_sockets_le_socket
0001:00485479  _zif_socket_clear_error
0001:00485527  _zif_socket_last_error
0001:0048563a  _zif_socket_shutdown
0001:00485758  _zm_deactivate_sockets
0001:004857d7  _zif_socket_get_option
0001:00485c66  _zif_socket_sendto
0001:00485f14  _zif_socket_strerror
0001:00485f84  _zif_socket_send
0001:00486127  _zif_socket_bind
0001:004863c8  _zif_socket_connect
0001:00486719  _zif_socket_create
0001:004868ad  _zif_socket_write
0001:004869f7  _zif_socket_close
0001:00486aa8  _zif_socket_listen
0001:00486be2  _zif_socket_set_block
0001:00486d1f  _zif_socket_set_nonblock
0001:00486e61  _zif_socket_accept
0001:0048702c  _zif_socket_create_listen
0001:0048761c  _zm_info_sockets
0001:00487bec  _zm_startup_sockets
0001:00488dc2  _zif_socket_read
0001:00489163  _zif_socket_select
0001:00489496  _zif_socket_create_pair
0001:00489760  _zif_socket_getpeername
0001:004899fb  _zif_socket_getsockname
0001:00489c78  _zif_socket_recv
0001:00489e65  _zif_socket_recvfrom
0001:0048a253  _zif_socket_set_option
0001:0048ab40  _sockets_functions
0002:00002c50  _sockets_module_entry
0002:00009e20  _inet_ntoa_lock
Module: U:\dev\php-5.3.20\ext\spl\php_spl.obj(php_spl.obj)
0002:00020860  _spl_globals_id
0001:0048b7a3  _zm_activate_spl
0001:0048b7d4  _zm_deactivate_spl
0001:0048b860  _zm_startup_spl
0001:0048b8fc  _zif_spl_classes
0001:0048c2c1  _zm_info_spl
0001:0048d705  _spl_build_class_list_string
0001:0048d75d  _php_spl_object_hash
0001:0048d88e  _zif_spl_object_hash
0001:0048d91f  _zif_spl_autoload_functions
0001:0048dbf8  _zif_spl_autoload_unregister
0001:0048e05e  _zif_spl_autoload_register
0001:0048e762  _zif_spl_autoload_call
0001:0048e9db  _zif_spl_autoload_extensions
0001:0048eaf7  _zif_spl_autoload
0001:0048f0d5  _zif_class_implements
0001:0048f1bb  _zif_class_parents
0001:0048f380  _spl_functions
0002:00002cb0  _spl_module_entry
Module: U:\dev\php-5.3.20\ext\spl\spl_functions.obj(spl_functions.obj)
0001:0048f850  _spl_gen_private_prop_name
0001:0048f894  _spl_add_class_name
0001:0048f977  _spl_add_interfaces
0001:0048f9d4  _spl_add_classes
0001:0048fa74  _spl_register_property
0001:0048fa80  _spl_register_sub_class
0001:0048fbd1  _spl_register_std_class
0001:0048fcfc  _spl_register_interface
Module: U:\dev\php-5.3.20\ext\spl\spl_engine.obj(spl_engine.obj)
0001:0048fe10  _spl_offset_convert_to_long
0001:0048ff47  _spl_instantiate
Module: U:\dev\php-5.3.20\ext\spl\spl_iterators.obj(spl_iterators.obj)
0002:00020870  _spl_ce_RecursiveIterator
0002:00020880  _spl_ce_RecursiveIteratorIterator
0002:00020890  _spl_ce_OuterIterator
0002:000208a0  _spl_ce_IteratorIterator
0002:000208b0  _spl_ce_FilterIterator
0002:000208c0  _spl_ce_RecursiveFilterIterator
0002:000208d0  _spl_ce_ParentIterator
0002:000208e0  _spl_ce_Countable
0002:000208f0  _spl_ce_SeekableIterator
0002:00020900  _spl_ce_LimitIterator
0002:00020910  _spl_ce_CachingIterator
0002:00020920  _spl_ce_RecursiveCachingIterator
0002:00020930  _spl_ce_NoRewindIterator
0002:00020940  _spl_ce_AppendIterator
0002:00020950  _spl_ce_InfiniteIterator
0002:00020960  _spl_ce_RegexIterator
0002:00020970  _spl_ce_RecursiveRegexIterator
0002:00020980  _spl_ce_EmptyIterator
0002:00020990  _spl_ce_RecursiveTreeIterator
0001:0049001b  _spl_iterator_apply
0001:0049101a  _zm_startup_spl_iterators
0001:0049a1b0  _spl_funcs_RecursiveIterator
0001:004928a7  _zif_iterator_count
0001:0049292c  _zim_spl_EmptyIterator_next
0001:00492970  _zim_spl_EmptyIterator_current
0001:004929e6  _zim_spl_EmptyIterator_key
0001:00492a35  _zim_spl_EmptyIterator_valid
0001:00492a6e  _zim_spl_EmptyIterator_rewind
0001:00492a87  _zim_spl_NoRewindIterator_rewind
0001:00492aa0  _zim_spl_RecursiveTreeIterator_getPrefix
0001:00492afc  _zim_spl_RecursiveIteratorIterator_getMaxDepth
0001:00492b86  _zim_spl_RecursiveIteratorIterator_setMaxDepth
0001:00492c01  _zim_spl_RecursiveIteratorIterator_nextElement
0001:00492c1a  _zim_spl_RecursiveIteratorIterator_endChildren
0001:00492c33  _zim_spl_RecursiveIteratorIterator_beginChildren
0001:00492c4c  _zim_spl_RecursiveIteratorIterator_callGetChildren
0001:00492d46  _zim_spl_RecursiveIteratorIterator_callHasChildren
0001:00492e52  _zim_spl_RecursiveIteratorIterator_endIteration
0001:00492e6b  _zim_spl_RecursiveIteratorIterator_beginIteration
0001:00492e84  _zim_spl_RecursiveIteratorIterator_getDepth
0001:00492ed1  _zim_spl_RecursiveIteratorIterator_next
0001:00492f2a  _zim_spl_RecursiveIteratorIterator_key
0001:00492fd9  _zim_spl_RecursiveIteratorIterator_valid
0001:0049303a  _zim_spl_RecursiveIteratorIterator_rewind
0001:00493099  _zif_iterator_apply
0001:0049337f  _zim_spl_AppendIterator_valid
0001:004933fd  _zim_spl_NoRewindIterator_next
0001:0049347b  _zim_spl_NoRewindIterator_key
0001:00493546  _zim_spl_NoRewindIterator_valid
0001:004935d1  _zim_spl_RecursiveCachingIterator_hasChildren
0001:0049364f  _zim_spl_CachingIterator_getFlags
0001:004936c5  _zim_spl_CachingIterator_valid
0001:0049373f  _zim_spl_LimitIterator_getPosition
0001:00493796  _zim_spl_LimitIterator_valid
0001:00493810  _zim_spl_RegexIterator_setPregFlags
0001:00493888  _zim_spl_RegexIterator_getPregFlags
0001:00493905  _zim_spl_RegexIterator_setFlags
0001:00493976  _zim_spl_RegexIterator_getFlags
0001:004939fd  _zim_spl_RegexIterator_setMode
0001:00493aa1  _zim_spl_RegexIterator_getMode
0001:00493b17  _zim_spl_RecursiveFilterIterator_hasChildren
0001:00493c2c  _zim_spl_dual_it_valid
0001:00493cdd  _zim_spl_RecursiveTreeIterator_setPrefixPart
0001:00493e74  _zim_spl_AppendIterator_getIteratorIndex
0001:00493ef9  _zim_spl_dual_it_key
0001:00493fa2  _zim_spl_RecursiveTreeIterator_getPostfix
0001:004948bf  _zim_spl_AppendIterator___construct
0001:00494908  _zim_spl_InfiniteIterator___construct
0001:00494951  _zim_spl_NoRewindIterator___construct
0001:0049499a  _zim_spl_IteratorIterator___construct
0001:004949e3  _zim_spl_RecursiveCachingIterator___construct
0001:00494a2c  _zim_spl_CachingIterator___construct
0001:00494a75  _zim_spl_LimitIterator___construct
0001:00494abe  _zim_spl_RecursiveRegexIterator___construct
0001:00494b07  _zim_spl_RegexIterator___construct
0001:00494b50  _zim_spl_ParentIterator___construct
0001:00494b99  _zim_spl_RecursiveFilterIterator___construct
0001:00494be2  _zim_spl_FilterIterator___construct
0001:00494c6c  _zim_spl_CachingIterator_count
0001:00494e1d  _zim_spl_CachingIterator_setFlags
0001:00494ffa  _zim_spl_CachingIterator_offsetExists
0001:0049520a  _zim_spl_CachingIterator_offsetUnset
0001:004954bc  _zim_spl_RecursiveRegexIterator_getChildren
0001:00495637  _zim_spl_RecursiveFilterIterator_getChildren
0001:004957c1  _zim_spl_RegexIterator_accept
0001:00495cee  _zim_spl_CachingIterator_hasNext
0001:00495d82  _zif_iterator_to_array
0001:00495e37  _zim_spl_RecursiveIteratorIterator_getInnerIterator
0001:00495ec6  _zim_spl_AppendIterator_getArrayIterator
0001:00495f6c  _zim_spl_RecursiveIteratorIterator_current
0001:00496011  _zim_spl_NoRewindIterator_current
0001:004960ee  _zim_spl_CachingIterator_offsetGet
0001:004963a4  _zim_spl_RecursiveCachingIterator_getChildren
0001:0049645a  _zim_spl_CachingIterator_getCache
0001:0049653d  _zim_spl_dual_it_current
0001:004965f3  _zim_spl_dual_it_getInnerIterator
0001:004966a9  _zim_spl_RecursiveIteratorIterator_getSubIterator
0001:00496754  _zim_spl_RecursiveTreeIterator_key
0001:00496a8e  _zim_spl_RecursiveTreeIterator_current
0001:00496c42  _zim_spl_RecursiveTreeIterator_getEntry
0001:00496ce2  _zim_spl_CachingIterator___toString
0001:00496e1f  _zim_spl_CachingIterator_offsetSet
0001:00497825  _zim_spl_RecursiveTreeIterator___construct
0001:0049786e  _zim_spl_RecursiveIteratorIterator___construct
0001:0049805b  _zim_spl_CachingIterator_next
0001:004980cf  _zim_spl_dual_it_rewind
0001:0049830e  _zim_spl_CachingIterator_rewind
0001:00498476  _spl_append_it_next_iterator
0001:0049869e  _spl_append_it_fetch
0001:004987e8  _zim_spl_AppendIterator_rewind
0001:00498882  _zim_spl_AppendIterator_append
0001:00498fc2  _zim_spl_LimitIterator_seek
0001:0049904f  _zim_spl_LimitIterator_rewind
0001:00499150  _spl_append_it_next
0001:00499225  _zim_spl_AppendIterator_next
0001:004992a4  _zim_spl_FilterIterator_rewind
0001:00499661  _zim_spl_LimitIterator_next
0001:0049989a  _zim_spl_InfiniteIterator_next
0001:00499ba3  _zim_spl_FilterIterator_next
0001:00499f54  _zim_spl_dual_it_next
0002:00002d10  _spl_recursive_it_iterator_funcs
Module: U:\dev\php-5.3.20\ext\spl\spl_array.obj(spl_array.obj)
0002:000209a0  _spl_ce_ArrayObject
0002:000209b0  _spl_handler_ArrayObject
0002:00020a20  _spl_ce_ArrayIterator
0002:00020a30  _spl_handler_ArrayIterator
0002:00020aa0  _spl_ce_RecursiveArrayIterator
0001:0049b844  _zm_startup_spl_array
0001:0049e450  _spl_array_serialize
0001:0049c09e  _spl_array_unserialize
0001:004a0770  _spl_array_object_count_elements
0001:0049bc29  _spl_array_get_iterator
0001:0049bcf0  _zim_spl_Array_setFlags
0001:0049bd4d  _zim_spl_Array_getFlags
0001:0049bd9d  _zim_spl_Array_setIteratorClass
0001:0049be14  _spl_array_unserialize_helper
0001:0049c1f8  _zim_spl_Array_unserialize
0001:0049c303  _zim_spl_Array_getIteratorClass
0001:0049c933  _spl_hash_verify_pos_ex
0001:0049d214  _zim_spl_Array_rewind
0001:0049d507  _zim_spl_Array___construct
0001:0049d620  _spl_array_iterator_key
0001:0049d7b5  _zim_spl_Array_key
0001:0049d800  _zim_spl_Array_getArrayCopy
0001:0049d91b  _zim_spl_Array_hasChildren
0001:0049dafd  _zim_spl_Array_valid
0001:0049dc8e  _zim_spl_Array_next
0001:0049dd9d  _zim_spl_Array_current
0001:0049df5f  _zim_spl_Array_getIterator
0001:0049e0a5  _spl_array_serialize_helper
0001:0049e4fa  _zim_spl_Array_serialize
0001:0049e607  _zim_spl_Array_getChildren
0001:0049ecbb  _zim_spl_Array_natcasesort
0001:0049ed08  _zim_spl_Array_natsort
0001:0049ed54  _zim_spl_Array_uksort
0001:0049eda0  _zim_spl_Array_uasort
0001:0049edeb  _zim_spl_Array_ksort
0001:0049ee36  _zim_spl_Array_asort
0001:0049ee7d  _zim_spl_Array_exchangeArray
0001:0049effd  _spl_hash_verify_pos
0001:0049f182  _zim_spl_Array_seek
0001:004a0540  _zim_spl_Array_offsetGet
0001:004a0717  _zim_spl_Array_count
0001:004a0e70  _zim_spl_Array_offsetUnset
0001:004a1457  _zim_spl_Array_offsetExists
0001:004a1a71  _spl_array_iterator_append
0001:004a1be5  _zim_spl_Array_append
0001:004a1c31  _zim_spl_Array_offsetSet
0002:00002d30  _spl_array_it_funcs
Module: U:\dev\php-5.3.20\ext\spl\spl_directory.obj(spl_directory.obj)
0002:00020ab0  _spl_ce_SplFileObject
0002:00020ac0  _spl_ce_SplFileInfo
0002:00020ad0  _spl_ce_DirectoryIterator
0002:00020ae0  _spl_ce_FilesystemIterator
0002:00020af0  _spl_ce_RecursiveDirectoryIterator
0002:00020b00  _spl_ce_GlobIterator
0002:00020b10  _spl_ce_SplTempFileObject
0001:004a2596  _zim_spl_SplFileInfo__bad_state_ex
0001:004a25bf  _zim_spl_SplFileObject_getChildren
0001:004a25d8  _zim_spl_SplFileObject_hasChildren
0001:004a2c49  _zm_startup_spl_directory
0001:004a5047  _spl_filesystem_dir_get_iterator
0001:004a4fd9  _spl_filesystem_tree_get_iterator
0001:004a3ba8  _spl_filesystem_object_get_method_check
0001:004a32c1  _zim_spl_SplFileObject_fseek
0001:004a33a7  _zim_spl_SplFileObject_setCsvControl
0001:004a34fa  _zim_spl_SplFileObject_getMaxLineLen
0001:004a3583  _zim_spl_SplFileObject_setMaxLineLen
0001:004a35f6  _zim_spl_SplFileObject_getFlags
0001:004a3646  _zim_spl_SplFileObject_setFlags
0001:004a3681  _zim_spl_SplFileObject_key
0001:004a36d5  _zim_spl_RecursiveDirectoryIterator_getSubPathname
0001:004a37a7  _zim_spl_RecursiveDirectoryIterator_getSubPath
0001:004a3839  _zim_spl_FilesystemIterator_setFlags
0001:004a3895  _zim_spl_FilesystemIterator_getFlags
0001:004a38ea  _zim_spl_SplFileInfo_setInfoClass
0001:004a396b  _zim_spl_SplFileInfo_setFileClass
0001:004a39ec  _zim_spl_DirectoryIterator_getFilename
0001:004a3a58  _zim_spl_DirectoryIterator_valid
0001:004a3aab  _zim_spl_DirectoryIterator_key
0001:004a3b14  _zim_spl_DirectoryIterator_rewind
0001:004a3c0e  _zim_spl_SplFileObject_valid
0001:004a3c92  _zim_spl_SplFileObject_eof
0001:004a3cf3  _zim_spl_DirectoryIterator_current
0001:004a409c  _zim_spl_SplFileObject_fgetcsv
0001:004a41ed  _zim_spl_SplFileObject_fgets
0001:004a4285  _zim_spl_SplFileObject_ftruncate
0001:004a4527  _zim_spl_SplFileObject_fstat
0001:004a45d5  _zim_spl_SplFileObject_fscanf
0001:004a468e  _zim_spl_SplFileObject_fgetss
0001:004a4799  _zim_spl_SplFileObject_flock
0001:004a4844  _zim_spl_SplFileObject_fwrite
0001:004a497a  _zim_spl_SplFileObject_fpassthru
0001:004a49b3  _zim_spl_SplFileObject_fgetc
0001:004a4a3a  _zim_spl_SplFileObject_ftell
0001:004a4a89  _zim_spl_SplFileObject_fflush
0001:004a4ad2  _zim_spl_SplFileObject_getCsvControl
0001:004a4b83  _zim_spl_SplTempFileObject___construct
0001:004a4ca7  _zim_spl_SplFileObject___construct
0001:004a4e28  _spl_filesystem_info_set_filename
0001:004a4f0a  _zim_spl_SplFileInfo___construct
0001:004a50d8  _zim_spl_GlobIterator_count
0001:004a5183  _zim_spl_DirectoryIterator_seek
0001:004a53e2  _zim_spl_SplFileInfo_getLinkTarget
0001:004a55fc  _zim_spl_DirectoryIterator_getBasename
0001:004a56aa  _zim_spl_DirectoryIterator_getExtension
0001:004a57bd  _spl_filesystem_object_get_path
0001:004a58c4  _zim_spl_SplFileInfo_getRealPath
0001:004a59e8  _zim_spl_SplFileInfo_getBasename
0001:004a5ac3  _zim_spl_SplFileInfo_getExtension
0001:004a5c07  _zim_spl_SplFileInfo_getFilename
0001:004a5cab  _zim_spl_SplFileInfo_getPath
0001:004a5fb2  _zim_spl_SplFileObject_current
0001:004a609a  _zim_spl_SplFileObject_next
0001:004a61d0  _zim_spl_SplFileObject_seek
0001:004a6283  _zim_spl_SplFileObject_rewind
0001:004a641d  _zim_spl_FilesystemIterator_rewind
0001:004a64d1  _zim_spl_DirectoryIterator_next
0001:004a694c  _spl_filesystem_object_construct
0001:004a6b16  _zim_spl_GlobIterator___construct
0001:004a6b54  _zim_spl_RecursiveDirectoryIterator___construct
0001:004a6b92  _zim_spl_FilesystemIterator___construct
0001:004a6bd0  _zim_spl_DirectoryIterator___construct
0001:004a6c0e  _zim_spl_DirectoryIterator_isDot
0001:004a6dc4  _zim_spl_FilesystemIterator_key
0001:004a6f08  _zim_spl_SplFileInfo_getInode
0001:004a7039  _zim_spl_SplFileInfo_getPerms
0001:004a716a  _zim_spl_SplFileInfo_getATime
0001:004a729d  _zim_spl_SplFileInfo_getGroup
0001:004a73ce  _zim_spl_SplFileInfo_getOwner
0001:004a74ff  _zim_spl_SplFileInfo_getSize
0001:004a7630  _zim_spl_RecursiveDirectoryIterator_getChildren
0001:004a78c6  _zim_spl_SplFileInfo_isLink
0001:004a79f8  _zim_spl_SplFileInfo_isDir
0001:004a7b29  _zim_spl_SplFileInfo_isFile
0001:004a7c5a  _zim_spl_SplFileInfo_isExecutable
0001:004a7d8d  _zim_spl_SplFileInfo_isReadable
0001:004a7ebe  _zim_spl_SplFileInfo_isWritable
0001:004a7fef  _zim_spl_SplFileInfo_getType
0001:004a8120  _zim_spl_SplFileInfo_getCTime
0001:004a8251  _zim_spl_SplFileInfo_getMTime
0001:004a8385  _zim_spl_RecursiveDirectoryIterator_hasChildren
0001:004a8608  _zim_spl_SplFileInfo_getPathInfo
0001:004a8836  _zim_spl_SplFileInfo_getPathname
0001:004a94ca  _zim_spl_SplFileInfo_getFileInfo
0001:004a9560  _zim_spl_SplFileInfo_openFile
0001:004a95a3  _zim_spl_FilesystemIterator_current
0002:00002d70  _spl_filesystem_tree_it_funcs
0002:00002d50  _spl_filesystem_dir_it_funcs
Module: U:\dev\php-5.3.20\ext\spl\spl_exceptions.obj(spl_exceptions.obj)
0002:00020b20  _spl_ce_LogicException
0002:00020b30  _spl_ce_BadFunctionCallException
0002:00020b40  _spl_ce_BadMethodCallException
0002:00020b50  _spl_ce_DomainException
0002:00020b60  _spl_ce_InvalidArgumentException
0002:00020b70  _spl_ce_LengthException
0002:00020b80  _spl_ce_OutOfRangeException
0002:00020b90  _spl_ce_RuntimeException
0002:00020ba0  _spl_ce_OutOfBoundsException
0002:00020bb0  _spl_ce_OverflowException
0002:00020bc0  _spl_ce_RangeException
0002:00020bd0  _spl_ce_UnderflowException
0002:00020be0  _spl_ce_UnexpectedValueException
0001:004aa80f  _zm_startup_spl_exceptions
Module: U:\dev\php-5.3.20\ext\spl\spl_observer.obj(spl_observer.obj)
0002:00020bf0  _spl_ce_SplObserver
0002:00020c00  _spl_ce_SplSubject
0002:00020c10  _spl_ce_SplObjectStorage
0002:00020c20  _spl_handler_SplObjectStorage
0002:00020c90  _spl_ce_MultipleIterator
0001:004aab23  _zm_startup_spl_observer
0001:004aae1e  _spl_object_storage_detach
0001:004ab235  _spl_object_storage_get
0001:004ab26c  _spl_object_storage_attach
0001:004ab339  _spl_object_storage_addall
0001:004ad57b  _spl_SplOjectStorage_free_storage
0001:004ab6ef  _zim_spl_MultipleIterator_setFlags
0001:004ab72b  _zim_spl_MultipleIterator_getFlags
0001:004ab778  _zim_spl_SplObjectStorage_next
0001:004ab7cf  _zim_spl_SplObjectStorage_setInfo
0001:004ab84e  _zim_spl_SplObjectStorage_key
0001:004ab89b  _zim_spl_SplObjectStorage_rewind
0001:004ab8f3  _zim_spl_SplObjectStorage_count
0001:004ab94a  _zim_spl_SplObjectStorage_removeAll
0001:004aba35  _zim_spl_SplObjectStorage_addAll
0001:004ababb  _zim_spl_SplObjectStorage_detach
0001:004abb32  _zim_spl_SplObjectStorage_attach
0001:004abba6  _zim_spl_MultipleIterator_valid
0001:004abd31  _zim_spl_MultipleIterator_next
0001:004abe4b  _zim_spl_MultipleIterator_rewind
0001:004ac3bf  _zim_spl_MultipleIterator_key
0001:004ac41f  _zim_spl_MultipleIterator_current
0001:004ac4bf  _zim_spl_MultipleIterator_attachIterator
0001:004ac61b  _zim_spl_MultipleIterator___construct
0001:004ac6e4  _zim_spl_SplObjectStorage_unserialize
0001:004acb2b  _zim_spl_SplObjectStorage_serialize
0001:004ad15a  _zim_spl_SplObjectStorage_valid
0001:004ad1bf  _zim_spl_SplObjectStorage_getInfo
0001:004ad25f  _zim_spl_SplObjectStorage_current
0001:004ad30f  _zim_spl_SplObjectStorage_offsetGet
0001:004ad3cf  _spl_object_storage_contains
0001:004ad3eb  _zim_spl_SplObjectStorage_contains
0001:004ad45e  _zim_spl_SplObjectStorage_removeAllExcept
Module: U:\dev\php-5.3.20\ext\spl\spl_dllist.obj(spl_dllist.obj)
0002:00020ca0  _spl_ce_SplDoublyLinkedList
0002:00020cb0  _spl_handler_SplDoublyLinkedList
0002:00020d20  _spl_ce_SplQueue
0002:00020d30  _spl_ce_SplStack
0001:004adfff  _zm_startup_spl_dllist
0001:004aea79  _spl_dllist_get_iterator
0001:004aeb17  _zim_spl_SplDoublyLinkedList_rewind
0001:004aebb2  _zim_spl_SplDoublyLinkedList_valid
0001:004aec05  _zim_spl_SplDoublyLinkedList_next
0001:004aec66  _zim_spl_SplDoublyLinkedList_prev
0001:004aecca  _zim_spl_SplDoublyLinkedList_key
0001:004aed17  _zim_spl_SplDoublyLinkedList_getIteratorMode
0001:004aeda8  _zim_spl_SplDoublyLinkedList_setIteratorMode
0001:004aee33  _zim_spl_SplDoublyLinkedList_count
0001:004aee85  _zim_spl_SplDoublyLinkedList_push
0001:004aef56  _zim_spl_SplDoublyLinkedList_offsetUnset
0001:004af0b8  _zim_spl_SplDoublyLinkedList_offsetExists
0001:004af269  _zim_spl_SplDoublyLinkedList_isEmpty
0001:004af2bf  _zim_spl_SplDoublyLinkedList_current
0001:004af379  _zim_spl_SplDoublyLinkedList_bottom
0001:004af428  _zim_spl_SplDoublyLinkedList_top
0001:004af500  _zim_spl_SplDoublyLinkedList_shift
0001:004af5de  _zim_spl_SplDoublyLinkedList_pop
0001:004af6b7  _zim_spl_SplDoublyLinkedList_offsetGet
0001:004af7dd  _zim_spl_SplDoublyLinkedList_offsetSet
0001:004af9b1  _zim_spl_SplDoublyLinkedList_unshift
0002:00002d90  _spl_dllist_it_funcs
Module: U:\dev\php-5.3.20\ext\spl\spl_heap.obj(spl_heap.obj)
0002:00020d40  _spl_ce_SplHeap
0002:00020d50  _spl_handler_SplHeap
0002:00020dc0  _spl_ce_SplMinHeap
0002:00020dd0  _spl_ce_SplMaxHeap
0002:00020de0  _spl_ce_SplPriorityQueue
0002:00020df0  _spl_handler_SplPriorityQueue
0001:004b02b6  _zm_startup_spl_heap
0001:004b05d3  _spl_heap_get_iterator
0001:004b054d  _spl_pqueue_get_iterator
0001:004b1234  _zim_spl_SplHeap_rewind
0001:004b124d  _zim_spl_SplHeap_valid
0001:004b12a5  _zim_spl_SplHeap_next
0001:004b1303  _zim_spl_SplHeap_key
0001:004b1359  _zim_spl_SplMaxHeap_compare
0001:004b13bc  _zim_spl_SplMinHeap_compare
0001:004b141f  _zim_spl_SplPriorityQueue_compare
0001:004b1482  _zim_spl_SplHeap_recoverFromCorruption
0001:004b14d5  _zim_spl_SplPriorityQueue_setExtractFlags
0001:004b152b  _zim_spl_SplHeap_isEmpty
0001:004b1583  _zim_spl_SplHeap_count
0001:004b16c7  _zim_spl_SplHeap_insert
0001:004b1917  _zim_spl_SplHeap_top
0001:004b19df  _zim_spl_SplPriorityQueue_top
0001:004b1af1  _zim_spl_SplPriorityQueue_current
0001:004b1bd9  _zim_spl_SplHeap_extract
0001:004b1cbc  _zim_spl_SplHeap_current
0001:004b1d65  _zim_spl_SplPriorityQueue_extract
0001:004b1e9c  _zim_spl_SplPriorityQueue_insert
0002:00002dd0  _spl_pqueue_it_funcs
0002:00002db0  _spl_heap_it_funcs
Module: U:\dev\php-5.3.20\ext\spl\spl_fixedarray.obj(spl_fixedarray.obj)
0002:00020e60  _spl_ce_SplFixedArray
0002:00020e70  _spl_handler_SplFixedArray
0001:004b25d1  _zm_startup_spl_fixedarray
0001:004b2715  _spl_fixedarray_get_iterator
0001:004b3010  _zim_spl_SplFixedArray_rewind
0001:004b3056  _zim_spl_SplFixedArray_valid
0001:004b30bc  _zim_spl_SplFixedArray_next
0001:004b30ff  _zim_spl_SplFixedArray_key
0001:004b314c  _zim_spl_SplFixedArray_getSize
0001:004b31ac  _zim_spl_SplFixedArray_count
0001:004b3234  _zim_spl_SplFixedArray___construct
0001:004b32d7  _zim_spl_SplFixedArray_setSize
0001:004b34bd  _zim_spl_SplFixedArray_toArray
0001:004b3780  _zim_spl_SplFixedArray_fromArray
0001:004b429e  _zim_spl_SplFixedArray_offsetExists
0001:004b432d  _zim_spl_SplFixedArray_offsetUnset
0001:004b43ec  _zim_spl_SplFixedArray_current
0001:004b4516  _zim_spl_SplFixedArray_offsetGet
0001:004b46e5  _zim_spl_SplFixedArray_offsetSet
0002:00002df0  _spl_fixedarray_it_funcs
Module: U:\dev\php-5.3.20\ext\standard\crypt_freesec.obj(crypt_freesec.obj)
0001:004b49c0  __crypt_extended_init
0001:004b5529  __crypt_extended_r
Module: U:\dev\php-5.3.20\ext\standard\crypt_blowfish.obj(crypt_blowfish.obj)
0001:004b7c4a  _php_crypt_blowfish_rn
Module: U:\dev\php-5.3.20\ext\standard\crypt_sha512.obj(crypt_sha512.obj)
0001:004b9e89  _php_sha512_crypt_r
0001:004bae6b  _php_sha512_crypt
Module: U:\dev\php-5.3.20\ext\standard\crypt_sha256.obj(crypt_sha256.obj)
0001:004bb843  ___php_mempcpy
0001:004bb86b  ___php_stpncpy
0001:004bb8b6  _php_sha256_crypt_r
0001:004bc883  _php_sha256_crypt
Module: U:\dev\php-5.3.20\ext\standard\php_crypt_r.obj(php_crypt_r.obj)
0002:00020ee0  _php_crypt_extended_init_lock
0001:004bca94  _php_md5_crypt_r
0001:004bcfaf  __crypt_extended_init_r
0001:004bcfe7  _php_shutdown_crypt_r
0001:004bcffc  _php_init_crypt_r
Module: U:\dev\php-5.3.20\ext\standard\array.obj(array.obj)
0002:00020ef0  _array_globals_id
0001:004bd148  _php_multisort_compare
0001:004bd305  _zif_array_chunk
0001:004bd56f  _zif_array_key_exists
0001:004bd78d  _zif_array_filter
0001:004bda05  _zif_array_values
0001:004bdb28  _zif_array_push
0001:004bddaf  _zif_array_search
0001:004bddde  _zif_in_array
0001:004bde0f  _zif_key
0001:004bdf04  _zif_array_rand
0001:004be1c0  _zif_array_multisort
0001:004be8e8  _zif_shuffle
0001:004becbe  _zif_array_slice
0001:004bf3b2  _zif_array_udiff_assoc
0001:004bf3e1  _zif_array_diff_assoc
0001:004bf410  _zif_array_diff_key
0001:004bf7aa  _zif_array_uintersect_assoc
0001:004bf7d9  _zif_array_intersect_assoc
0001:004bf808  _zif_array_intersect_key
0001:004bf837  _php_splice
0001:004bfbe3  _zif_array_change_key_case
0001:004bfd91  _zif_array_unshift
0001:004bfea1  _zif_array_reverse
0001:004c01b6  _zif_array_keys
0001:004c03c9  _zif_array_splice
0001:004c05f4  _zif_compact
0001:004c0705  _php_prefix_varname
0001:004c07cb  _zif_uksort
0001:004c098b  _zif_uasort
0001:004c0b4b  _zif_usort
0001:004c0d0b  _zif_rsort
0001:004c0da4  _zif_sort
0001:004c0e3d  _zif_arsort
0001:004c0ed6  _zif_asort
0001:004c0ff8  _zif_natcasesort
0001:004c1027  _zif_natsort
0001:004c1056  _zif_ksort
0001:004c10ef  _zif_krsort
0001:004c1192  _zif_count
0001:004c135b  _zm_shutdown_array
0001:004c146e  _zm_startup_array
0001:004c1a66  _zif_array_count_values
0001:004c1f3e  _zif_extract
0001:004c271c  _zif_array_fill
0001:004c2845  _zif_array_sum
0001:004c297a  _php_array_replace_recursive
0001:004c2cc2  _zif_array_map
0001:004c338f  _zif_array_combine
0001:004c359d  _zif_array_product
0001:004c3ac5  _zif_array_walk_recursive
0001:004c3c31  _zif_array_walk
0001:004c3dd2  _zif_array_pad
0001:004c41b4  _zif_min
0001:004c438f  _zif_max
0001:004c47ac  _zif_array_shift
0001:004c47db  _zif_array_pop
0001:004c4848  _zif_array_reduce
0001:004c4ac9  _zif_current
0001:004c4b6c  _php_array_merge
0001:004c537f  _zif_array_replace_recursive
0001:004c53bd  _zif_array_replace
0001:004c53fb  _zif_array_merge_recursive
0001:004c5439  _zif_array_merge
0001:004c5477  _zif_prev
0001:004c5536  _zif_next
0001:004c55f5  _zif_end
0001:004c56b4  _zif_reset
0001:004c65d9  _zif_array_udiff_uassoc
0001:004c661e  _zif_array_diff_uassoc
0001:004c6663  _zif_array_udiff
0001:004c66a8  _zif_array_diff
0001:004c66ed  _zif_array_diff_ukey
0001:004c752a  _zif_array_uintersect_uassoc
0001:004c756f  _zif_array_intersect_uassoc
0001:004c75b4  _zif_array_uintersect
0001:004c75f9  _zif_array_intersect
0001:004c763e  _zif_array_intersect_ukey
0001:004c76ad  _zif_range
0001:004c810e  _zif_array_fill_keys
0001:004c8421  _zif_array_flip
0001:004c874a  _zif_array_unique
Module: U:\dev\php-5.3.20\ext\standard\base64.obj(base64.obj)
0001:004c8a30  _php_base64_encode
0001:004c8bb5  _zif_base64_encode
0001:004c8c2b  _php_base64_decode_ex
0001:004c8df6  _zif_base64_decode
0001:004c8e7f  _php_base64_decode
Module: U:\dev\php-5.3.20\ext\standard\basic_functions.obj(basic_functions.obj)
0002:00020f00  _basic_globals_id
0001:004c9100  _php_get_nan
0001:004c910b  _php_get_inf
0001:004c9116  _zif_get_magic_quotes_runtime
0001:004c9137  _zif_get_magic_quotes_gpc
0001:004c9157  _zif_connection_aborted
0001:004c917e  _zif_connection_status
0001:004c91a2  _zif_sys_getloadavg
0001:004c9231  _zif_set_magic_quotes_runtime
0001:004c92bc  _zif_import_request_variables
0001:004c964d  _zif_parse_ini_string
0001:004c981b  _zif_parse_ini_file
0001:004c998e  _zif_is_uploaded_file
0001:004c9a5b  _zif_move_uploaded_file
0001:004c9cc2  _zif_unregister_tick_function
0001:004c9ef4  _zif_getprotobynumber
0001:004c9f73  _zif_getprotobyname
0001:004c9fd7  _zif_getservbyport
0001:004ca071  _zif_getservbyname
0001:004ca101  _zif_ignore_user_abort
0001:004ca1b2  _zif_print_r
0001:004ca28d  _zif_restore_include_path
0001:004ca2cf  _zif_ini_restore
0001:004ca321  _zif_get_include_path
0001:004ca3aa  _zif_ini_get
0001:004ca465  _zif_ini_get_all
0001:004ca787  _zif_php_strip_whitespace
0001:004ca957  _php_get_highlight_struct
0001:004caa52  _zif_register_shutdown_function
0001:004cacfa  _php_free_shutdown_functions
0001:004cadb3  _php_call_shutdown_functions
0001:004cae5b  _zif_error_get_last
0001:004cafc5  __php_error_log_ex
0001:004cb102  __php_error_log
0001:004cb159  _zif_error_log
0001:004cb25c  _zif_get_cfg_var
0001:004cb43a  _zif_get_current_user
0001:004cb4ca  _zif_time_sleep_until
0001:004cb6ba  _zif_time_nanosleep
0001:004cb84e  _zif_usleep
0001:004cb8fd  _zif_sleep
0001:004cb97b  _zif_flush
0001:004cba4f  _zif_putenv
0001:004cbe8e  _zif_getenv
0001:004cbf4e  _zif_long2ip
0001:004cc040  _php_inet_ntop
0001:004cc111  _zif_ip2long
0001:004cc1ac  _php_inet_pton
0001:004cc2bc  _zif_constant
0001:004cc35b  _zm_info_basic
0001:004cc39e  _zm_deactivate_basic
0001:004cc578  _zm_activate_basic
0001:004cc7a4  _zm_shutdown_basic
0001:004cca69  _zm_startup_basic
0001:004cd6b8  _zif_highlight_string
0001:004cd92c  _zif_forward_static_call
0001:004cdaef  _zif_call_user_method_array
0001:004cdd4b  _zif_call_user_method
0001:004cdf2d  _zif_call_user_func
0001:004ce044  _zif_forward_static_call_array
0001:004ce1a1  _zif_call_user_func_array
0001:004ce4ea  _zif_register_tick_function
0001:004cee50  _zif_ini_set
0001:004cf09e  _zif_set_include_path
0001:004cf1bc  _zif_highlight_file
0001:004cfc5b  _zif_getopt
0001:004d2090  _basic_functions
0002:00002fe0  _basic_functions_module
Module: U:\dev\php-5.3.20\ext\standard\browscap.obj(browscap.obj)
0002:00020f10  _browscap_globals_id
0001:004de0c1  _zm_shutdown_browscap
0001:004de0dd  _zm_deactivate_browscap
0001:004de417  _zif_get_browser
0001:004dea53  _zm_startup_browscap
0001:004deada  _OnChangeBrowscap
Module: U:\dev\php-5.3.20\ext\standard\crc32.obj(crc32.obj)
0001:004df3d2  _php_if_crc32
Module: U:\dev\php-5.3.20\ext\standard\crypt.obj(crypt.obj)
0001:004df870  _zif_crypt
0001:004dfe71  _zm_shutdown_crypt
0001:004dfee1  _zm_startup_crypt
Module: U:\dev\php-5.3.20\ext\standard\cyr_convert.obj(cyr_convert.obj)
0001:004e00d0  _zif_convert_cyr_string
Module: U:\dev\php-5.3.20\ext\standard\datetime.obj(datetime.obj)
0001:004e0ba9  _zif_strptime
0001:004e0db4  _php_std_date
0002:00003070  _mon_short_names
0002:000030a0  _day_full_names
0002:000030c0  _day_short_names
0002:00003040  _mon_full_names
Module: U:\dev\php-5.3.20\ext\standard\dir.obj(dir.obj)
0002:00020f20  _dir_globals_id
0001:004e0fc0  _zm_activate_dir
0001:004e1021  _zif_scandir
0001:004e12a5  _zif_glob
0001:004e1731  _php_if_readdir
0001:004e197e  _zif_getcwd
0001:004e1a0f  _zif_rewinddir
0001:004e1c12  _zif_chdir
0001:004e1e3d  _zif_closedir
0001:004e21d2  _zif_getdir
0001:004e2201  _zif_opendir
0001:004e22ba  _zm_startup_dir
Module: U:\dev\php-5.3.20\ext\standard\dl.obj(dl.obj)
0001:004e2690  _zm_info_dl
0001:004e28a9  _php_load_extension
0001:004e2c90  _php_dl
0001:004e2df6  _zif_dl
Module: U:\dev\php-5.3.20\ext\standard\dns.obj(dns.obj)
0001:004e2f82  _zif_gethostbynamel
0001:004e3036  _zif_gethostbyname
0001:004e30e7  _zif_gethostbyaddr
0001:004e31e3  _zif_gethostname
Module: U:\dev\php-5.3.20\ext\standard\exec.obj(exec.obj)
0001:004e32f8  _zif_proc_nice
0001:004e33d9  _zif_shell_exec
0001:004e351b  _php_escape_shell_arg
0001:004e3658  _zif_escapeshellarg
0001:004e36c1  _php_escape_shell_cmd
0001:004e3a6a  _zif_escapeshellcmd
0001:004e3b4a  _php_exec
0001:004e41cb  _zif_passthru
0001:004e41fa  _zif_system
0001:004e4229  _zif_exec
Module: U:\dev\php-5.3.20\ext\standard\file.obj(file.obj)
0002:00020f30  _file_globals_id
0001:004e4260  _php_le_stream_context
0001:004e429e  _zm_shutdown_file
0001:004e42a6  _zif_sys_get_temp_dir
0001:004e4384  _zif_fnmatch
0001:004e44e1  _php_next_meta_token
0001:004e4962  _zif_realpath
0001:004e4b22  _php_fgetcsv
0001:004e517f  _zif_fgetc
0001:004e524f  _zif_feof
0001:004e53f1  _zif_fgetcsv
0001:004e577a  _zif_fputcsv
0001:004e5f99  _zif_fwrite
0001:004e6154  _zif_fread
0001:004e6307  _php_copy_file_ctx
0001:004e65df  _php_copy_file_ex
0001:004e6610  _php_copy_file
0001:004e6655  _zif_copy
0001:004e6807  _php_if_fopen
0001:004e6988  _php_if_fstat
0001:004e76f5  _php_if_ftruncate
0001:004e7848  _zif_unlink
0001:004e7a5a  _zif_rename
0001:004e7c6a  _zif_fpassthru
0001:004e7d16  _zif_readfile
0001:004e7e65  _zif_umask
0001:004e7f0c  _zif_rmdir
0001:004e8019  _zif_mkdir
0001:004e8165  _zif_flock
0001:004e82ed  _php_mkdir_ex
0001:004e839b  _php_mkdir
0001:004e83c9  _zif_fseek
0001:004e849b  _zif_rewind
0001:004e8566  _zif_ftell
0001:004e8611  _zif_fflush
0001:004e86d7  _zif_fscanf
0001:004e8829  _zif_fgetss
0001:004e89d5  _zif_fgets
0001:004e8bf3  _zif_pclose
0001:004e8cce  _zif_fclose
0001:004e8dd7  _zif_popen
0001:004e90db  _php_if_tmpfile
0001:004e913a  _zif_tempnam
0001:004e931d  _zif_file_get_contents
0001:004e9625  _zif_file
0001:004e9be7  _zif_file_put_contents
0001:004ea381  _zif_get_meta_tags
0001:004eaed8  _zm_startup_file
Module: U:\dev\php-5.3.20\ext\standard\filestat.obj(filestat.obj)
0001:004ebc30  _zm_activate_filestat
0001:004ebc77  _zif_realpath_cache_get
0001:004ebe49  _zif_realpath_cache_size
0001:004ebe88  _zm_deactivate_filestat
0001:004ebfbf  _php_stat
0001:004ed53c  _php_if_stat
0001:004ed59b  _php_if_lstat
0001:004ed5fa  _zif_file_exists
0001:004ed659  _zif_is_link
0001:004ed6b8  _zif_is_dir
0001:004ed717  _zif_is_file
0001:004ed776  _zif_is_executable
0001:004ed7d5  _zif_is_readable
0001:004ed834  _zif_is_writable
0001:004ed893  _zif_filetype
0001:004ed8f2  _zif_filectime
0001:004ed951  _zif_filemtime
0001:004ed9b0  _zif_fileatime
0001:004eda0f  _zif_filegroup
0001:004eda6e  _zif_fileowner
0001:004edacd  _zif_filesize
0001:004edb2c  _zif_fileinode
0001:004edb8b  _zif_fileperms
0001:004edbea  _php_clear_stat_cache
0001:004edc99  _zif_clearstatcache
0001:004edd49  _zif_touch
0001:004edf5e  _zif_chmod
0001:004ee384  _zif_lchown
0001:004ee3bd  _zif_chown
0001:004ee646  _zif_lchgrp
0001:004ee675  _zif_chgrp
0001:004ee6a4  _zif_disk_free_space
0001:004ee77d  _zif_disk_total_space
Module: U:\dev\php-5.3.20\ext\standard\flock_compat.obj(flock_compat.obj)
0001:004ee850  _php_flock
Module: U:\dev\php-5.3.20\ext\standard\formatted_print.obj(formatted_print.obj)
0001:004f08a3  _zif_vfprintf
0001:004f09a5  _zif_fprintf
0001:004f0aa6  _zif_vsprintf
0001:004f0af4  _zif_user_sprintf
0001:004f0b3f  _zif_vprintf
0001:004f0bac  _zif_user_printf
Module: U:\dev\php-5.3.20\ext\standard\fsock.obj(fsock.obj)
0001:004f0fb8  _zif_pfsockopen
0001:004f0fe7  _zif_fsockopen
Module: U:\dev\php-5.3.20\ext\standard\head.obj(head.obj)
0001:004f1021  _zif_headers_list
0001:004f10d4  _zif_headers_sent
0001:004f137b  _php_setcookie
0001:004f1756  _zif_setrawcookie
0001:004f188b  _zif_setcookie
0001:004f19c3  _zif_header_remove
0001:004f1a35  _zif_header
0001:004f1ab1  _php_header
Module: U:\dev\php-5.3.20\ext\standard\html.obj(html.obj)
0001:004f1af0  _php_utf32_utf8
0001:004f1ed4  _zif_get_html_translation_table
0001:004f2144  _zif_htmlspecialchars_decode
0001:004f2415  _register_html_constants
0001:004f255c  _php_escape_html_entities_ex
0001:004f2e9b  _zif_htmlentities
0001:004f2eca  _zif_htmlspecialchars
0001:004f2ef9  _php_escape_html_entities
0001:004f2f56  _php_unescape_html_entities
0001:004f3632  _zif_html_entity_decode
Module: U:\dev\php-5.3.20\ext\standard\image.obj(image.obj)
0001:004f5ca7  _php_image_type_to_mime_type
0001:004f68c3  _php_getimagetype
0001:004f835f  _php_sig_gif
0001:004f836e  _php_sig_jpg
0001:004f8371  _php_sig_png
0001:004f8368  _php_sig_swf
0001:004f836b  _php_sig_swc
0001:004f8362  _php_sig_psd
0001:004f8366  _php_sig_bmp
0001:004f8381  _php_sig_jpc
0001:004f8379  _php_sig_tif_ii
0001:004f837d  _php_sig_tif_mm
0001:004f8390  _php_sig_iff
0001:004f8394  _php_sig_ico
0001:004f8384  _php_sig_jp2
0001:004f6c0e  _zif_getimagesize
0001:004f7acb  _zif_image_type_to_extension
0001:004f7e29  _zif_image_type_to_mime_type
0001:004f7fd8  _zm_startup_imagetypes
0001:004f83a0  _php_tiff_bytes_per_format
Module: U:\dev\php-5.3.20\ext\standard\info.obj(info.obj)
0001:004f84d1  _zif_php_ini_scanned_files
0001:004f850a  _zif_php_ini_loaded_file
0001:004f857b  _zif_php_sapi_name
0001:004f8614  _zif_zend_logo_guid
0001:004f868c  _zif_php_egg_logo_guid
0001:004f8704  _zif_php_real_logo_guid
0001:004f8754  _php_logo_guid
0001:004f87a2  _zif_php_logo_guid
0001:004f87f6  _zif_phpcredits
0001:004f8857  _zif_phpversion
0001:004f8a94  _register_phpinfo_constants
0001:004f8da5  _php_info_print_table_colspan_header
0001:004f8e71  _php_info_print_hr
0001:004f8ead  _php_info_print_table_end
0001:004f8ed9  _php_info_print_box_end
0001:004f8f2a  _php_info_print_table_start
0001:004f8f7e  _php_info_print_box_start
0001:004f9004  _php_info_print_table_header
0001:004f91e0  _php_info_html_esc
0001:004f9439  _php_info_print_table_row_ex
0001:004f9451  _php_info_print_table_row
0001:004f94b3  _php_info_print_module
0001:004f95ec  _php_info_html_esc_write
0001:004f9b43  _php_get_uname
0001:004f9be5  _zif_php_uname
0001:004f9c7e  _php_info_print_style
0001:004f9dc1  _php_print_info_htmlhead
0001:004fabd1  _php_print_info
0001:004fbf45  _zif_phpinfo
Module: U:\dev\php-5.3.20\ext\standard\iptc.obj(iptc.obj)
0001:004fbfea  _zif_iptcparse
0001:004fc3a9  _zif_iptcembed
Module: U:\dev\php-5.3.20\ext\standard\lcg.obj(lcg.obj)
0002:00020f40  _lcg_globals_id
0001:004fc89b  _zm_startup_lcg
0001:004fc8c9  _php_combined_lcg
0001:004fca39  _zif_lcg_value
Module: U:\dev\php-5.3.20\ext\standard\link.obj(link.obj)
0001:004fcaa8  _zif_link
0001:004fcd13  _zif_symlink
0001:004fd013  _zif_linkinfo
0001:004fd123  _zif_readlink
Module: U:\dev\php-5.3.20\ext\standard\mail.obj(mail.obj)
0001:004fd28f  _zm_info_mail
0001:004fd3f9  _php_mail
0001:004fd816  _zif_ezmlm_hash
0001:004fd946  _zif_mail
Module: U:\dev\php-5.3.20\ext\standard\math.obj(math.obj)
0001:004fde40  _zif_pi
0001:004fde54  __php_math_basetozval
0001:004fdf7a  _zif_rad2deg
0001:004fdfc5  _zif_deg2rad
0001:004fe010  _zif_is_nan
0001:004fe05d  _zif_fmod
0001:004fe0d5  __php_math_longtobase
0001:004fe15d  __php_math_zvaltobase
0001:004fe396  __php_math_basetolong
0001:004fe479  _zif_hypot
0001:004fe4ce  _zif_sqrt
0001:004fe52e  _zif_log10
0001:004fe595  _zif_log
0001:004fe685  _zif_log1p
0001:004fe6cc  _zif_expm1
0001:004fe713  _zif_exp
0001:004fe75f  _zif_pow
0001:004fe8c8  _zif_is_infinite
0001:004fe91c  _zif_is_finite
0001:004fe96b  _zif_atanh
0001:004fe9b2  _zif_acosh
0001:004fe9f9  _zif_asinh
0001:004fea40  _zif_tanh
0001:004fea87  _zif_cosh
0001:004feace  _zif_sinh
0001:004feb15  _zif_atan2
0001:004feb6a  _zif_atan
0001:004febb1  _zif_acos
0001:004febf8  _zif_asin
0001:004fec3f  _zif_tan
0001:004fec86  _zif_cos
0001:004feccd  _zif_sin
0001:004fed16  _zif_octdec
0001:004fee0f  _zif_hexdec
0001:004fef08  _zif_bindec
0001:004ff001  _zif_dechex
0001:004ff0eb  _zif_decoct
0001:004ff1d5  _zif_decbin
0001:004ff2f5  _zif_base_convert
0001:004ff480  _zif_abs
0001:004ff5ae  _zif_ceil
0001:004ff73c  _zif_floor
0001:004ff8d2  __php_math_round
0001:004ffebf  __php_math_number_format
0001:005000ed  _zif_number_format
0001:0050022b  _zif_round
Module: U:\dev\php-5.3.20\ext\standard\md5.obj(md5.obj)
0001:00500600  _make_digest_ex
0001:00500649  _make_digest
0001:00500d9a  _PHP_MD5Init
0001:00500dcb  _PHP_MD5Final
0001:00500f18  _PHP_MD5Update
0001:00500fe6  _php_if_md5_file
0001:005011c4  _php_if_md5
Module: U:\dev\php-5.3.20\ext\standard\metaphone.obj(metaphone.obj)
0001:00501314  _zif_metaphone
0002:00003150  __codes
Module: U:\dev\php-5.3.20\ext\standard\microtime.obj(microtime.obj)
0001:00502571  _zif_gettimeofday
0001:005025a0  _zif_microtime
Module: U:\dev\php-5.3.20\ext\standard\pack.obj(pack.obj)
0002:00020f50  _machine_little_endian
0001:005025e0  _zm_startup_pack
0001:00502854  _zif_unpack
0001:005036c3  _zif_pack
Module: U:\dev\php-5.3.20\ext\standard\pageinfo.obj(pageinfo.obj)
0001:00504970  _zif_getmypid
0001:0050499f  _php_statpage
0001:00504a2a  _php_getlastmod
0001:00504a54  _zif_getlastmod
0001:00504a89  _zif_getmyinode
0001:00504ad3  _php_getgid
0001:00504b10  _zif_getmygid
0001:00504b3f  _php_getuid
0001:00504b7c  _zif_getmyuid
Module: U:\dev\php-5.3.20\ext\standard\quot_print.obj(quot_print.obj)
0001:00504bb3  _zif_quoted_printable_decode
0001:00504e79  _php_quot_print_encode
0001:00504fdb  _zif_quoted_printable_encode
0001:00505067  _php_quot_print_decode
Module: U:\dev\php-5.3.20\ext\standard\rand.obj(rand.obj)
0001:00505670  _php_srand
0001:00505694  _php_mt_rand
0001:0050580d  _zif_mt_getrandmax
0001:00505846  _zif_getrandmax
0001:00505882  _zif_srand
0001:00505923  _php_rand
0001:005059b6  _zif_rand
0001:00505a64  _php_mt_srand
0001:00505bea  _zif_mt_rand
0001:00505d46  _zif_mt_srand
Module: U:\dev\php-5.3.20\ext\standard\soundex.obj(soundex.obj)
0001:00505df2  _zif_soundex
Module: U:\dev\php-5.3.20\ext\standard\string.obj(string.obj)
0001:00505f50  _php_strtoupper
0001:00505f78  _php_strtolower
0001:00505fa0  _php_strspn
0001:00505fdb  _php_strcspn
0001:0050601a  _php_strtr
0001:005061bc  _zif_ord
0001:005063ea  _zif_strcspn
0001:00506419  _zif_strspn
0001:005064af  _zif_substr_compare
0001:0050665b  _zif_strpbrk
0001:00506747  _zif_str_rot13
0001:005067c7  _zif_ucwords
0001:00506882  _zif_lcfirst
0001:00506911  _zif_ucfirst
0001:005069a5  _zif_substr
0001:00506ae2  _zif_strtolower
0001:00506b5d  _zif_strtoupper
0001:00506c11  _zif_str_split
0001:00506d4f  _zif_str_shuffle
0001:00506e1a  _zif_sscanf
0001:00506ed8  _zif_strrev
0001:00506feb  _zif_str_pad
0001:00507308  _zif_strnatcasecmp
0001:00507381  _zif_strnatcmp
0001:005073fa  _php_stripslashes
0001:00507550  _zif_stripslashes
0001:005075ca  _zif_count_chars
0001:005077a6  _zif_nl2br
0001:00507963  _php_char_to_str_ex
0001:00507c64  _php_char_to_str
0001:00508478  _zif_hebrevc
0001:005084a7  _zif_hebrev
0001:00508509  _zif_chunk_split
0001:00508793  _zif_bin2hex
0001:00508881  _zif_str_repeat
0001:005089e7  _zif_str_getcsv
0001:00508aff  _php_addslashes_ex
0001:00508c70  _php_addslashes
0001:00508ca7  _zif_addslashes
0001:00508d55  _zif_quotemeta
0001:00508f36  _php_tag_find
0001:00509063  _php_strip_tags_ex
0001:00509bc0  _php_strip_tags
0001:00509c11  _php_stripcslashes
0001:00509ee7  _zif_stripcslashes
0001:00509f53  _zif_similar_text
0001:0050a099  _zif_chr
0001:0050a126  _zif_strtok
0001:0050a3b4  _php_dirname
0001:0050a3c0  _zif_dirname
0001:0050a42b  _php_basename
0001:0050a5aa  _zif_basename
0001:0050a68f  _zif_wordwrap
0001:0050ac01  _zif_strcoll
0001:0050ac7c  _zif_nl_langinfo
0001:0050aef1  _zm_startup_nl_langinfo
0001:0050b993  _register_string_constants
0001:0050bc3c  _zm_shutdown_localeconv
0001:0050bc5d  _zm_startup_localeconv
0001:0050bc71  _localeconv_r
0001:0050bdb1  _zif_localeconv
0001:0050c191  _zif_parse_str
0001:0050c396  _zif_setlocale
0001:0050c870  _zif_strtr
0001:0050d02d  _php_implode
0001:0050d7d7  _zif_implode
0001:0050dada  _zif_pathinfo
0001:0050dfd3  _zif_strrchr
0001:0050e11d  _zif_strripos
0001:0050e492  _zif_strrpos
0001:0050e6cb  _zif_stripos
0001:0050e8c1  _zif_strip_tags
0001:0050eac3  _zif_substr_replace
0001:0050fae0  _php_addcslashes
0001:0050fe53  _zif_addcslashes
0001:0050ff2f  _php_trim
0001:0051039c  _zif_ltrim
0001:005103cb  _zif_rtrim
0001:005103fa  _zif_trim
0001:005104d7  _zif_substr_count
0001:0051075e  _php_explode_negative_limit
0001:005109e2  _php_stristr
0001:00510af7  _zif_stristr
0001:00510c9e  _php_explode
0001:00510ec7  _zif_explode
0001:00511036  _php_str_to_str_ex
0001:00511978  _php_str_to_str
0001:00512543  _zif_str_ireplace
0001:00512572  _zif_str_replace
0001:005125ba  _zif_str_word_count
0001:005129e6  _zif_strstr
0001:00512be5  _zif_strpos
Module: U:\dev\php-5.3.20\ext\standard\scanf.obj(scanf.obj)
0001:00512f09  _ValidateFormat
0001:00513545  _php_sscanf_internal
Module: U:\dev\php-5.3.20\ext\standard\syslog.obj(syslog.obj)
0001:00514916  _zif_syslog
0001:0051497f  _zif_closelog
0001:005149f3  _zm_shutdown_syslog
0001:00514a3d  _zif_openlog
0001:00514c4e  _zm_startup_syslog
0001:005179fe  _zif_define_syslog_variables
0001:00517a64  _zm_activate_syslog
Module: U:\dev\php-5.3.20\ext\standard\type.obj(type.obj)
0001:00517ad2  _zif_is_scalar
0001:00517b3c  _zif_is_callable
0001:00517c7a  _zif_is_numeric
0001:00517f55  _zif_is_object
0001:00517f84  _zif_is_array
0001:00517fb3  _zif_is_string
0001:00517fe2  _zif_is_float
0001:00518011  _zif_is_long
0001:00518040  _zif_is_bool
0001:0051806f  _zif_is_resource
0001:0051809e  _zif_is_null
0001:005180cd  _zif_strval
0001:0051818f  _zif_floatval
0001:0051820f  _zif_intval
0001:00518361  _zif_settype
0001:00518587  _zif_gettype
Module: U:\dev\php-5.3.20\ext\standard\uniqid.obj(uniqid.obj)
0001:0051877f  _zif_uniqid
Module: U:\dev\php-5.3.20\ext\standard\url.obj(url.obj)
0001:005188c0  _php_replace_controlchars_ex
0001:0051893f  _php_url_decode
0001:00518a14  _php_raw_url_decode
0001:00518ada  _zif_get_headers
0001:00518f2c  _zif_rawurldecode
0001:00518f97  _zif_urldecode
0001:00519002  _php_raw_url_encode
0001:005190da  _zif_rawurlencode
0001:0051913c  _php_url_encode
0001:005191f3  _zif_urlencode
0001:00519255  _php_replace_controlchars
0001:00519286  _php_url_parse_ex
0001:00519b28  _php_url_parse
0001:00519b54  _php_url_free
0001:00519c28  _zif_parse_url
Module: U:\dev\php-5.3.20\ext\standard\var.obj(var.obj)
0001:00519f53  _zif_memory_get_peak_usage
0001:00519fb6  _zif_memory_get_usage
0001:0051a03c  _zif_unserialize
0001:0051a5c5  _php_var_export_ex
0001:0051b4ea  _zif_var_export
0001:0051b5b4  _php_var_export
0001:0051c450  _php_debug_zval_dump
0001:0051c946  _zif_debug_zval_dump
0001:0051cc2c  _php_var_dump
0001:0051d07d  _zif_var_dump
0001:005212a2  _php_var_serialize
0001:005212d6  _zif_serialize
Module: U:\dev\php-5.3.20\ext\standard\versioning.obj(versioning.obj)
0001:0052149b  _php_canonicalize_version
0001:005216e2  _php_version_compare
0001:00521a1d  _zif_version_compare
Module: U:\dev\php-5.3.20\ext\standard\assert.obj(assert.obj)
0002:00020f58  _assert_globals_id
0001:00521e26  _zm_deactivate_assert
0001:00521eba  _zif_assert_options
0001:005224cc  _zif_assert
0001:00522a2f  _zm_info_assert
0001:00522a3b  _zm_shutdown_assert
0001:00522ac6  _zm_startup_assert
Module: U:\dev\php-5.3.20\ext\standard\strnatcmp.obj(strnatcmp.obj)
0001:00522f50  _strnatcmp_ex
Module: U:\dev\php-5.3.20\ext\standard\levenshtein.obj(levenshtein.obj)
0001:005235bd  _zif_levenshtein
Module: U:\dev\php-5.3.20\ext\standard\incomplete_class.obj(incomplete_class.obj)
0001:0052379c  _php_store_class_name
0001:0052384f  _php_lookup_class_name
0001:005238ee  _php_create_incomplete_class
Module: U:\dev\php-5.3.20\ext\standard\url_scanner_ex.obj(url_scanner_ex.obj)
0001:00523d40  _php_url_scanner_reset_vars
0001:00523d6a  _zm_activate_url_scanner_ex
0001:00523d8a  _zm_deactivate_url_scanner_ex
0001:00523f0d  _zm_shutdown_url_scanner_ex
0001:00523f29  _zm_startup_url_scanner_ex
0001:005247cf  _php_url_scanner_adapt_single_url
0001:00524a7e  _php_url_scanner_add_var
Module: U:\dev\php-5.3.20\ext\standard\ftp_fopen_wrapper.obj(ftp_fopen_wrapper.obj)
0001:00529b18  _php_stream_ftp_opendir
0001:0052a105  _php_stream_url_wrap_ftp
0002:000031f0  _php_stream_ftp_wrapper
Module: U:\dev\php-5.3.20\ext\standard\http_fopen_wrapper.obj(http_fopen_wrapper.obj)
0001:0052afb8  _php_stream_url_wrap_http_ex
0001:0052ea3c  _php_stream_url_wrap_http
0002:00003270  _php_stream_http_wrapper
Module: U:\dev\php-5.3.20\ext\standard\php_fopen_wrapper.obj(php_fopen_wrapper.obj)
0001:0052efcb  _php_stream_url_wrap_php
0002:000032f0  _php_stream_input_ops
0002:000032c0  _php_stream_output_ops
0002:00003320  _php_stream_php_wrapper
Module: U:\dev\php-5.3.20\ext\standard\credits.obj(credits.obj)
0001:005311c6  _php_print_credits
Module: U:\dev\php-5.3.20\ext\standard\css.obj(css.obj)
0001:00532491  _php_info_print_css
Module: U:\dev\php-5.3.20\ext\standard\var_unserializer.obj(var_unserializer.obj)
0001:00532670  _var_replace
0001:00532710  _var_push_dtor
0001:00532794  _var_destroy
0001:00532a4a  _php_var_unserialize
Module: U:\dev\php-5.3.20\ext\standard\ftok.obj(ftok.obj)
0001:00534748  _zif_ftok
Module: U:\dev\php-5.3.20\ext\standard\sha1.obj(sha1.obj)
0001:005348a0  _PHP_SHA1Init
0001:00535fbe  _PHP_SHA1Update
0001:00536093  _PHP_SHA1Final
0001:0053615f  _make_sha1_digest
0001:00536188  _zif_sha1_file
0001:00536370  _zif_sha1
Module: U:\dev\php-5.3.20\ext\standard\user_filters.obj(user_filters.obj)
0001:005364b0  _zif_user_filter_nop
0001:005364f4  _zif_stream_filter_register
0001:00536cbd  _zif_stream_get_filters
0001:00536dc5  _zif_stream_bucket_new
0001:0053701d  _zif_stream_bucket_make_writeable
0001:0053743f  _zif_stream_bucket_append
0001:0053746f  _zif_stream_bucket_prepend
0001:0053750e  _userfilter_filter
0001:00537912  _zm_deactivate_user_filters
0001:005379f8  _zm_startup_user_filters
Module: U:\dev\php-5.3.20\ext\standard\uuencode.obj(uuencode.obj)
0001:00537e80  _php_uuencode
0001:00538164  _zif_convert_uuencode
0001:005381da  _php_uudecode
0001:00538434  _zif_convert_uudecode
Module: U:\dev\php-5.3.20\ext\standard\filters.obj(filters.obj)
0001:00538e14  _zm_shutdown_standard_filters
0001:00539e0b  _zm_startup_standard_filters
0002:000033c0  _consumed_filter_factory
Module: U:\dev\php-5.3.20\ext\standard\proc_open.obj(proc_open.obj)
0001:0053bc5a  _zif_proc_get_status
0001:0053bebe  _zif_proc_close
0001:0053c067  _zif_proc_terminate
0001:0053c119  _zm_startup_proc_open
0001:0053c40b  _zif_proc_open
Module: U:\dev\php-5.3.20\ext\standard\streamsfuncs.obj(streamsfuncs.obj)
0001:0053d78a  _zif_stream_socket_shutdown
0001:0053d84e  _zif_stream_supports_lock
0001:0053d918  _zif_stream_set_read_buffer
0001:0053da17  _zif_stream_set_write_buffer
0001:0053db1b  _zif_stream_set_timeout
0001:0053dc39  _zif_stream_set_blocking
0001:0053dd12  _zif_stream_is_local
0001:0053de92  _zif_stream_resolve_include_path
0001:0053df5e  _zif_stream_socket_enable_crypto
0001:0053e159  _zif_stream_get_line
0001:0053e31a  _zif_stream_filter_remove
0001:0053e717  _zif_stream_filter_append
0001:0053e747  _zif_stream_filter_prepend
0001:0053ea22  _zif_stream_context_create
0001:0053ecb8  _zif_stream_context_set_default
0001:0053ed4f  _zif_stream_context_get_default
0001:0053eea5  _zif_stream_context_get_params
0001:0053f010  _zif_stream_context_set_params
0001:0053f0a6  _zif_stream_context_get_options
0001:0053f19b  _zif_stream_context_set_option
0001:0053f696  _zif_stream_select
0001:0053fc1d  _zif_stream_get_wrappers
0001:0053fd00  _zif_stream_get_transports
0001:0053fe35  _zif_stream_get_meta_data
0001:00540129  _zif_stream_copy_to_stream
0001:005402c4  _zif_stream_get_contents
0001:0054054a  _zif_stream_socket_sendto
0001:005406d1  _zif_stream_socket_get_name
0001:005407e3  _zif_stream_socket_pair
0001:00540945  _zif_stream_socket_accept
0001:00540b9c  _zif_stream_socket_recvfrom
0001:00540e00  _zif_stream_socket_client
0001:005411f0  _zif_stream_socket_server
Module: U:\dev\php-5.3.20\ext\standard\http.obj(http.obj)
0001:00541516  _php_url_encode_hash_ex
0001:005421a8  _zif_http_build_query
Module: U:\dev\php-5.3.20\ext\tokenizer\tokenizer.obj(tokenizer.obj)
0001:00542372  _zif_token_name
0001:005423df  _zif_token_get_all
0001:00542723  _zm_info_tokenizer
0001:00542750  _zm_startup_tokenizer
0001:00542790  _tokenizer_functions
0002:000034f0  _tokenizer_module_entry
Module: U:\dev\php-5.3.20\ext\tokenizer\tokenizer_data.obj(tokenizer_data.obj)
0001:00542868  _get_token_type_name
0001:00542e07  _tokenizer_register_constants
Module: U:\dev\php-5.3.20\ext\xml\xml.obj(xml.obj)
0002:00020f68  _xml_globals_id
0001:005445d4  _zif_xml_parser_get_option
0001:0054479d  _zif_xml_parser_set_option
0001:00544bb8  _zif_xml_parser_free
0001:00544c83  _zif_xml_get_current_byte_index
0001:00544d19  _zif_xml_get_current_column_number
0001:00544daf  _zif_xml_get_current_line_number
0001:00544e47  _zif_xml_error_string
0001:00544eb5  _zif_xml_get_error_code
0001:00544f50  _zif_xml_parse
0001:00545033  _zif_xml_parse_into_struct
0001:00546866  __xml_defaultHandler
0001:00547d81  __xml_endElementHandler
0001:005478fa  __xml_startElementHandler
0001:00546956  __xml_characterDataHandler
0001:00545201  _zif_xml_set_object
0001:005453cd  _zif_xml_set_end_namespace_decl_handler
0001:0054659d  __xml_endNamespaceDeclHandler
0001:00545483  _zif_xml_set_default_handler
0001:00545539  _zif_xml_set_character_data_handler
0001:005455f3  _zif_xml_set_element_handler
0001:005456c3  _zif_xml_set_start_namespace_decl_handler
0001:005465ff  __xml_startNamespaceDeclHandler
0001:00545779  _zif_xml_set_external_entity_ref_handler
0001:00546671  __xml_externalEntityRefHandler
0001:0054582f  _zif_xml_set_notation_decl_handler
0001:0054672a  __xml_notationDeclHandler
0001:005458e5  _zif_xml_set_unparsed_entity_decl_handler
0001:005467bc  __xml_unparsedEntityDeclHandler
0001:0054599b  _zif_xml_set_processing_instruction_handler
0001:005468c9  __xml_processingInstructionHandler
0001:00545c99  _zif_xml_parser_create_ns
0001:00545cc8  _zif_xml_parser_create
0001:0054610e  __xml_zval_strdup
0001:0054615f  _xml_utf8_decode
0001:0054649f  _zif_utf8_decode
0001:00546d65  _xml_utf8_encode
0001:00546eae  _zif_utf8_encode
0001:00546f67  _zm_info_xml
0001:00547295  _zm_startup_xml
0001:005481f0  _xml_functions
0002:000035b0  _xml_encodings
0002:00003550  _xml_module_entry
Module: U:\dev\php-5.3.20\ext\xml\compat.obj(compat.obj)
0001:00548c0c  _php_XML_SetUserData
0001:00548c1a  _XML_GetUserData
0001:00548c25  _php_XML_SetElementHandler
0001:00548c39  _php_XML_SetCharacterDataHandler
0001:00548c47  _php_XML_SetProcessingInstructionHandler
0001:00548c55  _php_XML_SetCommentHandler
0001:00548c63  _php_XML_SetDefaultHandler
0001:00548c71  _php_XML_SetUnparsedEntityDeclHandler
0001:00548c7f  _php_XML_SetNotationDeclHandler
0001:00548c8d  _php_XML_SetExternalEntityRefHandler
0001:00548c9b  _php_XML_SetStartNamespaceDeclHandler
0001:00548ca9  _php_XML_SetEndNamespaceDeclHandler
0001:00548cb7  _php_XML_GetErrorCode
0001:00548ccd  _php_XML_ErrorString
0001:00548ce6  _php_XML_GetCurrentLineNumber
0001:00548cf7  _php_XML_GetCurrentColumnNumber
0001:00548d08  _php_XML_GetCurrentByteIndex
0001:00548d1f  _php_XML_GetCurrentByteCount
0001:00548d3a  _php_XML_ExpatVersion
0001:00548d44  _php_XML_ParserFree
0001:00548d95  _php_XML_Parse
0001:00548de0  _php_XML_ParserCreate_MM
0001:00548e9d  _php_XML_ParserCreateNS
0001:00548ec9  _php_XML_ParserCreate
Module: U:\dev\php-5.3.20\ext\xmlreader\php_xmlreader.obj(php_xmlreader.obj)
0002:00020f78  _xmlreader_class_entry
0001:0054a510  _xmlreader_objects_clone
0001:0054a527  _zm_info_xmlreader
0001:0054a554  _zm_shutdown_xmlreader
0001:0054a5bb  _zim_xmlreader_moveToNextAttribute
0001:0054a5e7  _zim_xmlreader_moveToFirstAttribute
0001:0054a616  _zim_xmlreader_moveToElement
0001:0054a645  _zim_xmlreader_isValid
0001:0054a712  _zim_xmlreader_expand
0001:0054a95e  _zim_xmlreader_XML
0001:0054abcb  _zim_xmlreader_close
0001:0054ac17  _zim_xmlreader_setParserProperty
0001:0054ad3b  _zim_xmlreader_setSchema
0001:0054ae97  _zim_xmlreader_readString
0001:0054aec6  _zim_xmlreader_readOuterXml
0001:0054aef5  _zim_xmlreader_readInnerXml
0001:0054b033  _zim_xmlreader_lookupNamespace
0001:0054b062  _zim_xmlreader_getAttribute
0001:0054b0d4  _zim_xmlreader_next
0001:0054b200  _zim_xmlreader_read
0001:0054b2b9  _zim_xmlreader_moveToAttributeNs
0001:0054b3a0  _zim_xmlreader_moveToAttributeNo
0001:0054b437  _zim_xmlreader_moveToAttribute
0001:0054b4f9  _zim_xmlreader_getParserProperty
0001:0054b599  _zim_xmlreader_getAttributeNs
0001:0054b6c0  _zim_xmlreader_getAttributeNo
0001:0054b780  _xmlreader_objects_new
0001:0054b83a  _xmlreader_objects_free_storage
0001:0054b884  __xmlreader_get_valid_file_path
0001:0054b976  _zim_xmlreader_open
0001:0054bb53  _xmlreader_write_property
0001:0054bc67  _xmlreader_read_property
0001:0054be89  _xmlreader_get_property_ptr_ptr
0001:0054c0f2  _zim_xmlreader_setRelaxNGSchemaSource
0001:0054c121  _zim_xmlreader_setRelaxNGSchema
0001:0054c30c  _zm_startup_xmlreader
0002:00003660  _xmlreader_module_entry
Module: U:\dev\php-5.3.20\ext\xmlrpc\xmlrpc-epi-php.obj(xmlrpc-epi-php.obj)
0001:0054d26f  _xmlrpc_type_as_str
0001:0054d340  _zif_xmlrpc_is_fault
0001:0054d4d2  _set_zval_xmlrpc_type
0001:0054d705  _xmlrpc_str_as_vector_type
0001:0054d7e4  _xmlrpc_str_as_type
0001:0054d8ee  _zif_xmlrpc_set_type
0001:0054d992  _get_zval_xmlrpc_type
0001:0054daf0  _zif_xmlrpc_get_type
0001:0054e19f  _zif_xmlrpc_parse_method_descriptions
0001:0054e2f5  _zif_xmlrpc_server_register_introspection_callback
0001:0054e7ee  _zif_xmlrpc_server_add_introspection_data
0001:0054ed54  _zif_xmlrpc_encode_request
0001:0054eebe  _zif_xmlrpc_server_register_method
0001:0054efc2  _zif_xmlrpc_server_destroy
0001:0054f045  _zif_xmlrpc_server_create
0001:0054f12e  _zif_xmlrpc_encode
0001:0054f268  _zm_info_xmlrpc
0001:0054f314  _zm_startup_xmlrpc
0001:0054f905  _decode_request_worker
0001:0054f9f0  _zif_xmlrpc_decode
0001:0054fac0  _zif_xmlrpc_decode_request
0001:0054fb99  _zif_xmlrpc_server_call_method
0001:00550080  _xmlrpc_functions
0002:000036c0  _xmlrpc_module_entry
Module: U:\dev\php-5.3.20\ext\xmlwriter\php_xmlwriter.obj(php_xmlwriter.obj)
0002:00003720  _xmlwriter_module_entry
Module: U:\dev\php-5.3.20\ext\zip\php_zip.obj(php_zip.obj)
0001:00558ea6  _php_zip_pcre
0001:0055931e  _php_zip_glob
0002:00003780  _zip_module_entry
Module: U:\dev\php-5.3.20\ext\zip\zip_stream.obj(zip_stream.obj)
0001:0055c179  _php_stream_zip_opener
0001:0055c382  _php_stream_zip_open
0002:000037e0  _php_stream_zipio_ops
0002:00003810  _php_stream_zip_wrapper
Module: U:\dev\php-5.3.20\ext\zip\lib\zip_add.obj(zip_add.obj)
0001:0055c4a0  _zip_add
Module: U:\dev\php-5.3.20\ext\zip\lib\zip_error.obj(zip_error.obj)
0001:0055c500  __zip_error_clear
0001:0055c515  __zip_error_copy
0001:0055c52a  __zip_error_init
0001:0055c546  __zip_error_set
0001:0055c55d  __zip_error_set_from_source
0001:0055c595  __zip_error_get
0001:0055c5d9  __zip_error_fini
Module: U:\dev\php-5.3.20\ext\zip\lib\zip_fclose.obj(zip_fclose.obj)
0001:0055c600  _zip_fclose
Module: U:\dev\php-5.3.20\ext\zip\lib\zip_fread.obj(zip_fread.obj)
0001:0055c680  _zip_fread
Module: U:\dev\php-5.3.20\ext\zip\lib\zip_open.obj(zip_open.obj)
0001:0055ca94  __zip_open
0001:0055d2a7  _zip_open
Module: U:\dev\php-5.3.20\ext\zip\lib\zip_source_filep.obj(zip_source_filep.obj)
0001:0055d390  __zip_source_file_or_p
0001:0055d4f3  _zip_source_filep
Module: U:\dev\php-5.3.20\ext\zip\lib\zip_strerror.obj(zip_strerror.obj)
0001:0055d910  _zip_strerror
Module: U:\dev\php-5.3.20\ext\zip\lib\zip_close.obj(zip_close.obj)
0001:0055d920  __zip_changed
0001:0055dc8c  _zip_close
Module: U:\dev\php-5.3.20\ext\zip\lib\zip_error_get.obj(zip_error_get.obj)
0001:0055ede0  _zip_error_get
Module: U:\dev\php-5.3.20\ext\zip\lib\zip_file_error_get.obj(zip_file_error_get.obj)
0001:0055ee00  _zip_file_error_get
Module: U:\dev\php-5.3.20\ext\zip\lib\zip_free.obj(zip_free.obj)
0001:0055ee20  __zip_free
Module: U:\dev\php-5.3.20\ext\zip\lib\zip_rename.obj(zip_rename.obj)
0001:0055ef50  _zip_rename
Module: U:\dev\php-5.3.20\ext\zip\lib\zip_source_free.obj(zip_source_free.obj)
0001:0055f060  _zip_source_free
Module: U:\dev\php-5.3.20\ext\zip\lib\zip_unchange_all.obj(zip_unchange_all.obj)
0001:0055f110  _zip_unchange_all
Module: U:\dev\php-5.3.20\ext\zip\lib\zip_delete.obj(zip_delete.obj)
0001:0055f170  _zip_delete
Module: U:\dev\php-5.3.20\ext\zip\lib\zip_error_get_sys_type.obj(zip_error_get_sys_type.obj)
0001:0055f220  _zip_error_get_sys_type
Module: U:\dev\php-5.3.20\ext\zip\lib\zip_file_get_offset.obj(zip_file_get_offset.obj)
0001:0055f240  __zip_file_get_offset
Module: U:\dev\php-5.3.20\ext\zip\lib\zip_get_name.obj(zip_get_name.obj)
0001:0055f310  __zip_get_name
0001:0055f3d1  _zip_get_name
Module: U:\dev\php-5.3.20\ext\zip\lib\zip_replace.obj(zip_replace.obj)
0001:0055f400  __zip_replace
0001:0055f506  _zip_replace
Module: U:\dev\php-5.3.20\ext\zip\lib\zip_source_function.obj(zip_source_function.obj)
0001:0055f580  __zip_source_new
0001:0055f5e0  _zip_source_function
Module: U:\dev\php-5.3.20\ext\zip\lib\zip_unchange.obj(zip_unchange.obj)
0001:0055f610  __zip_unchange
0001:0055f765  _zip_unchange
Module: U:\dev\php-5.3.20\ext\zip\lib\zip_dirent.obj(zip_dirent.obj)
0001:0055f790  __zip_dirent_init
0001:0055f80c  __zip_read2
0001:0055f829  __zip_read4
0001:0055f858  __zip_u2d_time
0001:0055f939  __zip_dirent_write
0001:0055fb35  __zip_dirent_torrent_normalize
0001:0055fc1d  __zip_dirent_finalize
0001:0055fc63  __zip_cdir_free
0001:0055fd7c  __zip_cdir_new
0001:0055fea6  __zip_dirent_read
0001:005603e4  __zip_cdir_write
0001:0056050e  __zip_cdir_grow
Module: U:\dev\php-5.3.20\ext\zip\lib\zip_error_strerror.obj(zip_error_strerror.obj)
0001:005605ac  __zip_error_strerror
Module: U:\dev\php-5.3.20\ext\zip\lib\zip_filerange_crc.obj(zip_filerange_crc.obj)
0001:005606f0  __zip_filerange_crc
Module: U:\dev\php-5.3.20\ext\zip\lib\zip_file_strerror.obj(zip_file_strerror.obj)
0001:00560830  _zip_file_strerror
Module: U:\dev\php-5.3.20\ext\zip\lib\zip_get_num_files.obj(zip_get_num_files.obj)
0001:00560840  _zip_get_num_files
Module: U:\dev\php-5.3.20\ext\zip\lib\zip_get_archive_flag.obj(zip_get_archive_flag.obj)
0001:00560860  _zip_get_archive_flag
Module: U:\dev\php-5.3.20\ext\zip\lib\zip_set_archive_flag.obj(zip_set_archive_flag.obj)
0001:00560890  _zip_set_archive_flag
Module: U:\dev\php-5.3.20\ext\zip\lib\zip_set_name.obj(zip_set_name.obj)
0001:00560940  __zip_set_name
Module: U:\dev\php-5.3.20\ext\zip\lib\zip_source_zip.obj(zip_source_zip.obj)
0001:00560a70  _zip_source_zip
Module: U:\dev\php-5.3.20\ext\zip\lib\zip_unchange_data.obj(zip_unchange_data.obj)
0001:00560f00  __zip_unchange_data
Module: U:\dev\php-5.3.20\ext\zip\lib\zip_entry_free.obj(zip_entry_free.obj)
0001:00560f40  __zip_entry_free
Module: U:\dev\php-5.3.20\ext\zip\lib\zip_error_to_str.obj(zip_error_to_str.obj)
0001:00560fbc  _zip_error_to_str
Module: U:\dev\php-5.3.20\ext\zip\lib\zip_fopen.obj(zip_fopen.obj)
0001:00561070  _zip_fopen
Module: U:\dev\php-5.3.20\ext\zip\lib\zip_name_locate.obj(zip_name_locate.obj)
0001:005610c0  __zip_name_locate
0001:0056121d  _zip_name_locate
Module: U:\dev\php-5.3.20\ext\zip\lib\zip_source_buffer.obj(zip_source_buffer.obj)
0001:00561250  _zip_source_buffer
Module: U:\dev\php-5.3.20\ext\zip\lib\zip_stat.obj(zip_stat.obj)
0001:00561470  _zip_stat
Module: U:\dev\php-5.3.20\ext\zip\lib\zip_entry_new.obj(zip_entry_new.obj)
0001:005614d0  __zip_entry_new
Module: U:\dev\php-5.3.20\ext\zip\lib\zip_err_str.obj(zip_err_str.obj)
0001:00561870  __zip_err_str
0001:005618e0  __zip_nerr_str
0001:005618f0  __zip_err_type
Module: U:\dev\php-5.3.20\ext\zip\lib\zip_fopen_index.obj(zip_fopen_index.obj)
0001:00561960  _zip_fopen_index
Module: U:\dev\php-5.3.20\ext\zip\lib\zip_get_archive_comment.obj(zip_get_archive_comment.obj)
0001:00561990  _zip_get_archive_comment
Module: U:\dev\php-5.3.20\ext\zip\lib\zip_get_file_comment.obj(zip_get_file_comment.obj)
0001:005619e0  _zip_get_file_comment
Module: U:\dev\php-5.3.20\ext\zip\lib\zip_new.obj(zip_new.obj)
0001:00561a90  __zip_new
Module: U:\dev\php-5.3.20\ext\zip\lib\zip_source_file.obj(zip_source_file.obj)
0001:00561b50  _zip_source_file
Module: U:\dev\php-5.3.20\ext\zip\lib\zip_stat_index.obj(zip_stat_index.obj)
0001:00561be0  _zip_stat_index
Module: U:\dev\php-5.3.20\ext\zip\lib\zip_set_archive_comment.obj(zip_set_archive_comment.obj)
0001:00561d90  _zip_set_archive_comment
Module: U:\dev\php-5.3.20\ext\zip\lib\zip_set_file_comment.obj(zip_set_file_comment.obj)
0001:00561e40  _zip_set_file_comment
Module: U:\dev\php-5.3.20\ext\zip\lib\zip_unchange_archive.obj(zip_unchange_archive.obj)
0001:00561f30  _zip_unchange_archive
Module: U:\dev\php-5.3.20\ext\zip\lib\zip_memdup.obj(zip_memdup.obj)
0001:00561f70  __zip_memdup
Module: U:\dev\php-5.3.20\ext\zip\lib\zip_stat_init.obj(zip_stat_init.obj)
0001:00561fd0  _zip_stat_init
Module: U:\dev\php-5.3.20\ext\zip\lib\zip_add_dir.obj(zip_add_dir.obj)
0001:00562030  _zip_add_dir
Module: U:\dev\php-5.3.20\ext\zip\lib\zip_error_clear.obj(zip_error_clear.obj)
0001:005621a0  _zip_error_clear
Module: U:\dev\php-5.3.20\ext\zip\lib\zip_file_error_clear.obj(zip_file_error_clear.obj)
0001:005621b0  _zip_file_error_clear
Module: U:\dev\php-5.3.20\ext\zip\lib\zip_fdopen.obj(zip_fdopen.obj)
0001:005621c3  _zip_fdopen
Module: U:\dev\php-5.3.20\ext\zip\lib\zip_fopen_encrypted.obj(zip_fopen_encrypted.obj)
0001:00562250  _zip_fopen_encrypted
Module: U:\dev\php-5.3.20\ext\zip\lib\zip_fopen_index_encrypted.obj(zip_fopen_index_encrypted.obj)
0001:005622a0  _zip_fopen_index_encrypted
Module: U:\dev\php-5.3.20\ext\zip\lib\zip_get_compression_implementation.obj(zip_get_compression_implementation.obj)
0001:005626f0  _zip_get_compression_implementation
Module: U:\dev\php-5.3.20\ext\zip\lib\zip_get_encryption_implementation.obj(zip_get_encryption_implementation.obj)
0001:00562710  _zip_get_encryption_implementation
Module: U:\dev\php-5.3.20\ext\zip\lib\zip_get_file_extra.obj(zip_get_file_extra.obj)
0001:00562730  _zip_get_file_extra
Module: U:\dev\php-5.3.20\ext\zip\lib\zip_get_num_entries.obj(zip_get_num_entries.obj)
0001:005627e0  _zip_get_num_entries
Module: U:\dev\php-5.3.20\ext\zip\lib\zip_set_default_password.obj(zip_set_default_password.obj)
0001:00562820  _zip_set_default_password
Module: U:\dev\php-5.3.20\ext\zip\lib\zip_set_file_extra.obj(zip_set_file_extra.obj)
0001:00562890  _zip_set_file_extra
Module: U:\dev\php-5.3.20\ext\zip\lib\zip_source_close.obj(zip_source_close.obj)
0001:00562980  _zip_source_close
Module: U:\dev\php-5.3.20\ext\zip\lib\zip_source_crc.obj(zip_source_crc.obj)
0001:00562a10  _zip_source_crc
Module: U:\dev\php-5.3.20\ext\zip\lib\zip_source_deflate.obj(zip_source_deflate.obj)
0001:00562cb0  _zip_source_deflate
Module: U:\dev\php-5.3.20\ext\zip\lib\zip_source_error.obj(zip_source_error.obj)
0001:005633d0  _zip_source_error
Module: U:\dev\php-5.3.20\ext\zip\lib\zip_source_layered.obj(zip_source_layered.obj)
0001:005634a0  _zip_source_layered
Module: U:\dev\php-5.3.20\ext\zip\lib\zip_source_open.obj(zip_source_open.obj)
0001:005634d0  _zip_source_open
Module: U:\dev\php-5.3.20\ext\zip\lib\zip_source_pkware.obj(zip_source_pkware.obj)
0001:005636bf  _zip_source_pkware
Module: U:\dev\php-5.3.20\ext\zip\lib\zip_source_pop.obj(zip_source_pop.obj)
0001:00563a10  _zip_source_pop
Module: U:\dev\php-5.3.20\ext\zip\lib\zip_source_read.obj(zip_source_read.obj)
0001:00563ab0  _zip_source_read
Module: U:\dev\php-5.3.20\ext\zip\lib\zip_source_stat.obj(zip_source_stat.obj)
0001:00563b90  _zip_source_stat
Module: U:\dev\php-5.3.20\ext\mysqlnd\mysqlnd.obj(mysqlnd.obj)
0001:005642cf  _mysqlnd_get_client_info
0001:005642d9  _mysqlnd_get_client_version
0001:0056438d  _mysqlnd_field_type_name
0001:0056453e  __mysqlnd_init
0001:005645f4  _mysqlnd_connect
0001:005646ac  _mysqlnd_conn_get_methods
0001:005646b6  _mysqlnd_conn_set_methods
0001:005646c3  _mysqlnd_plugin_register
0001:005646d6  _mysqlnd_plugin_count
0001:005646e0  __mysqlnd_plugin_get_plugin_connection_data
0001:00564702  _mysqlnd_library_init
0001:00566630  _mysqlnd_library_end
0001:00566a17  _php_mysqlnd_conn_list_fields_pub
0001:005674fa  _php_mysqlnd_conn_list_method_pub
0001:00567625  _mysqlnd_old_escape_string
0001:00569595  _mysqlnd_stream_array_check_for_readiness
0001:00569736  __mysqlnd_poll
0001:005699a4  _mysqlnd_old_passwd
0001:005699a8  _mysqlnd_server_gone
0001:005699ac  _mysqlnd_out_of_sync
0001:005699b0  _mysqlnd_out_of_memory
0002:0001b7d0  _mysqlnd_global_stats
Module: U:\dev\php-5.3.20\ext\mysqlnd\mysqlnd_charset.obj(mysqlnd_charset.obj)
0001:00569f5e  _mysqlnd_find_charset_nr
0001:0056af20  _mysqlnd_charsets
0001:00569f80  _mysqlnd_cset_escape_quotes
0001:0056a047  _mysqlnd_cset_escape_slashes
0001:0056a1ac  _mysqlnd_find_charset_name
Module: U:\dev\php-5.3.20\ext\mysqlnd\mysqlnd_wireprotocol.obj(mysqlnd_wireprotocol.obj)
0001:0056c780  _php_mysqlnd_net_field_length
0001:0056c7e4  _php_mysqlnd_net_field_length_ll
0001:0056c856  _php_mysqlnd_net_store_length
0001:0056cdbb  _mysqlnd_protocol_free
0001:0056cde2  _mysqlnd_protocol_get_methods
0001:0056d588  _php_mysqlnd_cmd_write
0001:0056da38  __mysqlnd_plugin_get_plugin_protocol_data
0001:0056da5e  _mysqlnd_protocol_init
0001:0056dab7  _php_mysqlnd_rowp_read_binary_protocol
0001:0056e0cf  _php_mysqlnd_rowp_read_text_protocol
0001:0056e8d5  _php_mysqlnd_scramble
0001:00572770  _mysqlnd_empty_string
0001:00572780  _mysqlnd_read_header_name
0001:005727a0  _mysqlnd_read_body_name
0001:005728f0  _mysqlnd_command_to_text
Module: U:\dev\php-5.3.20\ext\mysqlnd\mysqlnd_loaddata.obj(mysqlnd_loaddata.obj)
0001:00572a00  _mysqlnd_local_infile_default
0001:00572a4b  _mysqlnd_handle_local_infile
0001:00572d5c  _mysqlnd_set_local_infile_handler
Module: U:\dev\php-5.3.20\ext\mysqlnd\mysqlnd_net.obj(mysqlnd_net.obj)
0001:005733f4  _php_mysqlnd_net_consume_uneaten_data_pub
0001:005734e4  _mysqlnd_net_get_methods
0001:00573dea  _mysqlnd_net_free
0001:00574194  __mysqlnd_plugin_get_plugin_net_data
0001:005741bd  _mysqlnd_net_init
0001:00574254  _php_mysqlnd_net_send_pub
Module: U:\dev\php-5.3.20\ext\mysqlnd\mysqlnd_statistics.obj(mysqlnd_statistics.obj)
0001:00574970  _mysqlnd_stats_reset_triggers
0001:005749ba  _mysqlnd_stats_set_trigger
0001:005749fb  _mysqlnd_stats_end
0001:00574a32  _mysqlnd_stats_init
0001:00574aa4  _mysqlnd_fill_stats_hash
0001:00574b6c  __mysqlnd_get_client_stats
0001:005759a0  _mysqlnd_stats_values_names
Module: U:\dev\php-5.3.20\ext\mysqlnd\mysqlnd_result.obj(mysqlnd_result.obj)
0001:005761b6  __mysqlnd_fetch_lengths
0001:005763f6  _mysqlnd_result_get_methods
0001:00578a3f  __mysqlnd_plugin_get_plugin_result_data
0001:00578a68  _mysqlnd_result_init
0001:00578acd  _php_mysqlnd_res_store_result_fetch_data_pub
0001:005791ca  _mysqlnd_query_read_result_set_header
Module: U:\dev\php-5.3.20\ext\mysqlnd\mysqlnd_result_meta.obj(mysqlnd_result_meta.obj)
0001:00579fe7  _mysqlnd_result_metadata_get_methods
0001:00579ff1  __mysqlnd_plugin_get_plugin_result_metadata_data
0001:0057a017  _mysqlnd_result_meta_init
Module: U:\dev\php-5.3.20\ext\mysqlnd\mysqlnd_debug.obj(mysqlnd_debug.obj)
0001:0057c31e  _mysqlnd_get_backtrace
0001:0057cdcd  __mysqlnd_efree
0001:0057cf53  __mysqlnd_erealloc
0001:0057d132  __mysqlnd_emalloc
0001:0057d2ef  __mysqlnd_malloc
0001:0057d4bb  __mysqlnd_pemalloc
0001:0057d73a  __mysqlnd_free
0001:0057d8c0  __mysqlnd_pefree
0001:0057dae3  __mysqlnd_realloc
0001:0057dcce  __mysqlnd_perealloc
0001:0057df85  __mysqlnd_calloc
0001:0057e14d  __mysqlnd_ecalloc
0001:0057e367  __mysqlnd_pecalloc
0001:0057e5e3  _mysqlnd_debug_init
0001:0057e69c  __mysqlnd_debug
0001:0057e72d  __mysqlnd_pestrndup
0001:0057e8f3  __mysqlnd_pestrdup
0002:00003b80  _mysqlnd_mysqlnd_debug_methods
0002:00003b40  _mysqlnd_debug_std_no_trace_funcs
0002:00003ba0  _mysqlnd_allocator
Module: U:\dev\php-5.3.20\ext\mysqlnd\mysqlnd_block_alloc.obj(mysqlnd_block_alloc.obj)
0001:0057ed7c  _mysqlnd_mempool_destroy
0001:0057edac  _mysqlnd_mempool_create
Module: U:\dev\php-5.3.20\ext\mysqlnd\php_mysqlnd.obj(php_mysqlnd.obj)
0002:00020f88  _mysqlnd_globals_id
0001:0057f100  _mysqlnd_minfo_print_hash
0001:0057f26b  _zm_info_mysqlnd
0002:00003be0  _mysqlnd_module_entry
Module: U:\dev\php-5.3.20\ext\mysqlnd\mysqlnd_ps.obj(mysqlnd_ps.obj)
0001:0057fd5b  _php_mysqlnd_stmt_free_parameter_bind_pub
0001:0057fd85  _php_mysqlnd_stmt_free_result_bind_pub
0001:0057fdaf  _mysqlnd_stmt_get_methods
0001:0057fdb9  _mysqlnd_stmt_set_methods
0001:00582742  _mysqlnd_fetch_stmt_row_cursor
0001:0058409b  _mysqlnd_stmt_fetch_row_buffered
0001:00583701  __mysqlnd_plugin_get_plugin_stmt_data
0001:00583727  __mysqlnd_stmt_init
0001:00584085  __mysqlnd_init_ps_subsystem
0001:005843b4  _mysqlnd_not_bound_as_blob
0001:005843b8  _mysqlnd_stmt_not_prepared
0002:00003c40  _mysqlnd_mysqlnd_stmt_methods
Module: U:\dev\php-5.3.20\ext\mysqlnd\mysqlnd_ps_codec.obj(mysqlnd_ps_codec.obj)
0002:00020f98  _mysqlnd_ps_fetch_functions
0001:00584420  __mysqlnd_init_ps_fetch_subsystem
0001:00584bb5  _ps_fetch_from_1_to_8_bytes
0001:005851a3  _mysqlnd_stmt_execute_generate_request
Module: U:\dev\php-5.3.20\TSRM\TSRM.obj(TSRM.obj)
0001:00586080  _tsrm_set_interpreter_context
0001:00586092  _tsrm_mutex_alloc
0001:00586099  _tsrm_mutex_unlock
0001:0058609e  _tsrm_set_new_thread_begin_handler
0001:005860b1  _tsrm_set_new_thread_end_handler
0001:005860c4  _tsrm_error_set
0001:005860d1  _tsrm_mutex_lock
0001:005860dd  _tsrm_mutex_free
0001:005860f2  _tsrm_thread_id
0001:00586101  _ts_free_id
0001:005861cf  _ts_free_worker_threads
0001:005862eb  _ts_free_thread
0001:005863ea  _tsrm_free_interpreter_context
0001:0058657b  _tsrm_new_interpreter_context
0001:005865b9  _ts_resource_ex
0001:00586669  _ts_allocate_id
0001:0058680e  _tsrm_shutdown
0001:00586982  _tsrm_startup
Module: U:\dev\php-5.3.20\TSRM\tsrm_strtok_r.obj(tsrm_strtok_r.obj)
0001:00586a70  _tsrm_strtok_r
Module: U:\dev\php-5.3.20\TSRM\tsrm_virtual_cwd.obj(tsrm_virtual_cwd.obj)
0002:00021f98  _cwd_globals_id
0002:00021fa8  _cwd_mutex
0002:00021fb8  _main_cwd_state
0001:00586b20  _realpath_cache_size
0001:00586b37  _realpath_cache_max_buckets
0001:00586b41  _realpath_cache_get_buckets
0001:00586b58  _realpath_cache_clean
0001:00586be3  _virtual_getcwd_ex
0001:00586d29  _virtual_getcwd
0001:00586d96  _virtual_chdir_file
0001:00587935  _virtual_file_ex
0001:00587fcb  _tsrm_realpath
0001:0058816c  _virtual_opendir
0001:00588215  _virtual_rmdir
0001:005882bd  _virtual_mkdir
0001:0058836c  _virtual_unlink
0001:00588414  _virtual_lstat
0001:005884c3  _virtual_stat
0001:00588572  _virtual_rename
0001:005886c1  _virtual_creat
0001:00588770  _virtual_open
0001:00588842  _virtual_chown
0001:00588918  _virtual_chmod
0001:005889c7  _virtual_utime
0001:00588a76  _virtual_access
0001:00588b25  _virtual_fopen
0001:00588be4  _virtual_filepath_ex
0001:00588c61  _virtual_filepath
0001:00588c8a  _virtual_realpath
0001:00588e08  _virtual_chdir
0001:00588e45  _virtual_popen
0001:00588ed5  _realpath_cache_del
0001:00588fdb  _virtual_cwd_shutdown
0001:00588ffd  _virtual_cwd_startup
0001:005890ef  _realpath_cache_lookup
Module: U:\dev\php-5.3.20\main\main.obj(main.obj)
0002:00021fc8  _core_globals_id
0001:00589201  _php_com_initialize
0001:00589206  _php_module_shutdown_for_exec
0001:0058920b  _php_lint_script
0001:005892bf  _php_handle_auth_data
0001:00589448  _php_handle_aborted_connection
0001:005894ba  _php_execute_simple_script
0001:0058961c  _php_execute_script
0001:00589957  _php_module_shutdown
0001:005899dd  _php_module_shutdown_wrapper
0001:00589a03  _php_request_shutdown_for_exec
0001:00589d37  _php_write
0001:0058a0be  _php_register_extensions
0001:0058a11a  _zm_info_php_core
0001:0058a157  _php_request_shutdown
0001:0058a620  _php_request_shutdown_for_hook
0001:0058a9a5  _php_request_startup_for_hook
0001:0058a9fb  _php_request_startup
0001:0058acc1  _php_on_timeout
0001:0058ada0  _php_stream_open_for_zend_ex
0001:0058aef3  _php_html_puts
0001:0058aeff  _php_printf
0001:0058b31a  _php_module_startup
0001:0058c0b9  _php_verror
0001:0058c6f7  _php_error_docref2
0001:0058c770  _php_error_docref1
0001:0058c7a6  _php_error_docref0
0001:0058cb0d  _zif_set_time_limit
0001:0058cc26  _php_log_err
0002:00003ce0  _php_register_internal_extensions_func
Module: U:\dev\php-5.3.20\main\snprintf.obj(snprintf.obj)
0001:0058f6a0  _ap_php_conv_10
0001:0058f73b  _ap_php_conv_p2
0001:0058f79c  _ap_php_asprintf
0001:0058f92c  _php_conv_fp
0001:00591213  _php_gcvt
0001:0059113b  _ap_php_vsnprintf
0001:00591161  _ap_php_vasprintf
0001:005911e5  _ap_php_snprintf
0001:00591511  _ap_php_vslprintf
0001:0059154e  _ap_php_slprintf
Module: U:\dev\php-5.3.20\main\spprintf.obj(spprintf.obj)
0001:00592c3f  _vspprintf
0001:00592c9b  _spprintf
Module: U:\dev\php-5.3.20\main\php_sprintf.obj(php_sprintf.obj)
0001:00592cd0  _php_sprintf
Module: U:\dev\php-5.3.20\main\safe_mode.obj(safe_mode.obj)
0001:00592d11  _php_get_current_user
0001:00592f0b  _php_checkuid_ex
0001:00593420  _php_checkuid
Module: U:\dev\php-5.3.20\main\fopen_wrappers.obj(fopen_wrappers.obj)
0001:00593451  _php_strip_url_passwd
0001:005934f6  _expand_filepath_ex
0001:00593725  _expand_filepath
0001:00593756  _php_resolve_path
0001:00593d44  _php_fopen_primary_script
0001:00594255  _php_check_safe_mode_include_dir
0001:00594357  _php_check_specific_open_basedir
0001:0059472d  _php_check_open_basedir_ex
0001:00594895  _php_check_open_basedir
0001:0059494f  _php_fopen_with_path
0001:00594d79  _OnUpdateBaseDir
Module: U:\dev\php-5.3.20\main\php_scandir.obj(php_scandir.obj)
0001:00594e70  _php_scandir
0001:00595012  _php_alphasort
Module: U:\dev\php-5.3.20\main\php_ini.obj(php_ini.obj)
0001:0059505d  _php_ini_has_per_dir_config
0001:00595067  _php_ini_has_per_host_config
0001:00595071  _php_ini_get_configuration_hash
0001:0059507b  _cfg_get_string
0001:005950ce  _cfg_get_entry
0001:00595102  _cfg_get_double
0001:00595184  _cfg_get_long
0001:00595208  _php_ini_activate_config
0001:005952ca  _php_ini_activate_per_host_config
0001:0059532f  _php_ini_activate_per_dir_config
0001:005953e6  _php_parse_user_ini_file
0001:00595548  _php_ini_register_extensions
0001:005955df  _php_shutdown_config
0001:0059562b  _config_zval_dtor
0001:005956bc  _php_init_config
0001:0059611a  _display_ini_entries
0002:0001b910  _php_ini_opened_path
0002:0001b918  _php_ini_scanned_files
0002:0001b914  _php_ini_scanned_path
Module: U:\dev\php-5.3.20\main\SAPI.obj(SAPI.obj)
0002:00021fd8  _sapi_globals_id
0002:00021fe8  _sapi_module
0001:00596a30  _sapi_initialize_empty_request
0001:00596a73  _sapi_flush
0001:00596aa2  _sapi_get_fd
0001:00596ac7  _sapi_force_http_10
0001:00596ae6  _sapi_get_target_uid
0001:00596b0b  _sapi_get_target_gid
0001:00596b30  _sapi_terminate_process
0001:00596b44  _sapi_get_request_time
0001:00596bac  _sapi_getenv
0001:00596c3a  _sapi_get_stat
0001:00596c9d  _sapi_register_input_filter
0001:00596cfa  _sapi_register_treat_data
0001:00596d4f  _sapi_register_default_post_reader
0001:00596da4  _sapi_unregister_post_entry
0001:00596e0b  _sapi_register_post_entry
0001:00596e87  _sapi_register_post_entries
0001:00596f16  _sapi_handle_post
0001:00596f9d  _sapi_free_header
0001:00597069  _sapi_apply_default_charset
0001:00597360  _sapi_header_op
0001:00597d8e  _sapi_add_header_ex
0001:00597dea  _sapi_deactivate
0001:00598006  _sapi_activate_headers_only
0001:00598158  _sapi_activate
0001:005984ac  _sapi_get_default_content_type
0001:0059856f  _sapi_get_default_content_type_header
0001:00598602  _sapi_send_headers
0001:00598924  _sapi_read_standard_form_data
0001:00598a9d  _sapi_shutdown
0001:00598aa9  _sapi_startup
Module: U:\dev\php-5.3.20\main\rfc1867.obj(rfc1867.obj)
0001:00599385  _destroy_uploaded_files_hash
0001:005994aa  _php_rfc1867_register_constants
0001:00599a4b  _rfc1867_post_handler
0002:0001b9d0  _php_rfc1867_callback
Module: U:\dev\php-5.3.20\main\php_content_types.obj(php_content_types.obj)
0001:0059b410  _php_setup_sapi_content_types
0001:0059b42d  _php_startup_sapi_content_types
0001:0059b47b  _php_default_post_reader
Module: U:\dev\php-5.3.20\main\mergesort.obj(mergesort.obj)
0001:0059b78d  _php_mergesort
Module: U:\dev\php-5.3.20\main\php_variables.obj(php_variables.obj)
0001:0059bff0  _php_default_input_filter
0001:0059c00a  _php_std_auto_global_callback
0001:0059c058  _php_startup_auto_globals
0001:0059ccec  _php_handle_special_queries
0001:0059cf28  _php_register_variable_ex
0001:0059da34  _php_register_variable_safe
0001:0059db0f  _php_default_treat_data
0001:0059df25  _php_std_post_handler
0001:0059e0aa  _php_register_variable
0001:0059e100  __php_import_environment_variables
0001:0059e31c  _php_hash_environment
0002:00003d80  _php_import_environment_variables
Module: U:\dev\php-5.3.20\main\php_ticks.obj(php_ticks.obj)
0001:0059f230  _php_run_ticks
0001:0059f2aa  _php_remove_tick_function
0001:0059f2ee  _php_add_tick_function
0001:0059f32a  _php_shutdown_ticks
0001:0059f34d  _php_deactivate_ticks
0001:0059f370  _php_startup_ticks
Module: U:\dev\php-5.3.20\main\network.obj(network.obj)
0001:0059f3b0  _php_sockaddr_size
0001:0059f51b  __php_emit_fd_setsize_warning
0001:0059f57b  _php_set_sock_blocking
0001:0059f5d6  __php_stream_sock_open_host
0001:0059f69b  _php_any_addr
0001:0059f6e2  __php_stream_sock_open_from_socket
0001:0059f7d9  _php_socket_strerror
0001:0059f99c  _php_network_populate_name_from_sockaddr
0001:0059fab5  _php_network_get_sock_name
0001:0059fb37  _php_network_get_peer_name
0001:0059fbd4  _php_network_parse_network_address_with_port
0001:0059fd80  _php_network_bind_socket_to_local_addr
0001:0059fec8  _php_network_connect_socket
0001:005a00e7  _php_network_connect_socket_to_host
0001:005a03c5  _php_network_accept_incoming
Module: U:\dev\php-5.3.20\main\php_open_temporary_file.obj(php_open_temporary_file.obj)
0001:005a0520  _php_shutdown_temporary_directory
0001:005a06c8  _php_get_temporary_directory
0001:005a074d  _php_open_temporary_fd_ex
0001:005a07ea  _php_open_temporary_fd
0001:005a081e  _php_open_temporary_file
Module: U:\dev\php-5.3.20\main\php_logos.obj(php_logos.obj)
0001:005a0880  _php_info_logos
0001:005a0960  _php_shutdown_info_logos
0001:005a0976  _php_unregister_info_logo
0001:005a09ba  _php_register_info_logo
0001:005a0ab4  _php_init_info_logos
Module: U:\dev\php-5.3.20\main\output.obj(output.obj)
0002:00022088  _output_globals_id
0001:005a5803  _php_default_output_func
0001:005a34cc  _php_output_activate
0001:005a3cec  _php_ub_body_write
0001:005a351c  _php_output_set_status
0001:005a3538  _php_body_write
0001:005a3552  _php_header_write
0001:005a3589  _php_start_implicit_flush
0001:005a35a1  _php_end_implicit_flush
0001:005a35b9  _php_get_output_start_filename
0001:005a35d0  _php_get_output_start_lineno
0001:005a35e7  _php_ob_get_length
0001:005a3617  _zif_ob_implicit_flush
0001:005a367f  _zif_ob_get_length
0001:005a36dd  _zif_ob_get_level
0001:005a3726  _zif_output_add_rewrite_var
0001:005a37be  _zif_output_reset_rewrite_vars
0001:005a39d7  _zif_ob_get_status
0001:005a3bd0  _zif_ob_list_handlers
0001:005a3c68  _php_ub_body_write_no_header
0001:005a3e00  _php_ob_get_buffer
0001:005a3e48  _zif_ob_get_contents
0001:005a3ef3  _php_ob_handler_used
0001:005a3fa3  _php_ob_init_conflict
0001:005a4071  _php_end_ob_buffer
0001:005a46b0  _zif_ob_get_clean
0001:005a47dc  _zif_ob_get_flush
0001:005a48c5  _zif_ob_end_clean
0001:005a499c  _zif_ob_end_flush
0001:005a4a73  _zif_ob_clean
0001:005a4b91  _zif_ob_flush
0001:005a4c68  _php_end_ob_buffers
0001:005a53ac  _php_start_ob_buffer
0001:005a5488  _zif_ob_start
0001:005a552d  _php_ob_set_internal_handler
0001:005a5631  _php_start_ob_buffer_named
0001:005a5737  _php_output_register_constants
0001:005a57d7  _php_output_startup
Module: U:\dev\php-5.3.20\main\getopt.obj(getopt.obj)
0001:005a599c  _php_getopt
0002:00003d90  _php_optidx
Module: U:\dev\php-5.3.20\main\streams\streams.obj(streams.obj)
0001:005a5e00  _php_file_le_stream
0001:005a5e0a  _php_file_le_pstream
0001:005a5e14  _php_file_le_stream_filter
0001:005a5e1e  __php_stream_get_url_stream_wrappers_hash
0001:005a5e40  _php_stream_get_url_stream_wrappers_hash_global
0001:005a5f7d  __php_stream_tell
0001:005a5f8b  __php_stream_set_option
0001:005a6009  __php_stream_eof
0001:005a6082  __php_stream_truncate_set_size
0001:005a60b3  _php_stream_notification_notify
0001:005a60f4  _php_stream_notification_free
0001:005a612b  _php_stream_dirent_alphasortr
0001:005a6147  _php_stream_dirent_alphasort
0001:005a6163  _php_unregister_url_stream_wrapper
0001:005a61a4  _php_stream_tidy_wrapper_error_log
0001:005a61f0  _php_stream_context_del_link
0001:005a62f9  _php_stream_context_set_link
0001:005a63e7  _php_register_url_stream_wrapper
0001:005a6496  _php_stream_context_get_link
0001:005a64fb  _php_stream_context_get_option
0001:005a6574  _php_stream_context_set_option
0001:005a6704  _php_stream_notification_alloc
0001:005a6720  _php_stream_context_alloc
0001:005a6798  _php_stream_from_persistent_id
0001:005a690d  _php_stream_context_free
0001:005a696a  _php_stream_context_set
0001:005a6ba5  _php_stream_locate_url_wrapper
0001:005a7069  __php_stream_stat_path
0001:005a7236  __php_stream_rmdir
0001:005a729c  __php_stream_mkdir
0001:005a73aa  _php_unregister_url_stream_wrapper_volatile
0001:005a7419  _php_register_url_stream_wrapper_volatile
0001:005a74fb  _php_shutdown_stream_hashes
0001:005a75c2  _php_shutdown_stream_wrappers
0001:005a762a  _php_init_stream_wrappers
0001:005a7820  __php_stream_stat
0001:005a79b3  __php_stream_write
0001:005a79fe  __php_stream_printf
0001:005a7a60  __php_stream_puts
0001:005a7ade  __php_stream_putc
0001:005a7b15  __php_stream_flush
0001:005a7c51  _php_stream_locate_eol
0001:005a7d3d  __php_stream_free
0001:005a810a  _php_stream_wrapper_log_error
0001:005a82d7  _php_stream_display_wrapper_errors
0001:005a85ff  __php_stream_open_wrapper_ex
0001:005a8b10  __php_stream_opendir
0001:005a8c09  _zm_deactivate_streams
0001:005a90b5  __php_stream_read
0001:005a91fe  __php_stream_readdir
0001:005a923d  __php_stream_scandir
0001:005a939f  __php_stream_copy_to_stream_ex
0001:005a9602  __php_stream_copy_to_stream
0001:005a9650  __php_stream_passthru
0001:005a9790  __php_stream_seek
0001:005a9aa5  __php_stream_getc
0001:005a9add  _php_stream_get_record
0001:005a9cd7  __php_stream_get_line
0001:005a9e87  __php_stream_alloc
0001:005aa00e  __php_stream_copy_to_mem
Module: U:\dev\php-5.3.20\main\streams\cast.obj(cast.obj)
0001:005aa2d0  _php_stream_mode_sanitize_fdopen_fopencookie
0001:005aa362  __php_stream_make_seekable
0001:005aa51a  __php_stream_cast
0001:005aa8da  __php_stream_open_wrapper_as_file
Module: U:\dev\php-5.3.20\main\streams\memory.obj(memory.obj)
0001:005aaabd  __php_stream_memory_get_buffer
0001:005ab11d  __php_stream_memory_create
0001:005ab194  __php_stream_memory_open
0001:005ab20a  __php_stream_temp_create
0001:005ab952  __php_stream_temp_open
0002:00003db0  _php_stream_memory_ops
0002:00003de0  _php_stream_temp_ops
0002:00003e10  _php_stream_rfc2397_ops
0002:00003e40  _php_stream_rfc2397_wops
0002:00003e70  _php_stream_rfc2397_wrapper
Module: U:\dev\php-5.3.20\main\streams\filter.obj(filter.obj)
0001:005ab9f0  _php_get_stream_filters_hash_global
0001:005ab9fa  __php_get_stream_filters_hash
0001:005aba1c  _php_stream_bucket_prepend
0001:005aba48  _php_stream_bucket_append
0001:005aba73  _php_stream_bucket_unlink
0001:005abac0  _php_stream_filter_prepend_ex
0001:005abaf1  __php_stream_filter_prepend
0001:005abb76  _php_stream_filter_free
0001:005abbb6  _php_stream_filter_remove
0001:005abc24  _php_stream_bucket_delref
0001:005abc8f  __php_stream_filter_flush
0001:005abf37  _php_stream_filter_create
0001:005ac122  _php_stream_filter_register_factory_volatile
0001:005ac220  _php_stream_filter_register_factory
0001:005ac270  _php_stream_filter_unregister_factory
0001:005ac2b1  _php_stream_bucket_new
0001:005ac3bf  _php_stream_filter_append_ex
0001:005ac6fd  __php_stream_filter_append
0001:005ac749  _php_stream_bucket_split
0001:005aca74  _php_stream_bucket_make_writeable
0001:005acba9  __php_stream_filter_alloc
Module: U:\dev\php-5.3.20\main\streams\plain_wrapper.obj(plain_wrapper.obj)
0001:005accff  _php_stream_parse_fopen_modes
0001:005adc9a  __php_stream_fopen_from_pipe
0001:005add10  __php_stream_fopen_from_file
0001:005ade9e  __php_stream_fopen_from_fd
0001:005adf9b  __php_stream_fopen
0001:005ae2df  __php_stream_fopen_with_path
0001:005ae86d  __php_stream_fopen_tmpfile
0001:005ae916  __php_stream_fopen_temporary_file
0002:00003e90  _php_stream_stdio_ops
0002:00003ec0  _php_plain_files_wrapper
Module: U:\dev\php-5.3.20\main\streams\userspace.obj(userspace.obj)
0001:005afda0  _zif_stream_wrapper_unregister
0001:005afeb5  _zif_stream_wrapper_restore
0001:005b0088  _zif_stream_wrapper_register
0001:005b17ac  _zm_startup_user_streams
0002:00003f70  _php_stream_userspace_dir_ops
0002:00003f40  _php_stream_userspace_ops
Module: U:\dev\php-5.3.20\main\streams\transports.obj(transports.obj)
0001:005b2920  _php_stream_xport_get_hash
0001:005b292a  _php_stream_xport_shutdown
0001:005b298b  _php_stream_xport_recvfrom
0001:005b2a42  _php_stream_xport_get_name
0001:005b2ae5  _php_stream_xport_accept
0001:005b2baf  _php_stream_xport_listen
0001:005b2c25  _php_stream_xport_connect
0001:005b2cbb  _php_stream_xport_bind
0001:005b2d7a  _php_stream_xport_sendto
0001:005b2e7f  _php_stream_xport_crypto_enable
0001:005b2f0a  _php_stream_xport_crypto_setup
0001:005b3074  __php_stream_xport_create
0001:005b361a  _php_stream_xport_unregister
0001:005b365b  _php_stream_xport_register
Module: U:\dev\php-5.3.20\main\streams\xp_socket.obj(xp_socket.obj)
0001:005b3f2f  _php_stream_generic_socket_factory
0002:00004000  _php_stream_socket_ops
0002:00004030  _php_stream_udp_socket_ops
0002:00004060  _php_stream_unix_socket_ops
0002:00004090  _php_stream_unixdg_socket_ops
0002:00003fd0  _php_stream_generic_socket_ops
Module: U:\dev\php-5.3.20\main\streams\mmap.obj(mmap.obj)
0001:005b4e70  __php_stream_mmap_unmap
0001:005b4eaa  __php_stream_mmap_unmap_ex
0001:005b4f00  __php_stream_mmap_range
Module: U:\dev\php-5.3.20\main\streams\glob_wrapper.obj(glob_wrapper.obj)
0001:005b4f70  __php_glob_stream_get_count
0001:005b503c  __php_glob_stream_get_pattern
0001:005b5088  __php_glob_stream_get_path
0002:000040c0  _php_glob_stream_ops
0002:000040f0  _php_glob_stream_wrapper
Module: U:\dev\php-5.3.20\main\internal_functions.obj(internal_functions.obj)
0001:005b5370  _php_register_internal_extensions
Module: U:\dev\php-5.3.20\Zend\zend_language_parser.obj(zend_language_parser.obj)
0001:005b572f  _zendparse
Module: U:\dev\php-5.3.20\Zend\zend_language_scanner.obj(zend_language_scanner.obj)
0002:00022098  _language_scanner_globals_id
0001:005c2c00  _zend_get_scanned_file_offset
0001:005c316f  _lex_scan
0001:005cb725  _zend_prepare_string_for_scanning
0001:005cb838  _open_file_for_scanning
0001:005cb9f1  _zend_destroy_file_handle
0001:005cba3d  _compile_filename
0001:005cbbf2  _shutdown_scanner
0001:005cbc89  _zend_restore_lexical_state
0001:005cbd6a  _zend_save_lexical_state
0001:005cbe0b  _highlight_string
0001:005cbec4  _highlight_file
0001:005cbf75  _compile_string
0001:005cc17f  _compile_file
0001:005cc356  _startup_scanner
Module: U:\dev\php-5.3.20\Zend\zend_ini_parser.obj(zend_ini_parser.obj)
0001:005cd154  _ini_parse
0001:005cdcdc  _zend_parse_ini_string
0001:005cdd65  _zend_parse_ini_file
Module: U:\dev\php-5.3.20\Zend\zend_ini_scanner.obj(zend_ini_scanner.obj)
0002:000220a8  _ini_scanner_globals_id
0001:005ce420  _zend_ini_scanner_get_lineno
0001:005ce43f  _zend_ini_scanner_get_filename
0001:005ce537  _ini_lex
0001:005d4ce4  _zend_ini_prepare_string_for_scanning
0001:005d4d3d  _zend_ini_open_file_for_scanning
0001:005d4db9  _shutdown_ini_scanner
Module: U:\dev\php-5.3.20\Zend\zend_alloc.obj(zend_alloc.obj)
0001:005d5605  _is_zend_mm
0001:005d561d  _zend_memory_usage
0001:005d5653  _zend_memory_peak_usage
0001:005d5686  _zend_mm_set_heap
0001:005d56a1  _zend_mm_get_storage
0001:005d56ac  _zend_mm_set_custom_handlers
0001:005d56cc  _start_memory_manager
0001:005d5753  _zend_set_memory_limit
0001:005d5893  __zend_mm_block_size
0001:005d58a5  __zend_mem_block_size
0001:005d58d2  _zend_strndup
0001:005d5964  __safe_realloc
0001:005d59ec  __safe_malloc
0001:005d5cd9  __efree
0001:005d5d24  __zend_mm_free
0001:005d691c  __emalloc
0001:005d6967  __estrndup
0001:005d69a3  __estrdup
0001:005d69e6  __safe_emalloc
0001:005d6a31  __ecalloc
0001:005d6a7b  __zend_mm_alloc
0001:005d6a8d  _zend_mm_shutdown
0001:005d6bc5  _shutdown_memory_manager
0001:005d6c9b  _zend_mm_startup_ex
0001:005d6fbf  _zend_mm_startup
0001:005d78ad  __erealloc
0001:005d7903  __safe_erealloc
0001:005d795d  __zend_mm_realloc
Module: U:\dev\php-5.3.20\Zend\zend_compile.obj(zend_compile.obj)
0002:000220b8  _zend_compile_file
0002:000220c8  _zend_compile_string
0001:005d79c0  _zend_auto_global_arm
0001:005d79d3  _zend_restore_compiled_filename
0001:005d79f0  _zend_get_compiled_filename
0001:005d7a0a  _zend_get_compiled_lineno
0001:005d7a24  _zend_is_compiling
0001:005d7a59  _zend_visibility_string
0001:005d7a84  _zend_do_declare_implicit_property
0001:005d7a89  _zend_get_compiled_variable_name
0001:005d7ac6  _zend_dirname
0001:005d7bae  _zend_verify_namespace
0001:005d7c27  _zend_unmangle_property_name
0001:005d7dce  _zend_do_verify_access_types
0001:005d7f2d  _zend_check_writable_variable
0001:005d7f7d  _zend_do_ticks
0001:005d7fed  _zend_do_extended_fcall_end
0001:005d8033  _zend_do_extended_fcall_begin
0001:005d8079  _zend_do_extended_info
0001:005d80bf  _zend_do_end_silence
0001:005d8118  _zend_do_begin_silence
0001:005d81a8  _zend_do_exit
0001:005d830b  _zend_do_include_or_eval
0001:005d83e0  _zend_do_cast
0001:005d8491  _zend_do_add_array_element
0001:005d854f  _zend_do_init_array
0001:005d865c  _zend_do_brk_cont
0001:005d86fe  _zend_do_throw
0001:005d87e2  _zend_do_clone
0001:005d888d  _zend_do_handle_exception
0001:005d88c8  _zend_do_add_variable
0001:005d89bc  _zend_do_add_string
0001:005d8bc3  _zend_do_abstract_method
0001:005d8d1b  _zend_do_echo
0001:005d8d74  _zend_do_print
0001:005d8e1f  _zend_do_unary_op
0001:005d8ed3  _zend_do_binary_op
0001:005d9123  _zend_is_auto_global
0001:005d919f  _zend_auto_global_disable_jit
0001:005d9242  _zend_get_class_fetch_type
0001:005d9333  _do_bind_function
0001:005d9458  _zend_set_compiled_filename
0001:005d953a  _zend_initialize_class_data
0001:005d988d  _zend_auto_global_dtor
0001:005d98a1  _zendlex
0001:005d99ab  _zend_register_auto_global
0001:005d9a44  _zend_do_qm_false
0001:005d9b41  _zend_do_qm_true
0001:005d9c97  _zend_do_begin_qm_op
0001:005d9d56  _zend_do_jmp_set_else
0001:005d9e55  _zend_do_jmp_set
0001:005d9f8e  _zend_do_instanceof
0001:005da0fd  _zend_do_unset
0001:005da1d7  _zend_do_case_after_statement
0001:005da28c  _zend_do_boolean_and_end
0001:005da361  _zend_do_boolean_and_begin
0001:005da451  _zend_do_boolean_or_end
0001:005da526  _zend_do_boolean_or_begin
0001:005da616  _zend_do_first_catch
0001:005da641  _zend_do_if_cond
0001:005da6dc  _zend_do_post_incdec
0001:005da834  _zend_do_pre_incdec
0001:005da99a  _zend_do_for_cond
0001:005daa30  _zend_do_assign_ref
0001:005dac37  _zend_do_binary_assign_op
0001:005dae4e  _zend_do_declare_end
0001:005daede  _zend_do_default_before_statement
0001:005dafb7  _zend_do_declare_begin
0001:005dafeb  _zend_do_begin_new_object
0001:005db0c0  _zend_do_push_object
0001:005db0f1  _zend_do_foreach_end
0001:005db249  _zend_do_pop_object
0001:005db2b6  _zend_do_for_before_statement
0001:005db5f1  _zend_do_try
0001:005db69c  _zend_do_build_full_name
0001:005db7b4  _zend_do_end_variable_parse
0001:005dbb0d  _zend_do_foreach_begin
0001:005dbe83  _zend_do_isset_or_isempty
0001:005dc122  _zend_do_pass_param
0001:005dc579  _zend_do_if_end
0001:005dc636  _zend_do_mark_last_catch
0001:005dc717  _zend_do_begin_variable_parse
0001:005dc76a  _zend_do_new_list_end
0001:005dc7a4  _zend_do_new_list_begin
0001:005dc7d4  _zend_do_list_init
0001:005dc895  _zend_do_end_catch
0001:005dc952  _zend_initialize_try_catch_element
0001:005dca5a  _zend_do_if_after_statement
0001:005dcb6a  _zend_do_add_list_element
0001:005dcc02  _zend_do_shell_exec
0001:005dcd70  _zend_do_end_function_call
0001:005dcf48  _zend_do_begin_dynamic_function_call
0001:005dd1bf  _zend_do_begin_method_call
0001:005dd39e  _zend_do_fetch_property
0001:005dd5d1  _fetch_array_dim
0001:005dd6d3  _fetch_string_offset
0001:005dd6df  _fetch_simple_variable_ex
0001:005dd92b  _fetch_simple_variable
0001:005dd95b  _fetch_array_begin
0001:005dd9a0  _zend_do_indirect_references
0001:005ddb7f  _zend_do_declare_property
0001:005ddd6a  _zend_mangle_property_name
0001:005dde9b  _zend_do_end_class_declaration
0001:005de0f1  _do_bind_class
0001:005de2bb  _zend_do_assign
0001:005df8fa  _function_add_ref
0001:005df995  _zend_do_return
0001:005dfbaf  _zend_release_labels
0001:005dfca2  _zend_do_end_function_declaration
0001:005dfe1d  _shutdown_compiler
0001:005dff17  _file_handle_dtor
0001:005dff42  _zend_init_compiler_data_structures
0001:005e0113  _init_compiler
0001:005e021a  _zend_do_declare_class_constant
0001:005e039a  _zend_do_label
0001:005e0532  _zend_do_fetch_global_variable
0001:005e0690  _zend_do_end_namespace
0001:005e07b8  _zend_do_end_compilation
0001:005e0835  _zend_do_halt_compiler_register
0001:005e09df  _zend_resolve_goto_label
0001:005e0b8c  _zend_do_goto
0001:005e0d0c  _zend_do_case_before_statement
0001:005e0f0d  _zend_do_declare_stmt
0001:005e104d  _zend_do_inherit_interfaces
0001:005e124a  _zend_do_implement_interface
0001:005e1585  _zend_do_inheritance
0001:005e1c85  _do_bind_inherited_class
0001:005e1da1  _zend_do_delayed_early_binding
0001:005e1f91  _zend_do_begin_namespace
0001:005e23dc  _zend_do_build_namespace_name
0001:005e2527  _zend_do_declare_constant
0001:005e27a0  _zend_do_begin_class_declaration
0001:005e2c15  _zend_resolve_non_class_name
0001:005e2e82  _zend_do_begin_function_call
0001:005e3303  _zend_do_begin_function_declaration
0001:005e3fe9  _zend_do_begin_lambda_function_declaration
0001:005e4108  _zend_do_free
0001:005e4242  _zend_do_end_new_object
0001:005e4310  _zend_do_fetch_static_variable
0001:005e45f1  _zend_do_fetch_lexical_variable
0001:005e4685  _zend_do_list_end
0001:005e4989  _zend_do_switch_end
0001:005e4b74  _zend_do_early_binding
0001:005e4ec9  _zend_do_while_cond
0001:005e5015  _zend_do_foreach_cont
0001:005e535a  _zend_do_switch_cond
0001:005e5426  _zend_do_do_while_begin
0001:005e549e  _zend_do_do_while_end
0001:005e5567  _zend_do_for_end
0001:005e5654  _zend_do_while_end
0001:005e57e8  _zend_do_use
0001:005e5d0b  _zend_resolve_class_name
0001:005e60c0  _zend_do_implements_interface
0001:005e61fb  _zend_do_fetch_class
0001:005e63e7  _zend_do_begin_catch
0001:005e6510  _zend_do_fetch_static_member
0001:005e67c0  _zend_do_fetch_constant
0001:005e6bfb  _zend_do_receive_arg
0001:005e6ffa  _zend_do_begin_class_member_function_call
0001:005e71db  _zend_do_add_static_array_element
Module: U:\dev\php-5.3.20\Zend\zend_constants.obj(zend_constants.obj)
0001:005e772e  _zend_register_constant
0001:005e78c9  _free_zend_constant
0001:005e7907  _zend_get_constant
0001:005e7bfa  _zend_get_constant_ex
0001:005e80fd  _zend_register_stringl_constant
0001:005e8153  _zend_register_string_constant
0001:005e81a2  _zend_register_double_constant
0001:005e81f2  _zend_register_long_constant
0001:005e837d  _zend_register_standard_constants
0001:005e8809  _copy_zend_constant
0001:005e884a  _clean_non_persistent_constants
0001:005e88a0  _zend_shutdown_constants
0001:005e88e6  _zend_startup_constants
0001:005e895c  _clean_module_constants
0001:005e8994  _zend_copy_constants
Module: U:\dev\php-5.3.20\Zend\zend_dynamic_array.obj(zend_dynamic_array.obj)
0001:005e89d0  _zend_dynamic_array_pop
0001:005e89e9  _zend_dynamic_array_get_element
0001:005e8a03  _zend_dynamic_array_push
0001:005e8a51  _zend_dynamic_array_init
Module: U:\dev\php-5.3.20\Zend\zend_execute_API.obj(zend_execute_API.obj)
0002:000220d8  _zend_execute
0002:000220e8  _zend_execute_internal
0001:005e8b29  _get_active_class_name
0001:005e8b94  _get_active_function_name
0001:005e8beb  _zend_get_executed_filename
0001:005e8c11  _zend_get_executed_lineno
0001:005e8c6c  _zend_is_executing
0001:005e8cd9  _zend_reset_all_cv
0001:005e8d8f  _zend_rebuild_symbol_table
0001:005e9711  __zval_ptr_dtor
0001:005e900d  _zend_verify_abstract_class
0001:005e926a  _zend_unset_timeout
0001:005e92f3  _zend_timeout
0001:005e9377  _zend_set_timeout
0001:005e943f  _execute_new_code
0001:005e96cc  __zval_internal_ptr_dtor
0001:005e9857  _zend_is_true
0001:005e9993  _shutdown_executor
0001:005e9f76  _shutdown_destructors
0001:005ea092  _init_executor
0001:005ea4a7  _zend_eval_stringl
0001:005ea79e  _zend_eval_stringl_ex
0001:005ea80a  _zend_eval_string_ex
0001:005ea852  _zend_eval_string
0001:005ea924  _zval_update_constant_ex
0001:005eb419  _zval_update_constant_inline_change
0001:005eb3c7  _zval_update_constant
0001:005eb3f0  _zval_update_constant_no_inline_change
0001:005eb442  _zend_delete_global_variable
0001:005eb7ef  _zend_call_function
0001:005ec4bb  _zend_lookup_class_ex
0001:005ecb7f  _zend_fetch_class
0001:005ecd90  _zend_lookup_class
0001:005ecdc0  _call_user_function_ex
0001:005ece21  _call_user_function
0001:005ecf60  _empty_fcall_info
0001:005ecf90  _empty_fcall_info_cache
Module: U:\dev\php-5.3.20\Zend\zend_highlight.obj(zend_highlight.obj)
0001:005ecff7  _zend_html_putc
0001:005ed18e  _zend_html_puts
0001:005ed1db  _zend_strip
0001:005ed387  _zend_highlight
Module: U:\dev\php-5.3.20\Zend\zend_llist.obj(zend_llist.obj)
0001:005ed580  _zend_llist_init
0001:005ed5ae  _zend_llist_apply
0001:005ed5e0  _zend_llist_apply_with_argument
0001:005ed617  _zend_llist_count
0001:005ed622  _zend_llist_get_first_ex
0001:005ed643  _zend_llist_get_last_ex
0001:005ed665  _zend_llist_get_next_ex
0001:005ed68e  _zend_llist_get_prev_ex
0001:005ed6b8  _zend_llist_apply_with_arguments
0001:005ed6f6  _zend_llist_sort
0001:005ed7b5  _zend_llist_apply_with_del
0001:005ed83b  _zend_llist_remove_tail
0001:005ed8a2  _zend_llist_destroy
0001:005ed8f8  _zend_llist_clean
0001:005ed91d  _zend_llist_del_element
0001:005ed9bd  _zend_llist_add_element
0001:005eda5f  _zend_llist_copy
0001:005edab6  _zend_llist_prepend_element
Module: U:\dev\php-5.3.20\Zend\zend_opcode.obj(zend_opcode.obj)
0001:005edb96  _zend_class_add_ref
0001:005edba4  _get_next_op_number
0001:005edbca  _get_unary_op
0001:005edbe5  _get_binary_op
0001:005edc1c  _print_class
0001:005edcaf  _pass_two
0001:005edc6e  _get_next_brk_cont_element
0001:005eded6  _init_op
0001:005edf91  _get_next_op
0001:005ee02f  _destroy_op_array
0001:005ee1ee  _destroy_zend_function
0001:005ee204  _destroy_zend_class
0001:005ee336  _zend_cleanup_class_data
0001:005ee40b  _zend_cleanup_function_data_full
0001:005ee430  _zend_cleanup_function_data
0001:005ee45a  _zend_function_dtor
0001:005ee485  _init_op_array
Module: U:\dev\php-5.3.20\Zend\zend_operators.obj(zend_operators.obj)
0001:005ee6c0  _instanceof_function
0001:005ee6e9  _instanceof_function_ex
0001:005ee773  _zend_str_tolower_copy
0001:005ee7b1  _zend_str_tolower
0001:005ee7d5  _zend_binary_strcasecmp
0001:005ee822  _zend_binary_strncasecmp
0001:005ee898  _zend_binary_zval_strcasecmp
0001:005ee8c4  _zend_binary_zval_strncasecmp
0001:005ee8f9  _zend_compare_objects
0001:005ee956  _zend_locale_sprintf_double
0001:005ee9b1  _zend_compare_symbol_tables
0001:005ee9f6  _zend_compare_arrays
0001:005eea0f  _zend_compare_symbol_tables_i
0001:005eeeda  _zend_binary_strncmp
0001:005eef39  _zend_binary_zval_strncmp
0001:005eef6e  _zend_binary_strcmp
0001:005eefa4  _zend_binary_zval_strcmp
0001:005eefd0  _is_identical_function
0001:005ef0df  _is_not_identical_function
0001:005ef176  _zend_str_tolower_dup
0001:005ef1c5  _decrement_function
0001:005ef2cf  _bitwise_not_function
0001:005ef409  _add_string_to_string
0001:005ef471  _add_char_to_string
0001:005ef5e5  _convert_to_object
0001:005ef65f  _zend_string_to_double
0001:005ef7a6  _zend_atol
0001:005ef8b1  _zend_atoi
0001:005ef9bd  _convert_to_null
0001:005efb40  _string_compare_function
0001:005efc04  _string_locale_compare_function
0001:005efcdc  _concat_function
0001:005efee0  _convert_to_array
0001:005f019f  _convert_to_double
0001:005f0408  _numeric_compare_function
0001:005f04af  _multi_convert_to_double_ex
0001:005f05ac  _convert_to_long_base
0001:005f0854  _convert_to_long
0001:005f0875  _multi_convert_to_long_ex
0001:005f091e  _bitwise_xor_function
0001:005f0c92  _bitwise_and_function
0001:005f100b  _bitwise_or_function
0001:005f13c0  _mod_function
0001:005f1747  __convert_to_string
0001:005f1a66  _multi_convert_to_string_ex
0001:005f1b1a  _convert_to_boolean
0001:005f1d4a  _zval_is_true
0001:005f1d6a  _boolean_xor_function
0001:005f1fb5  _boolean_not_function
0001:005f20e5  _shift_right_function
0001:005f23b0  _shift_left_function
0001:005f267c  _zendi_smart_strcmp
0001:005f2cfd  _increment_function
0001:005f3199  _convert_scalar_to_number
0001:005f3495  _compare_function
0001:005f4241  _is_smaller_or_equal_function
0001:005f428a  _is_smaller_function
0001:005f42cc  _is_not_equal_function
0001:005f4315  _is_equal_function
0001:005f435e  _div_function
0001:005f4705  _mul_function
0001:005f4a17  _sub_function
0001:005f4d10  _add_function
Module: U:\dev\php-5.3.20\Zend\zend_ptr_stack.obj(zend_ptr_stack.obj)
0001:005f50d0  _zend_ptr_stack_apply
0001:005f5104  _zend_ptr_stack_num_elements
0001:005f510e  _zend_ptr_stack_clean
0001:005f517f  _zend_ptr_stack_destroy
0001:005f51a9  _zend_ptr_stack_n_pop
0001:005f51fe  _zend_ptr_stack_n_push
0001:005f52d0  _zend_ptr_stack_init_ex
0001:005f535b  _zend_ptr_stack_init
Module: U:\dev\php-5.3.20\Zend\zend_stack.obj(zend_stack.obj)
0001:005f5380  _zend_stack_top
0001:005f53a9  _zend_stack_int_top
0001:005f53cb  _zend_stack_is_empty
0001:005f53dd  _zend_stack_base
0001:005f53e8  _zend_stack_count
0001:005f53f2  _zend_stack_apply
0001:005f547c  _zend_stack_apply_with_argument
0001:005f5510  _zend_stack_destroy
0001:005f555c  _zend_stack_del_top
0001:005f5582  _zend_stack_init
0001:005f55bb  _zend_stack_push
Module: U:\dev\php-5.3.20\Zend\zend_variables.obj(zend_variables.obj)
0001:005f5650  _zval_add_ref
0001:005f565e  _zend_print_variable
0001:005f5679  __zval_copy_ctor_func
0001:005f57b3  _zval_property_ctor
0001:005f5846  __zval_internal_dtor
0001:005f58a1  __zval_dtor_func
0001:005f5988  __zval_dtor_wrapper
Module: U:\dev\php-5.3.20\Zend\zend.obj(zend.obj)
0002:000220f8  _zend_uv
0002:00022108  _executor_globals_id
0002:00022118  _compiler_globals_id
0002:00022128  _zval_used_for_init
0002:00022138  _zend_vspprintf
0002:00022148  _zend_error_cb
0002:00022158  _zend_printf
0002:00022168  _zend_write
0002:00022178  _zend_fopen
0002:00022188  _zend_stream_open_function
0002:00022198  _zend_block_interruptions
0002:000221a8  _zend_unblock_interruptions
0002:000221b8  _zend_ticks_function
0002:000221c8  _zend_on_timeout
0002:000221d8  _zend_getenv
0002:000221e8  _zend_resolve_path
0001:005f59e0  _get_zend_version
0001:005f5a00  _zend_message_dispatcher
0001:005f5a1d  _zend_get_configuration_directive
0001:005f5a51  _zend_output_debug_string
0001:005f5a56  _free_estring
0001:005f5a7e  _zend_make_compiled_string_description
0001:005f5b05  _zend_set_utility_values
0001:005f5b3c  _zend_execute_scripts
0001:005f5e77  _zend_error
0001:005f6a7d  _zenderror
0001:005f6aa0  _zend_activate_modules
0001:005f6ac3  _zend_post_deactivate_modules
0001:005f6b03  _zend_deactivate_modules
0001:005f6b75  _zend_deactivate
0001:005f6ce6  _zend_call_destructors
0001:005f6d3e  _zend_activate
0001:005f6d89  _zend_append_version_info
0001:005f6e4c  __zend_bailout
0001:005f6f82  _zend_shutdown
0001:005f7457  _zend_post_startup
0001:005f75ae  _zend_register_standard_ini_entries
0001:005f76cf  _zend_startup
0001:005f7bd7  _zend_print_flat_zval_r
0001:005f7edc  _zend_make_printable_zval
0001:005f81cd  _zend_print_zval_ex
0001:005f825f  _zend_print_zval_r_ex
0001:005f870b  _zend_print_zval_r
0001:005f8735  _zend_print_zval
0001:005f5e77  _zend_error_noreturn
0002:0001baf0  _zend_standard_class_def
Module: U:\dev\php-5.3.20\Zend\zend_API.obj(zend_API.obj)
0002:000221f8  _module_registry
0001:005f8840  __zend_get_parameters_array_ex
0001:005f8894  _zend_get_type_by_const
0001:005f88ad  _zend_zval_type_name
0001:005f88f1  _module_registry_cleanup
0001:005f891c  _module_registry_unload_temp
0001:005f8931  _zend_fcall_info_args_save
0001:005f8957  _zend_save_error_handling
0001:005f8990  _zend_restore_error_handling
0001:005f8a30  _zend_replace_error_handling
0001:005f8b02  _zend_read_static_property
0001:005f8b9c  _add_assoc_function
0001:005f8bf6  _zend_get_class_entry
0001:005f8c24  _zend_get_object_classname
0001:005f8cb3  _zend_read_property
0001:005f8df2  _zend_update_property
0001:005f8eef  _zend_update_property_double
0001:005f8f5e  _zend_update_property_long
0001:005f8fcd  _zend_update_property_bool
0001:005f9044  _zend_update_property_null
0001:005f9099  _zend_update_property_stringl
0001:005f9128  _add_property_zval_ex
0001:005f91a6  _add_property_stringl_ex
0001:005f9287  _add_property_double_ex
0001:005f9340  _add_property_resource_ex
0001:005f93f3  _add_property_null_ex
0001:005f94a1  _add_property_bool_ex
0001:005f955a  _add_property_long_ex
0001:005f96a0  _zend_update_property_string
0001:005f973c  _add_property_string_ex
0001:005f982b  _zend_declare_class_constant
0001:005f9873  _zend_declare_class_constant_stringl
0001:005f9933  _zend_declare_class_constant_string
0001:005f997b  _zend_declare_class_constant_double
0001:005f9a04  _zend_declare_class_constant_bool
0001:005f9a98  _zend_declare_class_constant_long
0001:005f9b21  _zend_declare_class_constant_null
0001:005f9b8e  _zend_unregister_functions
0001:005f9c37  _zend_fcall_info_args_clear
0001:005f9c6b  _zend_fcall_info_args_restore
0001:005f9cd0  _zend_declare_property_ex
0001:005f9ffe  _zend_declare_property
0001:005fa044  _zend_declare_property_stringl
0001:005fa110  _zend_declare_property_string
0001:005fa1ec  _zend_declare_property_double
0001:005fa287  _zend_declare_property_long
0001:005fa31c  _zend_declare_property_bool
0001:005fa3b9  _zend_declare_property_null
0001:005fa441  _zend_register_class_alias_ex
0001:005fa4c4  _zend_get_module_version
0001:005fa532  _zend_get_module_started
0001:005fa57f  _zend_fcall_info_argv
0001:005fa5fd  _zend_fcall_info_argn
0001:005fa62b  _zend_fcall_info_argp
0001:005fa6a8  _zend_next_free_module
0001:005fa6bf  _zend_fcall_info_args
0001:005fa76e  _zend_fcall_info_call
0001:005fbbd7  _zend_is_callable_ex
0001:005fc245  _zend_fcall_info_init
0001:005fc2f7  _zend_is_callable
0001:005fc33f  _zend_disable_class
0001:005fc56b  __array_init
0001:005fc5b6  _zif_display_disabled_function
0001:005fc5de  _zend_set_hash_symbol
0001:005fc7c6  _zend_check_magic_method_implementation
0001:005fcc05  _zend_class_implements
0001:005fcc6b  _module_registry_request_startup
0001:005fccc7  _zend_get_parameters_ex
0001:005fcd4c  _module_destructor
0001:005fd023  _zend_register_functions
0001:005fdd81  _zend_disable_function
0001:005fdf3c  _zend_register_internal_interface
0001:005fdf53  _zend_register_internal_class
0001:005fdf67  _zend_register_internal_class_ex
0001:005fe091  _zend_register_module_ex
0001:005fe29d  _zend_register_internal_module
0001:005fe2c2  _zend_startup_modules
0001:005fe445  _zend_startup_module_ex
0001:005fe602  _zend_startup_module
0001:005fe653  _add_get_index_stringl
0001:005fe6e2  _add_get_index_string
0001:005fe77e  _add_get_index_double
0001:005fe7e8  _add_get_index_long
0001:005fe84c  _add_next_index_zval
0001:005fe888  _zend_copy_parameters_array
0001:005fe8ed  _add_next_index_stringl
0001:005fe97e  _add_next_index_string
0001:005fea1e  _zend_make_callable
0001:005feb16  _add_next_index_double
0001:005feb82  _add_next_index_resource
0001:005febe8  _add_next_index_bool
0001:005fec54  _add_next_index_null
0001:005fecb5  _add_next_index_long
0001:005fed1b  _add_index_zval
0001:005fed56  _add_index_stringl
0001:005fede6  _add_index_string
0001:005fee85  _add_index_double
0001:005feef0  _add_index_resource
0001:005fef55  _add_index_bool
0001:005fefc0  _add_index_null
0001:005ff020  _add_index_long
0001:005ff085  _zend_merge_properties
0001:005ff15b  _zend_wrong_param_count
0001:005ff5b8  _add_assoc_zval_ex
0001:005ff70a  _zend_update_class_constants
0001:005ffbe7  __object_and_properties_init
0001:005ffd16  __object_init_ex
0001:005ffd3f  __object_init
0001:005ffd62  __zend_get_parameters_array
0001:005ffe2b  _zend_get_parameters
0001:005fff12  _zend_update_static_property
0001:00600065  _zend_update_static_property_stringl
0001:006000e8  _zend_update_static_property_string
0001:00600178  _zend_update_static_property_double
0001:006001db  _zend_update_static_property_long
0001:0060023e  _zend_update_static_property_bool
0001:006002a9  _zend_update_static_property_null
0001:00601961  _zend_parse_method_parameters_ex
0001:00601ada  _zend_parse_method_parameters
0001:00601c38  _zend_parse_parameters
0001:00601cbd  _zend_parse_parameters_ex
0001:00601d45  _add_get_assoc_string_ex
0001:00601ed8  _add_get_assoc_stringl_ex
0001:00602072  _add_assoc_long_ex
0001:006021dc  _add_assoc_null_ex
0001:00602344  _add_assoc_bool_ex
0001:006024b4  _add_assoc_resource_ex
0001:00602622  _add_assoc_double_ex
0001:00602794  _add_assoc_string_ex
0001:00602929  _add_assoc_stringl_ex
Module: U:\dev\php-5.3.20\Zend\zend_extensions.obj(zend_extensions.obj)
0002:00022228  _zend_extensions
0001:00602b9e  _zend_get_resource_handle
0001:00602bdc  _zend_os2_module_error
0001:00602d8f  _zend_os2_query_symbol
0001:00602dc3  _zend_os2_load_module
0001:00602dfd  _zend_get_extension
0001:00602e47  _zend_extension_dispatch_message
0001:00602e91  _zend_extension_dtor
0001:00602eac  _zend_shutdown_extensions
0001:00602eda  _zend_startup_extensions
0001:00602f31  _zend_startup_extensions_mechanism
0001:00602f69  _zend_register_extension
0001:006031b7  _zend_load_extension
Module: U:\dev\php-5.3.20\Zend\zend_hash.obj(zend_hash.obj)
0001:006033f0  _zend_hash_set_apply_protection
0001:006033fe  _zend_hash_index_find
0001:0060343b  _zend_hash_index_exists
0001:00603475  _zend_hash_num_elements
0001:00603480  _zend_hash_get_pointer
0001:006034a9  _zend_hash_set_pointer
0001:00603501  _zend_hash_internal_pointer_reset_ex
0001:0060351d  _zend_hash_internal_pointer_end_ex
0001:00603539  _zend_hash_move_forward_ex
0001:0060355f  _zend_hash_move_backwards_ex
0001:00603585  _zend_hash_get_current_key_type_ex
0001:006035af  _zend_hash_get_current_data_ex
0001:006035d8  _zend_hash_minmax
0001:0060367a  _zend_hash_next_free_element
0001:00603685  _zend_hash_quick_exists
0001:00603710  _zend_hash_quick_find
0001:006037db  _zend_hash_compare
0001:00603c05  _zend_hash_reverse_apply
0001:00603c8c  _zend_hash_apply_with_argument
0001:00603d18  _zend_hash_apply
0001:00603d9b  _zend_hash_graceful_reverse_destroy
0001:00603de0  _zend_hash_graceful_destroy
0001:00603e24  _zend_hash_destroy
0001:00603f0b  _zend_hash_get_current_key_ex
0001:00603f8d  _zend_hash_apply_with_arguments
0001:00604047  _zend_hash_clean
0001:006040f8  _zend_hash_rehash
0001:00604159  _zend_hash_sort
0001:006043d0  __zend_hash_init
0001:006044ba  __zend_hash_init_ex
0001:006044f9  _zend_hash_func
0001:0060464e  _zend_get_hash_value
0001:006047a2  _zend_hash_exists
0001:00604945  _zend_hash_find
0001:00604af1  __zend_hash_index_update_or_next_insert
0001:00604eb6  __zend_hash_quick_add_or_update
0001:006052a2  _zend_hash_merge_ex
0001:0060535b  __zend_hash_merge
0001:00605458  _zend_hash_copy
0001:00605535  _zend_hash_update_current_key_ex
0001:00605dc9  __zend_hash_add_or_update
0001:006062b1  _zend_hash_add_empty_element
0001:006062f8  _zend_hash_del_key_or_index
Module: U:\dev\php-5.3.20\Zend\zend_list.obj(zend_list.obj)
0002:00022248  _le_index_ptr
0001:006065f6  __zend_list_addref
0001:0060663c  __zend_list_find
0001:00606692  _zend_rsrc_list_get_rsrc_type
0001:006066df  _zend_destroy_rsrc_list_dtors
0001:006066f3  _zend_init_rsrc_list_dtors
0001:00606731  _zend_init_rsrc_list
0001:00606b09  _list_entry_destructor
0001:0060679d  _zend_fetch_list_dtor_id
0001:00606818  _zend_register_list_destructors_ex
0001:00606899  _zend_register_list_destructors
0001:0060691b  _zend_clean_module_rsrc_dtors
0001:0060699e  _zend_destroy_rsrc_list
0001:006069aa  _zend_init_rsrc_plist
0001:00606a33  _plist_entry_destructor
0001:00606c67  _zend_fetch_resource
0001:00606e62  __zend_list_delete
0001:00606ef4  _zend_list_insert
0001:00606f85  _zend_register_resource
Module: U:\dev\php-5.3.20\Zend\zend_indent.obj(zend_indent.obj)
0001:0060703c  _zend_indent
Module: U:\dev\php-5.3.20\Zend\zend_builtin_functions.obj(zend_builtin_functions.obj)
0001:00609a34  _debug_print_backtrace_args
0001:00609ab6  _zend_startup_builtin_functions
0001:00609b07  _zm_startup_core
0001:0060a133  _zend_fetch_debug_backtrace
0002:00004220  _zend_builtin_module
Module: U:\dev\php-5.3.20\Zend\zend_sprintf.obj(zend_sprintf.obj)
0001:0060cc50  _zend_sprintf
Module: U:\dev\php-5.3.20\Zend\zend_ini.obj(zend_ini.obj)
0001:0060ccef  _OnUpdateStringUnempty
0001:0060cd2e  _OnUpdateString
0001:0060cd56  _OnUpdateReal
0001:0060cd95  _OnUpdateLongGEZero
0001:0060cdde  _OnUpdateLong
0001:0060ce28  _OnUpdateBool
0001:0060cecf  _display_link_numbers
0001:0060cf3e  _zend_ini_boolean_displayer_cb
0001:0060d04f  _zend_ini_color_displayer_cb
0001:0060d0e3  _zend_ini_string_ex
0001:0060d16f  _zend_ini_string
0001:0060d1b1  _zend_ini_double
0001:0060d236  _zend_ini_register_displayer
0001:0060d277  _zend_ini_long
0001:0060d41c  _zend_restore_ini_entry
0001:0060d513  _zend_alter_ini_entry_ex
0001:0060d72b  _zend_alter_ini_entry
0001:0060d781  _zend_ini_refresh_caches
0001:0060d7b9  _zend_unregister_ini_entries
0001:0060d7e4  _zend_register_ini_entries
0001:0060d94c  _zend_ini_sort_entries
0001:0060d9dd  _zend_ini_startup
0001:0060da51  _zend_copy_ini_directives
0001:0060db19  _zend_ini_deactivate
0001:0060db9f  _zend_ini_global_shutdown
0001:0060dbc3  _zend_ini_shutdown
Module: U:\dev\php-5.3.20\Zend\zend_qsort.obj(zend_qsort.obj)
0001:0060dc10  _zend_qsort
Module: U:\dev\php-5.3.20\Zend\zend_ts_hash.obj(zend_ts_hash.obj)
0001:0060e030  _zend_ts_hash_rehash
0001:0060e0e1  _zend_ts_hash_num_elements
0001:0060e10d  _zend_ts_hash_minmax
0001:0060e155  _zend_ts_hash_compare
0001:0060e1b4  _zend_ts_hash_sort
0001:0060e204  _zend_ts_hash_merge_ex
0001:0060e278  _zend_ts_hash_merge
0001:0060e2ec  _zend_ts_hash_copy_to_hash
0001:0060e33d  _zend_ts_hash_copy
0001:0060e3a4  _zend_ts_hash_index_exists
0001:0060e3d7  _zend_ts_hash_exists
0001:0060e411  _zend_ts_hash_index_find
0001:0060e44b  _zend_ts_hash_quick_find
0001:0060e493  _zend_ts_hash_find
0001:0060e4d4  _zend_ts_get_hash_value
0001:0060e50a  _zend_ts_hash_del_key_or_index
0001:0060e55a  _zend_ts_hash_reverse_apply
0001:0060e599  _zend_ts_hash_apply_with_arguments
0001:0060e5e5  _zend_ts_hash_apply_with_argument
0001:0060e631  _zend_ts_hash_apply
0001:0060e670  _zend_ts_hash_graceful_destroy
0001:0060e6b3  _zend_ts_hash_add_empty_element
0001:0060e6f5  __zend_ts_hash_index_update_or_next_insert
0001:0060e74c  __zend_ts_hash_quick_add_or_update
0001:0060e7b1  __zend_ts_hash_add_or_update
0001:0060e80f  _zend_ts_hash_clean
0001:0060e843  _zend_ts_hash_destroy
0001:0060e886  __zend_ts_hash_init_ex
0001:0060e8ec  __zend_ts_hash_init
Module: U:\dev\php-5.3.20\Zend\zend_stream.obj(zend_stream.obj)
0001:0060e9f3  _zend_compare_file_handles
0001:0060ea83  _zend_file_handle_dtor
0001:0060eb61  _zend_stream_open
0001:0060ebd2  _zend_stream_fixup
Module: U:\dev\php-5.3.20\Zend\zend_iterators.obj(zend_iterators.obj)
0001:0060efc7  _zend_iterator_unwrap
0001:0060f028  _zend_iterator_wrap
0001:0060f0a1  _zend_register_iterator_wrapper
Module: U:\dev\php-5.3.20\Zend\zend_interfaces.obj(zend_interfaces.obj)
0002:00022258  _zend_ce_traversable
0002:00022268  _zend_ce_aggregate
0002:00022278  _zend_ce_iterator
0002:00022288  _zend_ce_arrayaccess
0002:00022298  _zend_ce_serializable
0001:0060f1d7  _zend_user_it_invalidate_current
0001:0060f277  _zend_register_interfaces
0001:00610960  _zend_funcs_aggregate
0001:00610990  _zend_funcs_iterator
0001:00610a40  _zend_funcs_arrayaccess
0001:00610ab0  _zend_funcs_serializable
0001:00610151  _zend_user_serialize
0001:00610037  _zend_user_unserialize
0001:0061084a  _zend_user_it_get_new_iterator
0001:0060fbef  _zend_class_unserialize_deny
0001:0060fc51  _zend_class_serialize_deny
0001:0060fcef  _zend_call_method
0001:00610266  _zend_user_it_rewind
0001:006102e1  _zend_user_it_move_forward
0001:006103a1  _zend_user_it_get_current_key
0001:0061054d  _zend_user_it_get_current_data
0001:006105d1  _zend_user_it_valid
0001:00610793  _zend_user_it_new_iterator
0002:000042f0  _zend_interface_iterator_funcs_iterator
0002:0001c280  _zend_funcs_traversable
Module: U:\dev\php-5.3.20\Zend\zend_exceptions.obj(zend_exceptions.obj)
0002:000222a8  _default_exception_ce
0002:000222b8  _error_exception_ce
0002:000222c8  _zend_throw_exception_hook
0001:00610c00  _zend_exception_get_default
0001:00610c0a  _zend_get_error_exception
0001:00610c14  _zend_clear_exception
0001:00610d7b  _zend_exception_error
0001:006110bd  _zend_spprintf
0001:00611125  _zend_register_default_exception
0001:006116bf  _zend_exception_set_previous
0001:006117d3  _zend_throw_exception_internal
0001:00611943  _zend_throw_exception_object
0001:006119f9  _zend_throw_exception
0001:00611b03  _zend_throw_error_exception
0001:00611b63  _zend_throw_exception_ex
0001:00611be4  _zim_exception___clone
0001:00611c0b  _zend_exception_restore
0001:00611c79  _zend_exception_save
0001:00611d53  _zim_error_exception_getSeverity
0001:00611da7  _zim_exception_getTrace
0001:00611dfb  _zim_exception_getCode
0001:00611e4f  _zim_exception_getMessage
0001:00611ea3  _zim_exception_getLine
0001:00611ef7  _zim_exception_getFile
0001:00611f4b  _zim_exception_getPrevious
0001:00612075  _zim_exception___toString
0001:006124c3  _zim_exception_getTraceAsString
0001:00613009  _zim_error_exception___construct
0001:0061326a  _zim_exception___construct
Module: U:\dev\php-5.3.20\Zend\zend_strtod.obj(zend_strtod.obj)
0001:00613a95  _zend_hex_strtod
0001:00613b4a  _zend_oct_strtod
0001:00613c17  _zend_freedtoa
0001:006143d5  _zend_strtod
0001:00615463  _zend_dtoa
0001:006166a5  _zend_shutdown_strtod
0001:00616732  _zend_startup_strtod
Module: U:\dev\php-5.3.20\Zend\zend_gc.obj(zend_gc.obj)
0002:000222d8  _gc_globals_id
0001:00616939  _gc_globals_dtor
0001:0061693e  _gc_reset
0001:00616e91  _gc_remove_zval_from_buffer
0001:00616ef2  _gc_collect_cycles
0001:0061758f  _gc_zobj_possible_root
0001:006176ac  _gc_zval_possible_root
0001:006177db  _gc_init
0001:0061783a  _gc_globals_ctor
Module: U:\dev\php-5.3.20\Zend\zend_closures.obj(zend_closures.obj)
0002:000222e8  _zend_ce_closure
0001:006178f2  _zend_closure_get_closure
0001:00617942  _zend_get_closure_method_def
0001:0061795f  _zend_create_closure
0001:00617b58  _zim_Closure___construct
0001:00617e73  _zend_register_closure_ce
0001:00618168  _zend_get_closure_invoke_method
0001:006182b5  _zim_Closure___invoke
Module: U:\dev\php-5.3.20\Zend\zend_float.obj(zend_float.obj)
0001:006187a0  _zend_ensure_fpu_mode
0001:006187a5  _zend_shutdown_fpu
0001:006187e9  _zend_init_fpu
Module: U:\dev\php-5.3.20\Zend\zend_objects.obj(zend_objects.obj)
0001:00618830  _zend_object_std_init
0001:0061888b  _zend_objects_clone_members
0001:0061897b  _zend_objects_get_address
0001:00618987  _zend_objects_new
0001:00618e77  _zend_objects_free_object_storage
0001:00618b4d  _zend_objects_destroy_object
0001:006189df  _zend_objects_clone_obj
0001:00618e2e  _zend_object_std_dtor
Module: U:\dev\php-5.3.20\Zend\zend_object_handlers.obj(zend_object_handlers.obj)
0001:00618f44  _zend_check_protected
0001:00618f83  _zend_std_object_get_class
0001:00618f9f  _zend_std_get_properties
0001:00618fbc  _zend_std_get_debug_info
0001:006190f8  _zend_std_get_constructor
0001:006192a9  _zend_std_unset_static_property
0001:0061a213  _zend_std_call_user_call
0001:00619345  _zend_std_object_get_class_name
0001:00619fe3  _zend_std_callstatic_user_call
0001:0061940f  _zend_std_get_closure
0001:00619686  _zend_get_property_info
0001:006199fe  _zend_std_get_static_property
0001:00619b99  _zend_std_get_static_method
0001:00619eec  _zend_check_property_access
0001:0061a84f  _zend_std_read_property
0001:0061b126  _zend_std_read_dimension
0001:0061b561  _zend_check_private
0001:0061b6fc  _zend_std_cast_object_tostring
0002:00004310  _std_object_handlers
Module: U:\dev\php-5.3.20\Zend\zend_objects_API.obj(zend_objects_API.obj)
0001:0061c780  _zend_objects_store_call_destructors
0001:0061c7ef  _zend_objects_store_mark_destructed
0001:0061c81e  _zend_objects_store_free_object_storage
0001:0061c8d9  _zend_objects_store_get_refcount
0001:0061c8ff  _zend_objects_store_add_ref
0001:0061c925  _zend_objects_store_add_ref_by_handle
0001:0061c949  _zend_object_store_get_object
0001:0061c96f  _zend_object_store_get_object_by_handle
0001:0061c993  _zend_object_store_set_object
0001:0061c9bc  _zend_object_store_ctor_failed
0001:0061c9e7  _zend_get_std_object_handlers
0001:0061ca2d  _zend_object_proxy_get
0001:0061cad7  _zend_object_proxy_set
0001:0061cb49  _zend_objects_proxy_clone
0001:0061cb8a  _zend_objects_proxy_free_storage
0001:0061cbb4  _zend_objects_store_destroy
0001:0061cbfe  _zend_objects_store_del_ref_by_handle_ex
0001:0061ceab  _zend_objects_store_del_ref
0001:0061cf10  _zend_objects_store_put
0001:0061d021  _zend_object_create_proxy
0001:0061d0e3  _zend_objects_store_clone_obj
0001:0061d1b4  _zend_objects_store_init
Module: U:\dev\php-5.3.20\Zend\zend_default_classes.obj(zend_default_classes.obj)
0001:0061d200  _zend_register_default_classes
Module: U:\dev\php-5.3.20\Zend\zend_execute.obj(zend_execute.obj)
0002:000222f8  _zend_opcode_handlers
0001:0061d38b  _zend_get_compiled_variable_value
0001:0061d3ed  _execute_internal
0001:0061d4f4  _zend_init_opcodes_handlers
0001:0061d503  _zend_vm_set_opcode_handler
0001:0061d544  _zend_set_user_opcode_handler
0001:0061d56d  _zend_get_user_opcode_handler
0001:0061fb98  _execute
0001:00625337  _zend_get_zval_ptr_ptr
0001:00647b84  _zend_do_fcall
0001:006656d8  _zend_get_zval_ptr
Module: U:\usr\local446\lib\gcc\i386-pc-os2-emx\4.4.6\libgcc_eh.lib(emx-dllinit.obj)
0001:00685f80  _DLL_InitTerm
Module: U:\usr\lib\libend.lib(src/libend/386/endlink386.asm)
0002:00022380  _end
0002:00008da0  _edata
Module: U:\usr\lib\libend.lib(src/libend/386/end.asm)
0001:008bce00* _etext
0001:008bce00* __etext
0000:00000000* WEAK$ZERO
0002:00022380  __end
0002:00008da0  __edata
Module: U:\usr\local446\lib\gcc\i386-pc-os2-emx\4.4.6\libgcc.lib(_moddi3.obj)
0001:00685fc0  ___moddi3
Module: U:\usr\local446\lib\gcc\i386-pc-os2-emx\4.4.6\libgcc.lib(_divdi3.obj)
0001:00686180  ___divdi3
Module: U:\usr\local446\lib\gcc\i386-pc-os2-emx\4.4.6\libgcc.lib(_umoddi3.obj)
0001:006862c0  ___umoddi3
Module: U:\extras\lib\xml2.lib(xmlIO.obj)
0001:006863e0  _xmlCleanupInputCallbacks
0001:00686439* _xmlPopInputCallbacks
0001:0068648d  _xmlCleanupOutputCallbacks
0001:006864ee* _xmlFileMatch
0001:0068650c* _xmlRegisterInputCallbacks
0001:0068655e* _xmlRegisterOutputCallbacks
0001:006865b0  _xmlRegisterDefaultInputCallbacks
0001:00689f87* _xmlFileOpen
0001:00689e66* _xmlFileRead
0001:00689df4* _xmlFileClose
0001:00686947* _xmlIOHTTPMatch
0001:006873aa* _xmlIOHTTPOpen
0001:0068737d* _xmlIOHTTPRead
0001:006872f0* _xmlIOHTTPClose
0001:00686914* _xmlIOFTPMatch
0001:00687371* _xmlIOFTPOpen
0001:00687344* _xmlIOFTPRead
0001:00687338* _xmlIOFTPClose
0001:006866fb  _xmlRegisterDefaultOutputCallbacks
0001:00686790* _xmlRegisterHTTPPostCallbacks
0001:006868f6* _xmlSetExternalEntityLoader
0001:00686903* _xmlGetExternalEntityLoader
0001:00686972* _xmlNormalizeWindowsPath
0001:006869ae  _xmlParserGetDirectory
0001:00686a6a  _xmlOutputBufferGetSize
0001:00686a8b  _xmlOutputBufferGetContent
0001:00686aac  _xmlOutputBufferCreateFilenameDefault
0001:00689aca  ___xmlOutputBufferCreateFilename
0001:00686ad7  _xmlParserInputBufferCreateFilenameDefault
0001:006871c3  ___xmlParserInputBufferCreateFilename
0001:00686b18  _xmlParserInputBufferCreateStatic
0001:00686cf4  _xmlFreeParserInputBuffer
0001:00686d77  _xmlAllocOutputBufferInternal
0001:00686e36  _xmlOutputBufferCreateIO
0001:00686e69  _xmlOutputBufferCreateBuffer
0001:00686e99  _xmlOutputBufferCreateFd
0001:00686ece  _xmlOutputBufferCreateFile
0001:00686f13  _xmlAllocOutputBuffer
0001:00686fe4  _xmlAllocParserInputBuffer
0001:006870ad  _xmlParserInputBufferCreateIO
0001:006870e0  _xmlParserInputBufferCreateMem
0001:00687148  _xmlParserInputBufferCreateFd
0001:0068717d* _xmlParserInputBufferCreateFile
0001:006872ba  _xmlParserInputBufferCreateFilename
0001:006873c5* _xmlCheckFilename
0001:006875a8  _xmlLoadExternalEntity
0001:0068784b  ___xmlLoaderErr
0001:006879bb  _xmlCheckHTTPInput
0001:00687b4a  ___xmlIOErr
0001:006880d9* _xmlNoNetExternalEntityLoader
0001:006882a6  _xmlOutputBufferFlush
0001:006883d3  _xmlOutputBufferClose
0001:006884c8  _xmlOutputBufferWriteEscape
0001:006887b0  _xmlOutputBufferWrite
0001:006889b9  _xmlOutputBufferWriteString
0001:00688a1d  _xmlParserInputBufferGrow
0001:00688bc7  _xmlParserInputBufferRead
0001:00688c05  _xmlParserInputBufferPush
0001:00689a17* _xmlIOHTTPOpenW
0001:00689d85  _xmlOutputBufferCreateFilename
Module: U:\extras\lib\xml2.lib(uri.obj)
0001:0068a8ea  _xmlFreeURI
0001:0068a9a0* _xmlNormalizeURIPath
0001:0068ae3c  _xmlCreateURI
0001:0068ae91  _xmlURIUnescapeString
0001:0068b076  _xmlSaveUri
0001:0068bc48  _xmlURIEscapeStr
0001:0068bdc5* _xmlPrintURI
0001:0068cd1e  _xmlParseURIReference
0001:0068cd52  _xmlBuildRelativeURI
0001:0068d1d7  _xmlBuildURI
0001:0068d6c6  _xmlURIEscape
0001:0068da15  _xmlParseURIRaw
0001:0068da62  _xmlParseURI
0001:0068daac  _xmlCanonicPath
0001:0068db6f  _xmlPathToURI
Module: U:\extras\lib\xml2.lib(xmlstring.obj)
0001:0068dbf0  _xmlStrcmp
0001:0068dc42  _xmlStrEqual
0001:0068dc77  _xmlStrQEqual
0001:0068dcee  _xmlStrcasecmp
0001:0068dd4e  _xmlStrncasecmp
0001:0068ddb7  _xmlStrchr
0001:0068ddd9  _xmlStrcasestr
0001:0068de57  _xmlStrlen
0001:0068de77* _xmlUTF8Size
0001:0068deb7  _xmlUTF8Strlen
0001:0068df5b  _xmlGetUTF8Char
0001:0068e0a1  _xmlCheckUTF8
0001:0068e17f  _xmlUTF8Strsize
0001:0068e1c7  _xmlUTF8Strpos
0001:0068e240  _xmlUTF8Strndup
0001:0068e2d1  _xmlUTF8Strsub
0001:0068e35f* _xmlStrVPrintf
0001:0068e3a7  _xmlStrPrintf
0001:0068e3ef  _xmlCharStrndup
0001:0068e468  _xmlCharStrdup
0001:0068e49a  _xmlStrndup
0001:0068e503* _xmlStrsub
0001:0068e558  _xmlStrdup
0001:0068e58a  _xmlStrncat
0001:0068e639  _xmlStrcat
0001:0068e686  _xmlStrncatNew
0001:0068e783  _xmlStrncmp
0001:0068e7bf  _xmlUTF8Strloc
0001:0068e85b* _xmlUTF8Charcmp
0001:0068e89a  _xmlStrstr
Module: U:\extras\lib\xml2.lib(globals.obj)
0002:00022310+ _xmlLastError
0001:0068ea10* _xmlRegisterNodeDefault
0001:0068ea2d* _xmlDeregisterNodeDefault
0001:0068ea4a  ___xmlOutputBufferCreateFilenameValue
0001:0068ea71  ___xmlParserInputBufferCreateFilenameValue
0001:0068ea95  ___xmlDeregisterNodeDefaultValue
0001:0068eab9  ___xmlRegisterNodeDefaultValue
0001:0068eae1  ___xmlSubstituteEntitiesDefaultValue
0001:0068eb05  ___xmlSaveNoEmptyTags
0001:0068eb29  ___xmlPedanticParserDefaultValue
0001:0068eb51  ___xmlParserVersion
0001:0068eb71  ___xmlParserDebugEntities
0001:0068eb95  ___xmlLoadExtDtdDefaultValue
0001:0068ebb9  ___xmlLineNumbersDefaultValue
0001:0068ebe1  ___xmlKeepBlanksDefaultValue
0001:0068ec05  ___xmlTreeIndentString
0001:0068ec29  ___xmlIndentTreeOutput
0001:0068ec51  ___xmlGetWarningsDefaultValue
0001:0068ec75  ___xmlStructuredErrorContext
0001:0068ec99  ___xmlGenericErrorContext
0001:0068ecc1  ___xmlStructuredError
0001:0068ece5  ___xmlGenericError
0001:0068ed09  ___xmlDoValidityCheckingDefaultValue
0001:0068ed31  ___xmlDefaultSAXLocator
0001:0068ed53  ___xmlDefaultSAXHandler
0001:0068ed75  ___xmlDefaultBufferSize
0001:0068ed99  ___xmlBufferAllocScheme
0001:0068edc1* ___oldXMLWDcompatibility
0001:0068ede5  ___xmlLastError
0001:0068ee09  ___htmlDefaultSAXHandler
0001:0068ee31  ___docbDefaultSAXHandler
0001:0068ee55* _xmlThrDefSubstituteEntitiesDefaultValue
0001:0068ee8c* _xmlThrDefSaveNoEmptyTags
0001:0068eec3* _xmlThrDefPedanticParserDefaultValue
0001:0068eefa* _xmlThrDefParserDebugEntities
0001:0068ef31* _xmlThrDefLoadExtDtdDefaultValue
0001:0068ef68* _xmlThrDefLineNumbersDefaultValue
0001:0068ef9f* _xmlThrDefKeepBlanksDefaultValue
0001:0068efd6* _xmlThrDefTreeIndentString
0001:0068f00d* _xmlThrDefIndentTreeOutput
0001:0068f044* _xmlThrDefGetWarningsDefaultValue
0001:0068f07b* _xmlThrDefDoValidityCheckingDefaultValue
0001:0068f0b2* _xmlThrDefDefaultBufferSize
0001:0068f0e9* _xmlThrDefBufferAllocScheme
0001:0068f120* _xmlThrDefOutputBufferCreateFilenameDefault
0001:0068f162* _xmlThrDefParserInputBufferCreateFilenameDefault
0001:0068f1a4* _xmlThrDefDeregisterNodeDefault
0001:0068f1e5* _xmlThrDefRegisterNodeDefault
0001:0068f226* _xmlThrDefSetStructuredErrorFunc
0001:0068f260* _xmlThrDefSetGenericErrorFunc
0001:0068f2aa  _xmlCleanupGlobals
0001:0068f2d1  _xmlInitGlobals
0001:0068f2f4  _xmlInitializeGlobalState
0002:00004664* _xmlParserVersion
0002:00004674* _xmlKeepBlanksDefaultValue
0002:00004680* _xmlTreeIndentString
0002:0000467c* _xmlIndentTreeOutput
0002:00004670* _xmlGetWarningsDefaultValue
0002:00004678* _xmlGenericError
0002:00004700* _xmlDefaultSAXLocator
0002:00004690* _xmlDefaultSAXHandler
0002:0000466c* _xmlDefaultBufferSize
0002:00004668* _xmlBufferAllocScheme
0002:00004710* _htmlDefaultSAXHandler
0002:00004780* _docbDefaultSAXHandler
0002:00004650  _xmlFree
0002:00004654  _xmlMalloc
0002:00004658  _xmlMallocAtomic
0002:0000465c  _xmlRealloc
0002:00004660  _xmlMemStrdup
0002:0001ca1c* _xmlRegisterNodeDefaultValue
0002:0001ca20* _xmlDeregisterNodeDefaultValue
0002:0001ca28* _xmlOutputBufferCreateFilenameValue
0002:0001ca24* _xmlParserInputBufferCreateFilenameValue
0002:0001ca18* _xmlSubstituteEntitiesDefaultValue
0002:0001ca38* _xmlSaveNoEmptyTags
0002:0001ca10* _xmlPedanticParserDefaultValue
0002:0001ca04* _xmlParserDebugEntities
0002:0001ca0c* _xmlLoadExtDtdDefaultValue
0002:0001ca14* _xmlLineNumbersDefaultValue
0002:0001ca34* _xmlStructuredErrorContext
0002:0001ca30* _xmlGenericErrorContext
0002:0001ca2c* _xmlStructuredError
0002:0001ca08* _xmlDoValidityCheckingDefaultValue
0002:0001ca00* _oldXMLWDcompatibility
Module: U:\extras\lib\xml2.lib(error.obj)
0001:0068f65c* _xmlCtxtGetLastError
0001:0068f67b  _xmlCopyError
0001:0068f78d  _xmlGetLastError
0001:0068f7a9  _xmlResetError
0001:0068f821* _xmlCtxtResetLastError
0001:0068f84f  _xmlResetLastError
0001:0068f877  _initGenericErrorDefaultFunc
0001:0069103e  _xmlGenericErrorDefaultFunc
0001:006900e1* _xmlParserPrintFileContext
0001:00690103* _xmlParserPrintFileInfo
0001:00690175  _xmlSetGenericErrorFunc
0001:006901be  _xmlParserValidityWarning
0001:00690352  _xmlParserValidityError
0001:00690517  _xmlParserWarning
0001:006906d4  _xmlParserError
0001:00690887  _xmlSetStructuredErrorFunc
0001:006908c2  ___xmlRaiseError
0001:00690ecd  ___xmlSimpleError
Module: U:\extras\lib\xml2.lib(tree.obj)
0001:00691090  _xmlSplitQName3
0001:006910dd  _xmlSetNs
0001:006910ef  _xmlFreeNs
0001:00691132  _xmlFreeNsList
0001:00691156  _xmlGetIntSubset
0001:00691181* _xmlSetListDoc
0001:006911b8  _xmlSetTreeDoc
0001:00691224  _xmlGetLastChild
0001:00691241* _xmlChildElementCount
0001:00691288* _xmlFirstElementChild
0001:006912d6* _xmlLastElementChild
0001:00691326* _xmlPreviousElementSibling
0001:006913b1* _xmlNextElementSibling
0001:00691532  _xmlGetLineNo
0001:00691543  _xmlDocGetRootElement
0001:0069156a  _xmlNodeIsText
0001:00691581  _xmlIsBlankNode
0001:006915c9* _xmlBufferDetach
0001:006915f5* _xmlBufferSetAllocationScheme
0001:00691624  _xmlBufferFree
0001:00691676  _xmlBufferEmpty
0001:006916be  _xmlBufferContent
0001:006916ce* _xmlBufferLength
0001:006916df* _xmlGetDocCompressMode
0001:006916f3  _xmlSetDocCompressMode
0001:00691723  _xmlGetCompressMode
0001:0069172d* _xmlSetCompressMode
0001:006917ac* _xmlDOMWrapFreeCtxt
0001:006917db  _xmlNodeSetName
0001:00691deb* _xmlDOMWrapNewCtxt
0001:00691e43  _xmlBufferGrow
0001:00691f07  _xmlBufferCreateStatic
0001:00691f76  _xmlSearchNsByHref
0001:0069214f  _xmlSearchNs
0001:0069232b  _xmlGetNsList
0001:0069246d  _xmlNewNs
0001:00692629* _xmlCopyNamespace
0001:0069265c  _xmlCopyNamespaceList
0001:00692a93  _xmlReconciliateNs
0001:00692e24  _xmlGetNodePath
0001:0069353c  _xmlBufferShrink
0001:00693606* _xmlBufferResize
0001:0069379e  _xmlBufferCCat
0001:00693823  _xmlBufferWriteChar
0001:00693841  _xmlBufferAddHead
0001:00693939  _xmlBufferAdd
0001:006939e9  _xmlBufferCat
0001:00693a20  _xmlBufferWriteCHAR
0001:00693a43  _xmlBufferWriteQuotedString
0001:00693b67* _xmlBufferDump
0001:00693baa* _xmlBufferCreateSize
0001:00693c3b* _xmlGetBufferAllocationScheme
0001:00693c4a* _xmlSetBufferAllocationScheme
0001:00693c71  _xmlBufferCreate
0001:00693ced  _xmlTextConcat
0001:0069403e  _xmlHasNsProp
0001:0069406b  _xmlNewComment
0001:0069c089  _xmlStringComment
0001:006940f1  _xmlNewDocComment
0001:0069411c  _xmlNewText
0001:0069c07a  _xmlStringText
0001:006941a2  _xmlNewDocText
0001:00694423  _xmlNewNsPropEatName
0001:00694456  _xmlNewNsProp
0001:00694489  _xmlNewProp
0001:006944c4  _xmlNewDocFragment
0001:00694542* _xmlNewNodeEatName
0001:006945c1  _xmlNewNode
0001:00694654  _xmlNewDocPI
0001:0069471d  _xmlNewPI
0001:00694750  _xmlNewDoc
0001:0069483b  _xmlCreateIntSubset
0001:00694a41  _xmlNewDtd
0001:00694b25  _xmlNewCDataBlock
0001:00694bb1  _xmlNewTextLen
0001:00694c3d* _xmlNewDocTextLen
0001:00694c74  _xmlNewReference
0001:00694d7a  _xmlNewCharRef
0001:00694e4d  _xmlSplitQName2
0001:00694ef8  _xmlHasProp
0001:00694f96  _xmlBufGetNodeContent
0001:0069518a* _xmlNodeBufGetContent
0001:006951d8  _xmlUnlinkNode
0001:006953cd* _xmlDOMWrapRemoveNode
0001:006955a6  _xmlReplaceNode
0001:006956a2* _xmlNodeListGetRawString
0001:006957c7  _xmlNodeListGetString
0001:006959a4  _xmlGetNsProp
0001:006959da  _xmlNodeGetSpacePreserve
0001:00695a7a  _xmlNodeGetLang
0001:00695ac0  _xmlGetNoNsProp
0001:00695ae6  _xmlGetProp
0001:00695b32  _xmlNodeGetBase
0001:00695d71  _xmlNodeGetContent
0001:00695ea9  _xmlFreeDtd
0001:00696abe  _xmlFreeNode
0001:00696031  _xmlFreeDoc
0001:00696207  _xmlFreeNodeList
0001:00696a99  _xmlFreePropList
0001:006963c0  _xmlSetNsProp
0001:00696527  _xmlSetProp
0001:006965db  _xmlNodeSetBase
0001:006966ff* _xmlNodeSetSpacePreserve
0001:00696786* _xmlNodeSetLang
0001:006967db  _xmlFreeProp
0001:00696887* _xmlUnsetNsProp
0001:006968cf  _xmlUnsetProp
0001:0069690d* _xmlRemoveProp
0001:00696ccc* _xmlTextMerge
0001:00696e60  _xmlNodeAddContent
0001:00696d29  _xmlNodeAddContentLen
0001:00696e95  _xmlAddChild
0001:00697046  _xmlAddChildList
0001:00697145  _xmlAddSibling
0001:00697245  _xmlDocSetRootElement
0001:006972cb  _xmlAddNextSibling
0001:0069781e  _xmlNodeSetContent
0001:006973f8  _xmlStringGetNodeList
0001:00697947  _xmlNewDocNodeEatName
0001:006979df  _xmlNewDocNode
0001:00697a77  _xmlNewChild
0001:00697b61* _xmlNewDocRawNode
0001:00697bd6  _xmlNewTextChild
0001:00697cc1  _xmlNewDocProp
0001:00698022* _xmlCopyProp
0001:00698036  _xmlCopyPropList
0001:0069c07f  _xmlStringTextNoenc
0001:0069874e  _xmlCopyDoc
0001:006984d2  _xmlDocCopyNode
0001:006984ec  _xmlCopyNode
0001:00698505  _xmlCopyDtd
0001:0069884d  _xmlCopyNodeList
0001:00698860  _xmlDocCopyNodeList
0001:00698874  _xmlStringLenGetNodeList
0001:00698d20  _xmlNodeSetContentLen
0001:00698e5d  _xmlAddPrevSibling
0001:00698f85  _xmlValidateNMToken
0001:0069939e  _xmlValidateName
0001:00699735  _xmlValidateQName
0001:00699d0c  _xmlValidateNCName
0001:0069a0b4  _xmlBuildQName
0001:0069a404* _xmlDOMWrapCloneNode
0001:0069adb2* _xmlDOMWrapReconcileNamespaces
0001:0069b26d* _xmlDOMWrapAdoptNode
0002:0001cb40  ___xmlRegisterCallbacks
Module: U:\extras\lib\xml2.lib(valid.obj)
0001:0069c130  _xmlFreeValidCtxt
0001:0069c169* _xmlSprintfElementContent
0001:0069c16e  _xmlFreeEnumeration
0001:0069c208  _xmlValidateNotationDecl
0001:0069c235* _xmlValidGetPotentialChildren
0001:0069c5f6  _xmlValidatePushCData
0001:0069ca00  _xmlNewValidCtxt
0001:0069cb16  _xmlValidateDtdFinal
0001:0069cc0b  _xmlValidateDocumentFinal
0001:0069cc76  _xmlDumpNotationTable
0001:0069cca2* _xmlDumpAttributeTable
0001:0069ccce* _xmlDumpElementTable
0001:0069cd84  _xmlCreateEnumeration
0001:0069cdd5* _xmlCopyEnumeration
0001:0069cf42  _xmlValidateRoot
0001:0069d0f2  _xmlValidatePopElement
0001:0069d21e  _xmlSnprintfElementContent
0001:0069da23* _xmlValidateNamesValue
0001:0069dab0* _xmlValidateNameValue
0001:0069dbbf* _xmlValidateNmtokensValue
0001:0069dcb4* _xmlValidateAttributeValue
0001:0069dcc5* _xmlValidateNmtokenValue
0001:0069dcd6* _xmlGetDtdNotationDesc
0001:0069e0c8  _xmlValidateNotationUse
0001:0069e19e* _xmlGetRefs
0001:0069e1c6  _xmlGetID
0001:0069e56a  _xmlGetDtdQAttrDesc
0001:0069e5a6  _xmlGetDtdAttrDesc
0001:0069e64d  _xmlValidNormalizeAttributeValue
0001:0069e7e2  _xmlValidCtxtNormalizeAttributeValue
0001:0069ea09  _xmlIsRef
0001:0069eaa9  _xmlGetDtdQElementDesc
0001:0069eaca* _xmlGetDtdElementDesc
0001:0069eff4  _xmlValidateElementDecl
0001:0069f353  _xmlIsMixedElement
0001:0069f3b7* _xmlRemoveRef
0001:0069f4c8  _xmlFreeRefTable
0001:0069f4e3  _xmlFreeIDTable
0001:0069f4fe  _xmlFreeNotationTable
0001:0069f519  _xmlFreeAttributeTable
0001:0069f534  _xmlFreeElementTable
0001:0069f5a4  _xmlAddNotationDecl
0001:0069f759  _xmlAddRef
0001:0069f964  _xmlRemoveID
0001:0069fab6  _xmlFreeDocElementContent
0001:0069fba8* _xmlFreeElementContent
0001:0069fbd1  _xmlIsID
0001:0069fec5  _xmlAddID
0001:006a03e2  _xmlValidateOneNamespace
0001:006a0ca3  _xmlValidateOneAttribute
0001:006a124f* _xmlCopyDocElementContent
0001:006a1465* _xmlCopyElementContent
0001:006a17f5  _xmlDumpElementDecl
0001:006a19af* _xmlDumpNotationDecl
0001:006a1b4a  _xmlDumpAttributeDecl
0001:006a1dc2  _xmlCopyNotationTable
0001:006a1ddd  _xmlCopyAttributeTable
0001:006a1df8  _xmlCopyElementTable
0001:006a20db  _xmlAddElementDecl
0001:006a25b3  _xmlNewDocElementContent
0001:006a2748* _xmlNewElementContent
0001:006a2c98* _xmlValidBuildContentModel
0001:006a2f34  _xmlValidatePushElement
0001:006a3543  _xmlAddAttributeDecl
0001:006a3cc3  _xmlValidateAttributeDecl
0001:006a4889  _xmlValidateOneElement
0001:006a52ec* _xmlValidGetValidElements
0001:006a55da  _xmlValidateElement
0001:006a57b9  _xmlValidateDocument
0001:006a5953  _xmlValidateDtd
Module: U:\extras\lib\xml2.lib(relaxng.obj)
0001:006a5a30* _xmlRelaxParserSetFlag
0001:006a6405  _xmlRelaxNGSetParserErrors
0001:006a6429* _xmlRelaxNGGetParserErrors
0001:006a6465* _xmlRelaxNGSetParserStructuredErrors
0001:006a64ef  _xmlRelaxNGSetValidErrors
0001:006a6513  _xmlRelaxNGSetValidStructuredErrors
0001:006a6538* _xmlRelaxNGGetValidErrors
0001:006a72ff  _xmlRelaxNGNewValidCtxt
0001:006a73aa  _xmlRelaxNGNewMemParserCtxt
0001:006a7811  _xmlRelaxNGNewParserCtxt
0001:006a7877  _xmlRelaxNGFreeValidCtxt
0001:006a90db  _xmlRelaxNGValidatePopElement
0001:006a91a6  _xmlRelaxNGValidatePushCData
0001:006a9239  _xmlRelaxNGValidatePushElement
0001:006a9b95* _xmlRelaxNGDumpTree
0001:006b14e8  _xmlRelaxNGFree
0001:006b15de  _xmlRelaxNGFreeParserCtxt
0001:006b1d87* _xmlRelaxNGNewDocParserCtxt
0001:006b1e05  _xmlRelaxNGCleanupTypes
0001:006b23fe* _xmlRelaxNGDump
0001:006b2870* _xmlRelaxNGInitTypes
0001:006b29b7  _xmlRelaxNGParse
0001:006b57cf  _xmlRelaxNGValidateDoc
0001:006b5f8b  _xmlRelaxNGValidateFullElement
Module: U:\extras\lib\xml2.lib(parser.obj)
0001:006b6080* _xmlHasFeature
0001:006b6099  _xmlCheckLanguageID
0001:006b6315  _inputPop
0001:006b635d  _nodePop
0001:006b63a5* _namePop
0001:006b675e  _xmlStopParser
0001:006b6793* _xmlSetEntityReferenceFunc
0001:006b6b1c  _xmlCtxtUseOptions
0001:006b6e07* _namePush
0001:006b783b  _nodePush
0001:006b7989  _inputPush
0001:006b7a18  _xmlCreateMemoryParserCtxt
0001:006b7ac7* _xmlCreateURLParserCtxt
0001:006b7b7e  _xmlCreateFileParserCtxt
0001:006b7b99  _xmlCtxtReset
0001:006b7ee2* _xmlCtxtResetPush
0001:006b8166  _xmlCleanupParser
0001:006b81c1  _xmlInitParser
0001:006b836f* _xmlCreateDocParserCtxt
0001:006b83bf* _xmlSetupParserForBuffer
0001:006b856f* _xmlCreateEntityParserCtxt
0001:006b8a69* _xmlCreateIOParserCtxt
0001:006b8bc4  _xmlCreatePushParserCtxt
0001:006b8e8b* _xmlParseVersionNum
0001:006b96f3  _xmlPopInput
0001:006b9886* _xmlParseEncName
0001:006b9a48* _xmlParsePubidLiteral
0001:006b9d7e  _xmlPushInput
0001:006ba2c0  _xmlSplitQName
0001:006ba93b  _xmlParserHandlePEReference
0001:006bdb94* _xmlParseName
0001:006bb936* _xmlParseTextDecl
0001:006bace9* _xmlSkipBlankChars
0001:006bb10a* _xmlParseSDDecl
0001:006bb50b* _xmlParseEncodingDecl
0001:006bb781* _xmlParseVersionInfo
0001:006bbbdb* _xmlParseXMLDecl
0001:006bbfce* _xmlParseCDSect
0001:006bc617* _xmlParseComment
0001:006bd117* _xmlParseSystemLiteral
0001:006bd541* _xmlParseNmtoken
0001:006bd9b1* _xmlParseEnumerationType
0001:006be7a3* _xmlParsePEReference
0001:006bea70* _xmlParseEntityRef
0001:006bedb4* _xmlParsePITarget
0001:006bf7af* _xmlParseElementChildrenContentDecl
0001:006bf82a* _xmlParseNotationType
0001:006bfffe* _xmlParseEndTag
0001:006c003b* _xmlParseCharRef
0001:006c0494* _xmlParseExternalID
0001:006c07ad* _xmlParseDocTypeDecl
0001:006c09d4* _xmlParseNotationDecl
0001:006c0c7d* _xmlParseElementMixedContentDecl
0001:006c10f2* _xmlParseElementContentDecl
0001:006c1323* _xmlParseElementDecl
0001:006c170d* _xmlParseEnumeratedType
0001:006c181e* _xmlParseAttributeType
0001:006c1dd0* _xmlParsePI
0001:006c25b9* _xmlParseMisc
0001:006c2aba* _xmlParseCharData
0001:006c305d  _xmlStringLenDecodeEntities
0001:006c3f89  _xmlStringDecodeEntities
0001:006c652f* _xmlParseAttValue
0001:006c656b* _xmlParseAttribute
0001:006c6718* _xmlParseStartTag
0001:006c6c0d* _xmlParseElement
0001:006c7096* _xmlParseContent
0001:006c8d86* _xmlParseReference
0001:006c72b0* _xmlParseBalancedChunkMemoryRecover
0001:006c7680  _xmlParseBalancedChunkMemory
0001:006c76be  _xmlParseInNodeContext
0001:006c7fda* _xmlParseExternalEntity
0001:006c8046  _xmlParseCtxtExternalEntity
0001:006c8589* _xmlParseExtParsedEnt
0001:006c87eb* _xmlSAXParseEntity
0001:006c886a* _xmlParseEntity
0001:006c960f* _xmlParseDefaultDecl
0001:006c9a06* _xmlParseAttributeListDecl
0001:006ca284* _xmlParseEntityValue
0001:006ca8ca* _xmlParseEntityDecl
0001:006cba31* _xmlParseMarkupDecl
0001:006cd8b0  _xmlParseChunk
0001:006cde2f  _xmlParseDocument
0001:006ce362* _xmlCtxtReadIO
0001:006ce435* _xmlCtxtReadFd
0001:006ce4e7  _xmlCtxtReadMemory
0001:006ce59f  _xmlCtxtReadFile
0001:006ce614* _xmlCtxtReadDoc
0001:006ce68a* _xmlReadIO
0001:006ce74f* _xmlReadFd
0001:006ce811  _xmlReadMemory
0001:006ce85b  _xmlReadFile
0001:006ce89c* _xmlReadDoc
0001:006ce8e5* _xmlSAXParseDoc
0001:006ce973* _xmlParseDoc
0001:006ce996* _xmlRecoverDoc
0001:006ce9b9* _xmlSAXUserParseMemory
0001:006cea6f* _xmlSAXParseMemoryWithData
0001:006ceb1b* _xmlSAXParseMemory
0001:006ceb4b* _xmlRecoverMemory
0001:006ceb75* _xmlParseMemory
0001:006ceb9f* _xmlSAXUserParseFile
0001:006cec49* _xmlSAXParseFileWithData
0001:006ced2a* _xmlSAXParseFile
0001:006ced53* _xmlRecoverFile
0001:006ced76* _xmlParseFile
0001:006ced99  _xmlParseExternalSubset
0001:006cf0a4* _xmlSAXParseDTD
0001:006cf31a  _xmlParseDTD
0001:006cf33c* _xmlIOParseDTD
0002:00004810* _xmlParserMaxDepth
Module: U:\usr\local446\lib\gcc\i386-pc-os2-emx\4.4.6\libgcc.lib(_alloca.obj)
0001:006d00a0  __alloca
Module: U:\usr\local446\lib\gcc\i386-pc-os2-emx\4.4.6\libgcc.lib(_udivdi3.obj)
0001:006d00d0  ___udivdi3
Module: U:\extras\lib\libz.lib(deflate.obj)
0001:006d11f8* _deflateSetDictionary
0001:006d1324  _deflateReset
0001:006d1490* _deflateSetHeader
0001:006d14bc* _deflatePrime
0001:006d14f4* _deflateTune
0001:006d1534* _deflateBound
0001:006d1660  _deflate
0001:006d25ac  _deflateParams
0001:006d26a0  _deflateEnd
0001:006d2770  _deflateInit2_
0001:006d29f4  _deflateInit_
0001:006d2bf0* _deflateCopy
0001:006d2dc0* _deflate_copyright
Module: U:\extras\lib\libz.lib(crc32.obj)
0001:006d30ec  _get_crc_table
0001:006d30f8  _crc32
0001:006d33e0* _crc32_combine
0001:006d3404* _crc32_combine64
Module: U:\extras\lib\libz.lib(zutil.obj)
0001:006d5438  _zlibVersion
0001:006d5444* _zlibCompileFlags
0001:006d5450  _zError
0001:006d5510  _z_errmsg
0001:006d5464  _zcalloc
0001:006d547c  _zcfree
Module: U:\extras\lib\libz.lib(inflate.obj)
0001:006d5694  _inflateReset
0001:006d5740* _inflateReset2
0001:006d5884  _inflateInit2_
0001:006d5944  _inflateInit_
0001:006d5a08* _inflatePrime
0001:006d5c40  _inflate
0001:006d7ac8  _inflateEnd
0001:006d7b24* _inflateSetDictionary
0001:006d7c10* _inflateGetHeader
0001:006d7c40* _inflateSync
0001:006d7e3c* _inflateSyncPoint
0001:006d7e70* _inflateCopy
0001:006d7fd8* _inflateUndermine
0001:006d8004* _inflateMark
Module: U:\extras\lib\libz.lib(uncompr.obj)
0001:006d8908  _uncompress
Module: U:\extras\lib\libz.lib(compress.obj)
0001:006d89b8  _compress2
0001:006d8a64  _compress
0001:006d8b10* _compressBound
Module: U:\extras\lib\libz.lib(gzlib.obj)
0001:006d8f08  _gzopen
0001:006d8f20* _gzopen64
0001:006d8f40  _gzdopen
0001:006d8fa0* _gzbuffer
0001:006d8fdc* _gzrewind
0001:006d9088* _gzseek64
0001:006d925c  _gzseek
0001:006d9268* _gztell64
0001:006d92bc* _gztell
0001:006d9310* _gzoffset64
0001:006d9380* _gzoffset
0001:006d93f0  _gzeof
0001:006d9424* _gzerror
0001:006d9464* _gzclearerr
0001:006d94a4  _gz_error
Module: U:\extras\lib\libz.lib(gzclose.obj)
0001:006d9580  _gzclose
Module: U:\extras\lib\libz.lib(gzwrite.obj)
0001:006d9a10  _gzwrite
0001:006d9c18* _gzputc
0001:006d9cb4* _gzputs
0001:006d9cfc* _gzprintf
0001:006d9e90  _gzflush
0001:006d9f00* _gzsetparams
0001:006d9fa8  _gzclose_w
Module: U:\extras\lib\libz.lib(gzread.obj)
0001:006db3a0  _gzread
0001:006db588* _gzgetc
0001:006db610* _gzungetc
0001:006db6f0* _gzgets
0001:006db7fc  _gzdirect
0001:006db83c  _gzclose_r
Module: U:\extras\lib\xml2.lib(xpath.obj)
0001:006db8d0  _xmlXPathInit
0001:006db9ce  _xmlXPathIsNaN
0001:006dbb0e* _xmlXPathOrderDocElems
0001:006dbb68  _xmlXPathCmpNodes
0001:006dc7e5* _libxml_domnode_binary_insertion_sort
0001:006dc7f9* _xmlXPathNodeSetFreeNs
0001:006dc84e* _xmlXPathNodeSetDel
0001:006dc8de* _xmlXPathNodeSetRemove
0001:006dc957* _xmlXPathFreeNodeSet
0001:006dca23* _xmlXPathFreeNodeSetList
0001:006dca3a* _xmlXPathRegisterFuncLookup
0001:006dca52* _xmlXPathRegisterVariableLookup
0001:006dca6a* _xmlXPathCastBooleanToNumber
0001:006dca7c* _xmlXPathCastNumberToBoolean
0001:006dcab5* _xmlXPathCastNodeSetToBoolean
0001:006dcacb* _xmlXPathNextSelf
0001:006dcaec* _xmlXPathNextChild
0001:006dcb91* _xmlXPathNextDescendant
0001:006dcc29* _xmlXPathNextDescendantOrSelf
0001:006dcc69* _xmlXPathNextFollowingSibling
0001:006dcca7* _xmlXPathNextPrecedingSibling
0001:006dccf2* _xmlXPathNextFollowing
0001:006dcd68* _xmlXPathNextPreceding
0001:006dcec2* _xmlXPathNextAttribute
0001:006dcfb5* _xmlXPathCastBooleanToString
0001:006dd04f  _xmlXPathFreeObject
0001:006dd64a* _xmlXPathWrapExternal
0001:006dd6af* _xmlXPathNewCString
0001:006dd704* _xmlXPathWrapString
0001:006dd7c4* _xmlXPathWrapCString
0001:006dd7d1  _xmlXPathNewString
0001:006dd8ee  _xmlXPathNewBoolean
0001:006dd9c6* _xmlXPathNewFloat
0001:006dda9b* _xmlXPathWrapNodeSet
0001:006ddb5f* _xmlXPathNodeSetAddUnique
0001:006ddc67* _xmlXPathNodeSetAdd
0001:006ddd8d* _xmlXPathNodeSetCreate
0001:006dde74* _xmlXPathNewValueTree
0001:006dded5  _xmlXPathNewNodeSet
0001:006de016* _xmlXPathNewNodeSetList
0001:006de0c8  _valuePush
0001:006de169  _xmlXPathRoot
0001:006de1b1* _xmlXPathContextSetCache
0001:006de2bb  _xmlXPathEvaluatePredicateResult
0001:006de3b5  _xmlXPathNewParserContext
0001:006de65a* _xmlXPathEvalPredicate
0001:006de735* _xmlXPathCastStringToBoolean
0001:006de774* _xmlXPathCastToBoolean
0001:006de834* _xmlXPathConvertBoolean
0001:006de87f* _xmlXPathStringEvalNumber
0001:006deab6* _xmlXPathCastStringToNumber
0001:006deaeb* _xmlXPathIsNodeType
0001:006deb6e* _xmlXPathNextAncestor
0001:006ded36* _xmlXPathNextAncestorOrSelf
0001:006ded66* _xmlXPathNextParent
0001:006dee98* _xmlXPathNodeSetMerge
0001:006df060* _xmlXPathNodeSetAddNs
0001:006df19f  _xmlXPathNodeSetContains
0001:006df23c* _xmlXPathNodeLeadingSorted
0001:006df2e7* _xmlXPathLeadingSorted
0001:006df325* _xmlXPathHasSameNodes
0001:006df3af* _xmlXPathIntersection
0001:006df467* _xmlXPathDifference
0001:006e0705* _xmlXPathCastNodeToString
0001:006e0729* _xmlXPathCastNodeToNumber
0001:006e0b01* _xmlXPathNextNamespace
0001:006e0baa  _xmlXPathErr
0001:006e151a  _xmlXPathParseNCName
0001:006e162a  _xmlXPathParseName
0001:006e16e5* _xmlXPathFalseFunction
0001:006e1747* _xmlXPathTrueFunction
0001:006e17ac* _xmlXPathPositionFunction
0001:006e1830* _xmlXPathLastFunction
0001:006e18b4* _xmlXPatherror
0001:006e18fb  _valuePop
0001:006e199d  _xmlXPathObjectCopy
0001:006e1b6c* _xmlXPathRegisteredNsCleanup
0001:006e1b9b* _xmlXPathRegisteredVariablesCleanup
0001:006e1bc9* _xmlXPathRegisteredFuncsCleanup
0001:006e1bf7  _xmlXPathFreeContext
0001:006e1c79* _xmlXPathNsLookup
0001:006e464d  _xmlXPathRegisterNs
0001:006e46e3* _xmlXPathVariableLookupNS
0001:006e4751* _xmlXPathVariableLookup
0001:006e4796* _xmlXPathFunctionLookupNS
0001:006e47f1* _xmlXPathFunctionLookup
0001:006e4846* _xmlXPathRegisterVariableNS
0001:006e48d0* _xmlXPathRegisterVariable
0001:006e48f9  _xmlXPathRegisterFuncNS
0001:006e497d  _xmlXPathRegisterFunc
0001:006e4ab2* _xmlXPathRegisterAllFunctions
0001:006e8766* _xmlXPathBooleanFunction
0001:006e8de2* _xmlXPathCeilingFunction
0001:006e889c* _xmlXPathCountFunction
0001:006e8f38* _xmlXPathFloorFunction
0001:006e880b* _xmlXPathNotFunction
0001:006e8b2e* _xmlXPathNumberFunction
0001:006e8c3a* _xmlXPathRoundFunction
0001:006e8675* _xmlXPathSumFunction
0001:006e4d7c  _xmlXPathNewContext
0001:006e4e06* _xmlXPathDistinctSorted
0001:006e5011* _xmlXPathFreeCompExpr
0001:006e510d  _xmlXPathFreeParserContext
0001:006e515e* _xmlXPathCtxtCompile
0001:006e5211* _xmlXPathCompile
0001:006e522c* _xmlXPathIsInf
0001:006e54a1  _xmlXPathDebugDumpObject
0001:006e6aff* _xmlXPathDebugDumpCompExpr
0001:006e6f9e* _compute_minrun
0001:006e702a* _libxml_domnode_tim_sort
0001:006e7933* _xmlXPathNodeSetSort
0001:006e7953* _xmlXPathCastNodeSetToString
0001:006e799e* _xmlXPathCastNodeSetToNumber
0001:006e79df* _xmlXPathCastToNumber
0001:006e7a9b* _xmlXPathConvertNumber
0001:006e7ae2* _xmlXPathNodeTrailingSorted
0001:006e7bab* _xmlXPathTrailingSorted
0001:006e7be7* _xmlXPathTrailing
0001:006e7c60* _xmlXPathNodeTrailing
0001:006e7c87* _xmlXPathLeading
0001:006e7d00* _xmlXPathNodeLeading
0001:006e7d27* _xmlXPathDistinct
0001:006e7d84* _xmlXPathCastNumberToString
0001:006e81c4* _xmlXPathConvertString
0001:006e82ae  _xmlXPathCastToString
0001:006e89b4* _xmlXPathPopExternal
0001:006e8a49* _xmlXPathPopNodeSet
0001:006e8acd* _xmlXPathPopBoolean
0001:006e9054* _xmlXPathValueFlipSign
0001:006e93d2* _xmlXPathCompareValues
0001:006e9bd2* _xmlXPathNotEqualValues
0001:006e9db0* _xmlXPathEqualValues
0001:006e9f85* _xmlXPathModValues
0001:006ea06a* _xmlXPathDivValues
0001:006ea1fe* _xmlXPathMultValues
0001:006ea292* _xmlXPathSubValues
0001:006ea326* _xmlXPathAddValues
0001:006ef563* _xmlXPathConcatFunction
0001:006ef418* _xmlXPathContainsFunction
0001:006efa80  _xmlXPathIdFunction
0001:006eeaff* _xmlXPathLangFunction
0001:006efbf5* _xmlXPathLocalNameFunction
0001:006efeaa* _xmlXPathNamespaceURIFunction
0001:006eee9d* _xmlXPathNormalizeFunction
0001:006ee7a3* _xmlXPathStringFunction
0001:006ef675* _xmlXPathStringLengthFunction
0001:006ef2be* _xmlXPathStartsWithFunction
0001:006ef7c0* _xmlXPathSubstringFunction
0001:006ef196* _xmlXPathSubstringBeforeFunction
0001:006ef03e* _xmlXPathSubstringAfterFunction
0001:006eec60* _xmlXPathTranslateFunction
0001:006eda24  _xmlXPathEvalExpr
0001:006edb09  _xmlXPathEvalExpression
0001:006edccf  _xmlXPathEval
0001:006ee159* _xmlXPathCompiledEvalToBoolean
0001:006ee174* _xmlXPathCompiledEval
0001:006ee549* _xmlXPathPopNumber
0001:006ee5aa* _xmlXPathPopString
0002:00004880  _xmlXPathPINF
0002:00004888  _xmlXPathNINF
0002:0001cba0  _xmlXPathNAN
Module: U:\extras\lib\xml2.lib(HTMLtree.obj)
0001:006f03b3  _htmlIsBooleanAttr
0001:006f0613  _htmlNodeDumpFormatOutput
0001:006f0d98* _htmlDocContentDumpOutput
0001:006f0c59  _htmlDocContentDumpFormatOutput
0001:006f0dc1  _htmlNodeDumpOutput
0001:006f0dfc* _htmlNodeDumpFileFormat
0001:006f0eb2  _htmlNodeDumpFile
0001:006f0f23  _htmlSetMetaEncoding
0001:006f12af  _htmlSaveFileFormat
0001:006f13c0* _htmlSaveFileEnc
0001:006f1422  _htmlGetMetaEncoding
0001:006f16d3  _htmlSaveFile
0001:006f1799  _htmlDocDump
0001:006f1862  _htmlDocDumpMemoryFormat
0001:006f19bc* _htmlDocDumpMemory
0001:006f1a03  _htmlNodeDump
Module: U:\extras\lib\xml2.lib(HTMLparser.obj)
0001:006f1c6d  _htmlInitAutoClose
0001:006f1d31* _htmlEntityValueLookup
0001:006f1d6e* _htmlHandleOmittedElem
0001:006f1d81* _htmlCtxtUseOptions
0001:006f1edf  _htmlFreeParserCtxt
0001:006f2290* _htmlCtxtReset
0001:006f258f* _htmlAttrAllowed
0001:006f263b* _htmlElementAllowedHere
0001:006f2685* _htmlElementStatusHere
0001:006f2ec2* _htmlEntityLookup
0001:006f2f16* _htmlIsScriptAttribute
0001:006f2f63* _htmlAutoCloseTag
0001:006f2fda* _htmlIsAutoClosed
0001:006f304b  _htmlNewDocNoDtD
0001:006f312e* _htmlNewDoc
0001:006f33b2* _htmlEncodeEntities
0001:006f3623  _UTF8ToHtml
0001:006f39d2  _htmlTagLookup
0001:006f3a20* _htmlNodeStatus
0001:006f44f3* _htmlNewParserCtxt
0001:006f479a* _htmlCreatePushParserCtxt
0001:006f49b2  _htmlCreateMemoryParserCtxt
0001:006f4bd7  _htmlCreateFileParserCtxt
0001:006f63c7* _htmlParseEntityRef
0001:006f6da8* _htmlParseCharRef
0001:006f824a* _htmlParseChunk
0001:006f9b51  _htmlParseDocument
0001:006f9f91* _htmlCtxtReadIO
0001:006fa065* _htmlCtxtReadFd
0001:006fa110* _htmlCtxtReadMemory
0001:006fa1c8* _htmlCtxtReadFile
0001:006fa23d* _htmlCtxtReadDoc
0001:006fa2b3* _htmlReadIO
0001:006fa380* _htmlReadFd
0001:006fa447* _htmlReadMemory
0001:006fa4c7* _htmlReadFile
0001:006fa510* _htmlReadDoc
0001:006fa563* _htmlSAXParseFile
0001:006fa5d3  _htmlParseFile
0001:006fa5fd* _htmlSAXParseDoc
0001:006fa682* _htmlParseDoc
0001:006fa6ac  ___htmlParseContent
0001:006fa6e5* _htmlParseElement
Module: U:\extras\lib\xml2.lib(xinclude.obj)
0001:0070227f  _xmlXIncludeSetFlags
0001:00702752  _xmlXIncludeNewContext
0001:00702e48  _xmlXIncludeFreeContext
0001:0070485a  _xmlXIncludeProcessNode
0001:00705605* _xmlXIncludeProcessTreeFlags
0001:0070567c* _xmlXIncludeProcessTree
0001:00705697* _xmlXIncludeProcessTreeFlagsData
0001:00705713* _xmlXIncludeProcessFlagsData
0001:00705754  _xmlXIncludeProcessFlags
0001:00705776* _xmlXIncludeProcess
Module: U:\extras\lib\xml2.lib(xmlsave.obj)
0001:007058e5* _xmlSaveSetEscape
0001:007058fe* _xmlSaveSetAttrEscape
0001:00705fb8  _xmlNsListDumpOutput
0001:007060ec* _xmlIsXHTML
0001:0070619c* _xmlSaveFlush
0001:007061c0* _xmlSaveClose
0001:0070625f  _xmlBufAttrSerializeTxtContent
0001:007067bd* _xmlAttrSerializeTxtContent
0001:00706900* _xmlSaveToFilename
0001:0070694c* _xmlSaveToIO
0001:0070699e* _xmlSaveToBuffer
0001:00706a14* _xmlSaveToFd
0001:00706a58* _xmlBufDumpEntityDecl
0001:00706a98* _xmlBufDumpAttributeDecl
0001:00706ad8* _xmlBufDumpElementDecl
0001:00706b18* _xmlBufDumpNotationTable
0001:00708bf0* _xmlSaveTree
0001:00708c19  _xmlSaveFormatFileEnc
0001:00708cfd  _xmlSaveFile
0001:00708d27* _xmlSaveFormatFile
0001:00708d50* _xmlSaveFileEnc
0001:00708d79  _xmlSaveFormatFileTo
0001:00708e10* _xmlSaveFileTo
0001:00708e8f* _xmlDocFormatDump
0001:00708f78  _xmlDocDump
0001:00708fba* _xmlDocDumpFormatMemoryEnc
0001:00709169  _xmlDocDumpMemoryEnc
0001:00709199  _xmlDocDumpFormatMemory
0001:007091c9  _xmlDocDumpMemory
0001:007091fa* _xmlSaveDoc
0001:007092c0  _xmlNodeDumpOutput
0001:00709391  _xmlElemDump
0001:00709425* _xmlBufNodeDump
0001:00709504  _xmlNodeDump
Module: U:\extras\lib\xml2.lib(xmlschemas.obj)
0001:007099e4  _xmlSchemaFreeWildcard
0001:00709e0b* _xmlSchemaGetParserErrors
0001:0070a01c  _xmlSchemaIsValid
0001:0070a036  _xmlSchemaSetValidErrors
0001:0070a076  _xmlSchemaSetParserErrors
0001:0070a0b6  _xmlSchemaSetValidStructuredErrors
0001:0070a0f2* _xmlSchemaSetParserStructuredErrors
0001:0070a120* _xmlSchemaGetValidErrors
0001:0070a15d* _xmlSchemaSetValidOptions
0001:0070a193* _xmlSchemaValidCtxtGetOptions
0001:0070a47c  _xmlSchemaValidateSetLocator
0001:0070a4f2* _xmlSchemaValidCtxtGetParserCtxt
0001:0070a52f  _xmlSchemaNewFacet
0001:0070b43b* _xmlSchemaValidateSetFilename
0001:0070c0b7  _xmlSchemaFreeFacet
0001:0070c104  _xmlSchemaFreeType
0001:0070c501  _xmlSchemaFree
0001:0070d394  _xmlSchemaFreeValidCtxt
0001:0070d5ad  _xmlSchemaFreeParserCtxt
0001:0070d90d  _xmlSchemaSAXUnplug
0001:0070d963* _xmlSchemaNewDocParserCtxt
0001:0070d99a  _xmlSchemaNewMemParserCtxt
0001:0070d9d8  _xmlSchemaNewParserCtxt
0001:0070e861* _xmlSchemaDump
0001:0070ffe5  _xmlSchemaNewValidCtxt
0001:0071494e  _xmlSchemaSAXPlug
0001:00718a1e  _xmlSchemaCheckFacet
0001:0072eb7b  _xmlSchemaParse
0001:0072f7e9* _xmlSchemaValidateStream
0001:0072f913* _xmlSchemaValidateFile
0001:0072f96d  _xmlSchemaValidateDoc
0001:0072f9e3* _xmlSchemaValidateOneElement
Module: U:\extras\lib\xml2.lib(parserInternals.obj)
0001:0072fa90* _xmlParserInputRead
0001:0072fa9a  _xmlInitNodeInfoSeq
0001:0072faba* _xmlClearNodeInfoSeq
0001:0072faf2* _xmlParserFindNodeInfoIndex
0001:0072fb77* _xmlParserFindNodeInfo
0001:0072fbba* _xmlKeepBlanksDefault
0001:0072fbe5* _xmlSubstituteEntitiesDefault
0001:0072fc05* _xmlLineNumbersDefault
0001:0072fc25* _xmlPedanticParserDefault
0001:0072fc45  _xmlClearParserCtxt
0001:0072fdc2  ___xmlErrEncoding
0001:0072ff51  _xmlErrMemory
0001:007300c0  _xmlParserAddNodeInfo
0001:0073029a  _xmlNewInputStream
0001:00730379  _xmlNewInputFromFile
0001:00730517  _xmlNewStringInputStream
0001:00730684  _xmlNewEntityInputStream
0001:007307de  _xmlFreeInputStream
0001:00730862  _xmlFreeParserCtxt
0001:00730afa* _xmlInitParserCtxt
0001:00730ff8  _xmlNewParserCtxt
0001:0073136c  _xmlSwitchToEncoding
0001:00731380  _xmlSwitchInputEncoding
0001:00731429  _xmlSwitchEncoding
0001:0073177e  _xmlNewIOInputStream
0001:00731806  _xmlParserInputShrink
0001:007318da  _xmlParserInputGrow
0001:00731988* _xmlIsLetter
0001:00731a98* _xmlCheckVersion
0001:00731d4e  _xmlNextChar
0001:007320fb  _xmlCurrentChar
0001:0073249f  _xmlStringCurrentChar
0001:00732718  _xmlCopyCharMultiByte
0001:007327bf  _xmlCopyChar
Module: U:\extras\lib\xml2.lib(encoding.obj)
0001:00732a7a* _isolat1ToUTF8
0001:00732b94* _UTF8Toisolat1
0001:00733718  _xmlDetectCharEncoding
0001:007338ab* _xmlCleanupEncodingAliases
0001:00733938  _xmlGetCharEncodingName
0001:00733951  _xmlCleanupCharEncodingHandlers
0001:00733aa2  _xmlByteConsumed
0001:00733c62  _xmlCharEncCloseFunc
0001:00733cf3* _xmlCharEncFirstLineInt
0001:00733e4b* _xmlCharEncFirstLine
0001:00733f7a  _xmlCharEncOutFunc
0001:0073429a  _xmlCharEncInFunc
0001:0073440b  _xmlCharEncInput
0001:00734609  _xmlCharEncFirstLineInput
0001:0073480f  _xmlCharEncOutput
0001:00734bb1* _xmlAddEncodingAlias
0001:00734d84* _xmlGetEncodingAlias
0001:00734f25  _xmlParseCharEncoding
0001:007352e5  _xmlInitCharEncodingHandlers
0001:00735af9* _xmlNewCharEncodingHandler
0001:007354a4  _xmlFindCharEncodingHandler
0001:00735762  _xmlGetCharEncodingHandler
0001:00735a31* _xmlRegisterCharEncodingHandler
0001:00735ca9* _xmlDelEncodingAlias
Module: U:\extras\lib\xml2.lib(c14n.obj)
0001:007385fb* _xmlC14NExecute
0001:007387f2  _xmlC14NDocSaveTo
0001:00738877* _xmlC14NDocSave
0001:007389a1* _xmlC14NDocDumpMemory
Module: U:\extras\lib\xml2.lib(hash.obj)
0001:00738b6e  _xmlHashScanFull
0001:00738c32  _xmlHashScan
0001:00738c60  _xmlHashSize
0001:00738c74* _xmlHashScanFull3
0001:00738d74  _xmlHashScan3
0001:00738d80  _xmlHashLookup3
0001:00738e52  _xmlHashLookup2
0001:00738e7b  _xmlHashLookup
0001:00738ea5* _xmlHashRemoveEntry3
0001:00739026  _xmlHashRemoveEntry2
0001:00739056  _xmlHashRemoveEntry
0001:00739087* _xmlHashQLookup3
0001:007392c6  _xmlHashQLookup2
0001:00739305* _xmlHashQLookup
0001:00739346* _xmlHashUpdateEntry3
0001:00739664  _xmlHashUpdateEntry2
0001:0073969b  _xmlHashUpdateEntry
0001:007396d3  _xmlHashAddEntry3
0001:00739b6b  _xmlHashAddEntry2
0001:00739b9b  _xmlHashAddEntry
0001:00739bcc  _xmlHashFree
0001:00739d16  _xmlHashCreate
0001:00739d9a  _xmlHashCopy
0001:00739e5a  _xmlHashCreateDict
Module: U:\extras\lib\libssl.lib(ssl_lib.obj)
0001:0073e135  _ssl_undefined_function
0001:00739eb5  _SSL_clear
0001:0073e72d* _ssl_clear_cipher_ctx
0001:0073f0fa* _ssl_clear_hash_ctx
0001:0073a0dc* _SSL_CTX_set_ssl_version
0001:0073a1a3  _SSL_new
0001:0073cf39  _SSL_CTX_free
0001:0073a61a* _SSL_CTX_set_session_id_context
0001:0073a68b* _SSL_set_session_id_context
0001:0073a6fc* _SSL_CTX_set_generate_session_id
0001:0073a75d* _SSL_set_generate_session_id
0001:0073a7be  _SSL_has_matching_session_id
0001:0073a8c4* _SSL_CTX_set_purpose
0001:0073a8e4* _SSL_set_purpose
0001:0073a901* _SSL_CTX_set_trust
0001:0073a921* _SSL_set_trust
0001:0073a93e* _SSL_CTX_set1_param
0001:0073a95e* _SSL_set1_param
0001:0073a97b* _SSL_free
0001:0073acb4* _SSL_set_bio
0001:0073ad5a  _SSL_get_rbio
0001:0073ad65  _SSL_get_wbio
0001:0073ad70* _SSL_get_fd
0001:0073ad83* _SSL_get_rfd
0001:0073ade1* _SSL_get_wfd
0001:0073ae3f  _SSL_set_fd
0001:0073aede* _SSL_set_wfd
0001:0073b005* _SSL_set_rfd
0001:0073b12c* _SSL_get_finished
0001:0073b187* _SSL_get_peer_finished
0001:0073b1e2* _SSL_get_verify_mode
0001:0073b1f0* _SSL_get_verify_depth
0001:0073b206* _SSL_get_verify_callback
0001:0073b214* _SSL_CTX_get_verify_mode
0001:0073b222* _SSL_CTX_get_verify_depth
0001:0073b23b* _SSL_CTX_get_verify_callback
0001:0073b249* _SSL_set_verify
0001:0073b26c* _SSL_set_verify_depth
0001:0073b289* _SSL_set_read_ahead
0001:0073b297* _SSL_get_read_ahead
0001:0073b2a2* _SSL_pending
0001:0073b2bb* _SSL_get_peer_certificate
0001:0073b32d* _SSL_get_peer_cert_chain
0001:0073b37b  _SSL_copy_session_id
0001:0073b47f* _SSL_CTX_check_private_key
0001:0073b54a* _SSL_check_private_key
0001:0073b681  _SSL_accept
0001:0073e075* _SSL_set_accept_state
0001:0073b6af  _SSL_connect
0001:0073e0d5* _SSL_set_connect_state
0001:0073b6dd  _SSL_get_default_timeout
0001:0073b6f0  _SSL_read
0001:0073b772  _SSL_peek
0001:0073b7ea  _SSL_write
0001:0073b898  _SSL_shutdown
0001:0073ebeb  _SSL_state
0001:0073b90f* _SSL_renegotiate
0001:0073b93c* _SSL_renegotiate_pending
0001:0073b94f  _SSL_ctrl
0001:0073eaab  _SSL_version
0001:0073bc30* _SSL_callback_ctrl
0001:0073bc6f* _SSL_CTX_sessions
0001:0073bc7a  _SSL_CTX_ctrl
0001:0073bfc1* _SSL_CTX_callback_ctrl
0001:0073c002* _ssl_cipher_id_cmp
0001:0073c03e  _ssl_cipher_ptr_id_cmp
0001:0073c07e  _SSL_get_ciphers
0001:0073c0cb  _ssl_get_ciphers_by_id
0001:0073c118* _SSL_get_cipher_list
0001:0073c180* _SSL_CTX_set_cipher_list
0001:0073c20c* _SSL_set_cipher_list
0001:0073c29e* _SSL_get_shared_ciphers
0001:0073c389  _ssl_cipher_list_to_bytes
0001:0073c4aa  _ssl_bytes_to_cipher_list
0001:0073c6b7* _SSL_get_servername
0001:0073c6fd* _SSL_get_servername_type
0001:0073c842  _SSL_CTX_new
0001:0073d140* _SSL_CTX_set_default_passwd_cb
0001:0073d14e* _SSL_CTX_set_default_passwd_cb_userdata
0001:0073d15c* _SSL_CTX_set_cert_verify_callback
0001:0073d173* _SSL_CTX_set_verify
0001:0073d190* _SSL_CTX_set_verify_depth
0001:0073d1b0  _ssl_set_cert_masks
0001:0073d709  _ssl_check_srvr_ecc_cert_and_alg
0001:0073d957* _ssl_get_server_send_cert
0001:0073dad2* _ssl_get_sign_pkey
0001:0073db90  _ssl_update_cache
0001:0073dd02* _SSL_get_ssl_method
0001:0073dd0d  _SSL_set_ssl_method
0001:0073ddc9* _SSL_get_error
0001:0073ed4f* _SSL_want
0001:0073dfdc* _SSL_do_handshake
0001:0073e16e  _ssl_undefined_void_function
0001:0073e1a7  _ssl_undefined_const_function
0001:0073e1e0* _ssl_bad_method
0001:0073e22d* _SSL_get_version
0001:0073e26e* _SSL_dup
0001:0073eab5* _SSL_get_SSL_CTX
0001:0073ebdd* _SSL_get_info_callback
0001:0073ebcc* _SSL_set_info_callback
0001:0073e803* _SSL_get_certificate
0001:0073e829* _SSL_get_privatekey
0001:0073e850* _SSL_get_current_cipher
0001:0073e88b* _SSL_get_current_compression
0001:0073e8af* _SSL_get_current_expansion
0001:0073e8d3  _ssl_init_wbio_buffer
0001:0073ea09  _ssl_free_wbio_buffer
0001:0073ea5a* _SSL_CTX_set_quiet_shutdown
0001:0073ea6b* _SSL_CTX_get_quiet_shutdown
0001:0073ea79* _SSL_set_quiet_shutdown
0001:0073ea87* _SSL_get_quiet_shutdown
0001:0073ea92* _SSL_set_shutdown
0001:0073eaa0* _SSL_get_shutdown
0001:0073eac3* _SSL_set_SSL_CTX
0001:0073eb92* _SSL_CTX_set_default_verify_paths
0001:0073eba8* _SSL_CTX_load_verify_locations
0001:0073ebf6* _SSL_set_verify_result
0001:0073ec07* _SSL_get_verify_result
0001:0073ec15* _SSL_get_ex_new_index
0001:0073ec4c* _SSL_set_ex_data
0001:0073ec73* _SSL_get_ex_data
0001:0073ec93* _SSL_CTX_get_ex_new_index
0001:0073ecca* _SSL_CTX_set_ex_data
0001:0073ecf1* _SSL_CTX_get_ex_data
0001:0073ed11  _ssl_ok
0001:0073ed1b* _SSL_CTX_get_cert_store
0001:0073ed26* _SSL_CTX_set_cert_store
0001:0073ed5a* _SSL_CTX_set_tmp_rsa_callback
0001:0073ed7c* _SSL_set_tmp_rsa_callback
0001:0073ed9e* _SSL_CTX_set_tmp_dh_callback
0001:0073edc0* _SSL_set_tmp_dh_callback
0001:0073ede2* _SSL_CTX_set_tmp_ecdh_callback
0001:0073ee04* _SSL_set_tmp_ecdh_callback
0001:0073ee26* _SSL_CTX_use_psk_identity_hint
0001:0073eed7* _SSL_use_psk_identity_hint
0001:0073efd2* _SSL_get_psk_identity_hint
0001:0073f000* _SSL_get_psk_identity
0001:0073f02e* _SSL_set_psk_client_callback
0001:0073f03f* _SSL_CTX_set_psk_client_callback
0001:0073f050* _SSL_set_psk_server_callback
0001:0073f061* _SSL_CTX_set_psk_server_callback
0001:0073f072* _SSL_CTX_set_msg_callback
0001:0073f094* _SSL_set_msg_callback
0001:0073f0b6  _ssl_replace_hash
0001:0073f147  _OBJ_bsearch_ssl_cipher_id
0002:000048d0* _SSL_version_str
0002:000048e0  _ssl3_undef_enc_method
Module: U:\extras\lib\libssl.lib(s23_clnt.obj)
0001:0073f1ba  _SSLv23_client_method
0001:0073f1cf* _ssl23_connect
Module: U:\extras\lib\poll.lib(poll.obj)
0001:00740470  _poll
Module: U:\usr\lib\libc_dll.lib(accept.obj)
0001:00740880  _accept
Module: U:\usr\lib\libc_dll.lib(send.obj)
0001:00740960  _send
Module: U:\usr\lib\libc_dll.lib(recv.obj)
0001:00740a10  _recv
Module: U:\usr\lib\libc_dll.lib(socket.obj)
0001:00740ac0  _socket
Module: U:\usr\lib\libc_dll.lib(bind.obj)
0001:00740b40  _bind
Module: U:\usr\lib\libc_dll.lib(getsockname.obj)
0001:00740be0  _getsockname
Module: U:\usr\lib\libc_dll.lib(listen.obj)
0001:00740c80  _listen
Module: U:\extras\lib\xml2.lib(entities.obj)
0001:00740d20* _xmlDumpEntitiesTable
0001:00740ef4  _xmlDumpEntityDecl
0001:007411e6  _xmlEncodeSpecialChars
0001:0074134f  _xmlCopyEntitiesTable
0001:00741445  _xmlFreeEntitiesTable
0001:0074163c* _xmlCreateEntitiesTable
0001:00741c70  _xmlEncodeEntitiesReentrant
0001:00741c84  _xmlEncodeAttributeEntities
0001:00741c9b* _xmlGetDtdEntity
0001:00741cc3  _xmlGetParameterEntity
0001:00741ffe  _xmlAddDocEntity
0001:0074208b* _xmlNewEntity
0001:00742162  _xmlAddDtdEntity
0001:00742203  _xmlGetPredefinedEntity
0001:007422d5  _xmlGetDocEntity
Module: U:\usr\lib\libc_dll.lib(shutdown.obj)
0001:00742350  _shutdown
Module: U:\usr\lib\libc_dll.lib(getsockopt.obj)
0001:007423f0  _getsockopt
Module: U:\usr\lib\libc_dll.lib(sendto.obj)
0001:007424d0  _sendto
Module: U:\usr\lib\libc_dll.lib(connect.obj)
0001:00742580  _connect
Module: U:\usr\lib\libc_dll.lib(socketpair.obj)
0001:00742620  _socketpair
Module: U:\usr\lib\libc_dll.lib(getpeername.obj)
0001:007426e0  _getpeername
Module: U:\usr\lib\libc_dll.lib(recvfrom.obj)
0001:00742780  _recvfrom
Module: U:\usr\lib\libc_dll.lib(setsockopt.obj)
0001:00742850  _setsockopt
Module: U:\usr\lib\libc_dll.lib(syslog.obj)
0001:0074299c  _syslog
0001:00742a04* _vsyslog
0001:00742e61  _openlog
0001:00742eb0  _closelog
0001:00742ee4* _setlogmask
Module: U:\usr\local446\lib\gcc\i386-pc-os2-emx\4.4.6\libgcc.lib(_fixunsdfdi.obj)
0001:00742f10  ___fixunsdfdi
Module: U:\extras\lib\xml2.lib(xmlreader.obj)
0001:00743105* _xmlTextReaderReadState
0001:00743118  _xmlTextReaderMoveToAttributeNo
0001:00743192  _xmlTextReaderMoveToFirstAttribute
0001:007431d8  _xmlTextReaderMoveToNextAttribute
0001:00743244  _xmlTextReaderMoveToElement
0001:0074327b  _xmlTextReaderAttributeCount
0001:007432d7  _xmlTextReaderIsEmptyElement
0001:0074332f  _xmlTextReaderDepth
0001:00743371  _xmlTextReaderHasAttributes
0001:007433b1  _xmlTextReaderHasValue
0001:007433e8  _xmlTextReaderIsDefault
0001:007433f3* _xmlTextReaderQuoteChar
0001:00743401* _xmlTextReaderNormalization
0001:0074340f  _xmlTextReaderSetParserProp
0001:007434f1  _xmlTextReaderGetParserProp
0001:00743555* _xmlTextReaderGetParserLineNumber
0001:00743576* _xmlTextReaderGetParserColumnNumber
0001:00743597* _xmlTextReaderCurrentNode
0001:007435b1* _xmlTextReaderPreserve
0001:0074360b* _xmlTextReaderCurrentDoc
0001:0074363e* _xmlTextReaderIsNamespaceDecl
0001:0074366a* _xmlTextReaderStandalone
0001:00743729  _xmlTextReaderIsValid
0001:00743777* _xmlTextReaderGetErrorHandler
0001:00743799* _xmlReaderNewWalker
0001:00743952* _xmlReaderWalker
0001:007439bb* _xmlTextReaderByteConsumed
0001:007439df* _xmlTextReaderConstXmlVersion
0001:00743a29* _xmlTextReaderConstString
0001:00743a72  _xmlTextReaderConstNamespaceUri
0001:00743ae9  _xmlTextReaderConstPrefix
0001:00743b65* _xmlTextReaderConstEncoding
0001:00743bdc  _xmlTextReaderSetup
0001:0074413d* _xmlReaderNewIO
0001:007441c4* _xmlReaderNewFd
0001:0074422d* _xmlReaderNewMemory
0001:00744296* _xmlReaderNewDoc
0001:007442ec* _xmlReaderNewFile
0001:00744342* _xmlTextReaderNamespaceUri
0001:00744393* _xmlTextReaderPrefix
0001:007443ef* _xmlTextReaderSetStructuredErrorHandler
0001:00744578* _xmlTextReaderSetErrorHandler
0001:00744936* _xmlTextReaderLocatorBaseURI
0001:0074498b  _xmlTextReaderConstBaseUri
0001:007449e8* _xmlTextReaderBaseUri
0001:00744a12* _xmlTextReaderLocatorLineNumber
0001:00744cf7* _xmlTextReaderRelaxNGValidate
0001:00744d12* _xmlTextReaderRelaxNGValidateCtxt
0001:00744d2c  _xmlTextReaderRelaxNGSetSchema
0001:0074510f  _xmlTextReaderSchemaValidate
0001:0074512a* _xmlTextReaderSchemaValidateCtxt
0001:00745144* _xmlTextReaderSetSchema
0001:0074536d* _xmlTextReaderPreservePattern
0001:00745492  _xmlTextReaderConstXmlLang
0001:007454e7* _xmlTextReaderXmlLang
0001:00745508  _xmlTextReaderConstValue
0001:00745617* _xmlTextReaderValue
0001:007456f5  _xmlTextReaderGetAttributeNo
0001:007457e0  _xmlTextReaderConstName
0001:00745981  _xmlTextReaderConstLocalName
0001:007459e6* _xmlTextReaderName
0001:00745b4e* _xmlTextReaderLocalName
0001:00745ba8  _xmlTextReaderNodeType
0001:00745d03* _xmlTextReaderReadAttributeValue
0001:00745da8  _xmlTextReaderMoveToAttributeNs
0001:00745ebe  _xmlTextReaderMoveToAttribute
0001:00746071  _xmlTextReaderLookupNamespace
0001:00746631* _xmlTextReaderGetRemainder
0001:007466e1* _xmlTextReaderClose
0001:00746764  _xmlTextReaderGetAttributeNs
0001:00746824  _xmlTextReaderGetAttribute
0001:00746978  _xmlFreeTextReader
0001:00746b99  _xmlNewTextReader
0001:00746e70* _xmlReaderForIO
0001:00746f12* _xmlReaderForFd
0001:00746f92* _xmlReaderForMemory
0001:0074700c* _xmlReaderForDoc
0001:0074704b* _xmlNewTextReaderFilename
0001:007470ec  _xmlReaderForFile
0001:00747439  _xmlTextReaderExpand
0001:0074750c  _xmlTextReaderReadString
0001:007475a0  _xmlTextReaderReadOuterXml
0001:00747650  _xmlTextReaderReadInnerXml
0001:00747cb4  _xmlTextReaderRead
0001:00748801* _xmlTextReaderNextSibling
0001:0074884b  _xmlTextReaderNext
Module: U:\extras\lib\xmlrpc.lib(xmlrpc.obj)
0001:00748920  _XMLRPC_RequestGetMethodName
0001:00748931  _XMLRPC_RequestSetRequestType
0001:00748947  _XMLRPC_RequestGetRequestType
0001:00748958  _XMLRPC_RequestGetData
0001:00748968  _XMLRPC_RequestGetError
0001:00748979  _XMLRPC_RequestGetOutputOptions
0001:0074898a  _XMLRPC_SetValueInt
0001:007489a2  _XMLRPC_SetValueBoolean
0001:007489c0  _XMLRPC_CopyValue
0001:007489d0  _XMLRPC_SetValueDouble
0001:007489ec  _XMLRPC_GetValueString
0001:00748a04  _XMLRPC_GetValueStringLen
0001:00748a15  _XMLRPC_GetValueInt
0001:00748a31  _XMLRPC_GetValueBoolean
0001:00748a49  _XMLRPC_GetValueDouble
0001:00748a61  _XMLRPC_GetValueBase64
0001:00748a79  _XMLRPC_GetValueDateTime
0001:00748a91  _XMLRPC_GetValueDateTime_ISO8601
0001:00748aa9  _XMLRPC_GetValueID
0001:00748ac3  _XMLRPC_GetValueType
0001:00748ad6  _XMLRPC_GetVectorType
0001:00748af1  _XMLRPC_GetValueTypeEasy
0001:00748b82  _type_to_str
0001:00748c23  _XMLRPC_GetDefaultIdCase
0001:00748c2d* _XMLRPC_SetDefaultIdCase
0001:00748c3a  _XMLRPC_GetDefaultIdCaseComparison
0001:00748c44* _XMLRPC_SetDefaultIdCaseComparison
0001:00748c64  _XMLRPC_GetVersionString
0001:00748c6e* _XMLRPC_Free
0001:00748c83* _XMLRPC_ServerFindMethod
0001:00748cd0  _find_method
0001:00748d20  _XMLRPC_ServerRegisterMethod
0001:00748d86  _XMLRPC_VectorRewind
0001:00748daf  _XMLRPC_VectorNext
0001:00748dd8  _XMLRPC_CreateValueEmpty
0001:00748e1d  _XMLRPC_RequestNew
0001:00748e4e  _XMLRPC_ServerCreate
0001:00748e92* _XMLRPC_GetGlobalServer
0001:00748eb1  _XMLRPC_VectorSize
0001:00748eda  _XMLRPC_SetIsVector
0001:00748f77  _XMLRPC_RequestSetMethodName
0001:00748fac  _XMLRPC_SetValueBase64
0001:0074900f  _XMLRPC_SetValueString
0001:00749077  _XMLRPC_SetValueID_Case
0001:00749153  _XMLRPC_CreateValueDouble
0001:007491a5  _XMLRPC_CreateValueBase64
0001:007491fb  _XMLRPC_CreateValueBoolean
0001:0074924d  _XMLRPC_CreateValueInt
0001:00749299  _XMLRPC_CreateValueString
0001:007492f7  _XMLRPC_CreateVector
0001:00749352  _XMLRPC_SetValueDateTime_ISO8601
0001:007495ac  _XMLRPC_CreateValueDateTime_ISO8601
0001:0074960c* _XMLRPC_SetValueDateTime
0001:0074967a* _XMLRPC_CreateValueDateTime
0001:007496fd  _XMLRPC_CleanupValue
0001:00749810  _XMLRPC_ServerDestroy
0001:007498d1  _XMLRPC_RequestSetError
0001:00749910  _XMLRPC_RequestSetData
0001:0074994d  _XMLRPC_RequestFree
0001:00749a1e  _XMLRPC_AddValueToVector
0001:00749c37* _XMLRPC_UtilityCreateFault
0001:00749ddd  _XMLRPC_ServerCallMethod
0001:00749e76  _XMLRPC_DupValueNew
0001:00749fbf  _XMLRPC_VectorRemoveValue
0001:0074a033  _XMLRPC_VectorGetValueWithID_Case
0001:0074a0ad* _XMLRPC_GetValueFaultString
0001:0074a0e1* _XMLRPC_GetResponseFaultString
0001:0074a0f8* _XMLRPC_GetValueFaultCode
0001:0074a12c* _XMLRPC_GetResponseFaultCode
0001:0074a143* _XMLRPC_ValueIsFault
0001:0074a193* _XMLRPC_ResponseIsFault
0001:0074a1aa  _XMLRPC_AddValuesToVector
0001:0074a2bf  _XMLRPC_REQUEST_FromXML
0001:0074a3d5* _XMLRPC_VALUE_FromXML
0001:0074a415  _XMLRPC_REQUEST_ToXML
0001:0074a493  _XMLRPC_VALUE_ToXML
0001:0074a4d8  _XMLRPC_RequestSetOutputOptions
Module: U:\extras\lib\xmlrpc.lib(xmlrpc_introspection.obj)
0001:0074a5a4* _XMLRPC_ServerSetValidationLevel
0001:0074a5c2* _find_named_value
0001:0074a636* _validate_scalar
0001:0074a793* _validate_value
0001:0074a994* _validate_vector
0001:0074a887* _validate_method
0001:0074a912  _XMLRPC_ServerValidateRequest
0001:0074aaa9  _XMLRPC_ServerRegisterIntrospectionCallback
0001:0074ab12* _describe_method
0001:0074ac38* _xml_element_to_method_description
0001:0074b227  _XMLRPC_IntrospectionCreateDescription
0001:0074b2d6  _xi_register_system_methods
0001:0074b732  _XMLRPC_ServerAddIntrospectionData
Module: U:\extras\lib\xml2.lib(xmlwriter.obj)
0001:0074b9f0  _xmlTextWriterSetIndent
0001:0074ba16* _xmlTextWriterSetQuoteChar
0001:0074ba42  _xmlTextWriterSetIndentString
0001:0074ba89  _xmlTextWriterFlush
0001:0074bb36  _xmlTextWriterEndAttribute
0001:0074bb9c  _xmlTextWriterStartAttribute
0001:0074bd0e* _xmlTextWriterWriteDTDNotation
0001:0074c22c* _xmlTextWriterWriteDTDExternalEntityContents
0001:0074c546  _xmlTextWriterEndDTDEntity
0001:0074c603  _xmlTextWriterEndDTDAttlist
0001:0074c68f  _xmlTextWriterEndDTDElement
0001:0074c71f  _xmlTextWriterEndCDATA
0001:0074c785  _xmlTextWriterEndPI
0001:0074c884  _xmlTextWriterEndComment
0001:0074c947  _xmlTextWriterEndDTD
0001:0074caa0  _xmlTextWriterStartDTDEntity
0001:0074cc69* _xmlTextWriterWriteDTDExternalEntity
0001:0074cd2e  _xmlTextWriterStartDTDAttlist
0001:0074ced4  _xmlTextWriterStartDTDElement
0001:0074d124  _xmlTextWriterStartDTD
0001:0074d4b4  _xmlTextWriterStartAttributeNS
0001:0074d6ed  _xmlTextWriterWriteRaw
0001:0074e705* _xmlTextWriterWriteRawLen
0001:0074d718  _xmlTextWriterWriteString
0001:0074d7d1* _xmlTextWriterWriteDTDInternalEntity
0001:0074d83e  _xmlTextWriterWriteDTDEntity
0001:0074d8d2* _xmlTextWriterWriteVFormatDTDInternalEntity
0001:0074d929* _xmlTextWriterWriteFormatDTDInternalEntity
0001:0074d958  _xmlTextWriterWriteDTDAttlist
0001:0074d9b5* _xmlTextWriterWriteVFormatDTDAttlist
0001:0074da05* _xmlTextWriterWriteFormatDTDAttlist
0001:0074da2d  _xmlTextWriterWriteDTDElement
0001:0074da8a* _xmlTextWriterWriteVFormatDTDElement
0001:0074dada* _xmlTextWriterWriteFormatDTDElement
0001:0074db02  _xmlTextWriterWriteDTD
0001:0074db79* _xmlTextWriterWriteVFormatDTD
0001:0074dbd7* _xmlTextWriterWriteFormatDTD
0001:0074dc0d  _xmlTextWriterWriteAttributeNS
0001:0074dc7f* _xmlTextWriterWriteVFormatAttributeNS
0001:0074dcdd* _xmlTextWriterWriteFormatAttributeNS
0001:0074dd13  _xmlTextWriterWriteAttribute
0001:0074debc  _xmlTextWriterStartCDATA
0001:0074e0aa  _xmlTextWriterStartPI
0001:0074e3b6* _xmlTextWriterWriteBinHex
0001:0074e4d8* _xmlTextWriterWriteBase64
0001:0074e7c8  _xmlTextWriterFullEndElement
0001:0074e92d  _xmlTextWriterEndElement
0001:0074eacc  _xmlTextWriterEndDocument
0001:0074ec42  _xmlTextWriterStartElement
0001:0074ee3e  _xmlTextWriterStartElementNS
0001:0074efa6  _xmlTextWriterStartComment
0001:0074f0f9* _xmlTextWriterWriteVFormatAttribute
0001:0074f149* _xmlTextWriterWriteFormatAttribute
0001:0074f171  _xmlTextWriterWriteCDATA
0001:0074f1d3* _xmlTextWriterWriteVFormatCDATA
0001:0074f21c* _xmlTextWriterWriteFormatCDATA
0001:0074f23d  _xmlTextWriterWritePI
0001:0074f2a6* _xmlTextWriterWriteVFormatPI
0001:0074f2f6* _xmlTextWriterWriteFormatPI
0001:0074f31e  _xmlTextWriterWriteElement
0001:0074f378* _xmlTextWriterWriteVFormatElement
0001:0074f3c8* _xmlTextWriterWriteFormatElement
0001:0074f3f0  _xmlTextWriterWriteElementNS
0001:0074f464* _xmlTextWriterWriteVFormatElementNS
0001:0074f4c2* _xmlTextWriterWriteFormatElementNS
0001:0074f4f8* _xmlTextWriterWriteVFormatString
0001:0074f545* _xmlTextWriterWriteFormatString
0001:0074f575  _xmlTextWriterWriteComment
0001:0074f5fc* _xmlTextWriterWriteVFormatComment
0001:0074f660* _xmlTextWriterWriteFormatComment
0001:0074f681* _xmlTextWriterWriteVFormatRaw
0001:0074f6ca* _xmlTextWriterWriteFormatRaw
0001:0074f7b4  _xmlTextWriterStartDocument
0001:0074fac5  _xmlFreeTextWriter
0001:0074fcd3* _xmlNewTextWriter
0001:0074fea9* _xmlNewTextWriterPushParser
0001:0074ffe8* _xmlNewTextWriterTree
0001:0075011f* _xmlNewTextWriterDoc
0001:00750275  _xmlNewTextWriterMemory
0001:00750337  _xmlNewTextWriterFilename
Module: U:\usr\lib\libos2.lib(code2.obj)
0001:00750554  DosGetMessage
0001:00750540* __msgseg32
Module: U:\usr\local446\lib\gcc\i386-pc-os2-emx\4.4.6\libgcc.lib(emx-ctordtor.obj)
0001:00750570  ___ctordtorTerm
0001:007505a2  ___ctordtorInit
Module: U:\usr\local446\lib\gcc\i386-pc-os2-emx\4.4.6\libgcc_eh.lib(emx-eh.obj)
0001:00750615  ___ehInit
0001:007505e0* ___ehTerm
Module: U:\extras\lib\xml2.lib(buf.obj)
0001:00750650  _xmlBufDetach
0001:00750698  _xmlBufGetAllocationScheme
0001:007506ac  _xmlBufSetAllocationScheme
0001:00750709  _xmlBufFree
0001:0075075b  _xmlBufEmpty
0001:0075081b  _xmlBufContent
0001:00750834  _xmlBufEnd
0001:00750879  _xmlBufAddLen
0001:0075090d  _xmlBufErase
0001:00750997  _xmlBufLength
0001:007509d8  _xmlBufUse
0001:00750a19  _xmlBufAvail
0001:00750a61  _xmlBufIsEmpty
0001:00750ab0  _xmlBufResetInput
0001:00750b0c  _xmlBufSetInputBaseCur
0001:00750bda  _xmlBufGetInputBase
0001:00750c89  _xmlBufBackToBuffer
0001:00750dab  _xmlBufFromBuffer
0001:00750f49* _xmlBufInflate
0001:00750f7a  _xmlBufGrow
0001:00750fb4  _xmlBufCreateStatic
0001:0075103d  _xmlBufShrink
0001:0075115f* _xmlBufResize
0001:0075137b* _xmlBufCCat
0001:00751462* _xmlBufWriteChar
0001:007514b8  _xmlBufAddHead
0001:00751631  _xmlBufAdd
0001:00751742  _xmlBufMergeBuffer
0001:007517cf  _xmlBufCat
0001:00751833* _xmlBufWriteCHAR
0001:00751894  _xmlBufWriteQuotedString
0001:007519ef* _xmlBufDump
0001:00751a6f  _xmlBufCreateSize
0001:00751b23  _xmlBufCreate
Module: U:\extras\lib\xml2.lib(nanohttp.obj)
0001:00751bd0* _xmlNanoHTTPCleanup
0001:00751bfe  _xmlNanoHTTPReturnCode
0001:00751c12* _xmlNanoHTTPAuthHeader
0001:00751c23* _xmlNanoHTTPContentLength
0001:00751c37  _xmlNanoHTTPRedir
0001:00751c48  _xmlNanoHTTPEncoding
0001:00751c59  _xmlNanoHTTPMimeType
0001:0075219d* _xmlNanoHTTPScanProxy
0001:00752850  _xmlNanoHTTPClose
0001:00752867* _xmlNanoHTTPSave
0001:00752930  _xmlNanoHTTPRead
0001:00752a55* _xmlNanoHTTPInit
0001:00752c59* _xmlNanoHTTPMethodRedir
0001:0075399f  _xmlNanoHTTPMethod
0001:007539dd  _xmlNanoHTTPOpen
0001:00753a21* _xmlNanoHTTPFetch
0001:00753b1c* _xmlNanoHTTPOpenRedir
Module: U:\extras\lib\xml2.lib(nanoftp.obj)
0001:00753b80* _xmlNanoFTPCleanup
0001:00753be6* _xmlNanoFTPProxy
0001:00753c9a* _xmlNanoFTPFreeCtxt
0001:00753d31* _xmlNanoFTPQuit
0001:00753dd8  _xmlNanoFTPClose
0001:00754093* _xmlNanoFTPCheckResponse
0001:0075416f* _xmlNanoFTPGetResponse
0001:0075417e* _xmlNanoFTPCloseConnection
0001:0075429d  _xmlNanoFTPRead
0001:0075432e* _xmlNanoFTPDele
0001:00754407* _xmlNanoFTPCwd
0001:00754576* _xmlNanoFTPGetConnection
0001:00754946* _xmlNanoFTPGetSocket
0001:00754aac* _xmlNanoFTPGet
0001:00754c8e* _xmlNanoFTPList
0001:0075562a* _xmlNanoFTPConnect
0001:00755df2* _xmlNanoFTPNewCtxt
0001:00755ec0* _xmlNanoFTPScanProxy
0001:00755f9f* _xmlNanoFTPUpdateURL
0001:007560c1* _xmlNanoFTPInit
0001:00756173  _xmlNanoFTPOpen
0001:007561e2* _xmlNanoFTPConnectTo
Module: U:\extras\lib\xml2.lib(catalog.obj)
0001:00756250  _xmlCatalogGetDefaults
0001:0075625a* _xmlCatalogSetDebug
0001:0075640e* _xmlCatalogSetDefaultPrefer
0001:00756501* _xmlCatalogSetDefaults
0001:007575e3* _xmlNewCatalog
0001:0075763c* _xmlFreeCatalog
0001:007576a4  _xmlCatalogCleanup
0001:0075778d* _xmlInitializeCatalog
0001:007578f4  _xmlCatalogAddLocal
0001:0075798e  _xmlCatalogFreeLocal
0001:00758252* _xmlLoadACatalog
0001:00758341* _xmlLoadCatalog
0001:007583d0* _xmlLoadCatalogs
0001:00758482* _xmlLoadSGMLSuperCatalog
0001:007584f3* _xmlCatalogIsEmpty
0001:0075865c* _xmlConvertSGMLCatalog
0001:007586c2* _xmlCatalogConvert
0001:00758b65* _xmlACatalogDump
0001:00758ca5* _xmlCatalogDump
0001:00759013* _xmlParseCatalogFile
0001:00759fad* _xmlCatalogGetPublic
0001:0075a0b2* _xmlCatalogGetSystem
0001:0075a1e8  _xmlCatalogLocalResolve
0001:0075a305* _xmlACatalogResolve
0001:0075a3f3  _xmlCatalogResolve
0001:0075a437* _xmlACatalogResolvePublic
0001:0075a4bb* _xmlCatalogResolvePublic
0001:0075a4f7* _xmlACatalogResolveSystem
0001:0075a58e* _xmlCatalogResolveSystem
0001:0075ab25  _xmlCatalogLocalResolveURI
0001:0075ab9a* _xmlACatalogResolveURI
0001:0075ac1d  _xmlCatalogResolveURI
0001:0075ac6a* _xmlACatalogRemove
0001:0075ad70* _xmlCatalogRemove
0001:0075ae2a* _xmlACatalogAdd
0001:0075b34a* _xmlCatalogAdd
Module: U:\extras\lib\xml2.lib(xzlib.obj)
0001:0075b420  ___libxml2_xzclose
0001:0075c519  ___libxml2_xzread
0001:0075c855  ___libxml2_xzdopen
0001:0075c8b2  ___libxml2_xzopen
Module: U:\extras\lib\xml2.lib(threads.obj)
0001:0075c8d0  ___xmlGlobalInitMutexDestroy
0001:0075c8d5  _xmlInitThreads
0001:0075c8ef  _xmlCleanupThreads
0001:0075c935  ___xmlGlobalInitMutexLock
0001:0075c949  _xmlMutexLock
0001:0075c968  ___xmlGlobalInitMutexUnlock
0001:0075c97c  _xmlMutexUnlock
0001:0075c99b  _xmlIsMainThread
0001:0075ca18  _xmlGetThreadId
0001:0075ca31  _xmlRMutexLock
0001:0075cac9* _xmlLockLibrary
0001:0075cb02  _xmlFreeRMutex
0001:0075cb4d  _xmlFreeMutex
0001:0075cb8d  _xmlNewRMutex
0001:0075cbe8  _xmlNewMutex
0001:0075cc23  _xmlRMutexUnlock
0001:0075cc7d* _xmlUnlockLibrary
0001:0075ccb6  _xmlGetGlobalState
Module: U:\extras\lib\xml2.lib(SAX.obj)
0001:0075cd60  _initxmlDefaultSAXHandler
0001:0075ce3e  _inithtmlDefaultSAXHandler
0001:0075cf13  _initdocbDefaultSAXHandler
Module: U:\extras\lib\xml2.lib(SAX2.obj)
0001:0075cff0  _xmlSAX2GetPublicId
0001:0075cff7  _xmlSAX2GetSystemId
0001:0075d011  _xmlSAX2GetLineNumber
0001:0075d02b  _xmlSAX2GetColumnNumber
0001:0075d045  _xmlSAX2IsStandalone
0001:0075d066  _xmlSAX2HasInternalSubset
0001:0075d088  _xmlSAX2HasExternalSubset
0001:0075d0aa  _xmlSAX2SetDocumentLocator
0001:0075d0af  _xmlSAX2IgnorableWhitespace
0001:0075d0b4* _xmlSAXDefaultVersion
0001:0075d0d6  _xmlSAXVersion
0001:0075e7dc* _xmlSAX2StartElementNs
0001:0075e02d* _xmlSAX2EndElementNs
0001:00760655  _xmlSAX2InternalSubset
0001:0076043c  _xmlSAX2ExternalSubset
0001:007603c1  _xmlSAX2ResolveEntity
0001:007608b6  _xmlSAX2GetEntity
0001:007603a0  _xmlSAX2GetParameterEntity
0001:00760f7a  _xmlSAX2EntityDecl
0001:00760a99  _xmlSAX2AttributeDecl
0001:00760c97  _xmlSAX2ElementDecl
0001:00760de8  _xmlSAX2NotationDecl
0001:00761192  _xmlSAX2UnparsedEntityDecl
0001:0076027c  _xmlSAX2StartDocument
0001:007601a4  _xmlSAX2EndDocument
0001:0075dfca  _xmlSAX2Reference
0001:0075dd49  _xmlSAX2Characters
0001:0075d442  _xmlSAX2CDataBlock
0001:0075d575  _xmlSAX2ProcessingInstruction
0001:0075d4b2  _xmlSAX2Comment
0001:0075f9d0  _xmlSAX2StartElement
0001:0075e0c2  _xmlSAX2EndElement
0001:0075d1f2  _xmlSAX2InitDefaultSAXHandler
0001:0075d23f* _xmlSAX2InitHtmlDefaultSAXHandler
0001:0075d31d* _xmlSAX2InitDocbDefaultSAXHandler
0001:0075d3fb* _docbDefaultSAXHandlerInit
0001:0075d410  _htmlDefaultSAXHandlerInit
0001:0075d425  _xmlDefaultSAXHandlerInit
Module: U:\extras\lib\xml2.lib(dict.obj)
0001:00761555  _xmlDictOwns
0001:007615a2* _xmlDictSize
0001:007615c5  _xmlDictSetLimit
0001:007615dc* _xmlDictGetUsage
0001:00761996  _xmlDictExists
0001:00761be4  _xmlDictLookup
0001:00761f55  _xmlDictQLookup
0001:00762508  _xmlDictCleanup
0001:00762532  _xmlInitializeDict
0001:0076259e  _xmlDictFree
0001:007626ba  _xmlDictReference
0001:0076270b  ___xmlRandom
0001:0076274e  _xmlDictCreate
0001:007627f2* _xmlDictCreateSub
0002:0001d7f0* _rand_seed
Module: U:\extras\lib\xml2.lib(chvalid.obj)
0001:00762830  _xmlCharInRange
0001:007628cc* _xmlIsBaseChar
0001:00762b90  _xmlIsBaseCharGroup
0001:0076292d* _xmlIsBlank
0001:0076295b* _xmlIsChar
0001:007629b5* _xmlIsCombining
0001:00762bb0  _xmlIsCombiningGroup
0001:007629dc* _xmlIsDigit
0001:00762bc0  _xmlIsDigitGroup
0001:00762a0c* _xmlIsExtender
0001:00762bd0  _xmlIsExtenderGroup
0001:00762a3b* _xmlIsIdeographic
0001:00762a77* _xmlIsPubidChar
0001:00762a90  _xmlIsPubidChar_tab
0001:00762ba0* _xmlIsCharGroup
0001:00762be0* _xmlIsIdeographicGroup
Module: U:\extras\lib\xml2.lib(list.obj)
0001:00763214  _xmlListSearch
0001:00763237* _xmlListReverseSearch
0001:00763259  _xmlListRemoveFirst
0001:00763291* _xmlListRemoveLast
0001:007632c9* _xmlListRemoveAll
0001:007632fd* _xmlListClear
0001:00763324  _xmlListDelete
0001:0076335a  _xmlListEmpty
0001:00763375  _xmlListFront
0001:00763387* _xmlListEnd
0001:0076339a  _xmlListSize
0001:007633be  _xmlListPopFront
0001:007633db* _xmlListPopBack
0001:007633f9  _xmlLinkGetData
0001:0076340a* _xmlListReverse
0001:0076343e  _xmlListWalk
0001:00763483* _xmlListReverseWalk
0001:007634ee* _xmlListPushBack
0001:00763552  _xmlListPushFront
0001:007635b3  _xmlListAppend
0001:0076363c  _xmlListInsert
0001:007636c6* _xmlListCopy
0001:0076371f* _xmlListMerge
0001:00763792  _xmlListCreate
0001:00763859* _xmlListDup
0001:0076389e* _xmlListSort
Module: U:\extras\lib\xml2.lib(xmlregexp.obj)
0001:00763ab3  _xmlRegFreeExecCtxt
0001:00763bef  _xmlRegFreeRegexp
0001:00763d01  _xmlFreeAutomata
0001:00763d16  _xmlAutomataSetFlags
0001:00763d28  _xmlAutomataGetInitState
0001:00763d39  _xmlAutomataSetFinalState
0001:00763d5b* _xmlExpFree
0001:00763e1a* _xmlExpRef
0001:00763f1d* _xmlExpGetLanguage
0001:0076408d* _xmlExpGetStart
0001:007640cf* _xmlExpIsNillable
0001:007640e7* _xmlExpMaxToken
0001:007640fb* _xmlExpCtxtNbNodes
0001:0076410f* _xmlExpCtxtNbCons
0001:007643d6* _xmlExpDump
0001:00765cbb* _xmlExpParse
0001:00765f13* _xmlExpNewRange
0001:00765f76* _xmlExpNewSeq
0001:00765fdf* _xmlExpNewOr
0001:00766048* _xmlExpNewAtom
0001:007660a9* _xmlExpStringDerive
0001:00766100* _xmlExpFreeCtxt
0001:0076613d* _xmlExpNewCtxt
0001:00766c5e  _xmlAutomataNewCounterTrans
0001:00766ced  _xmlAutomataNewCountedTrans
0001:00766d2d  _xmlAutomataNewAllTrans
0001:00766e13  _xmlAutomataNewEpsilon
0001:00766e43  _xmlAutomataNewState
0001:00766f33  _xmlAutomataNewCounter
0001:00767289  _xmlRegNewExecCtxt
0001:007673cb* _xmlAutomataNewOnceTrans
0001:007674b6* _xmlAutomataNewCountTrans
0001:00767b85  _xmlAutomataNewTransition
0001:00767c6c  _xmlNewAutomata
0001:00767f20  _xmlAutomataNewOnceTrans2
0001:007680cd  _xmlAutomataNewCountTrans2
0001:007682dd  _xmlAutomataNewNegTrans
0001:0076848c  _xmlAutomataNewTransition2
0001:00768f39  _xmlRegExecPushString
0001:00768f55  _xmlRegExecPushString2
0001:0076a776* _xmlRegexpPrint
0001:0076b3b9  _xmlRegExecErrInfo
0001:0076b41c  _xmlRegExecNextValues
0001:0076bdee* _xmlExpSubsume
0001:0076be98* _xmlExpExpDerive
0001:0076d4a4  _xmlAutomataIsDeterminist
0001:0076d4be  _xmlRegexpIsDeterminist
0001:0076dc8b  _xmlAutomataCompile
0001:0076dcdf  _xmlRegexpCompile
0001:0076dd96  _xmlRegexpExec
0002:00004c00* _forbiddenExp
0002:00004c04* _emptyExp
Module: U:\extras\lib\xml2.lib(xmlschemastypes.obj)
0001:0076e440  _xmlSchemaIsBuiltInTypeFacet
0001:0076e5d3  _xmlSchemaValueAppend
0001:0076e5f2  _xmlSchemaValueGetNext
0001:0076e603  _xmlSchemaValueGetAsString
0001:0076e6e1  _xmlSchemaValueGetAsBoolean
0001:0076e6f9  _xmlSchemaFreeValue
0001:0076e81a* _xmlSchemaGetBuiltInListSimpleTypeItemType
0001:0076f4f8  _xmlSchemaGetFacetValueAsULong
0001:0076f50c  _xmlSchemaGetValType
0001:0076f51c  _xmlSchemaWhiteSpaceReplace
0001:0076f5cd  _xmlSchemaNewQNameValue
0001:0076f5ef  _xmlSchemaNewNOTATIONValue
0001:0076f61a* _xmlSchemaNewStringValue
0001:0076fd5c  _xmlSchemaCopyValue
0001:00770115  _xmlSchemaValidateLengthFacetWhtsp
0001:00770141* _xmlSchemaValidateLengthFacet
0001:00771321  _xmlSchemaCompareValuesWhtsp
0001:00771368  _xmlSchemaCompareValues
0001:0077183c  _xmlSchemaValidateFacetWhtsp
0001:00771868  _xmlSchemaValidateFacet
0001:007718bf  _xmlSchemaValidateListSimpleTypeFacet
0001:007719fa  _xmlSchemaCollapseString
0001:00771ca6  _xmlSchemaGetCanonValue
0001:00772ac6* _xmlSchemaGetCanonValueWhtsp
0001:00772c56  _xmlSchemaCleanupTypes
0001:00773167  _xmlSchemaInitTypes
0001:0077373c  _xmlSchemaGetPredefinedType
0001:0077377b  _xmlSchemaGetBuiltInType
0001:0077628e  _xmlSchemaValPredefTypeNode
0001:007762c3  _xmlSchemaValidatePredefinedType
0001:0077643d  _xmlSchemaValPredefTypeNodeNoNorm
Module: U:\extras\lib\xml2.lib(xmlmemory.obj)
0001:00776620* _xmlMemUsed
0001:0077662a* _xmlMemBlocks
0001:00776634* _xmlMemoryDump
0001:00776639* _xmlMemSetup
0001:00776683* _xmlMemGet
0001:007766ca* _xmlGcMemSetup
0001:0077671c* _xmlGcMemGet
0001:00776774  _xmlCleanupMemory
0001:007767d0  _xmlInitMemory
0001:0077687f  _xmlMemShow
0001:007768f3* _xmlMemDisplay
0001:0077696e* _xmlMemDisplayLast
0001:00776a6d* _xmlMallocBreakpoint
0001:00776ab3* _xmlMemStrdupLoc
0001:00776bdc* _xmlMemoryStrdup
0001:00776c37* _xmlMallocAtomicLoc
0001:00776d60* _xmlMallocLoc
0001:00776e86* _xmlMemMalloc
0001:00776ef9* _xmlMemFree
0001:00777043* _xmlReallocLoc
0001:007771db* _xmlMemRealloc
Module: U:\extras\lib\libz.lib(adler32.obj)
0001:00777210  _adler32
0001:00777480* _adler32_combine
0001:00777528* _adler32_combine64
Module: U:\extras\lib\libz.lib(trees.obj)
0001:00779990  __length_code
0001:00779790  __dist_code
0001:00778878  __tr_init
0001:00778950  __tr_stored_block
0001:007789fc  __tr_align
0001:00778d2c  __tr_flush_block
0001:007796f8* __tr_tally
Module: U:\extras\lib\libz.lib(inftrees.obj)
0001:0077a200  _inflate_table
0001:0077aa50* _inflate_copyright
Module: U:\extras\lib\libz.lib(inffast.obj)
0001:0077abd0  _inflate_fast
Module: U:\extras\lib\xml2.lib(xpointer.obj)
0001:0077b414* _xmlXPtrLocationSetDel
0001:0077b48e* _xmlXPtrLocationSetRemove
0001:0077b4ea  _xmlXPtrFreeLocationSet
0001:0077b573  _xmlXPtrAdvanceNode
0001:0077b65b* _xmlXPtrBuildNodeList
0001:0077c207  _xmlXPtrEval
0001:0077c8d0  _xmlXPtrNewContext
0001:0077d557* _xmlXPtrRangeToFunction
0001:0077ca50  _xmlXPtrWrapLocationSet
0001:0077cab2  _xmlXPtrLocationSetAdd
0001:0077cbd7  _xmlXPtrLocationSetMerge
0001:0077cc22  _xmlXPtrLocationSetCreate
0001:0077ccbd* _xmlXPtrEvalRangePredicate
0001:0077cf58* _xmlXPtrNewCollapsedRange
0001:0077cfc0* _xmlXPtrNewLocationSetNodeSet
0001:0077d445  _xmlXPtrNewRangeNodeObject
0001:0077d70d* _xmlXPtrNewRangeNodes
0001:0077d783* _xmlXPtrNewLocationSetNodes
0001:0077d8f8* _xmlXPtrNewRangeNodePoint
0001:0077d97e* _xmlXPtrNewRangePointNode
0001:0077d9fe* _xmlXPtrNewRangePoints
0001:0077da82  _xmlXPtrNewRange
Module: U:\extras\lib\xml2.lib(pattern.obj)
0001:0077ea2f  _xmlFreeStreamCtxt
0001:0077eb39  _xmlStreamPop
0001:0077eb9c  _xmlStreamWantsAnyNode
0001:0077ebc7  _xmlPatternStreamable
0001:0077ebf1  _xmlPatternMaxDepth
0001:0077ec56  _xmlPatternMinDepth
0001:0077eca1  _xmlPatternFromRoot
0001:0077ecd1  _xmlPatternGetStreamCtxt
0001:0077eed7  _xmlPatternMatch
0001:0077f951  _xmlStreamPushAttr
0001:0077f96d  _xmlStreamPushNode
0001:0077f988  _xmlStreamPush
0001:00780759  _xmlFreePattern
0001:0078083a  _xmlPatterncompile
0001:00781577  _xmlFreePatternList
Module: U:\extras\lib\xml2.lib(debugXML.obj)
0001:007815bb* _xmlBoolToText
0001:00781667* _xmlShellPrintXPathError
0001:00781801* _xmlShellDu
0001:00781998* _xmlShellPwd
0001:007819f8* _xmlShellValidate
0001:00781ae3* _xmlShellSave
0001:00781baa* _xmlShellWrite
0001:00781c6e* _xmlShellLoad
0001:00781d29* _xmlShellCat
0001:00781df1* _xmlShellBase
0001:00781ed8* _xmlLsCountNode
0001:00782b4c* _xmlDebugDumpDocumentHead
0001:00782bc5  _xmlDebugDumpString
0001:00782cc0* _xmlLsOneNode
0001:00783037* _xmlShellList
0001:00783d88* _xmlDebugDumpEntities
0001:00785302  _xmlDebugDumpOneNode
0001:00785372* _xmlDebugDumpAttrList
0001:00785466* _xmlShellPrintXPathResult
0001:0078546b* _xmlShellPrintNode
0001:00785477  _xmlDebugDumpAttr
0001:007854e7* _xmlShellDir
0001:00785d99* _xmlShell
0001:00787c80* _xmlDebugCheckDocument
0001:00787cfc* _xmlDebugDumpDocument
0001:00787d94* _xmlDebugDumpDTD
0001:00787e93* _xmlDebugDumpNodeList
0001:00787f24* _xmlDebugDumpNode
Module: U:\extras\lib\libcrypto.lib(err.obj)
0001:00788491* _ERR_get_implementation
0001:007884a3* _ERR_set_implementation
0001:00788ef6* _ERR_load_ERR_strings
0001:00788f9d* _ERR_load_strings
0001:00788fbc* _ERR_unload_strings
0001:00789001* _ERR_free_strings
0001:00789018  _ERR_put_error
0001:00789a83* _ERR_get_state
0001:00789175  _ERR_clear_error
0001:0078925a* _ERR_get_error
0001:00789296* _ERR_get_error_line
0001:007892d0  _ERR_get_error_line_data
0001:00789308  _ERR_peek_error
0001:00789344* _ERR_peek_error_line
0001:0078937e* _ERR_peek_error_line_data
0001:007893b6  _ERR_peek_last_error
0001:007893f2* _ERR_peek_last_error_line
0001:0078942c* _ERR_peek_last_error_line_data
0001:007896ae  _ERR_error_string_n
0001:007898e4* _ERR_lib_error_string
0001:0078992e* _ERR_func_error_string
0001:00789995* _ERR_reason_error_string
0001:0078985a* _ERR_error_string
0001:0078988c* _ERR_get_string_table
0001:007898a9* _ERR_get_err_state_table
0001:007898c7* _ERR_release_err_state_table
0001:00789a21* _ERR_remove_thread_state
0001:00789a6f* _ERR_remove_state
0001:00789bc0* _ERR_get_next_error_library
0001:00789bd7* _ERR_set_error_data
0001:00789c7c  _ERR_add_error_data
0001:00789d89  _ERR_set_mark
0001:00789de0  _ERR_pop_to_mark
Module: U:\extras\lib\libssl.lib(ssl_sess.obj)
0001:00789f70  _SSL_get_session
0001:00789f89* _SSL_get1_session
0001:0078a003* _SSL_SESSION_get_ex_new_index
0001:0078a03a* _SSL_SESSION_set_ex_data
0001:0078a061* _SSL_SESSION_get_ex_data
0001:0078a081  _SSL_SESSION_new
0001:0078a1df* _SSL_SESSION_get_id
0001:0078a263  _ssl_get_new_session
0001:0078b090  _SSL_SESSION_free
0001:0078a8fa* _ssl_get_prev_session
0001:0078ad95  _SSL_CTX_add_session
0001:0078af56  _SSL_CTX_remove_session
0001:0078b28c  _SSL_set_session
0001:0078b464* _SSL_SESSION_set_timeout
0001:0078b487* _SSL_SESSION_get_timeout
0001:0078b4a2* _SSL_SESSION_get_time
0001:0078b4bd* _SSL_SESSION_set_time
0001:0078b4de* _SSL_CTX_set_timeout
0001:0078b508* _SSL_CTX_get_timeout
0001:0078b520* _SSL_set_session_secret_cb
0001:0078b54f* _SSL_set_session_ticket_ext_cb
0001:0078b57e* _SSL_set_session_ticket_ext
0001:0078b762  _SSL_CTX_flush_sessions
0001:0078b80b  _ssl_clear_bad_session
0001:0078ba48* _SSL_CTX_sess_set_new_cb
0001:0078ba56* _SSL_CTX_sess_get_new_cb
0001:0078ba61* _SSL_CTX_sess_set_remove_cb
0001:0078ba6f* _SSL_CTX_sess_get_remove_cb
0001:0078ba7a* _SSL_CTX_sess_set_get_cb
0001:0078ba88* _SSL_CTX_sess_get_get_cb
0001:0078ba93* _SSL_CTX_set_info_callback
0001:0078baa4* _SSL_CTX_get_info_callback
0001:0078bab2* _SSL_CTX_set_client_cert_cb
0001:0078bac0* _SSL_CTX_get_client_cert_cb
0001:0078bacb* _SSL_CTX_set_client_cert_engine
0001:0078bb73* _SSL_CTX_set_cookie_generate_cb
0001:0078bb81* _SSL_CTX_set_cookie_verify_cb
0001:0078bba6* _PEM_read_bio_SSL_SESSION
0001:0078bbdf* _PEM_read_SSL_SESSION
0001:0078bc18* _PEM_write_bio_SSL_SESSION
0001:0078bc6b* _PEM_write_SSL_SESSION
Module: U:\extras\lib\libcrypto.lib(buffer.obj)
0001:0078bcc9  _BUF_MEM_new
0001:0078bd49  _BUF_MEM_free
0001:0078bd9d  _BUF_MEM_grow
0001:0078bef9  _BUF_MEM_grow_clean
0001:0078c088  _BUF_strdup
0001:0078c0b7  _BUF_strndup
0001:0078c1c6  _BUF_strlcpy
0001:0078c141  _BUF_memdup
0001:0078c216  _BUF_strlcat
0001:0078c25b* _BUF_reverse
Module: U:\extras\lib\libssl.lib(ssl_ciph.obj)
0001:0078d2a1* _ssl_load_ciphers
0001:0078d649  _ssl_cipher_get_evp
0001:0078d8f8  _ssl_get_handshake_digest
0001:0078ead6  _ssl_create_cipher_list
0001:0078f3db* _SSL_CIPHER_description
0001:0078f86e* _SSL_CIPHER_get_version
0001:0078f8ae* _SSL_CIPHER_get_name
0001:0078f8c6* _SSL_CIPHER_get_bits
0001:0078f8f8  _ssl3_comp_find
0001:0078f95e  _SSL_COMP_get_compression_methods
0001:0078f970* _SSL_COMP_add_compression_method
0001:0078fb01* _SSL_COMP_get_name
Module: U:\extras\lib\libcrypto.lib(stack.obj)
0001:0078fb50* _STACK_version
0001:0078fb79  _sk_set_cmp_func
0001:0078fbb3  _sk_dup
0001:0078fca0  _sk_new
0001:007901d6  _sk_free
0001:0078fc8c  _sk_new_null
0001:0078fd66  _sk_insert
0001:0078fe7f  _sk_delete_ptr
0001:0078fecb  _sk_delete
0001:0079028a  _sk_sort
0001:00790031  _sk_find
0001:00790053* _sk_find_ex
0001:00790075  _sk_push
0001:00790098* _sk_unshift
0001:007900ba* _sk_shift
0001:007900f2  _sk_pop
0001:0079012c  _sk_zero
0001:00790178  _sk_pop_free
0001:0079020a  _sk_num
0001:00790221  _sk_value
0001:00790253  _sk_set
0001:007902dd  _sk_is_sorted
Module: U:\extras\lib\libcrypto.lib(mem.obj)
0001:00790349* _CRYPTO_set_mem_functions
0001:007903c2* _CRYPTO_set_mem_ex_functions
0001:0079043b* _CRYPTO_set_locked_mem_functions
0001:00790482* _CRYPTO_set_locked_mem_ex_functions
0001:007904c9* _CRYPTO_set_mem_debug_functions
0001:0079050b* _CRYPTO_get_mem_functions
0001:00790567* _CRYPTO_get_mem_ex_functions
0001:007905c3* _CRYPTO_get_locked_mem_functions
0001:007905fc* _CRYPTO_get_locked_mem_ex_functions
0001:00790635* _CRYPTO_get_mem_debug_functions
0001:0079068f  _CRYPTO_malloc_locked
0001:00790767  _CRYPTO_free_locked
0001:007907bb  _CRYPTO_malloc
0001:00790893* _CRYPTO_strdup
0001:007908d5  _CRYPTO_realloc
0001:007909b8  _CRYPTO_realloc_clean
0001:00790ad3  _CRYPTO_free
0001:00790b2d* _CRYPTO_remalloc
0001:00790b67* _CRYPTO_set_mem_debug_options
0001:00790b86* _CRYPTO_get_mem_debug_options
Module: U:\extras\lib\libssl.lib(ssl_cert.obj)
0001:00790bd3  _SSL_get_ex_data_X509_STORE_CTX_idx
0001:00790cf1  _ssl_cert_new
0001:00790d84  _ssl_cert_dup
0001:00791225  _ssl_cert_free
0001:00791327  _ssl_cert_inst
0001:007913bc  _ssl_sess_cert_new
0001:00791450  _ssl_sess_cert_free
0001:00791547  _ssl_set_peer_cert_type
0001:00791570  _ssl_verify_cert_chain
0001:00791745* _SSL_dup_CA_list
0001:007917c8* _SSL_set_client_CA_list
0001:007917e8* _SSL_CTX_set_client_CA_list
0001:00791808* _SSL_CTX_get_client_CA_list
0001:00791816  _SSL_get_client_CA_list
0001:00791907* _SSL_add_client_CA
0001:00791927* _SSL_CTX_add_client_CA
0001:00791965* _SSL_load_client_CA_file
0001:00791b59* _SSL_add_file_cert_subjects_to_stack
0001:00791cf5* _SSL_add_dir_cert_subjects_to_stack
Module: U:\extras\lib\libcrypto.lib(cryptlib.obj)
0001:007920df* _CRYPTO_get_new_lockid
0001:007921ae* _CRYPTO_num_locks
0001:007921b8* _CRYPTO_get_new_dynlockid
0001:0079287d  _CRYPTO_lock
0001:0079246d* _CRYPTO_destroy_dynlockid
0001:007925ab* _CRYPTO_get_dynlock_value
0001:00792663* _CRYPTO_get_dynlock_create_callback
0001:0079266d* _CRYPTO_get_dynlock_lock_callback
0001:00792677* _CRYPTO_get_dynlock_destroy_callback
0001:00792681* _CRYPTO_set_dynlock_create_callback
0001:0079268e* _CRYPTO_set_dynlock_lock_callback
0001:0079269b* _CRYPTO_set_dynlock_destroy_callback
0001:007926a8* _CRYPTO_get_locking_callback
0001:007926b2* _CRYPTO_get_add_lock_callback
0001:007926bc* _CRYPTO_set_locking_callback
0001:007926c9* _CRYPTO_set_add_lock_callback
0001:007926d6* _CRYPTO_THREADID_set_numeric
0001:0079270a* _CRYPTO_THREADID_set_pointer
0001:00792756* _CRYPTO_THREADID_set_callback
0001:00792778* _CRYPTO_THREADID_get_callback
0001:00792782  _CRYPTO_THREADID_current
0001:007927d8  _CRYPTO_THREADID_cmp
0001:007927fa  _CRYPTO_THREADID_cpy
0001:0079281c  _CRYPTO_THREADID_hash
0001:00792827* _CRYPTO_get_id_callback
0001:00792831* _CRYPTO_set_id_callback
0001:0079283e* _CRYPTO_thread_id
0001:00792aaa  _OpenSSLDie
0001:00792924  _CRYPTO_add_lock
0001:007929d1* _CRYPTO_get_lock_name
0001:00792a32* _OPENSSL_ia32cap_loc
0001:00792a3c* _OPENSSL_cpuid_setup
0001:00792a41* _OPENSSL_showfatal
0001:00792a6a* _OPENSSL_isservice
0001:00792ad6* _OPENSSL_stderr
0002:0001f300* _OPENSSL_ia32cap_P
0002:0001f304* _OPENSSL_NONPIC_relocated
Module: U:\extras\lib\libcrypto.lib(x509_vpm.obj)
0001:00792b62  _X509_VERIFY_PARAM_new
0001:00792bb2  _X509_VERIFY_PARAM_free
0001:00792bd0  _X509_VERIFY_PARAM_inherit
0001:00792f1a* _X509_VERIFY_PARAM_set1_policies
0001:00792d78  _X509_VERIFY_PARAM_set1
0001:00792dbb* _X509_VERIFY_PARAM_set1_name
0001:00792dfe  _X509_VERIFY_PARAM_set_flags
0001:00792e36* _X509_VERIFY_PARAM_clear_flags
0001:00792e53* _X509_VERIFY_PARAM_get_flags
0001:00792e5e  _X509_VERIFY_PARAM_set_purpose
0001:00792e7b  _X509_VERIFY_PARAM_set_trust
0001:00792e98  _X509_VERIFY_PARAM_set_depth
0001:00792ea6  _X509_VERIFY_PARAM_set_time
0001:00792ec5* _X509_VERIFY_PARAM_add0_policy
0001:0079301b  _X509_VERIFY_PARAM_get_depth
0001:00793197* _X509_VERIFY_PARAM_add0_table
0001:00793241  _X509_VERIFY_PARAM_lookup
0001:007932a6* _X509_VERIFY_PARAM_table_cleanup
Module: U:\extras\lib\libcrypto.lib(ex_data.obj)
0001:0079334d* _CRYPTO_get_ex_data_implementation
0001:00793368* _CRYPTO_set_ex_data_implementation
0001:007940f1  _CRYPTO_get_ex_data
0001:0079400c  _CRYPTO_set_ex_data
0001:00793edb* _CRYPTO_ex_data_new_class
0001:00793efa* _CRYPTO_cleanup_all_ex_data
0001:00793f1a  _CRYPTO_get_ex_new_index
0001:00793f70  _CRYPTO_new_ex_data
0001:00793fa4  _CRYPTO_dup_ex_data
0001:00793fd8  _CRYPTO_free_ex_data
Module: U:\extras\lib\libcrypto.lib(lhash.obj)
0001:00794140* _lh_version
0001:00794171  _lh_new
0001:00794aab  _lh_strhash
0001:0079430e  _lh_free
0001:00794382  _lh_insert
0001:007944a0  _lh_delete
0001:0079457a  _lh_retrieve
0001:0079465b  _lh_doall
0001:0079468d  _lh_doall_arg
0001:00794b22  _lh_num_items
Module: U:\extras\lib\libcrypto.lib(bio_lib.obj)
0001:00794b4a  _BIO_new
0001:00794bdc  _BIO_set
0001:00794cd0  _BIO_free
0001:00794dd0  _BIO_vfree
0001:00794de3  _BIO_clear_flags
0001:00794dfb  _BIO_test_flags
0001:00794e09  _BIO_set_flags
0001:00794e1f* _BIO_get_callback
0001:00794e2a* _BIO_set_callback
0001:00794e38* _BIO_set_callback_arg
0001:00794e46* _BIO_get_callback_arg
0001:00794e51* _BIO_method_name
0001:00794e5e  _BIO_method_type
0001:00794e6a  _BIO_read
0001:00794fc5  _BIO_write
0001:0079512a  _BIO_puts
0001:00795280  _BIO_gets
0001:007953c6  _BIO_indent
0001:0079541e  _BIO_int_ctrl
0001:00795489  _BIO_ctrl
0001:0079544c* _BIO_ptr_ctrl
0001:0079559c  _BIO_callback_ctrl
0001:007956aa* _BIO_ctrl_pending
0001:007956d5* _BIO_ctrl_wpending
0001:00795700  _BIO_push
0001:0079576b  _BIO_pop
0001:007957f4* _BIO_get_retry_BIO
0001:0079584e  _BIO_get_retry_reason
0001:00795859  _BIO_find_type
0001:007958c4  _BIO_next
0001:007958dc  _BIO_free_all
0001:00795918* _BIO_dup_chain
0001:00795a50  _BIO_copy_next_retry
0001:00795a8c* _BIO_get_ex_new_index
0001:00795ac3* _BIO_set_ex_data
0001:00795ae7* _BIO_get_ex_data
0001:00795b04* _BIO_number_read
0001:00795b1c* _BIO_number_written
Module: U:\extras\lib\libcrypto.lib(x_exten.obj)
0001:00795bb0  _X509_EXTENSION_it
0001:00795c10  _X509_EXTENSIONS_it
0001:00795c2c* _d2i_X509_EXTENSION
0001:00795c55* _i2d_X509_EXTENSION
0001:00795c77  _X509_EXTENSION_new
0001:00795c8b  _X509_EXTENSION_free
0001:00795ca6  _d2i_X509_EXTENSIONS
0001:00795ccf  _i2d_X509_EXTENSIONS
0001:00795cf1  _X509_EXTENSION_dup
Module: U:\extras\lib\libcrypto.lib(ocsp_asn.obj)
0001:00795d90* _OCSP_SIGNATURE_it
0001:00795dac* _d2i_OCSP_SIGNATURE
0001:00795dd5* _i2d_OCSP_SIGNATURE
0001:00795df7* _OCSP_SIGNATURE_new
0001:00795e0b* _OCSP_SIGNATURE_free
0001:00795ec0* _OCSP_CERTID_it
0001:00795edc* _d2i_OCSP_CERTID
0001:00795f05* _i2d_OCSP_CERTID
0001:00795f27* _OCSP_CERTID_new
0001:00795f3b* _OCSP_CERTID_free
0001:00795fc0* _OCSP_ONEREQ_it
0001:00795fdc* _d2i_OCSP_ONEREQ
0001:00796005* _i2d_OCSP_ONEREQ
0001:00796027* _OCSP_ONEREQ_new
0001:0079603b* _OCSP_ONEREQ_free
0001:007960f0* _OCSP_REQINFO_it
0001:0079610c* _d2i_OCSP_REQINFO
0001:00796135* _i2d_OCSP_REQINFO
0001:00796157* _OCSP_REQINFO_new
0001:0079616b* _OCSP_REQINFO_free
0001:007961f0* _OCSP_REQUEST_it
0001:0079620c* _d2i_OCSP_REQUEST
0001:00796235* _i2d_OCSP_REQUEST
0001:00796257* _OCSP_REQUEST_new
0001:0079626b* _OCSP_REQUEST_free
0001:007962e0* _OCSP_RESPBYTES_it
0001:007962fc* _d2i_OCSP_RESPBYTES
0001:00796325* _i2d_OCSP_RESPBYTES
0001:00796347* _OCSP_RESPBYTES_new
0001:0079635b* _OCSP_RESPBYTES_free
0001:007963e0* _OCSP_RESPONSE_it
0001:007963fc* _d2i_OCSP_RESPONSE
0001:00796425* _i2d_OCSP_RESPONSE
0001:00796447* _OCSP_RESPONSE_new
0001:0079645b* _OCSP_RESPONSE_free
0001:007964d0* _OCSP_RESPID_it
0001:007964ec  _d2i_OCSP_RESPID
0001:00796515  _i2d_OCSP_RESPID
0001:00796537* _OCSP_RESPID_new
0001:0079654b  _OCSP_RESPID_free
0001:007965d0* _OCSP_REVOKEDINFO_it
0001:007965ec* _d2i_OCSP_REVOKEDINFO
0001:00796615* _i2d_OCSP_REVOKEDINFO
0001:00796637* _OCSP_REVOKEDINFO_new
0001:0079664b* _OCSP_REVOKEDINFO_free
0001:007966e0* _OCSP_CERTSTATUS_it
0001:007966fc* _d2i_OCSP_CERTSTATUS
0001:00796725* _i2d_OCSP_CERTSTATUS
0001:00796747* _OCSP_CERTSTATUS_new
0001:0079675b* _OCSP_CERTSTATUS_free
0001:00796830* _OCSP_SINGLERESP_it
0001:0079684c* _d2i_OCSP_SINGLERESP
0001:00796875* _i2d_OCSP_SINGLERESP
0001:00796897* _OCSP_SINGLERESP_new
0001:007968ab* _OCSP_SINGLERESP_free
0001:00796980* _OCSP_RESPDATA_it
0001:0079699c* _d2i_OCSP_RESPDATA
0001:007969c5* _i2d_OCSP_RESPDATA
0001:007969e7* _OCSP_RESPDATA_new
0001:007969fb* _OCSP_RESPDATA_free
0001:00796a90* _OCSP_BASICRESP_it
0001:00796aac* _d2i_OCSP_BASICRESP
0001:00796ad5* _i2d_OCSP_BASICRESP
0001:00796af7* _OCSP_BASICRESP_new
0001:00796b0b* _OCSP_BASICRESP_free
0001:00796b90  _OCSP_CRLID_it
0001:00796bac* _d2i_OCSP_CRLID
0001:00796bd5* _i2d_OCSP_CRLID
0001:00796bf7* _OCSP_CRLID_new
0001:00796c0b* _OCSP_CRLID_free
0001:00796c80  _OCSP_SERVICELOC_it
0001:00796c9c* _d2i_OCSP_SERVICELOC
0001:00796cc5* _i2d_OCSP_SERVICELOC
0001:00796ce7* _OCSP_SERVICELOC_new
0001:00796cfb* _OCSP_SERVICELOC_free
Module: U:\extras\lib\libcrypto.lib(x_name.obj)
0001:00796e00  _X509_NAME_ENTRY_it
0001:00796e1c* _d2i_X509_NAME_ENTRY
0001:00796e45* _i2d_X509_NAME_ENTRY
0001:00796e67  _X509_NAME_ENTRY_new
0001:00796e7b  _X509_NAME_ENTRY_free
0001:00796e96  _X509_NAME_ENTRY_dup
0001:00796ef0* _X509_NAME_ENTRIES_it
0001:00796f50* _X509_NAME_INTERNAL_it
0001:00796f70* _x509_name_ff
0001:00796fa0  _X509_NAME_it
0001:00796fbc  _d2i_X509_NAME
0001:00796fe5  _i2d_X509_NAME
0001:00797007  _X509_NAME_new
0001:0079701b  _X509_NAME_free
0001:00797036  _X509_NAME_dup
0001:00797af8  _X509_NAME_set
Module: U:\extras\lib\libcrypto.lib(bss_sock.obj)
0001:00797b67  _BIO_s_socket
0001:00797b71* _BIO_new_socket
0001:00797e46* _BIO_sock_should_retry
0001:00797e76* _BIO_sock_non_fatal_error
Module: U:\extras\lib\libcrypto.lib(x509_cmp.obj)
0001:00797ea0* _X509_issuer_and_serial_cmp
0001:00798176  _X509_NAME_cmp
0001:00797ef6* _X509_issuer_and_serial_hash
0001:00797ffd* _X509_issuer_name_cmp
0001:00798021  _X509_subject_name_cmp
0001:00798045  _X509_CRL_cmp
0001:00798069  _X509_CRL_match
0001:00798091  _X509_get_issuer_name
0001:0079809e* _X509_issuer_name_hash
0001:00798230  _X509_NAME_hash
0001:007980b6* _X509_issuer_name_hash_old
0001:007982b9* _X509_NAME_hash_old
0001:007980ce  _X509_get_subject_name
0001:007980db  _X509_get_serialNumber
0001:007980e8* _X509_subject_name_hash
0001:00798100* _X509_subject_name_hash_old
0001:00798118  _X509_cmp
0001:00798345  _X509_find_by_issuer_and_serial
0001:007983cd* _X509_find_by_subject
0001:0079842e  _X509_get_pubkey
0001:0079845c  _X509_get0_pubkey_bitstr
0001:00798484  _X509_check_private_key
Module: U:\extras\lib\libssl.lib(d1_both.obj)
0001:007987b4* _dtls1_do_write
0001:0079afb2  _dtls1_min_mtu
0001:00798df4* _dtls1_get_message
0001:0079b001  _dtls1_get_message_header
0001:00799edf* _dtls1_send_finished
0001:0079adc3* _dtls1_set_message_header
0001:0079a7af* _dtls1_buffer_message
0001:0079a0bb* _dtls1_send_change_cipher_spec
0001:0079a2bd* _dtls1_output_cert_chain
0001:0079a539  _dtls1_read_failed
0001:0079a5c6* _dtls1_get_queue_priority
0001:0079a603  _dtls1_retransmit_buffered_messages
0001:0079aa22* _dtls1_retransmit_message
0001:0079ad6c  _dtls1_clear_record_buffer
0001:0079b0ea  _dtls1_get_ccs_header
Module: U:\extras\lib\libssl.lib(s3_pkt.obj)
0001:0079b129  _ssl3_read_n
0001:0079bb3e  _ssl3_do_uncompress
0001:0079d422  _ssl3_send_alert
0001:0079bbbc  _ssl3_do_compress
0001:0079bc3a  _ssl3_write_bytes
0001:0079c236  _ssl3_write_pending
0001:0079c42d  _ssl3_read_bytes
0001:0079d2aa  _ssl3_do_change_cipher_spec
0001:0079d4f1  _ssl3_dispatch_alert
Module: U:\extras\lib\libcrypto.lib(x509_lu.obj)
0001:0079d68a* _X509_LOOKUP_new
0001:0079d71f* _X509_LOOKUP_free
0001:0079d763* _X509_LOOKUP_init
0001:0079d7a1* _X509_LOOKUP_shutdown
0001:0079d7df  _X509_LOOKUP_ctrl
0001:0079d839* _X509_LOOKUP_by_subject
0001:0079d896* _X509_LOOKUP_by_issuer_serial
0001:0079d8e9* _X509_LOOKUP_by_fingerprint
0001:0079d93c* _X509_LOOKUP_by_alias
0001:0079da18  _X509_STORE_new
0001:0079db9a  _X509_STORE_free
0001:0079dc61  _X509_STORE_add_lookup
0001:0079dd05* _X509_STORE_get_by_subject
0001:0079e2d4* _X509_OBJECT_retrieve_by_subject
0001:0079e0fd* _X509_OBJECT_up_ref_count
0001:0079de47  _X509_STORE_add_cert
0001:0079e7b1* _X509_OBJECT_retrieve_match
0001:0079e17a* _X509_OBJECT_free_contents
0001:0079dfa2  _X509_STORE_add_crl
0001:0079e2ab* _X509_OBJECT_idx_by_subject
0001:0079e317  _X509_STORE_get1_certs
0001:0079e569  _X509_STORE_get1_crls
0001:0079e8bd  _X509_STORE_CTX_get1_issuer
0001:0079eadc* _X509_STORE_set_flags
0001:0079eaf9* _X509_STORE_set_depth
0001:0079eb1b* _X509_STORE_set_purpose
0001:0079eb38* _X509_STORE_set_trust
0001:0079eb55* _X509_STORE_set1_param
0001:0079eb72* _X509_STORE_set_verify_cb
Module: U:\extras\lib\libcrypto.lib(names.obj)
0001:0079eb80* _EVP_add_cipher
0001:0079ebf8* _EVP_add_digest
0001:0079ed0d  _EVP_get_cipherbyname
0001:0079ed2e  _EVP_get_digestbyname
0001:0079ed4f* _EVP_cleanup
0001:0079ee15* _EVP_CIPHER_do_all
0001:0079ee44* _EVP_CIPHER_do_all_sorted
0001:0079eeea* _EVP_MD_do_all
0001:0079ef19* _EVP_MD_do_all_sorted
Module: U:\extras\lib\libcrypto.lib(rand_lib.obj)
0001:0079ef50  _RAND_set_rand_method
0001:0079ef85* _RAND_get_rand_method
0001:0079efee* _RAND_set_rand_engine
0001:0079f057* _RAND_cleanup
0001:0079f08b  _RAND_seed
0001:0079f0be  _RAND_add
0001:0079f10d  _RAND_bytes
0001:0079f149  _RAND_pseudo_bytes
0001:0079f185  _RAND_status
Module: U:\extras\lib\libcrypto.lib(x_x509.obj)
0001:0079f320  _X509_CINF_it
0001:0079f33c* _d2i_X509_CINF
0001:0079f365* _i2d_X509_CINF
0001:0079f387* _X509_CINF_new
0001:0079f39b* _X509_CINF_free
0001:0079f5c0  _X509_it
0001:0079f5dc  _d2i_X509
0001:0079f605  _i2d_X509
0001:0079f627* _X509_new
0001:0079f63b  _X509_free
0001:0079f656* _X509_dup
0001:0079f671* _X509_get_ex_new_index
0001:0079f6a8* _X509_set_ex_data
0001:0079f6cc* _X509_get_ex_data
0001:0079f6e9  _d2i_X509_AUX
0001:0079f774  _i2d_X509_AUX
Module: U:\extras\lib\libcrypto.lib(eng_init.obj)
0001:0079f7c0  _engine_unlocked_init
0001:0079f826  _engine_unlocked_finish
0001:0079f917  _ENGINE_init
0001:0079f9b1  _ENGINE_finish
Module: U:\extras\lib\libcrypto.lib(rsa_lib.obj)
0001:0079faa0* _RSA_version
0001:0079fac7  _RSA_new
0001:0079fb94* _RSA_new_method
0001:0079fae1* _RSA_set_default_method
0001:0079faee* _RSA_get_default_method
0001:0079fb0e* _RSA_get_method
0001:0079fb19* _RSA_set_method
0001:0079fe54  _RSA_free
0001:007a000d  _RSA_up_ref
0001:007a0050* _RSA_get_ex_new_index
0001:007a0087* _RSA_set_ex_data
0001:007a00ab* _RSA_get_ex_data
0001:007a00c8  _RSA_size
0001:007a00eb  _RSA_public_encrypt
0001:007a0120  _RSA_private_encrypt
0001:007a0155  _RSA_private_decrypt
0001:007a018a  _RSA_public_decrypt
0001:007a01bf  _RSA_flags
0001:007a01da* _RSA_blinding_off
0001:007a0226* _RSA_blinding_on
0001:007a03a5  _RSA_setup_blinding
0001:007a062a* _RSA_memory_lock
Module: U:\extras\lib\libcrypto.lib(dh_lib.obj)
0001:007a0820* _DH_version
0001:007a0852* _DH_set_default_method
0001:007a085f* _DH_get_default_method
0001:007a087f* _DH_set_method
0001:007a08f0  _DH_new
0001:007a090d* _DH_new_method
0001:007a0b81  _DH_free
0001:007a0cf2  _DH_up_ref
0001:007a0d35* _DH_get_ex_new_index
0001:007a0d6c* _DH_set_ex_data
0001:007a0d90* _DH_get_ex_data
0001:007a0dad  _DH_size
Module: U:\extras\lib\libcrypto.lib(p_lib.obj)
0001:007a0dd0  _EVP_PKEY_bits
0001:007a0e0d  _EVP_PKEY_size
0001:007a0e4a* _EVP_PKEY_save_parameters
0001:007a0eaf  _EVP_PKEY_copy_parameters
0001:007a0f66  _EVP_PKEY_missing_parameters
0001:007a0f9d  _EVP_PKEY_cmp_parameters
0001:007a0ff0  _EVP_PKEY_cmp
0001:007a1076  _EVP_PKEY_new
0001:007a1250  _EVP_PKEY_set_type
0001:007a127a  _EVP_PKEY_set_type_str
0001:007a12a3  _EVP_PKEY_assign
0001:007a12db* _EVP_PKEY_get0
0001:007a12e6  _EVP_PKEY_set1_RSA
0001:007a131f  _EVP_PKEY_get1_RSA
0001:007a1378  _EVP_PKEY_set1_DSA
0001:007a13b1  _EVP_PKEY_get1_DSA
0001:007a140a  _EVP_PKEY_set1_EC_KEY
0001:007a1443  _EVP_PKEY_get1_EC_KEY
0001:007a149e* _EVP_PKEY_set1_DH
0001:007a14d7* _EVP_PKEY_get1_DH
0001:007a1530  _EVP_PKEY_type
0001:007a1579  _EVP_PKEY_id
0001:007a1583* _EVP_PKEY_base_id
0001:007a1598  _EVP_PKEY_free
0001:007a16f4  _EVP_PKEY_print_public
0001:007a1768  _EVP_PKEY_print_private
0001:007a17db  _EVP_PKEY_print_params
0001:007a1843  _EVP_PKEY_get_default_digest_nid
Module: U:\extras\lib\libcrypto.lib(v3_purp.obj)
0001:007a19a1  _X509_check_purpose
0001:007a1b7a  _X509_PURPOSE_get_by_id
0001:007a1add  _X509_PURPOSE_get0
0001:007a1a5d  _X509_PURPOSE_set
0001:007a1ab5* _X509_PURPOSE_get_count
0001:007a1b2b* _X509_PURPOSE_get_by_sname
0001:007a1bd4* _X509_PURPOSE_add
0001:007a1e4a* _X509_PURPOSE_cleanup
0001:007a1ea4* _X509_PURPOSE_get_id
0001:007a1eae* _X509_PURPOSE_get0_name
0001:007a1eb9* _X509_PURPOSE_get0_sname
0001:007a1ec4* _X509_PURPOSE_get_trust
0001:007a1f3b* _X509_supported_extension
0001:007a282b  _X509_check_ca
0001:007a2cd8  _X509_check_issued
0001:007a2db2  _X509_check_akid
Module: U:\extras\lib\libcrypto.lib(obj_dat.obj)
0001:007b202f  _OBJ_bsearch_
0001:007b1291  _check_defer
0001:007b12b2  _OBJ_cleanup
0001:007b133d* _OBJ_new_nid
0001:007b1367* _OBJ_add_object
0001:007b157f  _OBJ_nid2obj
0001:007b1674  _OBJ_nid2sn
0001:007b176c  _OBJ_nid2ln
0001:007b1926  _OBJ_obj2nid
0001:007b19ce  _OBJ_txt2obj
0001:007b1f9e  _OBJ_sn2nid
0001:007b1f0d  _OBJ_ln2nid
0001:007b1b2b  _OBJ_obj2txt
0001:007b1ed3* _OBJ_txt2nid
0001:007b2066  _OBJ_bsearch_ex_
0001:007b2168* _OBJ_create_objects
0001:007b2335* _OBJ_create
0002:0001f420  _obj_cleanup_defer
Module: U:\extras\lib\libcrypto.lib(obj_xref.obj)
0002:00022350+ _sig_app
0002:00022360+ _sigx_app
0001:007b2762  _OBJ_find_sigid_algs
0001:007b2800  _OBJ_find_sigid_by_algs
0001:007b28b1* _OBJ_add_sigid
0001:007b29d9  _OBJ_sigid_free
Module: U:\extras\lib\libcrypto.lib(evp_enc.obj)
0001:007b2a30* _EVP_version
0001:007b2a57  _EVP_CIPHER_CTX_init
0001:007b2a84* _EVP_CIPHER_CTX_new
0001:007b2abf* _EVP_CipherInit
0001:007b2b9e  _EVP_CipherInit_ex
0001:007b38ee  _EVP_CIPHER_CTX_cleanup
0001:007b3a75  _EVP_CIPHER_CTX_ctrl
0001:007b2fca  _EVP_CipherUpdate
0001:007b31a2  _EVP_EncryptUpdate
0001:007b3544  _EVP_DecryptUpdate
0001:007b302c  _EVP_CipherFinal_ex
0001:007b3411  _EVP_EncryptFinal_ex
0001:007b36d7  _EVP_DecryptFinal_ex
0001:007b3072* _EVP_CipherFinal
0001:007b33d5* _EVP_EncryptFinal
0001:007b36b0  _EVP_DecryptFinal
0001:007b30b8* _EVP_EncryptInit
0001:007b30e8  _EVP_EncryptInit_ex
0001:007b311f* _EVP_DecryptInit
0001:007b314f  _EVP_DecryptInit_ex
0001:007b38ca* _EVP_CIPHER_CTX_free
0001:007b399c  _EVP_CIPHER_CTX_set_key_length
0001:007b3a41* _EVP_CIPHER_CTX_set_padding
0001:007b3b5f  _EVP_CIPHER_CTX_rand_key
0001:007b3bc1  _EVP_CIPHER_CTX_copy
Module: U:\extras\lib\libcrypto.lib(comp_lib.obj)
0001:007b3d7b  _COMP_CTX_new
0001:007b3e07  _COMP_CTX_free
0001:007b3e3f  _COMP_compress_block
0001:007b3eb4  _COMP_expand_block
Module: U:\extras\lib\libcrypto.lib(bf_buff.obj)
0001:007b3f37  _BIO_f_buffer
Module: U:\extras\lib\libcrypto.lib(x509_d2.obj)
0001:007b4d30  _X509_STORE_set_default_paths
0001:007b4de3  _X509_STORE_load_locations
Module: U:\extras\lib\libcrypto.lib(digest.obj)
0001:007b4ed0  _EVP_MD_CTX_init
0001:007b4efc  _EVP_MD_CTX_create
0001:007b4f37  _EVP_DigestInit
0001:007b4f64  _EVP_DigestInit_ex
0001:007b522d  _EVP_DigestUpdate
0001:007b5251  _EVP_DigestFinal
0001:007b52ac  _EVP_DigestFinal_ex
0001:007b5661  _EVP_MD_CTX_cleanup
0001:007b5362  _EVP_MD_CTX_copy
0001:007b5387  _EVP_MD_CTX_copy_ex
0001:007b55a9  _EVP_Digest
0001:007b5643  _EVP_MD_CTX_destroy
Module: U:\extras\lib\libssl.lib(s2_clnt.obj)
0001:007b577a  _SSLv2_client_method
0001:007b578e* _ssl2_connect
0001:007b791f* _ssl2_set_certificate
Module: U:\extras\lib\libssl.lib(s3_clnt.obj)
0001:007b7d5d  _SSLv3_client_method
0001:007b7d71  _ssl3_connect
0001:007b89ce* _ssl3_client_hello
0001:007b8e0f* _ssl3_get_server_hello
0001:007bdaeb* _ssl3_check_finished
0001:007b962d* _ssl3_get_server_certificate
0001:007b9d35* _ssl3_get_key_exchange
0001:007bd64f* _ssl3_check_cert_and_algorithm
0001:007bb09c* _ssl3_get_certificate_request
0001:007bbc0b* _ssl3_get_server_done
0001:007bd406* _ssl3_send_client_certificate
0001:007bbcbf* _ssl3_send_client_key_exchange
0001:007bcf5d* _ssl3_send_client_verify
0001:007bb5d0* _ssl3_get_new_session_ticket
0001:007bb94b* _ssl3_get_cert_status
0001:007bdb9a* _ssl_do_client_cert_cb
Module: U:\extras\lib\libssl.lib(t1_clnt.obj)
0001:007bdcfd  _TLSv1_client_method
Module: U:\extras\lib\libssl.lib(s3_both.obj)
0001:007bdd90  _ssl3_do_write
0001:007bdec7  _ssl3_send_finished
0001:007be090  _ssl3_get_finished
0001:007be2db  _ssl3_send_change_cipher_spec
0001:007be40c  _ssl3_output_cert_chain
0001:007be6d0  _ssl3_get_message
0001:007bebea  _ssl_cert_type
0001:007bec9e  _ssl_verify_alarm_type
0001:007befc1  _ssl3_setup_read_buffer
0001:007bf102  _ssl3_setup_write_buffer
0001:007bf232  _ssl3_setup_buffers
0001:007bf26b  _ssl3_release_write_buffer
0001:007bf2d1  _ssl3_release_read_buffer
Module: U:\extras\lib\libssl.lib(s3_enc.obj)
0001:007bf5a1  _ssl3_change_cipher_state
0001:007bfca6  _ssl3_setup_key_block
0001:007bfeda  _ssl3_cleanup_key_block
0001:007bff4c  _ssl3_enc
0001:007c0192  _ssl3_init_finished_mac
0001:007c0223  _ssl3_free_digest_list
0001:007c02ac  _ssl3_finish_mac
0001:007c0340  _ssl3_digest_cached_records
0001:007c0517  _ssl3_cert_verify_mac
0001:007c0548  _ssl3_final_finish_mac
0001:007c0815  _n_ssl3_mac
0001:007c0a6a  _ssl3_record_sequence_update
0001:007c0a9e  _ssl3_generate_master_secret
0001:007c0c32  _ssl3_alert_code
Module: U:\extras\lib\libssl.lib(s3_lib.obj)
0001:007c0f30* _ssl3_version_str
0001:007c15d9  _ssl3_default_timeout
0001:007c15e3  _ssl3_num_ciphers
0001:007c15ed  _ssl3_get_cipher
0001:007c1617  _ssl3_pending
0001:007c165d  _ssl3_new
0001:007c170c  _ssl3_free
0001:007c1868  _ssl3_clear
0001:007c1aa5  _ssl3_ctrl
0001:007c22de  _ssl3_callback_ctrl
0001:007c23a2  _ssl3_ctx_ctrl
0001:007c29f0  _ssl3_ctx_callback_ctrl
0001:007c2a85  _ssl3_get_cipher_by_char
0001:007c2aea  _ssl3_put_cipher_by_char
0001:007c2b34* _ssl3_choose_cipher
0001:007c3254* _ssl3_get_req_cert_type
0001:007c335e  _ssl3_shutdown
0001:007c3490  _ssl3_write
0001:007c3766  _ssl3_renegotiate_check
0001:007c36d3  _ssl3_read
0001:007c36fc  _ssl3_peek
0001:007c3725  _ssl3_renegotiate
0002:000051c0* _ssl3_ciphers
0002:000062a0  _SSLv3_enc_data
Module: U:\extras\lib\libssl.lib(t1_lib.obj)
0001:007c3810* _tls1_version_str
0001:007c3859  _tls1_default_timeout
0001:007c3863  _tls1_new
0001:007c3897  _tls1_free
0001:007c38c8  _tls1_clear
0001:007c38e4  _tls1_ec_curve_id2nid
0001:007c3909  _tls1_ec_nid2curve_id
0001:007c3b37  _ssl_add_clienthello_tlsext
0001:007c44ae* _ssl_add_serverhello_tlsext
0001:007c495d* _ssl_parse_clienthello_tlsext
0001:007c53d9  _ssl_parse_serverhello_tlsext
0001:007c58b2  _ssl_prepare_clienthello_tlsext
0001:007c5afe* _ssl_prepare_serverhello_tlsext
0001:007c5c40* _ssl_check_clienthello_tlsext
0001:007c5e3b  _ssl_check_serverhello_tlsext
0001:007c615f  _tls1_process_ticket
0002:000062e0  _TLSv1_enc_data
Module: U:\extras\lib\libssl.lib(s23_pkt.obj)
0001:007c6770  _ssl23_write_bytes
0001:007c680c  _ssl23_read_bytes
Module: U:\extras\lib\libssl.lib(s2_lib.obj)
0001:007c68b0* _ssl2_version_str
0001:007c6930* _ssl2_ciphers
0001:007c6a80  _ssl2_default_timeout
0001:007c6a8a  _ssl2_num_ciphers
0001:007c6a94  _ssl2_get_cipher
0001:007c6abe  _ssl2_pending
0001:007c6af3  _ssl2_new
0001:007c6c75  _ssl2_clear
0001:007c6c03  _ssl2_free
0001:007c6cee  _ssl2_ctrl
0001:007c6d11  _ssl2_callback_ctrl
0001:007c6d1b  _ssl2_ctx_ctrl
0001:007c6d25  _ssl2_ctx_callback_ctrl
0001:007c6d2f  _ssl2_get_cipher_by_char
0001:007c6da4  _ssl2_put_cipher_by_char
0001:007c6e66  _ssl2_generate_key_material
0001:007c70a4  _ssl2_return_error
0001:007c7108  _ssl2_write_error
0001:007c7214  _ssl2_shutdown
Module: U:\extras\lib\libssl.lib(s23_lib.obj)
0001:007c7230  _ssl23_default_timeout
0001:007c723a  _ssl23_num_ciphers
0001:007c7256  _ssl23_get_cipher
0001:007c728f  _ssl23_get_cipher_by_char
0001:007c72bc  _ssl23_put_cipher_by_char
0001:007c7308  _ssl23_read
0001:007c73b9  _ssl23_peek
0001:007c746a  _ssl23_write
Module: U:\extras\lib\xmlrpc.lib(queue.obj)
0001:007c7520  _Q_Init
0001:007c7553* _Q_AtHead
0001:007c756c* _Q_AtTail
0001:007c7586* _Q_IsEmpty
0001:007c75a0  _Q_Size
0001:007c75b1  _Q_Head
0001:007c75cf* _Q_Tail
0001:007c75ee  _Q_Next
0001:007c7611* _Q_Previous
0001:007c7630* _Q_Get
0001:007c7649* _Q_Put
0001:007c766e* _Q_Find
0001:007c77e6* _Q_Iter_Head
0001:007c77f6* _Q_Iter_Tail
0001:007c7807* _Q_Iter_Next
0001:007c7818* _Q_Iter_Prev
0001:007c7829* _Q_Iter_Get
0001:007c7839* _Q_Iter_Put
0001:007c7851* _Q_PopTail
0001:007c78cb* _Q_PopHead
0001:007c7943  _Q_Destroy
0001:007c7968  _Q_Iter_Del
0001:007c79fd* _Q_DelCur
0001:007c7a1d* _Q_Sort
0001:007c7b65* _Q_Seek
0001:007c7c16  _Q_PushTail
0001:007c7c8c* _Q_PushHead
0001:007c7cfd* _Q_Insert
Module: U:\extras\lib\xmlrpc.lib(simplestring.obj)
0001:007c7d40  _simplestring_clear
0001:007c7d58  _simplestring_addn
0001:007c7e4a  _simplestring_add
0001:007c7e8e  _simplestring_free
0001:007c7ebd  _simplestring_init
Module: U:\extras\lib\xmlrpc.lib(system_methods.obj)
0001:007c7f08  _xsm_register
Module: U:\extras\lib\xmlrpc.lib(xml_element.obj)
0001:007ca822* _xml_elem_serialize_to_stream
0001:007ca863  _xml_elem_serialize_to_string
0001:007ca8aa  _xml_elem_new
0001:007ca996  _xml_elem_free_non_recurse
0001:007caae1  _xml_elem_parse_buf
0001:007cad55  _xml_elem_free
Module: U:\extras\lib\xmlrpc.lib(xml_to_xmlrpc.obj)
0001:007cae29* _XMLRPC_to_xml_element_worker
0001:007cb388  _XMLRPC_REQUEST_to_xml_element
0001:007cb4af  _XMLRPC_VALUE_to_xml_element
0001:007cb4dd* _xml_element_to_XMLRPC_REQUEST_worker
0001:007cba15  _xml_element_to_XMLRPC_REQUEST
0001:007cba5a* _xml_element_to_XMLRPC_VALUE
Module: U:\extras\lib\xmlrpc.lib(xml_to_soap.obj)
0001:007cbbe4* _SOAP_to_xml_element_worker
0001:007cc376  _SOAP_REQUEST_to_xml_element
0001:007cc657* _SOAP_VALUE_to_xml_element
0001:007cc734* _xml_element_to_SOAP_REQUEST_worker
0001:007ccf11  _xml_element_to_SOAP_REQUEST
0001:007ccf66* _xml_element_to_SOAP_VALUE
Module: U:\extras\lib\xmlrpc.lib(xml_to_dandarpc.obj)
0001:007cd041* _DANDARPC_to_xml_element_worker
0001:007cd521  _DANDARPC_REQUEST_to_xml_element
0001:007cd653* _DANDARPC_VALUE_to_xml_element
0001:007cd66e* _xml_element_to_DANDARPC_REQUEST_worker
0001:007cda9a  _xml_element_to_DANDARPC_REQUEST
0001:007cdad7* _xml_element_to_DANDARPC_VALUE
Module: U:\usr\local446\lib\gcc\i386-pc-os2-emx\4.4.6\libgcc_eh.lib(unwind-dw2-fde.obj)
0001:007ce98f* ___deregister_frame_info_bases
0001:007ceafa* ___deregister_frame_info
0001:007ceb05  ___deregister_frame
0001:007ceb2a* ___register_frame_info_table_bases
0001:007cec1c* ___register_frame_info_table
0001:007cec47  ___register_frame_table
0001:007cec6a* __Unwind_Find_FDE
0001:007cee46* ___register_frame_info_bases
0001:007cef45* ___register_frame_info
0001:007cef70* ___register_frame
Module: U:\extras\lib\lzma.lib(liblzma_la-common.obj)
0001:007cefa0* _lzma_version_number
0001:007cefb0* _lzma_version_string
0001:007cefba  _lzma_next_filter_update
0001:007cf019  _lzma_code
0001:007cf28c* _lzma_get_check
0001:007cf2a9* _lzma_memusage
0001:007cf2fb* _lzma_memlimit_get
0001:007cf34d* _lzma_memlimit_set
0001:007cf3d1  _lzma_bufcpy
0001:007cf418  _lzma_free
0001:007cf444  _lzma_next_end
0001:007cf49f  _lzma_next_filter_init
0001:007cf4fa  _lzma_end
0001:007cf53d  _lzma_alloc
0001:007cf578  _lzma_strm_init
Module: U:\extras\lib\lzma.lib(liblzma_la-filter_decoder.obj)
0001:007cf661* _lzma_filter_decoder_is_supported
0001:007cf6a7  _lzma_properties_decode
0001:007cf74b  _lzma_raw_decoder_memusage
0001:007cf766  _lzma_raw_decoder_init
0001:007cf797* _lzma_raw_decoder
Module: U:\extras\lib\lzma.lib(liblzma_la-auto_decoder.obj)
0001:007cfa16  _lzma_auto_decoder
Module: U:\extras\lib\pthread.lib(my_os2key.obj)
0001:007cfbf0  _pthread_key_create
0001:007cfc12  _pthread_key_delete
0001:007cfc25  _pthread_getspecific
0001:007cfc38  _pthread_setspecific
Module: U:\extras\lib\pthread.lib(my_os2mutex.obj)
0001:007cfc60  _pthread_mutex_init
0001:007cfcd6  _pthread_mutex_destroy
0001:007cfd4a  _pthread_mutex_lock
0001:007cfdbd* _pthread_mutex_trylock
0001:007cfe4f  _pthread_mutex_unlock
0001:007cfead* _pthread_mutexattr_init
0001:007cff00* _pthread_mutexattr_destroy
0001:007cff46* _pthread_mutexattr_settype
0001:007cff90* _pthread_mutexattr_gettype
Module: U:\extras\lib\pthread.lib(my_os2thread.obj)
0001:007cffee* __pthreadInit
0001:007d01f9* _pthread_exit
0001:007d00bf* _pthread_create
0001:007d0265* _pthread_setprio
0001:007d0254  _pthread_equal
0001:007d028f* _pthread_dummy
0001:007d0297  _pthread_self
0001:007d030e* _pthread_join
0001:007d03a3* _pthread_cleanup_push
0001:007d03a8* _pthread_cleanup_pop
0001:007d03ad  _pthread_once
0001:007d041f* _pthread_yield
0001:007d0433* _pthread_setcancelstate
0001:007d043d* _pthread_setcanceltype
0001:007d0447* _pthread_testcancel
0001:007d044c* _pthread_atfork
0001:007d0456* _pthread_detach
0001:007d04ce* _pthread_kill
0001:007d0524* _pthread_cancel
Module: U:\extras\lib\pthread.lib(my_os2cond.obj)
0001:007d058e  _pthread_cond_init
0001:007d0673  _pthread_cond_destroy
0001:007d06e7  _pthread_cond_wait
0001:007d0799* _pthread_cond_timedwait
0001:007d08d8  _pthread_cond_signal
0001:007d093a* _pthread_cond_broadcast
Module: U:\extras\lib\xml2.lib(xmlunicode.obj)
0001:007d09b0* _xmlUCSIsAegeanNumbers
0001:007d09c6* _xmlUCSIsAlphabeticPresentationForms
0001:007d09dc* _xmlUCSIsArabic
0001:007d09f4* _xmlUCSIsArabicPresentationFormsA
0001:007d0a0c* _xmlUCSIsArabicPresentationFormsB
0001:007d0a24* _xmlUCSIsArmenian
0001:007d0a3a* _xmlUCSIsArrows
0001:007d0a50* _xmlUCSIsBasicLatin
0001:007d0a5e* _xmlUCSIsBengali
0001:007d0a74* _xmlUCSIsBlockElements
0001:007d0a8a* _xmlUCSIsBopomofo
0001:007d0aa0* _xmlUCSIsBopomofoExtended
0001:007d0ab6* _xmlUCSIsBoxDrawing
0001:007d0acc* _xmlUCSIsBraillePatterns
0001:007d0ae4* _xmlUCSIsBuhid
0001:007d0afa* _xmlUCSIsByzantineMusicalSymbols
0001:007d0b12* _xmlUCSIsCJKCompatibility
0001:007d0b2a* _xmlUCSIsCJKCompatibilityForms
0001:007d0b40* _xmlUCSIsCJKCompatibilityIdeographs
0001:007d0b58* _xmlUCSIsCJKCompatibilityIdeographsSupplement
0001:007d0b70* _xmlUCSIsCJKRadicalsSupplement
0001:007d0b86* _xmlUCSIsCJKSymbolsandPunctuation
0001:007d0b9c* _xmlUCSIsCJKUnifiedIdeographs
0001:007d0bb4* _xmlUCSIsCJKUnifiedIdeographsExtensionA
0001:007d0bcc* _xmlUCSIsCJKUnifiedIdeographsExtensionB
0001:007d0be4* _xmlUCSIsCherokee
0001:007d0bfa* _xmlUCSIsCombiningDiacriticalMarks
0001:007d0c10* _xmlUCSIsCombiningDiacriticalMarksforSymbols
0001:007d0c26* _xmlUCSIsCombiningHalfMarks
0001:007d0c3c* _xmlUCSIsCombiningMarksforSymbols
0001:007d0c52* _xmlUCSIsControlPictures
0001:007d0c68* _xmlUCSIsCurrencySymbols
0001:007d0c7e* _xmlUCSIsCypriotSyllabary
0001:007d0c94* _xmlUCSIsCyrillic
0001:007d0cac* _xmlUCSIsCyrillicSupplement
0001:007d0cc2* _xmlUCSIsDeseret
0001:007d0cd8* _xmlUCSIsDevanagari
0001:007d0cee* _xmlUCSIsDingbats
0001:007d0d06* _xmlUCSIsEnclosedAlphanumerics
0001:007d0d1e* _xmlUCSIsEnclosedCJKLettersandMonths
0001:007d0d36* _xmlUCSIsEthiopic
0001:007d0d4e* _xmlUCSIsGeneralPunctuation
0001:007d0d64* _xmlUCSIsGeometricShapes
0001:007d0d7a* _xmlUCSIsGeorgian
0001:007d0d90* _xmlUCSIsGothic
0001:007d0da6* _xmlUCSIsGreek
0001:007d0dbe* _xmlUCSIsGreekExtended
0001:007d0dd6* _xmlUCSIsGreekandCoptic
0001:007d0dee* _xmlUCSIsGujarati
0001:007d0e04* _xmlUCSIsGurmukhi
0001:007d0e1a* _xmlUCSIsHalfwidthandFullwidthForms
0001:007d0e32* _xmlUCSIsHangulCompatibilityJamo
0001:007d0e48* _xmlUCSIsHangulJamo
0001:007d0e60* _xmlUCSIsHangulSyllables
0001:007d0e78* _xmlUCSIsHanunoo
0001:007d0e8e* _xmlUCSIsHebrew
0001:007d0ea4* _xmlUCSIsHighPrivateUseSurrogates
0001:007d0eba* _xmlUCSIsHighSurrogates
0001:007d0ed2* _xmlUCSIsHiragana
0001:007d0ee8* _xmlUCSIsIPAExtensions
0001:007d0efe* _xmlUCSIsIdeographicDescriptionCharacters
0001:007d0f14* _xmlUCSIsKanbun
0001:007d0f2a* _xmlUCSIsKangxiRadicals
0001:007d0f42* _xmlUCSIsKannada
0001:007d0f58* _xmlUCSIsKatakana
0001:007d0f6e* _xmlUCSIsKatakanaPhoneticExtensions
0001:007d0f84* _xmlUCSIsKhmer
0001:007d0f9a* _xmlUCSIsKhmerSymbols
0001:007d0fb0* _xmlUCSIsLao
0001:007d0fc6* _xmlUCSIsLatin1Supplement
0001:007d0fda* _xmlUCSIsLatinExtendedA
0001:007d0ff0* _xmlUCSIsLatinExtendedB
0001:007d1008* _xmlUCSIsLatinExtendedAdditional
0001:007d1020* _xmlUCSIsLetterlikeSymbols
0001:007d1036* _xmlUCSIsLimbu
0001:007d104c* _xmlUCSIsLinearBIdeograms
0001:007d1062* _xmlUCSIsLinearBSyllabary
0001:007d1078* _xmlUCSIsLowSurrogates
0001:007d1090* _xmlUCSIsMalayalam
0001:007d10a6* _xmlUCSIsMathematicalAlphanumericSymbols
0001:007d10be* _xmlUCSIsMathematicalOperators
0001:007d10d6* _xmlUCSIsMiscellaneousMathematicalSymbolsA
0001:007d10ec* _xmlUCSIsMiscellaneousMathematicalSymbolsB
0001:007d1102* _xmlUCSIsMiscellaneousSymbols
0001:007d111a* _xmlUCSIsMiscellaneousSymbolsandArrows
0001:007d1132* _xmlUCSIsMiscellaneousTechnical
0001:007d114a* _xmlUCSIsMongolian
0001:007d1162* _xmlUCSIsMusicalSymbols
0001:007d117a* _xmlUCSIsMyanmar
0001:007d1192* _xmlUCSIsNumberForms
0001:007d11a8* _xmlUCSIsOgham
0001:007d11be* _xmlUCSIsOldItalic
0001:007d11d4* _xmlUCSIsOpticalCharacterRecognition
0001:007d11ea* _xmlUCSIsOriya
0001:007d1200* _xmlUCSIsOsmanya
0001:007d1216* _xmlUCSIsPhoneticExtensions
0001:007d122c* _xmlUCSIsPrivateUse
0001:007d1267* _xmlUCSIsPrivateUseArea
0001:007d127f* _xmlUCSIsRunic
0001:007d1295* _xmlUCSIsShavian
0001:007d12ab* _xmlUCSIsSinhala
0001:007d12c1* _xmlUCSIsSmallFormVariants
0001:007d12d7* _xmlUCSIsSpacingModifierLetters
0001:007d12ed* _xmlUCSIsSpecials
0001:007d1303* _xmlUCSIsSuperscriptsandSubscripts
0001:007d1319* _xmlUCSIsSupplementalArrowsA
0001:007d132f* _xmlUCSIsSupplementalArrowsB
0001:007d1345* _xmlUCSIsSupplementalMathematicalOperators
0001:007d135d* _xmlUCSIsSupplementaryPrivateUseAreaA
0001:007d1375* _xmlUCSIsSupplementaryPrivateUseAreaB
0001:007d138d* _xmlUCSIsSyriac
0001:007d13a3* _xmlUCSIsTagalog
0001:007d13b9* _xmlUCSIsTagbanwa
0001:007d13cf* _xmlUCSIsTags
0001:007d13e5* _xmlUCSIsTaiLe
0001:007d13fb* _xmlUCSIsTaiXuanJingSymbols
0001:007d1411* _xmlUCSIsTamil
0001:007d1427* _xmlUCSIsTelugu
0001:007d143d* _xmlUCSIsThaana
0001:007d1453* _xmlUCSIsThai
0001:007d1469* _xmlUCSIsTibetan
0001:007d1481* _xmlUCSIsUgaritic
0001:007d1497* _xmlUCSIsUnifiedCanadianAboriginalSyllabics
0001:007d14af* _xmlUCSIsVariationSelectors
0001:007d14c5* _xmlUCSIsVariationSelectorsSupplement
0001:007d14dd* _xmlUCSIsYiRadicals
0001:007d14f3* _xmlUCSIsYiSyllables
0001:007d150b* _xmlUCSIsYijingHexagramSymbols
0001:007d1521  _xmlUCSIsCatCc
0001:007d153d  _xmlUCSIsCatCo
0001:007d1583* _xmlUCSIsCatCs
0001:007d15bf  _xmlUCSIsCatMe
0001:007d15f9  _xmlUCSIsCatNl
0001:007d164b  _xmlUCSIsCatPc
0001:007d16a3  _xmlUCSIsCatPf
0001:007d16d9  _xmlUCSIsCatPi
0001:007d1713  _xmlUCSIsCatZl
0001:007d1724  _xmlUCSIsCatZp
0001:007d1735  _xmlUCSIsCatZs
0001:007d1802* _xmlUCSIsCat
0001:007d1832  _xmlUCSIsBlock
0001:007d1862  _xmlUCSIsCatZ
0001:007d187d  _xmlUCSIsCatSo
0001:007d1898  _xmlUCSIsCatSm
0001:007d18b3  _xmlUCSIsCatSk
0001:007d18ce  _xmlUCSIsCatSc
0001:007d18e9  _xmlUCSIsCatS
0001:007d1904  _xmlUCSIsCatPs
0001:007d191f  _xmlUCSIsCatPo
0001:007d193a  _xmlUCSIsCatPe
0001:007d1955  _xmlUCSIsCatPd
0001:007d1970  _xmlUCSIsCatP
0001:007d198b  _xmlUCSIsCatNo
0001:007d19a6  _xmlUCSIsCatNd
0001:007d19c1  _xmlUCSIsCatN
0001:007d19dc  _xmlUCSIsCatMn
0001:007d19f7  _xmlUCSIsCatMc
0001:007d1a12  _xmlUCSIsCatM
0001:007d1a2d  _xmlUCSIsCatLu
0001:007d1a48  _xmlUCSIsCatLt
0001:007d1a63  _xmlUCSIsCatLo
0001:007d1a7e  _xmlUCSIsCatLm
0001:007d1a99  _xmlUCSIsCatLl
0001:007d1ab4  _xmlUCSIsCatL
0001:007d1acf  _xmlUCSIsCatCf
0001:007d1aea  _xmlUCSIsCatC
Module: U:\extras\lib\libcrypto.lib(mem_dbg.obj)
0001:007d4f3e  _CRYPTO_mem_ctrl
0001:007d5129* _CRYPTO_is_mem_check_on
0001:007d51d0* _CRYPTO_dbg_set_options
0001:007d51dd* _CRYPTO_dbg_get_options
0001:007d5442  _CRYPTO_push_info_
0001:007d5549  _CRYPTO_pop_info
0001:007d558c* _CRYPTO_remove_all_info
0001:007d55cd* _CRYPTO_dbg_malloc
0001:007d57fb* _CRYPTO_dbg_free
0001:007d5883* _CRYPTO_dbg_realloc
0001:007d5da3* _CRYPTO_mem_leaks
0001:007d5ef5* _CRYPTO_mem_leaks_fp
0001:007d5fe0* _CRYPTO_mem_leaks_cb
Module: U:\extras\lib\libcrypto.lib(b_print.obj)
0001:007d74a4  _BIO_printf
0001:007d74d9* _BIO_vprintf
0001:007d75cd  _BIO_snprintf
0001:007d7601* _BIO_vsnprintf
Module: U:\extras\lib\libcrypto.lib(mem_clr.obj)
0001:007d7670  _OPENSSL_cleanse
0002:0001f530  _cleanse_ctr
Module: U:\extras\lib\libcrypto.lib(eng_pkey.obj)
0001:007d7700* _ENGINE_set_load_privkey_function
0001:007d7713* _ENGINE_set_load_pubkey_function
0001:007d7726* _ENGINE_set_load_ssl_client_cert_function
0001:007d7739* _ENGINE_get_load_privkey_function
0001:007d7744* _ENGINE_get_load_pubkey_function
0001:007d774f  _ENGINE_get_ssl_client_cert_function
0001:007d7765* _ENGINE_load_private_key
0001:007d78f4* _ENGINE_load_public_key
0001:007d7a83  _ENGINE_load_ssl_client_cert
Module: U:\extras\lib\libssl.lib(ssl_asn1.obj)
0001:007d7bf0  _i2d_SSL_SESSION
0001:007d8939  _d2i_SSL_SESSION
Module: U:\extras\lib\libcrypto.lib(pem_oth.obj)
0001:007d9eba  _PEM_ASN1_read_bio
Module: U:\extras\lib\libcrypto.lib(pem_lib.obj)
0001:007d9f80* _PEM_version
0001:007d9ffc  _PEM_def_callback
0001:007da14a  _PEM_proc_type
0001:007da1e3  _PEM_dek_info
0001:007da2d0  _PEM_ASN1_read
0001:007dc167  _pem_check_suffix
0001:007da777  _PEM_bytes_read_bio
0001:007db955  _PEM_read_bio
0001:007db10e  _PEM_get_EVP_CIPHER_INFO
0001:007daed4  _PEM_do_header
0001:007da8da  _PEM_ASN1_write
0001:007da9f5  _PEM_ASN1_write_bio
0001:007db5c1  _PEM_write_bio
0001:007db4f9* _PEM_write
0001:007db8aa* _PEM_read
Module: U:\extras\lib\libcrypto.lib(ameth_lib.obj)
0001:007dc280* _EVP_PKEY_asn1_get_count
0001:007dc2ab* _EVP_PKEY_asn1_get0
0001:007dc381  _EVP_PKEY_asn1_find
0001:007dc3f7  _EVP_PKEY_asn1_find_str
0001:007dc4e1* _EVP_PKEY_asn1_add0
0001:007dc545* _EVP_PKEY_asn1_add_alias
0001:007dc618* _EVP_PKEY_asn1_new
0001:007dc594  _EVP_PKEY_asn1_get0_info
0001:007dc601* _EVP_PKEY_get0_asn1
0001:007dc88a  _EVP_PKEY_asn1_free
0001:007dc7a1* _EVP_PKEY_asn1_copy
0001:007dc8e0* _EVP_PKEY_asn1_set_public
0001:007dc91b* _EVP_PKEY_asn1_set_private
0001:007dc93b* _EVP_PKEY_asn1_set_param
0001:007dc976* _EVP_PKEY_asn1_set_free
0001:007dc984* _EVP_PKEY_asn1_set_ctrl
Module: U:\extras\lib\libcrypto.lib(evp_lib.obj)
0001:007dc9a0  _EVP_CIPHER_param_to_asn1
0001:007dc9da  _EVP_CIPHER_asn1_to_param
0001:007dca31  _EVP_CIPHER_get_asn1_iv
0001:007dcd1b  _EVP_CIPHER_CTX_iv_length
0001:007dcae3  _EVP_CIPHER_set_asn1_iv
0001:007dcb4a  _EVP_CIPHER_type
0001:007dcd3e  _EVP_CIPHER_nid
0001:007dcc90  _EVP_CIPHER_block_size
0001:007dcc9b  _EVP_CIPHER_CTX_block_size
0001:007dcca8  _EVP_Cipher
0001:007dccd5  _EVP_CIPHER_CTX_cipher
0001:007dccdf  _EVP_CIPHER_flags
0001:007dccea  _EVP_CIPHER_CTX_flags
0001:007dccf7* _EVP_CIPHER_CTX_get_app_data
0001:007dcd02* _EVP_CIPHER_CTX_set_app_data
0001:007dcd10  _EVP_CIPHER_iv_length
0001:007dcd28  _EVP_CIPHER_key_length
0001:007dcd33  _EVP_CIPHER_CTX_key_length
0001:007dcd48* _EVP_CIPHER_CTX_nid
0001:007dcd54  _EVP_MD_block_size
0001:007dcd5f  _EVP_MD_type
0001:007dcd69  _EVP_MD_pkey_type
0001:007dcd74  _EVP_MD_size
0001:007dcdbb* _EVP_MD_flags
0001:007dcdc6  _EVP_MD_CTX_md
0001:007dcddd  _EVP_MD_CTX_set_flags
0001:007dcdf3  _EVP_MD_CTX_clear_flags
0001:007dce0b  _EVP_MD_CTX_test_flags
0001:007dce1b* _EVP_CIPHER_CTX_set_flags
0001:007dce31* _EVP_CIPHER_CTX_clear_flags
0001:007dce49* _EVP_CIPHER_CTX_test_flags
Module: U:\extras\lib\libcrypto.lib(c_zlib.obj)
0001:007dce68  _COMP_zlib
0001:007dce7a* _COMP_zlib_cleanup
Module: U:\extras\lib\libcrypto.lib(e_null.obj)
0001:007dceb4  _EVP_enc_null
Module: U:\extras\lib\libcrypto.lib(x509_vfy.obj)
0001:007dcf00* _X509_version
0001:007dcf3c  _X509_verify_cert
0001:007dfc85* _X509_get_pubkey_parameters
0001:007df8bb* _X509_cmp_time
0001:007e0202  _X509_STORE_CTX_init
0001:007e0783* _X509_STORE_CTX_set0_param
0001:007e05f1  _X509_STORE_CTX_cleanup
0001:007df8a0* _X509_cmp_current_time
0001:007dfbac* _X509_time_adj
0001:007dfb8a  _X509_gmtime_adj
0001:007dfbd5* _X509_time_adj_ex
0001:007dfdfd  _X509_STORE_CTX_get_ex_new_index
0001:007dfe34  _X509_STORE_CTX_set_ex_data
0001:007dfe5b* _X509_STORE_CTX_get_ex_data
0001:007dfe7b* _X509_STORE_CTX_get_error
0001:007dfe86* _X509_STORE_CTX_set_error
0001:007dfe94* _X509_STORE_CTX_get_error_depth
0001:007dfe9f* _X509_STORE_CTX_get_current_cert
0001:007dfeaa* _X509_STORE_CTX_get_chain
0001:007dfeb5* _X509_STORE_CTX_get1_chain
0001:007dff47* _X509_STORE_CTX_get0_current_issuer
0001:007dff52* _X509_STORE_CTX_get0_current_crl
0001:007dff5d* _X509_STORE_CTX_get0_parent_ctx
0001:007dff68* _X509_STORE_CTX_set_cert
0001:007dff76* _X509_STORE_CTX_set_chain
0001:007dff84* _X509_STORE_CTX_set0_crls
0001:007dff92  _X509_STORE_CTX_set_purpose
0001:007dffe6* _X509_STORE_CTX_purpose_inherit
0001:007dffbc* _X509_STORE_CTX_set_trust
0001:007e015e* _X509_STORE_CTX_new
0001:007e01dc* _X509_STORE_CTX_free
0001:007e05d9* _X509_STORE_CTX_trusted_stack
0001:007e06c5* _X509_STORE_CTX_set_depth
0001:007e06e2* _X509_STORE_CTX_set_flags
0001:007e06ff* _X509_STORE_CTX_set_time
0001:007e071c  _X509_STORE_CTX_set_verify_cb
0001:007e072a* _X509_STORE_CTX_get0_policy_tree
0001:007e0735* _X509_STORE_CTX_get_explicit_policy
0001:007e0740  _X509_STORE_CTX_set_default
0001:007e0778  _X509_STORE_CTX_get0_param
Module: U:\extras\lib\libcrypto.lib(dh_asn1.obj)
0001:007e0880* _DHparams_it
0001:007e089c  _d2i_DHparams
0001:007e08c5  _i2d_DHparams
0001:007e08e7  _DHparams_dup
Module: U:\extras\lib\libcrypto.lib(bn_lib.obj)
0001:007e0910* _BN_version
0001:007e093e* _BN_set_params
0001:007e0a05* _BN_get_params
0001:007e0a43  _BN_value_one
0001:007e0a57* _BN_options
0001:007e0aa4  _BN_num_bits_word
0001:007e0b15  _BN_num_bits
0001:007e0b5f  _BN_clear_free
0001:007e0be1  _BN_free
0001:007e0c49  _BN_init
0001:007e0c75  _BN_new
0001:007e0ec7* _bn_dup_expand
0001:007e0fb2  _BN_dup
0001:007e0f53  _bn_expand2
0001:007e1007  _BN_copy
0001:007e1140* _BN_swap
0001:007e11fa  _BN_clear
0001:007e1245* _BN_get_word
0001:007e1275  _BN_set_word
0001:007e12dc  _BN_bin2bn
0001:007e144b  _BN_bn2bin
0001:007e14d2  _BN_ucmp
0001:007e155e  _BN_cmp
0001:007e1674  _BN_set_bit
0001:007e176c* _BN_clear_bit
0001:007e1841  _BN_is_bit_set
0001:007e18ae  _BN_mask_bits
0001:007e19a3  _BN_set_negative
0001:007e19ce  _bn_cmp_words
0001:007e1a65  _bn_cmp_part_words
Module: U:\extras\lib\libcrypto.lib(ec_key.obj)
0001:007e1c29  _EC_KEY_new
0001:007e1cdb* _EC_KEY_new_by_curve_name
0001:007e1d28  _EC_KEY_free
0001:007e1deb* _EC_KEY_copy
0001:007e2036  _EC_KEY_dup
0001:007e207e  _EC_KEY_up_ref
0001:007e20c1  _EC_KEY_generate_key
0001:007e22aa* _EC_KEY_check_key
0001:007e2631  _EC_KEY_get0_group
0001:007e263c  _EC_KEY_set_group
0001:007e267b  _EC_KEY_get0_private_key
0001:007e2686  _EC_KEY_set_private_key
0001:007e26c5  _EC_KEY_get0_public_key
0001:007e26d0  _EC_KEY_set_public_key
0001:007e2719  _EC_KEY_get_enc_flags
0001:007e2724  _EC_KEY_set_enc_flags
0001:007e2732  _EC_KEY_get_conv_form
0001:007e273d* _EC_KEY_set_conv_form
0001:007e276d  _EC_KEY_get_key_method_data
0001:007e2798  _EC_KEY_insert_key_method_data
0001:007e283e* _EC_KEY_set_asn1_flag
0001:007e2865* _EC_KEY_precompute_mult
Module: U:\extras\lib\libcrypto.lib(bss_file.obj)
0001:007e28c7  _BIO_new_file
0001:007e2a7f  _BIO_s_file
0001:007e2a23  _BIO_new_fp
Module: U:\extras\lib\libcrypto.lib(pem_x509.obj)
0001:007e30fc  _PEM_read_bio_X509
0001:007e3135* _PEM_read_X509
0001:007e316e  _PEM_write_bio_X509
0001:007e31c1* _PEM_write_X509
Module: U:\extras\lib\libcrypto.lib(o_dir.obj)
0001:007e3220  _OPENSSL_DIR_read
0001:007e3238  _OPENSSL_DIR_end
Module: U:\extras\lib\libcrypto.lib(a_object.obj)
0001:007e3250* _i2d_ASN1_OBJECT
0001:007e3319  _a2d_ASN1_OBJECT
0001:007e37b0  _i2t_ASN1_OBJECT
0001:007e37e8  _i2a_ASN1_OBJECT
0001:007e38e3  _d2i_ASN1_OBJECT
0001:007e39a9  _c2i_ASN1_OBJECT
0001:007e3bb2  _ASN1_OBJECT_new
0001:007e3c50  _ASN1_OBJECT_free
0001:007e3d06  _ASN1_OBJECT_create
Module: U:\extras\lib\libcrypto.lib(x509_trs.obj)
0001:007e3dbc* _X509_TRUST_set_default
0001:007e3dd7  _X509_check_trust
0001:007e3eb7  _X509_TRUST_get_by_id
0001:007e3e70* _X509_TRUST_get0
0001:007e3e48* _X509_TRUST_get_count
0001:007e3f1c  _X509_TRUST_set
0001:007e3f74* _X509_TRUST_add
0001:007e41b3* _X509_TRUST_cleanup
0001:007e4206* _X509_TRUST_get_flags
0001:007e4211* _X509_TRUST_get0_name
0001:007e421c* _X509_TRUST_get_trust
Module: U:\extras\lib\libcrypto.lib(obj_lib.obj)
0001:007e43da  _OBJ_dup
0001:007e4647  _OBJ_cmp
Module: U:\extras\lib\libcrypto.lib(tasn_typ.obj)
0001:007e46b0  _ASN1_INTEGER_it
0001:007e46cc  _d2i_ASN1_INTEGER
0001:007e46f5  _i2d_ASN1_INTEGER
0001:007e4717  _ASN1_INTEGER_new
0001:007e472b  _ASN1_INTEGER_free
0001:007e4760  _ASN1_ENUMERATED_it
0001:007e477c  _d2i_ASN1_ENUMERATED
0001:007e47a5* _i2d_ASN1_ENUMERATED
0001:007e47c7* _ASN1_ENUMERATED_new
0001:007e47db  _ASN1_ENUMERATED_free
0001:007e4810  _ASN1_BIT_STRING_it
0001:007e482c  _d2i_ASN1_BIT_STRING
0001:007e4855  _i2d_ASN1_BIT_STRING
0001:007e4877  _ASN1_BIT_STRING_new
0001:007e488b  _ASN1_BIT_STRING_free
0001:007e48c0  _ASN1_OCTET_STRING_it
0001:007e48dc  _d2i_ASN1_OCTET_STRING
0001:007e4905  _i2d_ASN1_OCTET_STRING
0001:007e4927  _ASN1_OCTET_STRING_new
0001:007e493b  _ASN1_OCTET_STRING_free
0001:007e4960  _ASN1_NULL_it
0001:007e497c* _d2i_ASN1_NULL
0001:007e49a5* _i2d_ASN1_NULL
0001:007e49c7  _ASN1_NULL_new
0001:007e49db* _ASN1_NULL_free
0001:007e4a10  _ASN1_OBJECT_it
0001:007e4a40  _ASN1_UTF8STRING_it
0001:007e4a5c* _d2i_ASN1_UTF8STRING
0001:007e4a85* _i2d_ASN1_UTF8STRING
0001:007e4aa7  _ASN1_UTF8STRING_new
0001:007e4abb  _ASN1_UTF8STRING_free
0001:007e4af0* _ASN1_PRINTABLESTRING_it
0001:007e4b0c* _d2i_ASN1_PRINTABLESTRING
0001:007e4b35* _i2d_ASN1_PRINTABLESTRING
0001:007e4b57* _ASN1_PRINTABLESTRING_new
0001:007e4b6b* _ASN1_PRINTABLESTRING_free
0001:007e4ba0* _ASN1_T61STRING_it
0001:007e4bbc* _d2i_ASN1_T61STRING
0001:007e4be5* _i2d_ASN1_T61STRING
0001:007e4c07* _ASN1_T61STRING_new
0001:007e4c1b* _ASN1_T61STRING_free
0001:007e4c50  _ASN1_IA5STRING_it
0001:007e4c6c* _d2i_ASN1_IA5STRING
0001:007e4c95* _i2d_ASN1_IA5STRING
0001:007e4cb7* _ASN1_IA5STRING_new
0001:007e4ccb* _ASN1_IA5STRING_free
0001:007e4d00* _ASN1_GENERALSTRING_it
0001:007e4d1c* _d2i_ASN1_GENERALSTRING
0001:007e4d45* _i2d_ASN1_GENERALSTRING
0001:007e4d67* _ASN1_GENERALSTRING_new
0001:007e4d7b* _ASN1_GENERALSTRING_free
0001:007e4db0* _ASN1_UTCTIME_it
0001:007e4dcc* _d2i_ASN1_UTCTIME
0001:007e4df5* _i2d_ASN1_UTCTIME
0001:007e4e17* _ASN1_UTCTIME_new
0001:007e4e2b* _ASN1_UTCTIME_free
0001:007e4e60  _ASN1_GENERALIZEDTIME_it
0001:007e4e7c* _d2i_ASN1_GENERALIZEDTIME
0001:007e4ea5* _i2d_ASN1_GENERALIZEDTIME
0001:007e4ec7  _ASN1_GENERALIZEDTIME_new
0001:007e4edb* _ASN1_GENERALIZEDTIME_free
0001:007e4f10* _ASN1_VISIBLESTRING_it
0001:007e4f2c* _d2i_ASN1_VISIBLESTRING
0001:007e4f55* _i2d_ASN1_VISIBLESTRING
0001:007e4f77* _ASN1_VISIBLESTRING_new
0001:007e4f8b* _ASN1_VISIBLESTRING_free
0001:007e4fc0* _ASN1_UNIVERSALSTRING_it
0001:007e4fdc* _d2i_ASN1_UNIVERSALSTRING
0001:007e5005* _i2d_ASN1_UNIVERSALSTRING
0001:007e5027* _ASN1_UNIVERSALSTRING_new
0001:007e503b* _ASN1_UNIVERSALSTRING_free
0001:007e5070* _ASN1_BMPSTRING_it
0001:007e508c* _d2i_ASN1_BMPSTRING
0001:007e50b5* _i2d_ASN1_BMPSTRING
0001:007e50d7* _ASN1_BMPSTRING_new
0001:007e50eb* _ASN1_BMPSTRING_free
0001:007e5110  _ASN1_ANY_it
0001:007e5140  _ASN1_SEQUENCE_it
0001:007e515c  _d2i_ASN1_TYPE
0001:007e5185  _i2d_ASN1_TYPE
0001:007e51a7  _ASN1_TYPE_new
0001:007e51bb  _ASN1_TYPE_free
0001:007e51f0  _ASN1_PRINTABLE_it
0001:007e520c* _d2i_ASN1_PRINTABLE
0001:007e5235* _i2d_ASN1_PRINTABLE
0001:007e5257* _ASN1_PRINTABLE_new
0001:007e526b* _ASN1_PRINTABLE_free
0001:007e52a0  _DISPLAYTEXT_it
0001:007e52bc* _d2i_DISPLAYTEXT
0001:007e52e5* _i2d_DISPLAYTEXT
0001:007e5307* _DISPLAYTEXT_new
0001:007e531b* _DISPLAYTEXT_free
0001:007e5350  _DIRECTORYSTRING_it
0001:007e536c* _d2i_DIRECTORYSTRING
0001:007e5395* _i2d_DIRECTORYSTRING
0001:007e53b7* _DIRECTORYSTRING_new
0001:007e53cb* _DIRECTORYSTRING_free
0001:007e5400  _ASN1_BOOLEAN_it
0001:007e5430* _ASN1_TBOOLEAN_it
0001:007e5460  _ASN1_FBOOLEAN_it
0001:007e54a0  _ASN1_OCTET_STRING_NDEF_it
0001:007e54f0* _ASN1_SEQUENCE_ANY_it
0001:007e5540* _ASN1_SET_ANY_it
0001:007e555c  _d2i_ASN1_SEQUENCE_ANY
0001:007e5585  _i2d_ASN1_SEQUENCE_ANY
0001:007e55a7* _d2i_ASN1_SET_ANY
0001:007e55d0  _i2d_ASN1_SET_ANY
Module: U:\extras\lib\libcrypto.lib(tasn_dec.obj)
0001:007e5680  _ASN1_tag2bit
0001:007e56a2  _ASN1_item_d2i
0001:007e576b  _ASN1_item_ex_d2i
0001:007e5710* _ASN1_template_d2i
0001:007e6f94* _asn1_ex_c2i
Module: U:\extras\lib\libcrypto.lib(tasn_enc.obj)
0001:007e7af0  _ASN1_item_ndef_i2d
0001:007e7b19  _ASN1_item_i2d
0001:007e7c34  _ASN1_item_ex_i2d
0001:007e815c* _ASN1_template_i2d
0001:007e8941* _asn1_ex_i2c
Module: U:\extras\lib\libcrypto.lib(tasn_new.obj)
0001:007e8be0  _ASN1_item_new
0001:007e8c0f  _ASN1_item_ex_new
0001:007e915c* _ASN1_template_new
0001:007e9272* _ASN1_primitive_new
Module: U:\extras\lib\libcrypto.lib(tasn_fre.obj)
0001:007e9460  _ASN1_item_free
0001:007e9482  _ASN1_item_ex_free
0001:007e9833  _ASN1_template_free
0001:007e98d9  _ASN1_primitive_free
Module: U:\extras\lib\libcrypto.lib(a_dup.obj)
0001:007e9a28  _ASN1_dup
0001:007e9afc  _ASN1_item_dup
Module: U:\extras\lib\libcrypto.lib(x_algor.obj)
0001:007e9c10  _X509_ALGOR_it
0001:007e9c60  _X509_ALGORS_it
0001:007e9c7c  _d2i_X509_ALGOR
0001:007e9ca5* _i2d_X509_ALGOR
0001:007e9cc7  _X509_ALGOR_new
0001:007e9cdb  _X509_ALGOR_free
0001:007e9cf6* _d2i_X509_ALGORS
0001:007e9d1f  _i2d_X509_ALGORS
0001:007e9d41* _X509_ALGOR_dup
0001:007e9d5c  _X509_ALGOR_set0
0001:007e9e1c  _X509_ALGOR_get0
Module: U:\extras\lib\libcrypto.lib(v3_genn.obj)
0001:007e9ec0* _OTHERNAME_it
0001:007e9edc* _d2i_OTHERNAME
0001:007e9f05* _i2d_OTHERNAME
0001:007e9f27  _OTHERNAME_new
0001:007e9f3b* _OTHERNAME_free
0001:007e9fb0* _EDIPARTYNAME_it
0001:007e9fcc* _d2i_EDIPARTYNAME
0001:007e9ff5* _i2d_EDIPARTYNAME
0001:007ea017* _EDIPARTYNAME_new
0001:007ea02b* _EDIPARTYNAME_free
0001:007ea1a0  _GENERAL_NAME_it
0001:007ea1bc* _d2i_GENERAL_NAME
0001:007ea1e5* _i2d_GENERAL_NAME
0001:007ea207  _GENERAL_NAME_new
0001:007ea21b  _GENERAL_NAME_free
0001:007ea280  _GENERAL_NAMES_it
0001:007ea29c* _d2i_GENERAL_NAMES
0001:007ea2c5* _i2d_GENERAL_NAMES
0001:007ea2e7  _GENERAL_NAMES_new
0001:007ea2fb  _GENERAL_NAMES_free
0001:007ea316* _GENERAL_NAME_dup
0001:007ea33b  _GENERAL_NAME_cmp
0001:007ea45c* _OTHERNAME_cmp
0001:007ea4c0* _GENERAL_NAME_set0_value
0001:007ea546* _GENERAL_NAME_get0_value
0001:007ea5c7* _GENERAL_NAME_set0_othername
0001:007ea614* _GENERAL_NAME_get0_otherName
Module: U:\extras\lib\libcrypto.lib(v3_info.obj)
0001:007ea660  _v3_info
0001:007ea810* _AUTHORITY_INFO_ACCESS_it
0001:007ea6a0  _v3_sinfo
0001:007ea730  _ACCESS_DESCRIPTION_it
0001:007ea74c* _d2i_ACCESS_DESCRIPTION
0001:007ea775* _i2d_ACCESS_DESCRIPTION
0001:007ea797* _ACCESS_DESCRIPTION_new
0001:007ea7ab* _ACCESS_DESCRIPTION_free
0001:007ea82c* _d2i_AUTHORITY_INFO_ACCESS
0001:007ea855* _i2d_AUTHORITY_INFO_ACCESS
0001:007ea877* _AUTHORITY_INFO_ACCESS_new
0001:007ea88b  _AUTHORITY_INFO_ACCESS_free
0001:007eacf6* _i2a_ACCESS_DESCRIPTION
Module: U:\extras\lib\libcrypto.lib(a_strex.obj)
0001:007ebbcb  _X509_NAME_print_ex
0001:007ebc1c* _X509_NAME_print_ex_fp
0001:007ebca1  _ASN1_STRING_print_ex
0001:007ebcca* _ASN1_STRING_print_ex_fp
0001:007ebcf3  _ASN1_STRING_to_UTF8
Module: U:\extras\lib\libcrypto.lib(asn1_lib.obj)
0001:007ebdc0* _ASN1_version
0001:007ebe31* _ASN1_check_infinite_end
0001:007ebe4b  _ASN1_const_check_infinite_end
0001:007ebe70  _ASN1_get_object
0001:007ec132  _ASN1_put_object
0001:007ec232  _ASN1_put_eoc
0001:007ec2e5  _ASN1_object_size
0001:007ec3bf* _asn1_Finish
0001:007ec3d2  _asn1_const_Finish
0001:007ec3e5  _asn1_GetSequence
0001:007ec4ea  _ASN1_STRING_copy
0001:007ec59a  _ASN1_STRING_set
0001:007ec545  _ASN1_STRING_dup
0001:007ec6f9  _ASN1_STRING_new
0001:007ec796  _ASN1_STRING_free
0001:007ec6c8  _ASN1_STRING_set0
0001:007ec70d  _ASN1_STRING_type_new
0001:007ec7d7  _ASN1_STRING_cmp
0001:007ec859  _asn1_add_error
0001:007ec8cf* _ASN1_STRING_length
0001:007ec8d9* _ASN1_STRING_length_set
0001:007ec8e6* _ASN1_STRING_type
0001:007ec8f1  _ASN1_STRING_data
Module: U:\extras\lib\libcrypto.lib(x509_obj.obj)
0001:007ec918  _X509_NAME_oneline
Module: U:\extras\lib\libcrypto.lib(m_md5.obj)
0001:007ece0c  _EVP_md5
Module: U:\extras\lib\libcrypto.lib(m_sha1.obj)
0001:007ececc  _EVP_sha1
0001:007ecf9c* _EVP_sha224
0001:007ecffc  _EVP_sha256
0001:007ed0cc* _EVP_sha384
0001:007ed12c* _EVP_sha512
Module: U:\extras\lib\libcrypto.lib(x_pubkey.obj)
0001:007ed1e0  _X509_PUBKEY_it
0001:007ed1fc* _d2i_X509_PUBKEY
0001:007ed225* _i2d_X509_PUBKEY
0001:007ed247* _X509_PUBKEY_new
0001:007ed25b* _X509_PUBKEY_free
0001:007ed281  _X509_PUBKEY_set
0001:007ed3b6  _X509_PUBKEY_get
0001:007ed590  _d2i_PUBKEY
0001:007ed606  _i2d_PUBKEY
0001:007ed662  _d2i_RSA_PUBKEY
0001:007ed6e8  _i2d_RSA_PUBKEY
0001:007ed773  _d2i_DSA_PUBKEY
0001:007ed7f9  _i2d_DSA_PUBKEY
0001:007ed884  _d2i_EC_PUBKEY
0001:007ed90a  _i2d_EC_PUBKEY
0001:007ed995  _X509_PUBKEY_set0_param
0001:007eda34  _X509_PUBKEY_get0_param
Module: U:\extras\lib\libssl.lib(d1_pkt.obj)
0001:007ee2e1* _dtls1_get_record
0001:007ee6b5* _dtls1_read_bytes
0001:007eff94* _dtls1_reset_seq_numbers
0001:007ef56b* _dtls1_write_app_data_bytes
0001:007ef72c  _dtls1_write_bytes
0001:007ef793* _do_dtls1_write
0001:007efd4e* _dtls1_dispatch_alert
Module: U:\extras\lib\libcrypto.lib(pqueue.obj)
0001:007f00b9  _pitem_new
0001:007f011d  _pitem_free
0001:007f0139  _pqueue_new
0001:007f018b  _pqueue_free
0001:007f01a7  _pqueue_insert
0001:007f025b  _pqueue_peek
0001:007f0265  _pqueue_pop
0001:007f028e  _pqueue_find
0001:007f034b* _pqueue_print
0001:007f03fb  _pqueue_iterator
0001:007f040e  _pqueue_next
0001:007f0444  _pqueue_size
Module: U:\extras\lib\libssl.lib(d1_lib.obj)
0001:007f0480* _dtls1_version_str
0001:007f04ca* _dtls1_default_timeout
0001:007f04dd* _dtls1_new
0001:007f085d* _dtls1_free
0001:007f08ed* _dtls1_clear
0001:007f0a57* _dtls1_ctrl
0001:007f0bc4* _dtls1_get_timeout
0001:007f0e07  _dtls1_handle_timeout
0001:007f0ef3* _dtls1_listen
0001:007f0ae7* _dtls1_get_cipher
0001:007f0b18* _dtls1_start_timer
0001:007f0cfc  _dtls1_is_timer_expired
0001:007f0d3b* _dtls1_double_timeout
0001:007f0d8a* _dtls1_stop_timer
0002:00006f70* _DTLSv1_enc_data
Module: U:\extras\lib\libcrypto.lib(x_crl.obj)
0001:007f1000* _X509_REVOKED_it
0001:007f1160  _X509_CRL_INFO_it
0001:007f1860  _X509_CRL_it
0001:007f187c* _d2i_X509_REVOKED
0001:007f18a5* _i2d_X509_REVOKED
0001:007f18c7* _X509_REVOKED_new
0001:007f18db* _X509_REVOKED_free
0001:007f18f6* _d2i_X509_CRL_INFO
0001:007f191f* _i2d_X509_CRL_INFO
0001:007f1941* _X509_CRL_INFO_new
0001:007f1955* _X509_CRL_INFO_free
0001:007f1970  _d2i_X509_CRL
0001:007f1999  _i2d_X509_CRL
0001:007f19bb* _X509_CRL_new
0001:007f19cf  _X509_CRL_free
0001:007f19ea* _X509_CRL_dup
0001:007f1a2f* _X509_CRL_add0_revoked
0001:007f1ac3  _X509_CRL_verify
0001:007f1af7* _X509_CRL_get0_by_serial
0001:007f1b3a  _X509_CRL_get0_by_cert
0001:007f1dde* _X509_CRL_set_default_method
0001:007f1dfd* _X509_CRL_METHOD_new
0001:007f1e61* _X509_CRL_METHOD_free
0001:007f1e83* _X509_CRL_set_meth_data
0001:007f1e91* _X509_CRL_get_meth_data
Module: U:\extras\lib\libcrypto.lib(o_names.obj)
0001:007f1edf* _OBJ_NAME_init
0001:007f1f3f* _OBJ_NAME_new_index
0001:007f21ce  _OBJ_NAME_get
0001:007f2279  _OBJ_NAME_add
0001:007f239e* _OBJ_NAME_remove
0001:007f24af  _OBJ_NAME_do_all
0001:007f2556  _OBJ_NAME_do_all_sorted
0001:007f267a  _OBJ_NAME_cleanup
Module: U:\extras\lib\libcrypto.lib(evp_pbe.obj)
0001:007f28b5  _EVP_PBE_CipherInit
0001:007f2cd6  _EVP_PBE_find
0001:007f2bac* _EVP_PBE_alg_add_type
0001:007f2c6c* _EVP_PBE_alg_add
0001:007f2dba  _EVP_PBE_cleanup
Module: U:\extras\lib\libcrypto.lib(tb_rand.obj)
0001:007f2df4* _ENGINE_unregister_RAND
0001:007f2e23* _ENGINE_register_RAND
0001:007f2e6f* _ENGINE_register_all_RAND
0001:007f2ea0* _ENGINE_set_default_RAND
0001:007f2eec  _ENGINE_get_default_RAND
0001:007f2f09  _ENGINE_get_RAND
0001:007f2f14* _ENGINE_set_RAND
Module: U:\extras\lib\libcrypto.lib(md_rand.obj)
0001:007f2f30* _RAND_version
0001:007f2f58  _RAND_SSLeay
0002:00006fe0* _rand_ssleay_meth
Module: U:\extras\lib\libcrypto.lib(x_val.obj)
0001:007f3bf0  _X509_VAL_it
0001:007f3c0c* _d2i_X509_VAL
0001:007f3c35* _i2d_X509_VAL
0001:007f3c57* _X509_VAL_new
0001:007f3c6b* _X509_VAL_free
Module: U:\extras\lib\libcrypto.lib(x_x509a.obj)
0001:007f3d30* _X509_CERT_AUX_it
0001:007f3d4c  _d2i_X509_CERT_AUX
0001:007f3d75  _i2d_X509_CERT_AUX
0001:007f3d97* _X509_CERT_AUX_new
0001:007f3dab  _X509_CERT_AUX_free
0001:007f3e07* _X509_alias_set1
0001:007f3ebe* _X509_keyid_set1
0001:007f3f75* _X509_alias_get0
0001:007f3fba* _X509_keyid_get0
0001:007f3fff* _X509_add1_trust_object
0001:007f4076* _X509_add1_reject_object
0001:007f40f1* _X509_trust_clear
0001:007f4134* _X509_reject_clear
0001:007f41d0* _X509_CERT_PAIR_it
0001:007f41ec  _d2i_X509_CERT_PAIR
0001:007f4215  _i2d_X509_CERT_PAIR
0001:007f4237* _X509_CERT_PAIR_new
0001:007f424b* _X509_CERT_PAIR_free
Module: U:\extras\lib\libcrypto.lib(v3_akeya.obj)
0001:007f42e0  _AUTHORITY_KEYID_it
0001:007f42fc* _d2i_AUTHORITY_KEYID
0001:007f4325* _i2d_AUTHORITY_KEYID
0001:007f4347  _AUTHORITY_KEYID_new
0001:007f435b  _AUTHORITY_KEYID_free
Module: U:\extras\lib\libcrypto.lib(v3_crld.obj)
0001:007f4380  _v3_crld
0001:007f50f0* _CRL_DIST_POINTS_it
0001:007f43c0  _v3_freshest_crl
0001:007f4f87* _DIST_POINT_NAME_new
0001:007f5077* _DIST_POINT_new
0001:007f508b* _DIST_POINT_free
0001:007f4f20* _DIST_POINT_NAME_it
0001:007f4f3c* _d2i_DIST_POINT_NAME
0001:007f4f65* _i2d_DIST_POINT_NAME
0001:007f4f9b* _DIST_POINT_NAME_free
0001:007f5010* _DIST_POINT_it
0001:007f502c* _d2i_DIST_POINT
0001:007f5055* _i2d_DIST_POINT
0001:007f510c* _d2i_CRL_DIST_POINTS
0001:007f5135* _i2d_CRL_DIST_POINTS
0001:007f5157* _CRL_DIST_POINTS_new
0001:007f516b  _CRL_DIST_POINTS_free
0001:007f5250* _ISSUING_DIST_POINT_it
0001:007f526c* _d2i_ISSUING_DIST_POINT
0001:007f5295* _i2d_ISSUING_DIST_POINT
0001:007f52b7* _ISSUING_DIST_POINT_new
0001:007f52cb  _ISSUING_DIST_POINT_free
0001:007f52f0  _v3_idp
0001:007f5a2a  _DIST_POINT_set_dpname
Module: U:\extras\lib\libcrypto.lib(pcy_cache.obj)
0001:007f5f60  _policy_cache_free
0001:007f5fb3  _policy_cache_set
0001:007f601e  _policy_cache_find_data
Module: U:\extras\lib\libcrypto.lib(v3_ncons.obj)
0001:007f60d0  _v3_name_constraints
0001:007f61f0* _NAME_CONSTRAINTS_it
0001:007f6170* _GENERAL_SUBTREE_it
0001:007f620c* _GENERAL_SUBTREE_new
0001:007f6220* _GENERAL_SUBTREE_free
0001:007f623b* _NAME_CONSTRAINTS_new
0001:007f624f  _NAME_CONSTRAINTS_free
0001:007f67a8  _NAME_CONSTRAINTS_check
Module: U:\extras\lib\libcrypto.lib(eng_lib.obj)
0001:007f6eaa  _ENGINE_new
0001:007f6f4f* _engine_set_all_null
0001:007f6ffd  _engine_free_util
0001:007f70fa  _ENGINE_free
0001:007f7190  _engine_cleanup_add_first
0001:007f71db  _engine_cleanup_add_last
0001:007f7238* _ENGINE_cleanup
0001:007f727c* _ENGINE_get_ex_new_index
0001:007f72b3* _ENGINE_set_ex_data
0001:007f72d7* _ENGINE_get_ex_data
0001:007f72f4* _ENGINE_set_id
0001:007f7342* _ENGINE_set_name
0001:007f7391* _ENGINE_set_destroy_function
0001:007f73a4* _ENGINE_set_init_function
0001:007f73b7* _ENGINE_set_finish_function
0001:007f73ca* _ENGINE_set_ctrl_function
0001:007f73dd* _ENGINE_set_flags
0001:007f73f0* _ENGINE_set_cmd_defns
0001:007f7403* _ENGINE_get_id
0001:007f740d* _ENGINE_get_name
0001:007f7418* _ENGINE_get_destroy_function
0001:007f7423* _ENGINE_get_init_function
0001:007f742e* _ENGINE_get_finish_function
0001:007f7439* _ENGINE_get_ctrl_function
0001:007f7444* _ENGINE_get_flags
0001:007f744f* _ENGINE_get_cmd_defns
0001:007f745a* _ENGINE_get_static_state
Module: U:\extras\lib\libcrypto.lib(rsa_eay.obj)
0001:007f7488  _RSA_PKCS1_SSLeay
Module: U:\extras\lib\libcrypto.lib(tb_rsa.obj)
0001:007f9544* _ENGINE_unregister_RSA
0001:007f9573* _ENGINE_register_RSA
0001:007f95bf* _ENGINE_register_all_RSA
0001:007f95f0* _ENGINE_set_default_RSA
0001:007f963c  _ENGINE_get_default_RSA
0001:007f9659  _ENGINE_get_RSA
0001:007f9664* _ENGINE_set_RSA
Module: U:\extras\lib\libcrypto.lib(bn_blind.obj)
0001:007f968b* _BN_BLINDING_new
0001:007f97c7  _BN_BLINDING_free
0001:007f9841* _BN_BLINDING_update
0001:007f9be4  _BN_BLINDING_create_param
0001:007f99bc* _BN_BLINDING_convert
0001:007f99e5  _BN_BLINDING_convert_ex
0001:007f9ad1* _BN_BLINDING_invert
0001:007f9afa  _BN_BLINDING_invert_ex
0001:007f9ba7* _BN_BLINDING_get_thread_id
0001:007f9bb2* _BN_BLINDING_set_thread_id
0001:007f9bc0  _BN_BLINDING_thread_id
0001:007f9bcb* _BN_BLINDING_get_flags
0001:007f9bd6* _BN_BLINDING_set_flags
Module: U:\extras\lib\libcrypto.lib(bn_ctx.obj)
0001:007f9e50* _BN_CTX_init
0001:007f9e98  _BN_CTX_new
0001:007f9f32  _BN_CTX_free
0001:007f9f67  _BN_CTX_start
0001:007f9feb  _BN_CTX_end
0001:007fa057  _BN_CTX_get
Module: U:\extras\lib\libcrypto.lib(bn_add.obj)
0001:007fa530  _BN_add
0001:007fa799  _BN_usub
0001:007fa60b  _BN_uadd
0001:007fa9b2  _BN_sub
Module: U:\extras\lib\libcrypto.lib(bn_mul.obj)
0001:007fab20* _bn_sub_part_words
0001:007fae64* _bn_add_part_words
0001:007fb2ac* _bn_mul_recursive
0001:007fcf6c* _bn_mul_normal
0001:007fb9da* _bn_mul_part_recursive
0001:007fc1fa* _bn_mul_low_recursive
0001:007fd10f* _bn_mul_low_normal
0001:007fc3db* _bn_mul_high
0001:007fcb0e  _BN_mul
Module: U:\extras\lib\libcrypto.lib(bn_gcd.obj)
0001:007fd220  _BN_gcd
0001:007fd510  _BN_mod_inverse
Module: U:\extras\lib\libcrypto.lib(dh_key.obj)
0001:007fe180  _DH_generate_key
0001:007fe199  _DH_compute_key
0001:007fe1d2  _DH_OpenSSL
Module: U:\extras\lib\libcrypto.lib(tb_dh.obj)
0001:007fe774* _ENGINE_unregister_DH
0001:007fe7a3* _ENGINE_register_DH
0001:007fe7ef* _ENGINE_register_all_DH
0001:007fe820* _ENGINE_set_default_DH
0001:007fe86c  _ENGINE_get_default_DH
0001:007fe889  _ENGINE_get_DH
0001:007fe894* _ENGINE_set_DH
Module: U:\extras\lib\libcrypto.lib(dsa_lib.obj)
0001:007fe8b0* _DSA_version
0001:007fe8d7* _DSA_set_default_method
0001:007fe8e4* _DSA_get_default_method
0001:007fe904  _DSA_new
0001:007fe993* _DSA_new_method
0001:007fe918* _DSA_set_method
0001:007febf3  _DSA_free
0001:007fed4c  _DSA_up_ref
0001:007fed8f  _DSA_size
0001:007fee0b* _DSA_get_ex_new_index
0001:007fee42* _DSA_set_ex_data
0001:007fee66* _DSA_get_ex_data
0001:007fee83* _DSA_dup_DH
Module: U:\extras\lib\libcrypto.lib(x_attrib.obj)
0001:007ff000* _X509_ATTRIBUTE_SET_it
0001:007ff060  _X509_ATTRIBUTE_it
0001:007ff07c* _d2i_X509_ATTRIBUTE
0001:007ff0a5* _i2d_X509_ATTRIBUTE
0001:007ff0c7  _X509_ATTRIBUTE_new
0001:007ff0db  _X509_ATTRIBUTE_free
0001:007ff0f6  _X509_ATTRIBUTE_dup
0001:007ff111  _X509_ATTRIBUTE_create
Module: U:\extras\lib\libcrypto.lib(x509_v3.obj)
0001:007ff1f0  _X509v3_get_ext_count
0001:007ff210  _X509v3_get_ext_by_NID
0001:007ff24c  _X509v3_get_ext_by_OBJ
0001:007ff2c3  _X509v3_get_ext_by_critical
0001:007ff342  _X509v3_get_ext
0001:007ff37f  _X509v3_delete_ext
0001:007ff3cc  _X509v3_add_ext
0001:007ff502  _X509_EXTENSION_create_by_NID
0001:007ff588  _X509_EXTENSION_create_by_OBJ
0001:007ff673* _X509_EXTENSION_set_object
0001:007ff6b0* _X509_EXTENSION_set_critical
0001:007ff6df* _X509_EXTENSION_set_data
0001:007ff72a  _X509_EXTENSION_get_object
0001:007ff741  _X509_EXTENSION_get_data
0001:007ff759  _X509_EXTENSION_get_critical
Module: U:\extras\lib\libcrypto.lib(x509_ext.obj)
0001:007ff790* _X509_CRL_get_ext_count
0001:007ff7a8  _X509_CRL_get_ext_by_NID
0001:007ff7ce* _X509_CRL_get_ext_by_OBJ
0001:007ff7f4* _X509_CRL_get_ext_by_critical
0001:007ff81a  _X509_CRL_get_ext
0001:007ff839* _X509_CRL_delete_ext
0001:007ff858  _X509_CRL_get_ext_d2i
0001:007ff885* _X509_CRL_add1_ext_i2d
0001:007ff8b9* _X509_CRL_add_ext
0001:007ff8e7  _X509_get_ext_count
0001:007ff8ff  _X509_get_ext_by_NID
0001:007ff925* _X509_get_ext_by_OBJ
0001:007ff94b* _X509_get_ext_by_critical
0001:007ff971  _X509_get_ext
0001:007ff990* _X509_delete_ext
0001:007ff9af* _X509_add_ext
0001:007ff9dd  _X509_get_ext_d2i
0001:007ffa0a* _X509_add1_ext_i2d
0001:007ffa3e* _X509_REVOKED_get_ext_count
0001:007ffa54* _X509_REVOKED_get_ext_by_NID
0001:007ffa78* _X509_REVOKED_get_ext_by_OBJ
0001:007ffa9c* _X509_REVOKED_get_ext_by_critical
0001:007ffac0* _X509_REVOKED_get_ext
0001:007ffadd* _X509_REVOKED_delete_ext
0001:007ffafa* _X509_REVOKED_add_ext
0001:007ffb26  _X509_REVOKED_get_ext_d2i
0001:007ffb51* _X509_REVOKED_add1_ext_i2d
Module: U:\extras\lib\libcrypto.lib(x_all.obj)
0001:007ffb90  _X509_verify
0001:007ffbcd* _X509_REQ_verify
0001:007ffc0a* _NETSCAPE_SPKI_verify
0001:007ffc47* _X509_sign
0001:007ffca5  _X509_REQ_sign
0001:007ffcf1* _X509_CRL_sign
0001:007ffd4f* _NETSCAPE_SPKI_sign
0001:007ffd9b* _d2i_X509_fp
0001:007ffdbd* _i2d_X509_fp
0001:007ffddf  _d2i_X509_bio
0001:007ffe01* _i2d_X509_bio
0001:007ffe23* _d2i_X509_CRL_fp
0001:007ffe45* _i2d_X509_CRL_fp
0001:007ffe67  _d2i_X509_CRL_bio
0001:007ffe89* _i2d_X509_CRL_bio
0001:007ffeab* _d2i_PKCS7_fp
0001:007ffecd* _i2d_PKCS7_fp
0001:007ffeef* _d2i_PKCS7_bio
0001:007fff11* _i2d_PKCS7_bio
0001:007fff33* _d2i_X509_REQ_fp
0001:007fff55* _i2d_X509_REQ_fp
0001:007fff77* _d2i_X509_REQ_bio
0001:007fff99* _i2d_X509_REQ_bio
0001:007fffbb* _d2i_RSAPrivateKey_fp
0001:007fffdd* _i2d_RSAPrivateKey_fp
0001:007fffff* _d2i_RSAPublicKey_fp
0001:00800021* _d2i_RSA_PUBKEY_fp
0001:0080004d* _i2d_RSAPublicKey_fp
0001:0080006f* _i2d_RSA_PUBKEY_fp
0001:00800092  _d2i_RSAPrivateKey_bio
0001:008000b4* _i2d_RSAPrivateKey_bio
0001:008000d6* _d2i_RSAPublicKey_bio
0001:008000f8* _d2i_RSA_PUBKEY_bio
0001:00800124* _i2d_RSAPublicKey_bio
0001:00800146* _i2d_RSA_PUBKEY_bio
0001:00800169* _d2i_DSAPrivateKey_fp
0001:00800195* _i2d_DSAPrivateKey_fp
0001:008001b8* _d2i_DSA_PUBKEY_fp
0001:008001e4* _i2d_DSA_PUBKEY_fp
0001:00800207* _d2i_DSAPrivateKey_bio
0001:00800233* _i2d_DSAPrivateKey_bio
0001:00800256* _d2i_DSA_PUBKEY_bio
0001:00800282* _i2d_DSA_PUBKEY_bio
0001:008002a5* _d2i_EC_PUBKEY_fp
0001:008002d1* _i2d_EC_PUBKEY_fp
0001:008002f4* _d2i_ECPrivateKey_fp
0001:00800320* _i2d_ECPrivateKey_fp
0001:00800343* _d2i_EC_PUBKEY_bio
0001:0080036f* _i2d_EC_PUBKEY_bio
0001:00800392* _d2i_ECPrivateKey_bio
0001:008003be* _i2d_ECPrivateKey_bio
0001:008003e1* _X509_pubkey_digest
0001:0080043a  _X509_digest
0001:0080046a  _X509_CRL_digest
0001:0080049a* _X509_REQ_digest
0001:008004ca* _X509_NAME_digest
0001:008004fa* _PKCS7_ISSUER_AND_SERIAL_digest
0001:0080052a* _d2i_PKCS8_fp
0001:00800556* _i2d_PKCS8_fp
0001:00800579  _d2i_PKCS8_bio
0001:008005a5  _i2d_PKCS8_bio
0001:008005c8* _d2i_PKCS8_PRIV_KEY_INFO_fp
0001:008005f4* _i2d_PKCS8_PRIV_KEY_INFO_fp
0001:00800617* _i2d_PKCS8PrivateKeyInfo_fp
0001:0080065d* _i2d_PrivateKey_fp
0001:00800680* _d2i_PrivateKey_fp
0001:008006ac* _i2d_PUBKEY_fp
0001:008006cf* _d2i_PUBKEY_fp
0001:008006fb* _d2i_PKCS8_PRIV_KEY_INFO_bio
0001:00800727  _i2d_PKCS8_PRIV_KEY_INFO_bio
0001:0080074a* _i2d_PKCS8PrivateKeyInfo_bio
0001:00800790* _i2d_PrivateKey_bio
0001:008007b3  _d2i_PrivateKey_bio
0001:008007df* _i2d_PUBKEY_bio
0001:00800802* _d2i_PUBKEY_bio
Module: U:\extras\lib\libcrypto.lib(a_int.obj)
0001:00800830* _ASN1_INTEGER_dup
0001:00800843  _ASN1_INTEGER_cmp
0001:008008a2  _i2c_ASN1_INTEGER
0001:00800a74  _c2i_ASN1_INTEGER
0001:00800ca6  _d2i_ASN1_UINTEGER
0001:00800e72  _ASN1_INTEGER_set
0001:00800fae  _ASN1_INTEGER_get
0001:00801058  _BN_to_ASN1_INTEGER
0001:008011c9  _ASN1_INTEGER_to_BN
Module: U:\extras\lib\libcrypto.lib(v3_bcons.obj)
0001:00801250  _v3_bcons
0001:008012e0* _BASIC_CONSTRAINTS_it
0001:008012fc* _d2i_BASIC_CONSTRAINTS
0001:00801325* _i2d_BASIC_CONSTRAINTS
0001:00801347* _BASIC_CONSTRAINTS_new
0001:0080135b  _BASIC_CONSTRAINTS_free
Module: U:\extras\lib\libcrypto.lib(v3_pcia.obj)
0001:008015c0* _PROXY_POLICY_it
0001:008015dc* _d2i_PROXY_POLICY
0001:00801605* _i2d_PROXY_POLICY
0001:00801627* _PROXY_POLICY_new
0001:0080163b* _PROXY_POLICY_free
0001:008016d0  _PROXY_CERT_INFO_EXTENSION_it
0001:008016ec* _d2i_PROXY_CERT_INFO_EXTENSION
0001:00801715* _i2d_PROXY_CERT_INFO_EXTENSION
0001:00801737  _PROXY_CERT_INFO_EXTENSION_new
0001:0080174b  _PROXY_CERT_INFO_EXTENSION_free
Module: U:\extras\lib\libcrypto.lib(a_octet.obj)
0001:00801770  _ASN1_OCTET_STRING_dup
0001:00801783  _ASN1_OCTET_STRING_cmp
0001:0080179d  _ASN1_OCTET_STRING_set
Module: U:\extras\lib\libcrypto.lib(bn_word.obj)
0001:008017c0  _BN_mod_word
0001:00801844  _BN_div_word
0001:00801964  _BN_add_word
0001:00801abc  _BN_sub_word
0001:00801c36  _BN_mul_word
Module: U:\extras\lib\libcrypto.lib(bn_shift.obj)
0001:00801d10  _BN_lshift1
0001:00801e2a  _BN_rshift1
0001:00801f6b  _BN_lshift
0001:00802150  _BN_rshift
Module: U:\extras\lib\libcrypto.lib(bn_print.obj)
0001:008023bc* _BN_bn2hex
0001:008024f0  _BN_bn2dec
0001:00802773  _BN_hex2bn
0001:008029e8  _BN_dec2bn
0001:00802c1a  _BN_asc2bn
0001:00802ca9* _BN_print_fp
0001:00802d17* _BN_print
Module: U:\extras\lib\libcrypto.lib(tb_cipher.obj)
0001:00802e20* _ENGINE_unregister_ciphers
0001:00802e4f* _ENGINE_register_ciphers
0001:00802ec7* _ENGINE_register_all_ciphers
0001:00802ef8* _ENGINE_set_default_ciphers
0001:00802f70  _ENGINE_get_cipher_engine
0001:00802f97  _ENGINE_get_cipher
0001:0080300e* _ENGINE_get_ciphers
0001:00803019* _ENGINE_set_ciphers
Module: U:\extras\lib\libcrypto.lib(by_file.obj)
0001:00803045  _X509_LOOKUP_file
0001:008035d8* _X509_load_cert_crl_file
0001:0080316a  _X509_load_cert_file
0001:008033a0  _X509_load_crl_file
0002:00007070* _x509_file_lookup
Module: U:\extras\lib\libcrypto.lib(by_dir.obj)
0001:00803785  _X509_LOOKUP_hash_dir
0002:000070a0* _x509_dir_lookup
Module: U:\extras\lib\libcrypto.lib(tb_digest.obj)
0001:00804220* _ENGINE_unregister_digests
0001:0080424f* _ENGINE_register_digests
0001:008042c7* _ENGINE_register_all_digests
0001:008042f8* _ENGINE_set_default_digests
0001:00804370  _ENGINE_get_digest_engine
0001:00804397  _ENGINE_get_digest
0001:0080440e* _ENGINE_get_digests
0001:00804419* _ENGINE_set_digests
Module: U:\extras\lib\libcrypto.lib(pmeth_lib.obj)
0001:008044a0* _EVP_PKEY_meth_find
0001:00804b0b  _EVP_PKEY_CTX_free
0001:00804757* _EVP_PKEY_meth_new
0001:008048a1  _EVP_PKEY_meth_free
0001:008048c7  _EVP_PKEY_CTX_new
0001:008048e9  _EVP_PKEY_CTX_new_id
0001:0080490b  _EVP_PKEY_CTX_dup
0001:00804aa7* _EVP_PKEY_meth_add0
0001:00804b94  _EVP_PKEY_CTX_ctrl
0001:00804cf3* _EVP_PKEY_CTX_ctrl_str
0001:00804e06* _EVP_PKEY_CTX_get_operation
0001:00804e11* _EVP_PKEY_CTX_set0_keygen_info
0001:00804e28* _EVP_PKEY_CTX_set_data
0001:00804e36* _EVP_PKEY_CTX_get_data
0001:00804e41* _EVP_PKEY_CTX_get0_pkey
0001:00804e4c* _EVP_PKEY_CTX_get0_peerkey
0001:00804e57* _EVP_PKEY_CTX_set_app_data
0001:00804e65* _EVP_PKEY_CTX_get_app_data
0001:00804e70* _EVP_PKEY_meth_set_init
0001:00804e7e* _EVP_PKEY_meth_set_copy
0001:00804e8c* _EVP_PKEY_meth_set_cleanup
0001:00804e9a* _EVP_PKEY_meth_set_paramgen
0001:00804eb1* _EVP_PKEY_meth_set_keygen
0001:00804ec8* _EVP_PKEY_meth_set_sign
0001:00804edf* _EVP_PKEY_meth_set_verify
0001:00804ef6* _EVP_PKEY_meth_set_verify_recover
0001:00804f0d* _EVP_PKEY_meth_set_signctx
0001:00804f24* _EVP_PKEY_meth_set_verifyctx
0001:00804f3b* _EVP_PKEY_meth_set_encrypt
0001:00804f52* _EVP_PKEY_meth_set_decrypt
0001:00804f69* _EVP_PKEY_meth_set_derive
0001:00804f80* _EVP_PKEY_meth_set_ctrl
0002:0001fb40* _app_pkey_methods
Module: U:\extras\lib\libssl.lib(s2_enc.obj)
0001:00805016  _ssl2_enc_init
0001:00805335  _ssl2_enc
0001:008053ca  _ssl2_mac
Module: U:\extras\lib\libssl.lib(s2_pkt.obj)
0001:00805b9e  _ssl2_read
0001:00805bc7  _ssl2_peek
0001:00805ec8  _ssl2_write
0001:0080657a  _ssl2_part_read
0001:00806656  _ssl2_do_write
Module: U:\extras\lib\libssl.lib(ssl_rsa.obj)
0001:0080679a  _SSL_use_certificate
0001:0080683a* _SSL_use_certificate_file
0001:008069f3* _SSL_use_certificate_ASN1
0001:00806a74* _SSL_use_RSAPrivateKey
0001:00806d2a* _SSL_use_RSAPrivateKey_file
0001:00806edd* _SSL_use_RSAPrivateKey_ASN1
0001:00806f64  _SSL_use_PrivateKey
0001:0080700a* _SSL_use_PrivateKey_file
0001:008071bd* _SSL_use_PrivateKey_ASN1
0001:0080724b* _SSL_CTX_use_certificate
0001:008074db* _SSL_CTX_use_certificate_file
0001:00807688* _SSL_CTX_use_certificate_ASN1
0001:00807709* _SSL_CTX_use_RSAPrivateKey
0001:00807826* _SSL_CTX_use_RSAPrivateKey_file
0001:008079cd* _SSL_CTX_use_RSAPrivateKey_ASN1
0001:00807a54* _SSL_CTX_use_PrivateKey
0001:00807af4* _SSL_CTX_use_PrivateKey_file
0001:00807c9b* _SSL_CTX_use_PrivateKey_ASN1
0001:00807d29* _SSL_CTX_use_certificate_chain_file
Module: U:\extras\lib\libcrypto.lib(p_sign.obj)
0001:00807f79  _EVP_SignFinal
Module: U:\extras\lib\libcrypto.lib(ec_curve.obj)
0001:0080c2f3  _EC_GROUP_new_by_curve_name
0001:0080c3a8* _EC_get_builtin_curves
Module: U:\extras\lib\libcrypto.lib(ec_lib.obj)
0001:0080c45f  _EC_GROUP_new
0001:0080c5cf  _EC_GROUP_free
0001:0080d567  _EC_EX_DATA_free_all_data
0001:0080d720  _EC_POINT_free
0001:0080c665  _EC_GROUP_clear_free
0001:0080d5bb* _EC_EX_DATA_clear_free_all_data
0001:0080d758  _EC_POINT_clear_free
0001:0080c744  _EC_GROUP_copy
0001:0080d312  _EC_EX_DATA_set_data
0001:0080d60f  _EC_POINT_new
0001:0080d7c1  _EC_POINT_copy
0001:0080ca41  _EC_GROUP_dup
0001:0080cac2  _EC_GROUP_method_of
0001:0080cacc  _EC_METHOD_get_field_type
0001:0080cad6  _EC_GROUP_set_generator
0001:0080cbe6  _EC_GROUP_get0_generator
0001:0080cbf1  _EC_GROUP_get_order
0001:0080cc27  _EC_GROUP_get_cofactor
0001:0080cc5d  _EC_GROUP_set_curve_name
0001:0080cc6b  _EC_GROUP_get_curve_name
0001:0080cc76  _EC_GROUP_set_asn1_flag
0001:0080cc84  _EC_GROUP_get_asn1_flag
0001:0080cc8f  _EC_GROUP_set_point_conversion_form
0001:0080cc9d  _EC_GROUP_get_point_conversion_form
0001:0080cca8  _EC_GROUP_set_seed
0001:0080cd4b  _EC_GROUP_get0_seed
0001:0080cd56  _EC_GROUP_get_seed_len
0001:0080cd61  _EC_GROUP_set_curve_GFp
0001:0080cdd4  _EC_GROUP_get_curve_GFp
0001:0080ce47  _EC_GROUP_set_curve_GF2m
0001:0080ceba  _EC_GROUP_get_curve_GF2m
0001:0080cf2d  _EC_GROUP_get_degree
0001:0080cf84* _EC_GROUP_check_discriminant
0001:0080cfe2  _EC_GROUP_cmp
0001:0080e40e  _EC_POINT_cmp
0001:0080d40d  _EC_EX_DATA_get_data
0001:0080d459  _EC_EX_DATA_free_data
0001:0080d4e0* _EC_EX_DATA_clear_free_data
0001:0080d86f  _EC_POINT_dup
0001:0080d8cf* _EC_POINT_method_of
0001:0080d8d9  _EC_POINT_set_to_infinity
0001:0080d978  _EC_POINT_set_Jprojective_coordinates_GFp
0001:0080da33* _EC_POINT_get_Jprojective_coordinates_GFp
0001:0080daee  _EC_POINT_set_affine_coordinates_GFp
0001:0080dba2  _EC_POINT_set_affine_coordinates_GF2m
0001:0080dc56  _EC_POINT_get_affine_coordinates_GFp
0001:0080dd0a  _EC_POINT_get_affine_coordinates_GF2m
0001:0080ddbe  _EC_POINT_set_compressed_coordinates_GFp
0001:0080de72  _EC_POINT_set_compressed_coordinates_GF2m
0001:0080df26  _EC_POINT_point2oct
0001:0080dfe1  _EC_POINT_oct2point
0001:0080e095  _EC_POINT_add
0001:0080e168  _EC_POINT_dbl
0001:0080e223  _EC_POINT_invert
0001:0080e2c9  _EC_POINT_is_at_infinity
0001:0080e368  _EC_POINT_is_on_curve
0001:0080e4c9  _EC_POINT_make_affine
0001:0080e56f  _EC_POINTs_make_affine
0001:0080e63b* _EC_POINTs_mul
0001:0080e6c0  _EC_POINT_mul
0001:0080e71e  _EC_GROUP_precompute_mult
0001:0080e770  _EC_GROUP_have_precompute_mult
Module: U:\extras\lib\libcrypto.lib(rsa_sign.obj)
0001:0080e7cb  _RSA_sign
0001:0080eadd  _int_rsa_verify
0001:0080ef59  _RSA_verify
Module: U:\extras\lib\libcrypto.lib(m_dss1.obj)
0001:0080f09c  _EVP_dss1
Module: U:\extras\lib\libcrypto.lib(p_verify.obj)
0001:0080f0bb  _EVP_VerifyFinal
Module: U:\extras\lib\libcrypto.lib(m_ecdsa.obj)
0001:0080f38c  _EVP_ecdsa
Module: U:\extras\lib\libcrypto.lib(ech_key.obj)
0001:0080f3a0  _ECDH_compute_key
Module: U:\extras\lib\libcrypto.lib(pmeth_fn.obj)
0001:0080f3fb  _EVP_PKEY_sign_init
0001:0080f494  _EVP_PKEY_sign
0001:0080f5cc  _EVP_PKEY_verify_init
0001:0080f665  _EVP_PKEY_verify
0001:0080f725* _EVP_PKEY_verify_recover_init
0001:0080f7be* _EVP_PKEY_verify_recover
0001:0080f8f6  _EVP_PKEY_encrypt_init
0001:0080f98f  _EVP_PKEY_encrypt
0001:0080fac9  _EVP_PKEY_decrypt_init
0001:0080fb62  _EVP_PKEY_decrypt
0001:0080fc9c* _EVP_PKEY_derive_init
0001:0080fd35  _EVP_PKEY_derive_set_peer
0001:0080ffcf* _EVP_PKEY_derive
Module: U:\extras\lib\libcrypto.lib(dsa_sign.obj)
0001:00810100* _DSA_do_sign
0001:00810127  _DSA_sign
0001:0081019c  _DSA_sign_setup
Module: U:\extras\lib\libcrypto.lib(ecs_sign.obj)
0001:008101d0* _ECDSA_do_sign
0001:00810201* _ECDSA_do_sign_ex
0001:00810251  _ECDSA_sign
0001:00810297* _ECDSA_sign_ex
0001:0081031a  _ECDSA_sign_setup
Module: U:\extras\lib\libcrypto.lib(x509type.obj)
0001:00810370  _X509_certificate_type
Module: U:\extras\lib\libcrypto.lib(bss_mem.obj)
0001:008104ae  _BIO_s_mem
0001:008104c2  _BIO_new_mem_buf
Module: U:\extras\lib\libcrypto.lib(rsa_asn1.obj)
0001:00810c50  _RSAPrivateKey_it
0001:00810cc0  _RSAPublicKey_it
0001:00810cdc  _d2i_RSAPrivateKey
0001:00810d05  _i2d_RSAPrivateKey
0001:00810d27  _d2i_RSAPublicKey
0001:00810d50  _i2d_RSAPublicKey
0001:00810d72* _RSAPublicKey_dup
0001:00810d8d  _RSAPrivateKey_dup
Module: U:\extras\lib\libssl.lib(t1_enc.obj)
0001:008114e8  _tls1_change_cipher_state
0001:00811d48  _tls1_setup_key_block
0001:00812018  _tls1_enc
0001:008123f4  _tls1_cert_verify_mac
0001:0081251b  _tls1_final_finish_mac
0001:00812733  _tls1_mac
0001:008129ed  _tls1_generate_master_secret
0001:00812abd  _tls1_alert_code
Module: U:\extras\lib\libssl.lib(t1_reneg.obj)
0001:00812dbb  _ssl_add_clienthello_renegotiate_ext
0001:00812e73  _ssl_parse_clienthello_renegotiate_ext
0001:00812fec  _ssl_add_serverhello_renegotiate_ext
0001:00813189  _ssl_parse_serverhello_renegotiate_ext
Module: U:\extras\lib\libcrypto.lib(hmac.obj)
0001:00813459  _HMAC_Init_ex
0001:0081370b* _HMAC_Init
0001:00813810  _HMAC_CTX_init
0001:00813752  _HMAC_Update
0001:00813776  _HMAC_Final
0001:00813842  _HMAC_CTX_copy
0001:008138e7  _HMAC_CTX_cleanup
0001:00813934  _HMAC
0001:008139e0  _HMAC_CTX_set_flags
Module: U:\extras\lib\libcrypto.lib(e_aes.obj)
0001:00813cc4  _EVP_aes_128_cbc
0001:00813d04* _EVP_aes_128_cfb128
0001:00813d44* _EVP_aes_128_ofb
0001:00813d84* _EVP_aes_128_ecb
0001:00814024* _EVP_aes_192_cbc
0001:00814064* _EVP_aes_192_cfb128
0001:008140a4* _EVP_aes_192_ofb
0001:008140e4* _EVP_aes_192_ecb
0001:00814384* _EVP_aes_256_cbc
0001:008143c4* _EVP_aes_256_cfb128
0001:00814404* _EVP_aes_256_ofb
0001:00814444* _EVP_aes_256_ecb
0001:00814544* _EVP_aes_128_cfb1
0001:00814644* _EVP_aes_192_cfb1
0001:00814744* _EVP_aes_256_cfb1
0001:00814824* _EVP_aes_128_cfb8
0001:00814904* _EVP_aes_192_cfb8
0001:008149e4* _EVP_aes_256_cfb8
Module: U:\extras\lib\xmlrpc.lib(encodings.obj)
0001:00814bfc  _utf8_decode
0001:00814c1e* _utf8_encode
Module: U:\extras\lib\expat.lib(xmlparse.obj)
0001:00814c73* _XML_UseParserAsHandlerArg
0001:00814c7e* _XML_UseForeignDTD
0001:00814ca8* _XML_SetReturnNSTriplet
0001:00814ccc  _XML_SetUserData
0001:00814ce7* _XML_GetBase
0001:00814cf5* _XML_GetSpecifiedAttributeCount
0001:00814d03* _XML_GetIdAttributeIndex
0001:00814d11  _XML_SetElementHandler
0001:00814d25* _XML_SetStartElementHandler
0001:00814d33* _XML_SetEndElementHandler
0001:00814d41  _XML_SetCharacterDataHandler
0001:00814d4f* _XML_SetProcessingInstructionHandler
0001:00814d5d* _XML_SetCommentHandler
0001:00814d6b* _XML_SetCdataSectionHandler
0001:00814d7f* _XML_SetStartCdataSectionHandler
0001:00814d8d* _XML_SetEndCdataSectionHandler
0001:00814d9b* _XML_SetDefaultHandler
0001:00814db0* _XML_SetDefaultHandlerExpand
0001:00814dc5* _XML_SetDoctypeDeclHandler
0001:00814dd9* _XML_SetStartDoctypeDeclHandler
0001:00814de7* _XML_SetEndDoctypeDeclHandler
0001:00814df5* _XML_SetUnparsedEntityDeclHandler
0001:00814e03* _XML_SetNotationDeclHandler
0001:00814e11* _XML_SetNamespaceDeclHandler
0001:00814e25* _XML_SetStartNamespaceDeclHandler
0001:00814e33* _XML_SetEndNamespaceDeclHandler
0001:00814e41* _XML_SetNotStandaloneHandler
0001:00814e4f* _XML_SetExternalEntityRefHandler
0001:00814e5d* _XML_SetExternalEntityRefHandlerArg
0001:00814e74* _XML_SetSkippedEntityHandler
0001:00814e82* _XML_SetUnknownEncodingHandler
0001:00814e99* _XML_SetElementDeclHandler
0001:00814eaa* _XML_SetAttlistDeclHandler
0001:00814ebb* _XML_SetEntityDeclHandler
0001:00814ecc* _XML_SetXmlDeclHandler
0001:00814edd* _XML_SetParamEntityParsing
0001:00814f07* _XML_SetHashSalt
0001:00814f31* _XML_StopParser
0001:00814fa8* _XML_ResumeParser
0001:00815091  _XML_GetErrorCode
0001:0081509f  _XML_GetCurrentByteIndex
0001:008150be  _XML_GetCurrentByteCount
0001:008150e0* _XML_GetInputContext
0001:00815111  _XML_GetCurrentLineNumber
0001:0081516a  _XML_GetCurrentColumnNumber
0001:008151c0* _XML_FreeContentModel
0001:008151d5* _XML_MemMalloc
0001:008151ea* _XML_MemRealloc
0001:00815205* _XML_MemFree
0001:0081521a  _XML_ErrorString
0001:0081523f* _XML_ExpatVersion
0001:00815249* _XML_ExpatVersionInfo
0001:00815267* _XML_GetFeatureList
0001:0081535f* _XML_DefaultCurrent
0001:00815b26  _XML_ParserFree
0001:00815f76* _XML_GetParsingStatus
0001:00815fbc* _XML_GetBuffer
0001:008165df* _XML_SetBase
0001:00816629* _XML_SetEncoding
0001:0081735f* _XML_ParseBuffer
0001:008174c8  _XML_Parse
0001:0081819f* _XML_ExternalEntityParserCreate
0001:00818832* _XML_ParserCreate_MM
0001:0081884e* _XML_ParserCreateNS
0001:00818876  _XML_ParserCreate
0001:00818899* _XML_ParserReset
Module: U:\extras\lib\xmlrpc.lib(base64.obj)
0001:0081e3b0  _buffer_delete
0001:0081e3e5* _buffer_add
0001:0081e436* _buffer_new
0001:0081e468  _base64_decode
0001:0081e5f2  _base64_encode
Module: U:\extras\lib\lzma.lib(liblzma_la-filter_common.obj)
0001:0081e780  _lzma_raw_coder_memusage
0001:0081e8f1  _lzma_raw_coder_init
0001:0081eb51* _lzma_filters_copy
Module: U:\extras\lib\lzma.lib(liblzma_la-lzma_decoder.obj)
0001:0081f0a6  _lzma_lzma_lclppb_decode
0001:0081f121  _lzma_lzma_decoder_create
0001:0081f211  _lzma_lzma_props_decode
0001:0081f296  _lzma_lzma_decoder_memusage_nocheck
0001:0081f2b3  _lzma_lzma_decoder_memusage
0001:0081f2e9  _lzma_lzma_decoder_init
Module: U:\extras\lib\lzma.lib(liblzma_la-lzma2_decoder.obj)
0001:00822d30  _lzma_lzma2_props_decode
0001:00822db3  _lzma_lzma2_decoder_memusage
0001:00822dce  _lzma_lzma2_decoder_init
Module: U:\extras\lib\lzma.lib(liblzma_la-x86.obj)
0001:00823457  _lzma_simple_x86_decoder_init
0001:008234bb* _lzma_simple_x86_encoder_init
Module: U:\extras\lib\lzma.lib(liblzma_la-simple_decoder.obj)
0001:00823550  _lzma_simple_props_decode
Module: U:\extras\lib\lzma.lib(liblzma_la-powerpc.obj)
0001:0082369e  _lzma_simple_powerpc_decoder_init
0001:008236e7* _lzma_simple_powerpc_encoder_init
Module: U:\extras\lib\lzma.lib(liblzma_la-ia64.obj)
0001:00823963  _lzma_simple_ia64_decoder_init
0001:008239ac* _lzma_simple_ia64_encoder_init
Module: U:\extras\lib\lzma.lib(liblzma_la-arm.obj)
0001:00823b1b  _lzma_simple_arm_decoder_init
0001:00823b64* _lzma_simple_arm_encoder_init
Module: U:\extras\lib\lzma.lib(liblzma_la-armthumb.obj)
0001:00823cab  _lzma_simple_armthumb_decoder_init
0001:00823cf4* _lzma_simple_armthumb_encoder_init
Module: U:\extras\lib\lzma.lib(liblzma_la-sparc.obj)
0001:00823e31  _lzma_simple_sparc_decoder_init
0001:00823e7a* _lzma_simple_sparc_encoder_init
Module: U:\extras\lib\lzma.lib(liblzma_la-delta_decoder.obj)
0001:00823f73  _lzma_delta_props_decode
0001:00823fbf  _lzma_delta_decoder_init
Module: U:\extras\lib\lzma.lib(liblzma_la-delta_common.obj)
0001:00823fe0  _lzma_delta_coder_memusage
0001:00824014  _lzma_delta_coder_init
Module: U:\extras\lib\lzma.lib(liblzma_la-alone_decoder.obj)
0001:00824168  _lzma_alone_decoder_init
0001:00824254* _lzma_alone_decoder
Module: U:\extras\lib\lzma.lib(liblzma_la-stream_decoder.obj)
0001:008245de  _lzma_stream_decoder_init
0001:00824763* _lzma_stream_decoder
Module: U:\extras\lib\pthread.lib(my_os2tls.obj)
0002:00022370+ _tls_bits
0001:00824e56  _TlsAlloc
0001:008251c8* _TlsAllocThreadLocalMemory
0001:00824f95  _TlsFree
0001:00825044  _TlsGetValue
0001:008250a8  _TlsSetValue
0001:008252fa* _TlsFreeThreadLocalMemory
0002:0001fb90* _tls_storage
0002:0001fb94* _tls_mutex
Module: U:\extras\lib\libcrypto.lib(evp_key.obj)
0001:00825390* _EVP_set_pw_prompt
0001:008253c9  _EVP_get_pw_prompt
0001:008253e3* _EVP_read_pw_string
0001:00825413  _EVP_read_pw_string_min
0001:00825536  _EVP_BytesToKey
Module: U:\extras\lib\libcrypto.lib(encode.obj)
0001:00825850  _EVP_EncodeInit
0001:008258a7  _EVP_EncodeUpdate
0001:00825ace  _EVP_EncodeBlock
0001:00825a69  _EVP_EncodeFinal
0001:00825c12  _EVP_DecodeInit
0001:00825c5f  _EVP_DecodeUpdate
0001:00825f09  _EVP_DecodeBlock
0001:00826085  _EVP_DecodeFinal
Module: U:\extras\lib\libcrypto.lib(rsa_ameth.obj)
0001:00826b00  _rsa_asn1_meths
Module: U:\extras\lib\libcrypto.lib(dh_ameth.obj)
0001:00827947* _DHparams_print
0001:008279a0  _dh_asn1_meth
Module: U:\extras\lib\libcrypto.lib(dsa_ameth.obj)
0001:00828cc0  _dsa_asn1_meths
Module: U:\extras\lib\libcrypto.lib(ec_ameth.obj)
0001:0082a210  _eckey_asn1_meth
Module: U:\extras\lib\libcrypto.lib(hm_ameth.obj)
0001:0082a400  _hmac_asn1_meth
Module: U:\extras\lib\libcrypto.lib(tb_asnmth.obj)
0001:0082a460* _ENGINE_unregister_pkey_asn1_meths
0001:0082a48f* _ENGINE_register_pkey_asn1_meths
0001:0082a507* _ENGINE_register_all_pkey_asn1_meths
0001:0082a538* _ENGINE_set_default_pkey_asn1_meths
0001:0082a5b0  _ENGINE_get_pkey_asn1_meth_engine
0001:0082a5d7  _ENGINE_get_pkey_asn1_meth
0001:0082a64e* _ENGINE_get_pkey_asn1_meths
0001:0082a659* _ENGINE_set_pkey_asn1_meths
0001:0082a66c  _engine_pkey_asn1_meths_free
0001:0082a6f7* _ENGINE_get_pkey_asn1_meth_str
0001:0082a89e  _ENGINE_pkey_asn1_find_str
Module: U:\extras\lib\libcrypto.lib(evp_asn1.obj)
0001:0082a940  _ASN1_TYPE_set_octetstring
0001:0082a9b2  _ASN1_TYPE_get_octetstring
0001:0082aa4a* _ASN1_TYPE_set_int_octetstring
0001:0082abb7* _ASN1_TYPE_get_int_octetstring
Module: U:\extras\lib\libcrypto.lib(pcy_tree.obj)
0001:0082bb32  _X509_policy_tree_free
0001:0082bc17  _X509_policy_check
Module: U:\extras\lib\libcrypto.lib(a_utctm.obj)
0001:0082bde0  _ASN1_UTCTIME_check
0001:0082c028* _ASN1_UTCTIME_set_string
0001:0082c09a* _ASN1_UTCTIME_set
0001:0082c0e8  _ASN1_UTCTIME_adj
0001:0082c2bb* _ASN1_UTCTIME_cmp_time_t
Module: U:\extras\lib\libcrypto.lib(a_gentm.obj)
0001:0082c700  _ASN1_GENERALIZEDTIME_check
0001:0082c9a0* _ASN1_GENERALIZEDTIME_set_string
0001:0082ca12* _ASN1_GENERALIZEDTIME_set
0001:0082ca60  _ASN1_GENERALIZEDTIME_adj
Module: U:\extras\lib\libcrypto.lib(a_time.obj)
0001:0082cc80  _ASN1_TIME_it
0001:0082cc9c* _d2i_ASN1_TIME
0001:0082ccc5* _i2d_ASN1_TIME
0001:0082cce7* _ASN1_TIME_new
0001:0082ccfb  _ASN1_TIME_free
0001:0082cd16* _ASN1_TIME_set
0001:0082cd49  _ASN1_TIME_adj
0001:0082ce2c  _ASN1_TIME_check
0001:0082ce6f* _ASN1_TIME_to_generalizedtime
0001:0082cfb0* _ASN1_TIME_set_string
Module: U:\extras\lib\libcrypto.lib(x_bignum.obj)
0001:0082d040  _BIGNUM_it
0001:0082d060  _CBIGNUM_it
Module: U:\extras\lib\libcrypto.lib(x_long.obj)
0001:0082d1f0  _LONG_it
0001:0082d220  _ZLONG_it
Module: U:\extras\lib\libcrypto.lib(bn_rand.obj)
0001:0082d752  _BN_rand
0001:0082d782  _BN_pseudo_rand
0001:0082d7b2* _BN_bntest_rand
0001:0082da40  _BN_rand_range
0001:0082da62  _BN_pseudo_rand_range
Module: U:\extras\lib\libcrypto.lib(tasn_utl.obj)
0001:0082da90  _asn1_get_choice_selector
0001:0082dab0  _asn1_set_choice_selector
0001:0082dae9  _asn1_do_lock
0001:0082dbd9  _asn1_enc_init
0001:0082dc19  _asn1_enc_free
0001:0082dc6f  _asn1_enc_save
0001:0082dd14  _asn1_enc_restore
0001:0082dd98  _asn1_get_field_ptr
0001:0082ddc9  _asn1_do_adb
Module: U:\extras\lib\libcrypto.lib(a_type.obj)
0001:0082dee0  _ASN1_TYPE_get
0001:0082df05  _ASN1_TYPE_set
0001:0082df61  _ASN1_TYPE_set1
0001:0082e00b  _ASN1_TYPE_cmp
Module: U:\extras\lib\libcrypto.lib(a_bitstr.obj)
0001:0082e090  _ASN1_BIT_STRING_set
0001:0082e0b1  _i2c_ASN1_BIT_STRING
0001:0082e271  _c2i_ASN1_BIT_STRING
0001:0082e43d  _ASN1_BIT_STRING_set_bit
0001:0082e61f  _ASN1_BIT_STRING_get_bit
0001:0082e694* _ASN1_BIT_STRING_check
Module: U:\extras\lib\libcrypto.lib(v3_alt.obj)
0001:0082e710  _v3_alt
0001:0082e7b8  _i2v_GENERAL_NAMES
0001:0082e895  _i2v_GENERAL_NAME
0001:0082ec20  _GENERAL_NAME_print
0001:0082f5c9  _v2i_GENERAL_NAME
0001:0082f4f2  _v2i_GENERAL_NAMES
0001:0082f975  _v2i_GENERAL_NAME_ex
0001:0082f601* _a2i_GENERAL_NAME
Module: U:\extras\lib\libcrypto.lib(a_utf8.obj)
0001:0082fd50  _UTF8_getc
0001:00830200  _UTF8_putc
Module: U:\extras\lib\libcrypto.lib(asn1_par.obj)
0001:0083126e  _ASN1_tag2str
0001:0083065e* _ASN1_parse
0001:0083069e  _ASN1_parse_dump
Module: U:\extras\lib\libcrypto.lib(x509name.obj)
0001:00831490* _X509_NAME_get_text_by_NID
0001:008314d3* _X509_NAME_get_text_by_OBJ
0001:008315c7* _X509_NAME_get_index_by_OBJ
0001:00831646  _X509_NAME_get_entry
0001:00831e01  _X509_NAME_ENTRY_get_data
0001:00831569  _X509_NAME_entry_count
0001:0083158b  _X509_NAME_get_index_by_NID
0001:00831687  _X509_NAME_delete_entry
0001:00831776* _X509_NAME_add_entry_by_OBJ
0001:00831bd2* _X509_NAME_ENTRY_create_by_OBJ
0001:008318d4  _X509_NAME_add_entry
0001:008317e7* _X509_NAME_add_entry_by_NID
0001:00831b4b* _X509_NAME_ENTRY_create_by_NID
0001:00831858  _X509_NAME_add_entry_by_txt
0001:00831aa1* _X509_NAME_ENTRY_create_by_txt
0001:00831c86* _X509_NAME_ENTRY_set_object
0001:00831cf7* _X509_NAME_ENTRY_set_data
0001:00831dea  _X509_NAME_ENTRY_get_object
Module: U:\extras\lib\libcrypto.lib(t_x509.obj)
0001:00831e20* _X509_print_fp
0001:00831e53* _X509_print_ex_fp
0001:00832091* _X509_print_ex
0001:00831ef7* _X509_print
0001:00832b9d* _ASN1_TIME_print
0001:0083297a* _X509_signature_print
0001:0083276c* _X509_ocspid_print
0001:00832a9d  _ASN1_STRING_print
0001:00832fd1  _ASN1_UTCTIME_print
0001:00832c57  _ASN1_GENERALIZEDTIME_print
0001:00833269  _X509_NAME_print
Module: U:\extras\lib\libcrypto.lib(a_mbstr.obj)
0001:008333e0  _ASN1_mbstring_copy
0001:0083343f  _ASN1_mbstring_ncopy
Module: U:\extras\lib\libcrypto.lib(md5_dgst.obj)
0001:00833e00  _MD5_Update
0001:008341a6* _md5_block_data_order
0001:00833fb7* _MD5_Transform
0001:00833fd9  _MD5_Final
0001:00834130* _MD5_version
0001:00834157  _MD5_Init
Module: U:\extras\lib\libcrypto.lib(sha1dgst.obj)
0001:00834e40* _SHA1_version
0001:00834e68  _SHA1_Update
0001:0083501f* _SHA1_Transform
0001:00835041  _SHA1_Final
0001:0083520f  _SHA1_Init
Module: U:\extras\lib\libcrypto.lib(sha256.obj)
0001:008379d0* _SHA256_version
0001:008379fb  _SHA224_Init
0001:00837a7c  _SHA256_Init
0001:00837afd* _SHA224
0001:00837c00  _SHA256_Update
0001:00837dd9  _SHA256_Final
0001:00837b61* _SHA256
0001:00837bc5* _SHA224_Update
0001:00837be6* _SHA224_Final
0001:00837db7* _SHA256_Transform
Module: U:\extras\lib\libcrypto.lib(sha512.obj)
0001:0083a400* _SHA512_version
0001:0083a42b  _SHA384_Init
0001:0083a4f8  _SHA512_Init
0001:0083a5c5  _SHA512_Final
0001:0083a9d7* _SHA384_Final
0001:0083a9f1  _SHA512_Update
0001:0083abaa* _SHA384_Update
0001:0083abcb* _SHA512_Transform
0001:0083abed* _SHA384
0001:0083ac5d* _SHA512
Module: U:\extras\lib\libssl.lib(d1_enc.obj)
0001:0083b8f5  _dtls1_enc
Module: U:\extras\lib\libcrypto.lib(a_enum.obj)
0001:0083bd19* _ASN1_ENUMERATED_set
0001:0083be55  _ASN1_ENUMERATED_get
0001:0083beff* _BN_to_ASN1_ENUMERATED
0001:0083c055  _ASN1_ENUMERATED_to_BN
Module: U:\extras\lib\libcrypto.lib(a_verify.obj)
0001:0083c0eb* _ASN1_verify
0001:0083c2b1  _ASN1_item_verify
Module: U:\extras\lib\libcrypto.lib(p5_crpt.obj)
0001:0083c520* _PKCS5_PBE_add
0001:0083c58b  _PKCS5_PBE_keyivgen
Module: U:\extras\lib\libcrypto.lib(p12_crpt.obj)
0001:0083c900* _PKCS12_PBE_add
0001:0083c910  _PKCS12_PBE_keyivgen
Module: U:\extras\lib\libcrypto.lib(p5_crpt2.obj)
0001:0083cba0* _PKCS5_PBKDF2_HMAC
0001:0083cd8d* _PKCS5_PBKDF2_HMAC_SHA1
0001:0083cdf3  _PKCS5_v2_PBE_keyivgen
Module: U:\extras\lib\libcrypto.lib(eng_table.obj)
0001:0083d330* _ENGINE_get_table_flags
0001:0083d33a* _ENGINE_set_table_flags
0001:0083d407  _engine_table_register
0001:0083d6c8  _engine_table_unregister
0001:0083d7a5  _engine_table_cleanup
0001:0083d829  _engine_table_select
0001:0083da4b  _engine_table_doall
Module: U:\extras\lib\libcrypto.lib(eng_list.obj)
0001:0083e0f2* _ENGINE_remove
0001:0083dd83  _ENGINE_get_first
0001:0083ddf3* _ENGINE_get_last
0001:0083de63  _ENGINE_get_next
0001:0083df1f* _ENGINE_get_prev
0001:0083dfdb* _ENGINE_add
0001:0083e308* _ENGINE_by_id
0001:0083e573* _ENGINE_up_ref
Module: U:\extras\lib\libcrypto.lib(rand_os2.obj)
0001:0083e60b  _RAND_poll
Module: U:\extras\lib\libcrypto.lib(v3_conf.obj)
0001:0083ea21* _X509V3_EXT_nconf
0001:0083eb0d* _X509V3_EXT_nconf_nid
0001:0083efcf  _X509V3_EXT_i2d
0001:0083f3ad* _X509V3_EXT_add_nconf_sk
0001:0083f475* _X509V3_EXT_add_nconf
0001:0083f4b5* _X509V3_EXT_CRL_add_nconf
0001:0083f4f5* _X509V3_EXT_REQ_add_nconf
0001:0083f577* _X509V3_get_string
0001:0083f606  _X509V3_get_section
0001:0083f691* _X509V3_string_free
0001:0083f6ca  _X509V3_section_free
0001:0083f73e  _X509V3_set_nconf
0001:0083f756* _X509V3_set_ctx
0001:0083f787* _X509V3_EXT_conf
0001:0083f7c1* _X509V3_EXT_conf_nid
0001:0083f836* _X509V3_set_conf_lhash
0001:0083f84e* _X509V3_EXT_add_conf
0001:0083f888* _X509V3_EXT_CRL_add_conf
0001:0083f8c2* _X509V3_EXT_REQ_add_conf
Module: U:\extras\lib\libcrypto.lib(v3_utl.obj)
0001:0083f991  _X509V3_add_value
0001:0083fad8  _X509V3_add_value_uchar
0001:0083faf9  _X509V3_conf_free
0001:0083fb66  _X509V3_add_value_bool
0001:0083fbaa* _X509V3_add_value_bool_nf
0001:0083fbd9  _i2s_ASN1_ENUMERATED
0001:0083fc66  _i2s_ASN1_INTEGER
0001:0083fcf3  _s2i_ASN1_INTEGER
0001:0083fea3  _X509V3_add_value_int
0001:0083ff3e  _X509V3_get_value_bool
0001:00840103  _X509V3_get_value_int
0001:0084017f  _X509V3_parse_list
0001:008404ee  _hex_to_string
0001:008405d2  _string_to_hex
0001:00840826  _name_cmp
0001:008408a4* _X509_get1_email
0001:00840906* _X509_get1_ocsp
0001:008409c7* _X509_REQ_get1_email
0001:00840c13* _X509_email_free
0001:00840c2f  _a2i_IPADDRESS
0001:00840dce* _a2i_ipadd
0001:00840ca0  _a2i_IPADDRESS_NC
0001:00841264  _X509V3_NAME_from_section
Module: U:\extras\lib\libcrypto.lib(pcy_data.obj)
0001:00841390  _policy_data_free
0001:008413f6  _policy_data_new
Module: U:\extras\lib\libcrypto.lib(v3_cpols.obj)
0001:00841520  _v3_cpols
0001:00841590* _CERTIFICATEPOLICIES_it
0001:00841680* _POLICYINFO_it
0001:008415ac* _d2i_CERTIFICATEPOLICIES
0001:008415d5* _i2d_CERTIFICATEPOLICIES
0001:008415f7* _CERTIFICATEPOLICIES_new
0001:0084160b* _CERTIFICATEPOLICIES_free
0001:008417f0* _POLICYQUALINFO_it
0001:0084169c* _d2i_POLICYINFO
0001:008416c5* _i2d_POLICYINFO
0001:008416e7* _POLICYINFO_new
0001:008416fb  _POLICYINFO_free
0001:008418e0* _USERNOTICE_it
0001:0084180c* _d2i_POLICYQUALINFO
0001:00841835* _i2d_POLICYQUALINFO
0001:00841857* _POLICYQUALINFO_new
0001:0084186b  _POLICYQUALINFO_free
0001:008419d0* _NOTICEREF_it
0001:008418fc* _d2i_USERNOTICE
0001:00841925* _i2d_USERNOTICE
0001:00841947* _USERNOTICE_new
0001:0084195b* _USERNOTICE_free
0001:008419ec* _d2i_NOTICEREF
0001:00841a15* _i2d_NOTICEREF
0001:00841a37* _NOTICEREF_new
0001:00841a4b* _NOTICEREF_free
0001:00842b3c* _X509_POLICY_NODE_print
Module: U:\extras\lib\libcrypto.lib(pcy_map.obj)
0001:00842c30  _policy_cache_set_mapping
Module: U:\extras\lib\libcrypto.lib(v3_pcons.obj)
0001:00842e00  _v3_policy_constraints
0001:00842eb0* _POLICY_CONSTRAINTS_it
0001:00842ecc* _POLICY_CONSTRAINTS_new
0001:00842ee0  _POLICY_CONSTRAINTS_free
Module: U:\extras\lib\libcrypto.lib(tb_pkmeth.obj)
0001:00843160* _ENGINE_unregister_pkey_meths
0001:0084318f* _ENGINE_register_pkey_meths
0001:00843207* _ENGINE_register_all_pkey_meths
0001:00843238* _ENGINE_set_default_pkey_meths
0001:008432b0  _ENGINE_get_pkey_meth_engine
0001:008432d7  _ENGINE_get_pkey_meth
0001:0084334e* _ENGINE_get_pkey_meths
0001:00843359* _ENGINE_set_pkey_meths
0001:0084336c  _engine_pkey_meths_free
Module: U:\extras\lib\libcrypto.lib(bn_exp.obj)
0001:00843409* _BN_exp
0001:008435c9  _BN_mod_exp
0001:00844826  _BN_mod_exp_mont_word
0001:00843b6d  _BN_mod_exp_mont
0001:008436b3* _BN_mod_exp_recp
0001:008442ac* _BN_mod_exp_mont_consttime
0001:00844d4c* _BN_mod_exp_simple
Module: U:\extras\lib\libcrypto.lib(rsa_pk1.obj)
0001:0084516a  _RSA_padding_add_PKCS1_type_1
0001:0084521b  _RSA_padding_check_PKCS1_type_1
0001:008453bb  _RSA_padding_add_PKCS1_type_2
0001:008454b3  _RSA_padding_check_PKCS1_type_2
Module: U:\extras\lib\libcrypto.lib(rsa_oaep.obj)
0001:0084562b  _RSA_padding_add_PKCS1_OAEP
0001:008458b5  _RSA_padding_check_PKCS1_OAEP
0001:00845bc6  _PKCS1_MGF1
Module: U:\extras\lib\libcrypto.lib(rsa_ssl.obj)
0001:00845d8a  _RSA_padding_add_SSLv23
0001:00845ea4  _RSA_padding_check_SSLv23
Module: U:\extras\lib\libcrypto.lib(rsa_none.obj)
0001:0084607b  _RSA_padding_add_none
0001:00846117  _RSA_padding_check_none
Module: U:\extras\lib\libcrypto.lib(bn_mont.obj)
0001:008461b0  _BN_mod_mul_montgomery
0001:00846740  _BN_from_montgomery
0001:008467b8  _BN_MONT_CTX_new
0001:00846804* _BN_MONT_CTX_init
0001:0084685f  _BN_MONT_CTX_free
0001:008468b2  _BN_MONT_CTX_set
0001:00846b23  _BN_MONT_CTX_copy
0001:00846bc9  _BN_MONT_CTX_set_locked
Module: U:\extras\lib\libcrypto.lib(rsa_x931.obj)
0001:00846d0b  _RSA_padding_add_X931
0001:00846dd9  _RSA_padding_check_X931
0001:00846f63  _RSA_X931_hash_id
Module: U:\extras\lib\libcrypto.lib(bn_div.obj)
0001:00846fc9  _BN_div
Module: U:\extras\lib\libcrypto.lib(bn_mod.obj)
0001:00847d10  _BN_nnmod
0001:00847d88  _BN_mod_add
0001:00847dd4  _BN_mod_add_quick
0001:00847e36* _BN_mod_sub
0001:00847e82  _BN_mod_sub_quick
0001:00847ed8  _BN_mod_mul
0001:00847f93  _BN_mod_sqr
0001:00847fe7* _BN_mod_lshift1
0001:0084802c  _BN_mod_lshift1_quick
0001:00848087* _BN_mod_lshift
0001:0084813b  _BN_mod_lshift_quick
Module: U:\extras\lib\libcrypto.lib(bn_asm.obj)
0001:00848280  _bn_mul_add_words
0001:00848750  _bn_mul_words
0001:00848b6d  _bn_sqr_words
0001:00848dc4  _bn_div_words
0001:00848f51  _bn_add_words
0001:00849103  _bn_sub_words
0001:008492aa  _bn_mul_comba8
0001:0084eaec  _bn_mul_comba4
0001:0084ff7e  _bn_sqr_comba8
0001:0085351c  _bn_sqr_comba4
Module: U:\extras\lib\libcrypto.lib(dh_check.obj)
0001:00854120* _DH_check
0001:008542fd  _DH_check_pub_key
Module: U:\extras\lib\libcrypto.lib(dsa_ossl.obj)
0001:008543f3  _DSA_OpenSSL
Module: U:\extras\lib\libcrypto.lib(tb_dsa.obj)
0001:00854f24* _ENGINE_unregister_DSA
0001:00854f53* _ENGINE_register_DSA
0001:00854f9f* _ENGINE_register_all_DSA
0001:00854fd0* _ENGINE_set_default_DSA
0001:0085501c  _ENGINE_get_default_DSA
0001:00855039  _ENGINE_get_DSA
0001:00855044* _ENGINE_set_DSA
Module: U:\extras\lib\libcrypto.lib(v3_lib.obj)
0001:00855069* _X509V3_EXT_add
0001:00855188  _X509V3_EXT_get_nid
0001:0085521c  _X509V3_EXT_get
0001:0085524c* _X509V3_EXT_add_list
0001:0085527f* _X509V3_EXT_add_alias
0001:0085536b* _X509V3_EXT_cleanup
0001:008553b3* _X509V3_add_standard_extensions
0001:008553bd  _X509V3_EXT_d2i
0001:00855443  _X509V3_get_d2i
0001:0085556b  _X509V3_add1_i2d
Module: U:\extras\lib\libcrypto.lib(x_req.obj)
0001:00855840  _X509_REQ_INFO_it
0001:0085585c* _d2i_X509_REQ_INFO
0001:00855885* _i2d_X509_REQ_INFO
0001:008558a7* _X509_REQ_INFO_new
0001:008558bb* _X509_REQ_INFO_free
0001:00855970  _X509_REQ_it
0001:0085598c  _d2i_X509_REQ
0001:008559b5  _i2d_X509_REQ
0001:008559d7  _X509_REQ_new
0001:008559eb  _X509_REQ_free
0001:00855a06* _X509_REQ_dup
Module: U:\extras\lib\libcrypto.lib(x_spki.obj)
0001:00855a90  _NETSCAPE_SPKAC_it
0001:00855aac* _d2i_NETSCAPE_SPKAC
0001:00855ad5* _i2d_NETSCAPE_SPKAC
0001:00855af7* _NETSCAPE_SPKAC_new
0001:00855b0b* _NETSCAPE_SPKAC_free
0001:00855b90* _NETSCAPE_SPKI_it
0001:00855bac* _d2i_NETSCAPE_SPKI
0001:00855bd5* _i2d_NETSCAPE_SPKI
0001:00855bf7* _NETSCAPE_SPKI_new
0001:00855c0b* _NETSCAPE_SPKI_free
Module: U:\extras\lib\libcrypto.lib(a_sign.obj)
0001:00855c39* _ASN1_sign
0001:00855fa4  _ASN1_item_sign
Module: U:\extras\lib\libcrypto.lib(a_d2i_fp.obj)
0001:0085632b  _ASN1_d2i_fp
0001:008563cf  _ASN1_d2i_bio
0001:0085643d  _ASN1_item_d2i_bio
0001:008564b2  _ASN1_item_d2i_fp
Module: U:\extras\lib\libcrypto.lib(a_i2d_fp.obj)
0001:008568bb  _ASN1_i2d_fp
0001:00856958  _ASN1_i2d_bio
0001:00856a46  _ASN1_item_i2d_fp
0001:00856ae3  _ASN1_item_i2d_bio
Module: U:\extras\lib\libcrypto.lib(pk7_asn1.obj)
0001:00856f80* _PKCS7_SIGNED_it
0001:00857340* _PKCS7_ENVELOPE_it
0001:008576e0* _PKCS7_SIGN_ENVELOPE_it
0001:008578c0* _PKCS7_DIGEST_it
0001:008577c0* _PKCS7_ENCRYPT_it
0001:00856de0  _PKCS7_it
0001:00856dfc  _d2i_PKCS7
0001:00856e25  _i2d_PKCS7
0001:00856e47  _PKCS7_new
0001:00856e5b  _PKCS7_free
0001:00856e76* _i2d_PKCS7_NDEF
0001:00856e98* _PKCS7_dup
0001:00857150* _PKCS7_SIGNER_INFO_it
0001:00856f9c* _d2i_PKCS7_SIGNED
0001:00856fc5* _i2d_PKCS7_SIGNED
0001:00856fe7  _PKCS7_SIGNED_new
0001:00856ffb  _PKCS7_SIGNED_free
0001:00857240  _PKCS7_ISSUER_AND_SERIAL_it
0001:0085716c* _d2i_PKCS7_SIGNER_INFO
0001:00857195* _i2d_PKCS7_SIGNER_INFO
0001:008571b7  _PKCS7_SIGNER_INFO_new
0001:008571cb  _PKCS7_SIGNER_INFO_free
0001:0085725c* _d2i_PKCS7_ISSUER_AND_SERIAL
0001:00857285* _i2d_PKCS7_ISSUER_AND_SERIAL
0001:008572a7* _PKCS7_ISSUER_AND_SERIAL_new
0001:008572bb* _PKCS7_ISSUER_AND_SERIAL_free
0001:008574a0* _PKCS7_RECIP_INFO_it
0001:008575a0* _PKCS7_ENC_CONTENT_it
0001:0085735c* _d2i_PKCS7_ENVELOPE
0001:00857385* _i2d_PKCS7_ENVELOPE
0001:008573a7  _PKCS7_ENVELOPE_new
0001:008573bb* _PKCS7_ENVELOPE_free
0001:008574bc* _d2i_PKCS7_RECIP_INFO
0001:008574e5* _i2d_PKCS7_RECIP_INFO
0001:00857507  _PKCS7_RECIP_INFO_new
0001:0085751b  _PKCS7_RECIP_INFO_free
0001:008575bc* _d2i_PKCS7_ENC_CONTENT
0001:008575e5* _i2d_PKCS7_ENC_CONTENT
0001:00857607* _PKCS7_ENC_CONTENT_new
0001:0085761b* _PKCS7_ENC_CONTENT_free
0001:008576fc* _d2i_PKCS7_SIGN_ENVELOPE
0001:00857725* _i2d_PKCS7_SIGN_ENVELOPE
0001:00857747  _PKCS7_SIGN_ENVELOPE_new
0001:0085775b* _PKCS7_SIGN_ENVELOPE_free
0001:008577dc* _d2i_PKCS7_ENCRYPT
0001:00857805* _i2d_PKCS7_ENCRYPT
0001:00857827  _PKCS7_ENCRYPT_new
0001:0085783b* _PKCS7_ENCRYPT_free
0001:008578dc* _d2i_PKCS7_DIGEST
0001:00857905* _i2d_PKCS7_DIGEST
0001:00857927  _PKCS7_DIGEST_new
0001:0085793b* _PKCS7_DIGEST_free
0001:008579a0  _PKCS7_ATTR_SIGN_it
0001:008579f0  _PKCS7_ATTR_VERIFY_it
0001:00857a0c* _PKCS7_print_ctx
Module: U:\extras\lib\libcrypto.lib(dsa_asn1.obj)
0001:00857b30* _DSA_SIG_it
0001:00857b4c  _d2i_DSA_SIG
0001:00857b75  _i2d_DSA_SIG
0001:00857b97  _DSA_SIG_new
0001:00857bab  _DSA_SIG_free
0001:00857ce0* _DSAPrivateKey_it
0001:00857cfc  _d2i_DSAPrivateKey
0001:00857d25  _i2d_DSAPrivateKey
0001:00857db0* _DSAparams_it
0001:00857dcc  _d2i_DSAparams
0001:00857df5  _i2d_DSAparams
0001:00857e70* _dsa_pub_internal_it
0001:00857ee0* _DSAPublicKey_it
0001:00857efc* _d2i_DSAPublicKey
0001:00857f25  _i2d_DSAPublicKey
0001:00857f47* _DSAparams_dup
Module: U:\extras\lib\libcrypto.lib(ec_asn1.obj)
0001:00857f70  _EC_GROUP_get_basis_type
0001:00857fe0* _EC_GROUP_get_trinomial_basis
0001:00858073* _EC_GROUP_get_pentanomial_basis
0001:008581a0* _X9_62_PENTANOMIAL_it
0001:008581bc* _X9_62_PENTANOMIAL_new
0001:008581d0* _X9_62_PENTANOMIAL_free
0001:00858310* _X9_62_CHARACTERISTIC_TWO_it
0001:0085832c* _X9_62_CHARACTERISTIC_TWO_new
0001:00858340* _X9_62_CHARACTERISTIC_TWO_free
0001:00858430* _X9_62_FIELDID_it
0001:008584b0* _X9_62_CURVE_it
0001:00858590* _ECPARAMETERS_it
0001:008585ac* _ECPARAMETERS_new
0001:008585c0* _ECPARAMETERS_free
0001:00858670* _ECPKPARAMETERS_it
0001:0085868c* _d2i_UC_ECPKPARAMETERS
0001:008586b5* _i2d_UC_ECPKPARAMETERS
0001:008586d7* _ECPKPARAMETERS_new
0001:008586eb* _ECPKPARAMETERS_free
0001:00858790* _EC_PRIVATEKEY_it
0001:008587ac* _d2i_EC_PRIVATEKEY
0001:008587d5* _i2d_EC_PRIVATEKEY
0001:008587f7* _EC_PRIVATEKEY_new
0001:0085880b* _EC_PRIVATEKEY_free
0001:0085a40c  _d2i_ECPKParameters
0001:0085a502  _i2d_ECPKParameters
0001:0085a5c7  _d2i_ECPrivateKey
0001:0085a94d  _i2d_ECPrivateKey
0001:0085adf7  _i2d_ECParameters
0001:0085ae4d  _d2i_ECParameters
0001:0085af5b  _o2i_ECPublicKey
0001:0085b0b4  _i2o_ECPublicKey
Module: U:\extras\lib\libcrypto.lib(a_digest.obj)
0001:0085b27b* _ASN1_digest
0001:0085b347  _ASN1_item_digest
Module: U:\extras\lib\libcrypto.lib(x_sig.obj)
0001:0085b410  _X509_SIG_it
0001:0085b42c  _d2i_X509_SIG
0001:0085b455  _i2d_X509_SIG
0001:0085b477  _X509_SIG_new
0001:0085b48b  _X509_SIG_free
Module: U:\extras\lib\libcrypto.lib(p8_pkey.obj)
0001:0085b5b0  _PKCS8_PRIV_KEY_INFO_it
0001:0085b5cc  _d2i_PKCS8_PRIV_KEY_INFO
0001:0085b5f5  _i2d_PKCS8_PRIV_KEY_INFO
0001:0085b617  _PKCS8_PRIV_KEY_INFO_new
0001:0085b62b  _PKCS8_PRIV_KEY_INFO_free
0001:0085b646  _PKCS8_pkey_set0
0001:0085b72e  _PKCS8_pkey_get0
Module: U:\extras\lib\libcrypto.lib(evp_pkey.obj)
0001:0085b801  _EVP_PKCS82PKEY
0001:0085b9ad  _EVP_PKEY2PKCS8
0001:0085b9c8* _EVP_PKEY2PKCS8_broken
0001:0085bb33* _PKCS8_set_broken
0001:0085bba2* _EVP_PKEY_get_attr_count
0001:0085bbb8* _EVP_PKEY_get_attr_by_NID
0001:0085bbdc* _EVP_PKEY_get_attr_by_OBJ
0001:0085bc00* _EVP_PKEY_get_attr
0001:0085bc1d* _EVP_PKEY_delete_attr
0001:0085bc3a* _EVP_PKEY_add1_attr
0001:0085bc67* _EVP_PKEY_add1_attr_by_OBJ
0001:0085bca9* _EVP_PKEY_add1_attr_by_NID
0001:0085bceb* _EVP_PKEY_add1_attr_by_txt
Module: U:\extras\lib\libcrypto.lib(i2d_pr.obj)
0001:0085bd39  _i2d_PrivateKey
Module: U:\extras\lib\libcrypto.lib(d2i_pr.obj)
0001:0085bdf9  _d2i_PrivateKey
0001:0085bfc1  _d2i_AutoPrivateKey
Module: U:\extras\lib\libcrypto.lib(x509_def.obj)
0001:0085c120* _X509_get_default_private_dir
0001:0085c132  _X509_get_default_cert_area
0001:0085c14a  _X509_get_default_cert_dir
0001:0085c165  _X509_get_default_cert_file
0001:0085c17c  _X509_get_default_cert_dir_env
0001:0085c194  _X509_get_default_cert_file_env
Module: U:\extras\lib\libcrypto.lib(pem_xaux.obj)
0001:0085c1b4  _PEM_read_bio_X509_AUX
0001:0085c1ed* _PEM_read_X509_AUX
0001:0085c226* _PEM_write_bio_X509_AUX
0001:0085c279* _PEM_write_X509_AUX
0001:0085c2dd* _PEM_read_bio_X509_CERT_PAIR
0001:0085c316* _PEM_read_X509_CERT_PAIR
0001:0085c34f* _PEM_write_bio_X509_CERT_PAIR
0001:0085c3a2* _PEM_write_X509_CERT_PAIR
Module: U:\extras\lib\libcrypto.lib(pem_all.obj)
0001:0085c414* _PEM_read_bio_X509_REQ
0001:0085c44d* _PEM_read_X509_REQ
0001:0085c486* _PEM_write_bio_X509_REQ
0001:0085c4d9* _PEM_write_X509_REQ
0001:0085c544* _PEM_write_bio_X509_REQ_NEW
0001:0085c597* _PEM_write_X509_REQ_NEW
0001:0085c5f3  _PEM_read_bio_X509_CRL
0001:0085c62c* _PEM_read_X509_CRL
0001:0085c665* _PEM_write_bio_X509_CRL
0001:0085c6b8* _PEM_write_X509_CRL
0001:0085c711* _PEM_read_bio_PKCS7
0001:0085c74a* _PEM_read_PKCS7
0001:0085c783* _PEM_write_bio_PKCS7
0001:0085c7d6* _PEM_write_PKCS7
0001:0085c835* _PEM_read_bio_NETSCAPE_CERT_SEQUENCE
0001:0085c86e* _PEM_read_NETSCAPE_CERT_SEQUENCE
0001:0085c8a7* _PEM_write_bio_NETSCAPE_CERT_SEQUENCE
0001:0085c8fa* _PEM_write_NETSCAPE_CERT_SEQUENCE
0001:0085c9a6  _PEM_read_bio_RSAPrivateKey
0001:0085c9e4* _PEM_read_RSAPrivateKey
0001:0085ca32  _PEM_write_bio_RSAPrivateKey
0001:0085ca80* _PEM_write_RSAPrivateKey
0001:0085cadd* _PEM_read_bio_RSAPublicKey
0001:0085cb16* _PEM_read_RSAPublicKey
0001:0085cb4f* _PEM_write_bio_RSAPublicKey
0001:0085cba2* _PEM_write_RSAPublicKey
0001:0085cc00* _PEM_read_bio_RSA_PUBKEY
0001:0085cc39* _PEM_read_RSA_PUBKEY
0001:0085cc72* _PEM_write_bio_RSA_PUBKEY
0001:0085ccc5* _PEM_write_RSA_PUBKEY
0001:0085cd71* _PEM_read_bio_DSAPrivateKey
0001:0085cdbf* _PEM_write_bio_DSAPrivateKey
0001:0085ce0d* _PEM_write_DSAPrivateKey
0001:0085ce5b* _PEM_read_bio_DSA_PUBKEY
0001:0085ce94* _PEM_read_DSA_PUBKEY
0001:0085cecd* _PEM_write_bio_DSA_PUBKEY
0001:0085cf20* _PEM_write_DSA_PUBKEY
0001:0085cf73* _PEM_read_DSAPrivateKey
0001:0085cfc0* _PEM_read_bio_DSAparams
0001:0085cff9* _PEM_read_DSAparams
0001:0085d032* _PEM_write_bio_DSAparams
0001:0085d085* _PEM_write_DSAparams
0001:0085d131* _PEM_read_bio_ECPrivateKey
0001:0085d17d* _PEM_read_bio_ECPKParameters
0001:0085d1b6* _PEM_read_ECPKParameters
0001:0085d1ef* _PEM_write_bio_ECPKParameters
0001:0085d242* _PEM_write_ECPKParameters
0001:0085d2a4* _PEM_write_bio_ECPrivateKey
0001:0085d2f2* _PEM_write_ECPrivateKey
0001:0085d340* _PEM_read_bio_EC_PUBKEY
0001:0085d379* _PEM_read_EC_PUBKEY
0001:0085d3b2* _PEM_write_bio_EC_PUBKEY
0001:0085d405* _PEM_write_EC_PUBKEY
0001:0085d458* _PEM_read_ECPrivateKey
0001:0085d4a4* _PEM_read_bio_DHparams
0001:0085d4dd* _PEM_read_DHparams
0001:0085d516* _PEM_write_bio_DHparams
0001:0085d569* _PEM_write_DHparams
0001:0085d5bc* _PEM_read_bio_PUBKEY
0001:0085d5f5* _PEM_read_PUBKEY
0001:0085d62e* _PEM_write_bio_PUBKEY
0001:0085d681* _PEM_write_PUBKEY
Module: U:\extras\lib\libcrypto.lib(pem_info.obj)
0001:0085d6eb* _PEM_X509_INFO_read
0001:0085d7f8  _PEM_X509_INFO_read_bio
0001:0085df3d* _PEM_X509_INFO_write_bio
Module: U:\extras\lib\libcrypto.lib(x_info.obj)
0001:0085e1e9  _X509_INFO_new
0001:0085e298  _X509_INFO_free
Module: U:\extras\lib\libcrypto.lib(rsa_pmeth.obj)
0001:0085f420  _rsa_pkey_meth
Module: U:\extras\lib\libcrypto.lib(dh_pmeth.obj)
0001:0085f8d0  _dh_pkey_meth
Module: U:\extras\lib\libcrypto.lib(dsa_pmeth.obj)
0001:00860050  _dsa_pkey_meth
Module: U:\extras\lib\libcrypto.lib(ec_pmeth.obj)
0001:008607d0  _ec_pkey_meth
Module: U:\extras\lib\libcrypto.lib(hm_pmeth.obj)
0001:00860ce0  _hmac_pkey_meth
Module: U:\extras\lib\libcrypto.lib(pem_pkey.obj)
0001:00860d8d  _PEM_read_bio_PrivateKey
0001:008610b2* _PEM_write_bio_PrivateKey
0001:00861183* _PEM_read_bio_Parameters
0001:00861306* _PEM_write_bio_Parameters
0001:008613a5  _PEM_read_PrivateKey
0001:00861449* _PEM_write_PrivateKey
Module: U:\extras\lib\libcrypto.lib(ec_cvt.obj)
0001:008614f0  _EC_GROUP_new_curve_GFp
0001:00861603  _EC_GROUP_new_curve_GF2m
Module: U:\extras\lib\libcrypto.lib(ec_mult.obj)
0001:00861c82  _ec_wNAF_mul
0001:00862a5b  _ec_wNAF_precompute_mult
0001:00863092  _ec_wNAF_have_precompute_mult
Module: U:\extras\lib\libcrypto.lib(dsa_vrf.obj)
0001:008630d0* _DSA_do_verify
0001:008630fe  _DSA_verify
Module: U:\extras\lib\libcrypto.lib(ecs_vrf.obj)
0001:00863180* _ECDSA_do_verify
0001:008631c9  _ECDSA_verify
Module: U:\extras\lib\libcrypto.lib(ech_lib.obj)
0001:00863240* _ECDH_version
0001:00863268* _ECDH_set_default_method
0001:00863275* _ECDH_get_default_method
0001:00863295* _ECDH_set_method
0001:008634bf  _ecdh_check
0001:0086353d* _ECDH_get_ex_new_index
0001:00863574* _ECDH_set_ex_data
0001:008635b3* _ECDH_get_ex_data
Module: U:\extras\lib\libcrypto.lib(ecs_lib.obj)
0001:008635f0* _ECDSA_version
0001:00863619* _ECDSA_set_default_method
0001:00863626* _ECDSA_get_default_method
0001:00863646* _ECDSA_set_method
0001:00863870  _ecdsa_check
0001:008638ee  _ECDSA_size
0001:008639ef* _ECDSA_get_ex_new_index
0001:00863a26* _ECDSA_set_ex_data
0001:00863a65* _ECDSA_get_ex_data
Module: U:\extras\lib\libcrypto.lib(ecs_asn1.obj)
0001:00863af0* _ECDSA_SIG_it
0001:00863b0c  _d2i_ECDSA_SIG
0001:00863b35  _i2d_ECDSA_SIG
0001:00863b57  _ECDSA_SIG_new
0001:00863b6b  _ECDSA_SIG_free
Module: U:\extras\lib\libcrypto.lib(pmeth_gn.obj)
0001:00863b9b* _EVP_PKEY_paramgen_init
0001:00863c34* _EVP_PKEY_paramgen
0001:00863d26* _EVP_PKEY_keygen_init
0001:00863dbf* _EVP_PKEY_keygen
0001:00863eb1* _EVP_PKEY_CTX_set_cb
0001:00863ebf* _EVP_PKEY_CTX_get_cb
0001:00863f02  _evp_pkey_set_cb_translate
0001:00863f2c* _EVP_PKEY_CTX_get_keygen_info
0001:00863f67  _EVP_PKEY_new_mac_key
Module: U:\extras\lib\libcrypto.lib(m_sigver.obj)
0001:0086420e  _EVP_DigestSignInit
0001:00864245  _EVP_DigestVerifyInit
0001:0086427c  _EVP_DigestSignFinal
0001:00864416  _EVP_DigestVerifyFinal
Module: U:\extras\lib\libcrypto.lib(aes_cbc.obj)
0001:00864510  _AES_cbc_encrypt
Module: U:\extras\lib\libcrypto.lib(aes_cfb.obj)
0001:00864580  _AES_cfb128_encrypt
0001:008645c6  _AES_cfb1_encrypt
0001:0086460c  _AES_cfb8_encrypt
Module: U:\extras\lib\libcrypto.lib(aes_ecb.obj)
0001:00864660  _AES_ecb_encrypt
Module: U:\extras\lib\libcrypto.lib(aes_ofb.obj)
0001:008646b0  _AES_ofb128_encrypt
Module: U:\extras\lib\libcrypto.lib(aes_core.obj)
0001:00866818  _AES_set_encrypt_key
0001:00866eb5  _AES_set_decrypt_key
0001:00867278  _AES_encrypt
0001:008678d7  _AES_decrypt
Module: U:\extras\lib\expat.lib(xmlrole.obj)
0001:00869890  _XmlPrologStateInit
0001:008698b3  _XmlPrologStateInitExternalEntity
Module: U:\extras\lib\expat.lib(xmltok.obj)
0001:0087887f  _XmlUtf8Encode
0001:0087891f* _XmlUtf16Encode
0001:00878967  _XmlSizeOfUnknownEncoding
0001:00878b9c  _XmlInitUnknownEncoding
0001:008790c2  _XmlGetUtf8InternalEncoding
0001:008790cc* _XmlGetUtf16InternalEncoding
0001:00879133  _XmlInitEncoding
0001:00879225  _XmlParseXmlDecl
0001:00879275  _XmlGetUtf8InternalEncodingNS
0001:0087927f* _XmlGetUtf16InternalEncodingNS
0001:008792e6  _XmlInitEncodingNS
0001:008793d8  _XmlParseXmlDeclNS
0001:00879428  _XmlInitUnknownEncodingNS
Module: U:\extras\lib\lzma.lib(liblzma_la-lz_decoder.obj)
0001:0087b330  _lzma_lz_decoder_memusage
0001:0087b342  _lzma_lz_decoder_uncompressed
0001:0087b5e7  _lzma_lz_decoder_init
Module: U:\extras\lib\lzma.lib(liblzma_la-simple_coder.obj)
0001:0087b820  _lzma_simple_coder_init
Module: U:\extras\lib\lzma.lib(liblzma_la-index_hash.obj)
0001:0087bce0  _lzma_index_hash_size
0001:0087bde1  _lzma_index_hash_decode
0001:0087c228  _lzma_index_hash_append
0001:0087c323  _lzma_index_hash_end
0001:0087c32f  _lzma_index_hash_init
Module: U:\extras\lib\lzma.lib(liblzma_la-stream_flags_decoder.obj)
0001:0087c460  _lzma_stream_footer_decode
0001:0087c507  _lzma_stream_header_decode
Module: U:\extras\lib\lzma.lib(liblzma_la-stream_flags_common.obj)
0001:0087c5a0  _lzma_stream_flags_compare
0001:0087c650  _lzma_header_magic
0001:0087c656  _lzma_footer_magic
Module: U:\extras\lib\lzma.lib(liblzma_la-check.obj)
0001:0087c660  _lzma_check_is_supported
0001:0087c676  _lzma_check_size
0001:0087c68f  _lzma_check_finish
0001:0087c6da  _lzma_check_update
0001:0087c761  _lzma_check_init
Module: U:\extras\lib\lzma.lib(liblzma_la-block_header_decoder.obj)
0001:0087c7d0  _lzma_block_header_decode
Module: U:\extras\lib\lzma.lib(liblzma_la-block_decoder.obj)
0001:0087ca20  _lzma_block_decoder_init
0001:0087cbd1* _lzma_block_decoder
Module: U:\extras\lib\lzma.lib(liblzma_la-block_util.obj)
0001:0087cfc0  _lzma_block_unpadded_size
0001:0087d06f* _lzma_block_total_size
0001:0087d0a1* _lzma_block_compressed_size
Module: U:\extras\lib\libcrypto.lib(ui_lib.obj)
0001:0087d120  _UI_new
0001:0087d13d* _UI_new_method
0001:0087e174* _UI_get_default_method
0001:0087d257  _UI_free
0001:0087d5ce  _UI_add_input_string
0001:0087d61c* _UI_dup_input_string
0001:0087d6be  _UI_add_verify_string
0001:0087d70b* _UI_dup_verify_string
0001:0087d7ac* _UI_add_input_boolean
0001:0087d7f9* _UI_dup_input_boolean
0001:0087d9d6* _UI_add_info_string
0001:0087da28* _UI_dup_info_string
0001:0087dace* _UI_add_error_string
0001:0087db20* _UI_dup_error_string
0001:0087dbcf* _UI_construct_prompt
0001:0087dd3a* _UI_add_user_data
0001:0087dd57* _UI_get0_user_data
0001:0087dd62* _UI_get0_result
0001:0087e3f9  _UI_get0_result_string
0001:0087de69  _UI_process
0001:0087e013* _UI_ctrl
0001:0087e0ef* _UI_get_ex_new_index
0001:0087e126* _UI_set_ex_data
0001:0087e14a* _UI_get_ex_data
0001:0087e167* _UI_set_default_method
0001:0087e194* _UI_get_method
0001:0087e19e* _UI_set_method
0001:0087e1b0* _UI_create_method
0001:0087e20b* _UI_destroy_method
0001:0087e234* _UI_method_set_opener
0001:0087e254* _UI_method_set_writer
0001:0087e274* _UI_method_set_flusher
0001:0087e294* _UI_method_set_reader
0001:0087e2b4* _UI_method_set_closer
0001:0087e2d4* _UI_method_set_prompt_constructor
0001:0087e2f4* _UI_method_get_opener
0001:0087e30c* _UI_method_get_writer
0001:0087e324* _UI_method_get_flusher
0001:0087e33c* _UI_method_get_reader
0001:0087e354* _UI_method_get_closer
0001:0087e36c* _UI_method_get_prompt_constructor
0001:0087e384  _UI_get_string_type
0001:0087e39b  _UI_get_input_flags
0001:0087e3b3  _UI_get0_output_string
0001:0087e3cb  _UI_get0_action_string
0001:0087e423  _UI_get0_test_string
0001:0087e44c* _UI_get_result_minsize
0001:0087e476* _UI_get_result_maxsize
0001:0087e4c6  _UI_set_result
Module: U:\extras\lib\libcrypto.lib(t_pkey.obj)
0001:0087e7d9  _ASN1_bn_print
Module: U:\extras\lib\libcrypto.lib(pk7_lib.obj)
0001:0087ea2a  _PKCS7_ctrl
0001:0087ebab* _PKCS7_content_new
0001:0087ecd1  _PKCS7_set_type
0001:0087ec18* _PKCS7_set_content
0001:0087ef6d* _PKCS7_set0_type_other
0001:0087ef94* _PKCS7_add_signer
0001:0087f15d* _PKCS7_add_certificate
0001:0087f285* _PKCS7_add_crl
0001:0087f3ad* _PKCS7_SIGNER_INFO_set
0001:0087f562* _PKCS7_add_signature
0001:0087f648* _PKCS7_set_digest
0001:0087f71f* _PKCS7_get_signer_info
0001:0087f768  _PKCS7_SIGNER_INFO_get0_algs
0001:0087f7a0  _PKCS7_RECIP_INFO_get0_alg
0001:0087f7b6* _PKCS7_add_recipient
0001:0087f8b1* _PKCS7_RECIP_INFO_set
0001:0087f81a* _PKCS7_add_recipient_info
0001:0087fa9f* _PKCS7_cert_from_signer_info
0001:0087faeb* _PKCS7_set_cipher
0001:0087fbb5  _PKCS7_stream
Module: U:\extras\lib\libcrypto.lib(cms_sd.obj)
0001:0087fdec* _CMS_SignedData_init
0001:008809ba* _CMS_get0_SignerInfos
0001:0088011f  _cms_set1_SignerIdentifier
0001:00880287  _cms_SignerIdentifier_get0_signer_id
0001:008802e7  _cms_SignerIdentifier_cert_cmp
0001:0088039c* _CMS_add1_signer
0001:008818ef* _CMS_add_standard_smimecap
0001:00881711* _CMS_add_smimecap
0001:00880fc2* _CMS_SignerInfo_sign
0001:008809e3* _CMS_get0_signers
0001:00880a84* _CMS_SignerInfo_set1_signer_cert
0001:00880b0a* _CMS_SignerInfo_get0_signer_id
0001:00880b35* _CMS_SignerInfo_cert_cmp
0001:00880b52* _CMS_set1_signers_certs
0001:00880cc7  _CMS_SignerInfo_get0_algs
0001:00880f42  _cms_SignedData_final
0001:00881276* _CMS_SignerInfo_verify
0001:00881414  _cms_SignedData_init_bio
0001:008814e3* _CMS_SignerInfo_verify_content
0001:0088177c* _CMS_add_simple_smimecap
Module: U:\extras\lib\libcrypto.lib(cms_env.obj)
0001:00881b6d* _CMS_get0_RecipientInfos
0001:00881b96* _CMS_RecipientInfo_type
0001:00881ba0* _CMS_EnvelopedData_create
0001:00881c41* _CMS_add1_recipient_cert
0001:00881ed8  _CMS_RecipientInfo_ktri_get0_algs
0001:00881f5d* _CMS_RecipientInfo_ktri_get0_signer_id
0001:00881fcd* _CMS_RecipientInfo_ktri_cert_cmp
0001:00882029* _CMS_RecipientInfo_set0_pkey
0001:008824fc* _CMS_RecipientInfo_kekri_id_cmp
0001:008825b2* _CMS_add0_recipient_key
0001:00882858* _CMS_RecipientInfo_kekri_get0_id
0001:00882937* _CMS_RecipientInfo_set0_key
0001:00882df7* _CMS_RecipientInfo_decrypt
0001:00882e68  _cms_EnvelopedData_init_bio
Module: U:\extras\lib\libcrypto.lib(ec_print.obj)
0001:0088300b  _EC_POINT_point2bn
0001:008830f6* _EC_POINT_bn2point
0001:00883228* _EC_POINT_point2hex
0001:00883397* _EC_POINT_hex2point
Module: U:\extras\lib\libcrypto.lib(eck_prn.obj)
0001:0088340a* _ECPKParameters_print_fp
0001:0088370c  _ECPKParameters_print
0001:008834a7* _EC_KEY_print_fp
0001:008835da* _EC_KEY_print
0001:00883544* _ECParameters_print_fp
0001:0088363f* _ECParameters_print
Module: U:\extras\lib\libcrypto.lib(a_bytes.obj)
0001:008840ea* _d2i_ASN1_type_bytes
0001:008842de  _i2d_ASN1_bytes
0001:008843ca* _d2i_ASN1_bytes
Module: U:\extras\lib\libcrypto.lib(pcy_node.obj)
0001:00884878  _policy_node_cmp_new
0001:0088488d  _tree_find_sk
0001:008848d5  _level_find_node
0001:0088494f  _level_add_node
0001:00884a84  _policy_node_free
0001:00884a97  _policy_node_match
Module: U:\extras\lib\libcrypto.lib(pcy_lib.obj)
0001:00884b50* _X509_policy_tree_level_count
0001:00884b68* _X509_policy_tree_get0_level
0001:00884b98* _X509_policy_tree_get0_policies
0001:00884bb0  _X509_policy_tree_get0_user_policies
0001:00884bdd* _X509_policy_level_node_count
0001:00884c2a* _X509_policy_level_get0_node
0001:00884c6f* _X509_policy_node_get0_policy
0001:00884c89* _X509_policy_node_get0_qualifiers
0001:00884ca3* _X509_policy_node_get0_parent
Module: U:\extras\lib\libcrypto.lib(o_time.obj)
0001:00884cc0  _OPENSSL_gmtime
0001:00884d0d  _OPENSSL_gmtime_adj
Module: U:\extras\lib\libcrypto.lib(asn1_gen.obj)
0001:008851e0* _ASN1_generate_nconf
0001:00885232  _ASN1_generate_v3
Module: U:\extras\lib\libcrypto.lib(a_bool.obj)
0001:00886bd0* _i2d_ASN1_BOOLEAN
0001:00886c55  _d2i_ASN1_BOOLEAN
Module: U:\extras\lib\libcrypto.lib(b_dump.obj)
0001:00886d30* _BIO_dump_cb
0001:00886d93* _BIO_dump_indent_cb
0001:00887149* _BIO_dump_fp
0001:00887172* _BIO_dump_indent_fp
0001:008871c3* _BIO_dump
0001:008871ec  _BIO_dump_indent
Module: U:\extras\lib\libcrypto.lib(a_strnid.obj)
0001:00887220* _ASN1_STRING_set_default_mask
0001:0088722d* _ASN1_STRING_get_default_mask
0001:0088725b* _ASN1_STRING_set_default_mask_asc
0001:00887366  _ASN1_STRING_set_by_NID
0001:00887641* _ASN1_STRING_TABLE_get
0001:008876cb* _ASN1_STRING_TABLE_add
0001:00887817* _ASN1_STRING_TABLE_cleanup
Module: U:\extras\lib\libcrypto.lib(a_print.obj)
0001:00887870  _ASN1_PRINTABLE_type
0001:0088797e* _ASN1_UNIVERSALSTRING_to_string
Module: U:\extras\lib\libcrypto.lib(err_prn.obj)
0001:00887a92  _ERR_print_errors_cb
0001:00887c05* _ERR_print_errors_fp
0001:00887c41  _ERR_print_errors
Module: U:\extras\lib\libcrypto.lib(v3_prn.obj)
0001:00887c79* _X509V3_EXT_val_prn
0001:00887dea* _X509V3_EXT_print
0001:0088805d  _X509V3_extensions_print
0001:00888336* _X509V3_EXT_print_fp
Module: U:\extras\lib\libcrypto.lib(t_x509a.obj)
0001:0088841f  _X509_CERT_AUX_print
Module: U:\extras\lib\libcrypto.lib(p5_pbe.obj)
0001:00888770* _PBEPARAM_it
0001:0088878c  _d2i_PBEPARAM
0001:008887b5* _i2d_PBEPARAM
0001:008887d7* _PBEPARAM_new
0001:008887eb  _PBEPARAM_free
0001:0088880f* _PKCS5_pbe_set0_algor
0001:00888a24  _PKCS5_pbe_set
Module: U:\extras\lib\libcrypto.lib(p12_key.obj)
0001:00888aba  _PKCS12_key_gen_asc
0001:00888bab* _PKCS12_key_gen_uni
Module: U:\extras\lib\libcrypto.lib(p5_pbev2.obj)
0001:00889110* _PBE2PARAM_it
0001:0088912c  _d2i_PBE2PARAM
0001:00889155* _i2d_PBE2PARAM
0001:00889177* _PBE2PARAM_new
0001:0088918b  _PBE2PARAM_free
0001:00889220* _PBKDF2PARAM_it
0001:0088923c  _d2i_PBKDF2PARAM
0001:00889265* _i2d_PBKDF2PARAM
0001:00889287* _PBKDF2PARAM_new
0001:0088929b  _PBKDF2PARAM_free
0001:008892c1* _PKCS5_pbe2_set_iv
0001:008897fd  _PKCS5_pbe2_set
Module: U:\extras\lib\libcrypto.lib(eng_ctrl.obj)
0001:00889c72* _ENGINE_ctrl
0001:00889e5b* _ENGINE_cmd_is_executable
0001:00889ef3* _ENGINE_ctrl_cmd
0001:00889ff6  _ENGINE_ctrl_cmd_string
Module: U:\extras\lib\libcrypto.lib(conf_lib.obj)
0001:0088a370* _CONF_version
0001:0088a398  _CONF_set_nconf
0001:0088a3cc* _CONF_set_default_method
0001:0088a3ec* _CONF_load
0001:0088a4f5* _CONF_load_bio
0001:0088a474* _CONF_load_fp
0001:0088a897* _NCONF_load_bio
0001:0088a53b  _CONF_get_section
0001:0088a8f6  _NCONF_get_section
0001:0088a574  _CONF_get_string
0001:0088a990  _NCONF_get_string
0001:0088a5c9* _CONF_get_number
0001:0088aa56* _NCONF_get_number_e
0001:0088a647  _CONF_free
0001:0088a796* _NCONF_free_data
0001:0088a66c* _CONF_dump_fp
0001:0088a6e6* _CONF_dump_bio
0001:0088aba9* _NCONF_dump_bio
0001:0088a712  _NCONF_new
0001:0088a775  _NCONF_free
0001:0088a7b7  _NCONF_load
0001:0088a816* _NCONF_load_fp
0001:0088ab2f* _NCONF_dump_fp
Module: U:\extras\lib\libcrypto.lib(x509_req.obj)
0001:0088ac1b* _X509_to_X509_REQ
0001:0088ad51* _X509_REQ_get_pubkey
0001:0088ad7f* _X509_REQ_check_private_key
0001:0088aef4* _X509_REQ_extension_nid
0001:0088af36* _X509_REQ_get_extension_nids
0001:0088af40* _X509_REQ_set_extension_nids
0001:0088af4d  _X509_REQ_get_extensions
0001:0088b1e5* _X509_REQ_get_attr_by_NID
0001:0088b231* _X509_REQ_get_attr
0001:0088b067* _X509_REQ_add_extensions_nid
0001:0088b1ab  _X509_REQ_add_extensions
0001:0088b1cd* _X509_REQ_get_attr_count
0001:0088b20b* _X509_REQ_get_attr_by_OBJ
0001:0088b250* _X509_REQ_delete_attr
0001:0088b26f* _X509_REQ_add1_attr
0001:0088b29e* _X509_REQ_add1_attr_by_OBJ
0001:0088b2e2* _X509_REQ_add1_attr_by_NID
0001:0088b326* _X509_REQ_add1_attr_by_txt
Module: U:\extras\lib\libcrypto.lib(conf_mod.obj)
0001:0088b3d5* _CONF_modules_load
0001:0088b4f6* _CONF_modules_load_file
0001:0088be76* _CONF_get1_default_config_file
0001:0088bc20* _CONF_modules_unload
0001:0088bcfa* _CONF_modules_finish
0001:0088bd9e* _CONF_module_add
0001:0088bdd7* _CONF_modules_free
0001:0088bdf0* _CONF_imodule_get_name
0001:0088bdfb* _CONF_imodule_get_value
0001:0088be06* _CONF_imodule_get_usr_data
0001:0088be11* _CONF_imodule_set_usr_data
0001:0088be1f* _CONF_imodule_get_module
0001:0088be29* _CONF_imodule_get_flags
0001:0088be34* _CONF_imodule_set_flags
0001:0088be42* _CONF_module_get_usr_data
0001:0088be4d* _CONF_module_set_usr_data
0001:0088bf47  _CONF_parse_list
Module: U:\extras\lib\libcrypto.lib(v3_pmaps.obj)
0001:0088c0a0  _v3_policy_mappings
0001:0088c190* _POLICY_MAPPINGS_it
0001:0088c140* _POLICY_MAPPING_it
0001:0088c1ac* _POLICY_MAPPING_new
0001:0088c1c0  _POLICY_MAPPING_free
Module: U:\extras\lib\libcrypto.lib(bn_sqr.obj)
0001:0088c510  _BN_sqr
0001:0088c7b3* _bn_sqr_normal
0001:0088c8e2* _bn_sqr_recursive
Module: U:\extras\lib\libcrypto.lib(bn_recp.obj)
0001:0088cb90  _BN_RECP_CTX_init
0001:0088cbcf* _BN_RECP_CTX_new
0001:0088cc1b  _BN_RECP_CTX_free
0001:0088cc5d  _BN_RECP_CTX_set
0001:0088ccb8  _BN_mod_mul_reciprocal
0001:0088cd88* _BN_div_recp
0001:0088d0b3* _BN_reciprocal
Module: U:\extras\lib\libcrypto.lib(bn_prime.obj)
0001:0088e140  _BN_GENCB_call
0001:0088e1c0  _BN_generate_prime_ex
0001:0088e50b  _BN_is_prime_fasttest_ex
0001:0088e4db  _BN_is_prime_ex
Module: U:\extras\lib\libcrypto.lib(bn_exp2.obj)
0001:0088efba  _BN_mod_exp2_mont
Module: U:\extras\lib\libcrypto.lib(v3_bitst.obj)
0001:0088f940  _v3_nscert
0001:0088f9b8* _i2v_ASN1_BIT_STRING
0001:0088fa34* _v2i_ASN1_BIT_STRING
0001:0088f980  _v3_key_usage
Module: U:\extras\lib\libcrypto.lib(v3_ia5.obj)
0001:0088fc10  _v3_ns_ia5_list
Module: U:\extras\lib\libcrypto.lib(v3_skey.obj)
0001:0088ff50  _v3_skey_id
0001:0088ff88* _i2s_ASN1_OCTET_STRING
0001:0088ffb1* _s2i_ASN1_OCTET_STRING
Module: U:\extras\lib\libcrypto.lib(v3_pku.obj)
0001:00890230  _v3_pkey_usage_period
0001:008902c0* _PKEY_USAGE_PERIOD_it
0001:008902dc* _d2i_PKEY_USAGE_PERIOD
0001:00890305* _i2d_PKEY_USAGE_PERIOD
0001:00890327* _PKEY_USAGE_PERIOD_new
0001:0089033b* _PKEY_USAGE_PERIOD_free
Module: U:\extras\lib\libcrypto.lib(v3_int.obj)
0001:00890440  _v3_crl_num
0001:00890480  _v3_delta_crl
0001:008904e0  _v3_inhibit_anyp
Module: U:\extras\lib\libcrypto.lib(v3_akey.obj)
0001:00890520  _v3_akey_id
Module: U:\extras\lib\libcrypto.lib(v3_extku.obj)
0001:00890a00  _v3_ext_ku
0001:00890ab0* _EXTENDED_KEY_USAGE_it
0001:00890a40  _v3_ocsp_accresp
0001:00890acc* _d2i_EXTENDED_KEY_USAGE
0001:00890af5* _i2d_EXTENDED_KEY_USAGE
0001:00890b17* _EXTENDED_KEY_USAGE_new
0001:00890b2b* _EXTENDED_KEY_USAGE_free
Module: U:\extras\lib\libcrypto.lib(v3_enum.obj)
0001:00890e80  _v3_crl_reason
0001:00890eb8* _i2s_ASN1_ENUMERATED_TABLE
Module: U:\extras\lib\libcrypto.lib(v3_ocsp.obj)
0001:00890f20  _v3_ocsp_crlid
0001:00890f60  _v3_ocsp_acutoff
0001:00890fa0  _v3_crl_invdate
0001:00890fe0  _v3_crl_hold
0001:00891020  _v3_ocsp_nonce
0001:00891060  _v3_ocsp_nocheck
0001:008910a0  _v3_ocsp_serviceloc
Module: U:\extras\lib\libcrypto.lib(v3_sxnet.obj)
0001:00891630  _v3_sxnet
0001:00891790* _SXNET_it
0001:008916b0* _SXNETID_it
0001:008916cc* _d2i_SXNETID
0001:008916f5* _i2d_SXNETID
0001:00891717* _SXNETID_new
0001:0089172b* _SXNETID_free
0001:008917ac* _d2i_SXNET
0001:008917d5* _i2d_SXNET
0001:008917f7* _SXNET_new
0001:0089180b* _SXNET_free
0001:008919c0* _SXNET_add_id_asc
0001:00891ad6* _SXNET_add_id_INTEGER
0001:00891a3e* _SXNET_add_id_ulong
0001:00891dfd* _SXNET_get_id_INTEGER
0001:00891ce1* _SXNET_get_id_asc
0001:00891d62* _SXNET_get_id_ulong
Module: U:\extras\lib\libcrypto.lib(v3_pci.obj)
0001:00891e70  _v3_pci
Module: U:\extras\lib\libcrypto.lib(pk7_doit.obj)
0001:00893423  _PKCS7_dataInit
0001:00893a16* _PKCS7_dataDecode
0001:008951a5  _PKCS7_get_signed_attribute
0001:008948f2* _PKCS7_SIGNER_INFO_sign
0001:00894348  _PKCS7_dataFinal
0001:00894b69* _PKCS7_dataVerify
0001:00894d31* _PKCS7_signatureVerify
0001:00895294* _PKCS7_digest_from_attributes
0001:0089510d* _PKCS7_get_issuer_and_serial
0001:008951c2* _PKCS7_get_attribute
0001:008952c5* _PKCS7_set_signed_attributes
0001:00895371* _PKCS7_set_attributes
0001:0089541d  _PKCS7_add_signed_attribute
0001:00895448* _PKCS7_add_attribute
Module: U:\extras\lib\libcrypto.lib(tasn_prn.obj)
0001:008955db* _ASN1_PCTX_new
0001:0089566f* _ASN1_PCTX_free
0001:00895682* _ASN1_PCTX_get_flags
0001:0089568c* _ASN1_PCTX_set_flags
0001:00895699* _ASN1_PCTX_get_nm_flags
0001:008956a4* _ASN1_PCTX_set_nm_flags
0001:008956b2* _ASN1_PCTX_get_cert_flags
0001:008956bd* _ASN1_PCTX_set_cert_flags
0001:008956cb* _ASN1_PCTX_get_oid_flags
0001:008956d6* _ASN1_PCTX_set_oid_flags
0001:008956e4* _ASN1_PCTX_get_str_flags
0001:008956ef* _ASN1_PCTX_set_str_flags
0001:008956fd  _ASN1_item_print
0001:00895d4f* _asn1_template_print_ctx
0002:000086e0* _default_pctx
Module: U:\extras\lib\libcrypto.lib(ec2_smpl.obj)
0001:008966e0  _EC_GF2m_simple_method
0001:008966ea* _ec_GF2m_simple_group_init
0001:00896723* _ec_GF2m_simple_group_finish
0001:00896757* _ec_GF2m_simple_group_clear_finish
0001:008967c7* _ec_GF2m_simple_group_copy
0001:008969ce  _ec_GF2m_simple_group_set_curve
0001:00896be8* _ec_GF2m_simple_group_get_curve
0001:00896c6d* _ec_GF2m_simple_group_get_degree
0001:00896c84* _ec_GF2m_simple_group_check_discriminant
0001:00896d65* _ec_GF2m_simple_point_init
0001:00896d9c* _ec_GF2m_simple_point_finish
0001:00896dce* _ec_GF2m_simple_point_clear_finish
0001:00896e0a* _ec_GF2m_simple_point_copy
0001:00896e8c* _ec_GF2m_simple_point_set_to_infinity
0001:00896eb9* _ec_GF2m_simple_point_set_affine_coordinates
0001:00896fba* _ec_GF2m_simple_point_get_affine_coordinates
0001:008970d7* _ec_GF2m_simple_set_compressed_coordinates
0001:00897424* _ec_GF2m_simple_point2oct
0001:0089786f* _ec_GF2m_simple_oct2point
0001:00897cf6* _ec_GF2m_simple_add
0001:00898287* _ec_GF2m_simple_dbl
0001:008982b6* _ec_GF2m_simple_invert
0001:0089832b* _ec_GF2m_simple_is_at_infinity
0001:0089833e* _ec_GF2m_simple_is_on_curve
0001:0089855c* _ec_GF2m_simple_cmp
0001:00898754* _ec_GF2m_simple_make_affine
0001:0089889b* _ec_GF2m_simple_points_make_affine
0001:008988ed* _ec_GF2m_simple_field_mul
0001:0089891f* _ec_GF2m_simple_field_sqr
0001:0089894a* _ec_GF2m_simple_field_div
Module: U:\extras\lib\libcrypto.lib(x509_att.obj)
0001:00898a20  _X509at_get_attr_count
0001:00898a33  _X509at_get_attr_by_NID
0001:00898a6f  _X509at_get_attr_by_OBJ
0001:00898ae6  _X509at_get_attr
0001:00898b23  _X509at_delete_attr
0001:00898b71  _X509at_add1_attr
0001:00898c76  _X509at_add1_attr_by_OBJ
0001:00898edc* _X509_ATTRIBUTE_create_by_OBJ
0001:00898cd9  _X509at_add1_attr_by_NID
0001:00898e4f* _X509_ATTRIBUTE_create_by_NID
0001:00898d3c  _X509at_add1_attr_by_txt
0001:00898fc2* _X509_ATTRIBUTE_create_by_txt
0001:00898d9f  _X509at_get0_data_by_OBJ
0001:0089928a* _X509_ATTRIBUTE_count
0001:008992d9* _X509_ATTRIBUTE_get0_data
0001:0089906c* _X509_ATTRIBUTE_set1_object
0001:008990a9* _X509_ATTRIBUTE_set1_data
0001:008992c2* _X509_ATTRIBUTE_get0_object
0001:0089934c* _X509_ATTRIBUTE_get0_type
Module: U:\extras\lib\libcrypto.lib(nsseq.obj)
0001:00899440* _NETSCAPE_CERT_SEQUENCE_it
0001:0089945c  _d2i_NETSCAPE_CERT_SEQUENCE
0001:00899485  _i2d_NETSCAPE_CERT_SEQUENCE
0001:008994a7* _NETSCAPE_CERT_SEQUENCE_new
0001:008994bb* _NETSCAPE_CERT_SEQUENCE_free
Module: U:\extras\lib\libcrypto.lib(x_pkey.obj)
0001:008994e0* _i2d_X509_PKEY
0001:008994f3* _d2i_X509_PKEY
0001:00899783  _X509_PKEY_new
0001:0089989b  _X509_PKEY_free
Module: U:\extras\lib\libcrypto.lib(rsa_pss.obj)
0001:00899972  _RSA_verify_PKCS1_PSS
0001:00899dc3  _RSA_padding_add_PKCS1_PSS
Module: U:\extras\lib\libcrypto.lib(rsa_gen.obj)
0001:0089a0f0  _RSA_generate_key_ex
Module: U:\extras\lib\libcrypto.lib(dh_gen.obj)
0001:0089a970  _DH_generate_parameters_ex
Module: U:\extras\lib\libcrypto.lib(dsa_gen.obj)
0001:0089ac70* _DSA_generate_parameters_ex
0001:0089ad49  _dsa_builtin_paramgen
Module: U:\extras\lib\libcrypto.lib(dsa_key.obj)
0001:0089b680  _DSA_generate_key
Module: U:\extras\lib\libcrypto.lib(p12_p8d.obj)
0001:0089b870  _PKCS8_decrypt
Module: U:\extras\lib\libcrypto.lib(pem_pk8.obj)
0001:0089b8b0* _PEM_write_bio_PKCS8PrivateKey_nid
0001:0089b8fd  _PEM_write_bio_PKCS8PrivateKey
0001:0089b94a* _i2d_PKCS8PrivateKey_bio
0001:0089b997* _i2d_PKCS8PrivateKey_nid_bio
0001:0089c045* _PEM_write_bio_PKCS8
0001:0089c169* _PEM_write_bio_PKCS8_PRIV_KEY_INFO
0001:0089bbf4* _d2i_PKCS8PrivateKey_bio
0001:0089bd56* _i2d_PKCS8PrivateKey_fp
0001:0089bda3* _i2d_PKCS8PrivateKey_nid_fp
0001:0089bdf0* _PEM_write_PKCS8PrivateKey_nid
0001:0089be3d* _PEM_write_PKCS8PrivateKey
0001:0089bf35* _d2i_PKCS8PrivateKey_fp
0001:0089bfd3* _PEM_read_bio_PKCS8
0001:0089c00c* _PEM_read_PKCS8
0001:0089c098* _PEM_write_PKCS8
0001:0089c0f7* _PEM_read_bio_PKCS8_PRIV_KEY_INFO
0001:0089c130* _PEM_read_PKCS8_PRIV_KEY_INFO
0001:0089c1bc* _PEM_write_PKCS8_PRIV_KEY_INFO
Module: U:\extras\lib\libcrypto.lib(ecp_nist.obj)
0001:0089c210  _EC_GFp_nist_method
0001:0089c21a* _ec_GFp_nist_group_copy
0001:0089c251* _ec_GFp_nist_group_set_curve
0001:0089c3f1* _ec_GFp_nist_field_mul
0001:0089c4dc* _ec_GFp_nist_field_sqr
Module: U:\extras\lib\libcrypto.lib(ecp_mont.obj)
0001:0089c660  _EC_GFp_mont_method
0001:0089c66a* _ec_GFp_mont_group_init
0001:0089c69d* _ec_GFp_mont_group_finish
0001:0089c706* _ec_GFp_mont_group_clear_finish
0001:0089c76f* _ec_GFp_mont_group_copy
0001:0089c8bd* _ec_GFp_mont_group_set_curve
0001:0089cac6* _ec_GFp_mont_field_mul
0001:0089cb3b* _ec_GFp_mont_field_sqr
0001:0089cbb0* _ec_GFp_mont_field_encode
0001:0089cc2e* _ec_GFp_mont_field_decode
0001:0089cc9c* _ec_GFp_mont_field_set_to_one
Module: U:\extras\lib\libcrypto.lib(ech_ossl.obj)
0001:0089cdc4  _ECDH_OpenSSL
Module: U:\extras\lib\libcrypto.lib(tb_ecdh.obj)
0001:0089d264* _ENGINE_unregister_ECDH
0001:0089d293* _ENGINE_register_ECDH
0001:0089d2df* _ENGINE_register_all_ECDH
0001:0089d310* _ENGINE_set_default_ECDH
0001:0089d35c  _ENGINE_get_default_ECDH
0001:0089d379  _ENGINE_get_ECDH
0001:0089d384* _ENGINE_set_ECDH
Module: U:\extras\lib\libcrypto.lib(ecs_ossl.obj)
0001:0089d3b5  _ECDSA_OpenSSL
Module: U:\extras\lib\libcrypto.lib(tb_ecdsa.obj)
0001:0089e454* _ENGINE_unregister_ECDSA
0001:0089e483* _ENGINE_register_ECDSA
0001:0089e4cf* _ENGINE_register_all_ECDSA
0001:0089e500* _ENGINE_set_default_ECDSA
0001:0089e54c  _ENGINE_get_default_ECDSA
0001:0089e569  _ENGINE_get_ECDSA
0001:0089e574* _ENGINE_set_ECDSA
Module: U:\extras\lib\libcrypto.lib(cbc128.obj)
0001:0089e590  _CRYPTO_cbc128_encrypt
0001:0089e6bc  _CRYPTO_cbc128_decrypt
Module: U:\extras\lib\libcrypto.lib(cfb128.obj)
0001:0089e880  _CRYPTO_cfb128_encrypt
0001:0089ec80  _CRYPTO_cfb128_1_encrypt
0001:0089ed5d  _CRYPTO_cfb128_8_encrypt
Module: U:\extras\lib\libcrypto.lib(ofb128.obj)
0001:0089edc0  _CRYPTO_ofb128_encrypt
Module: U:\extras\lib\lzma.lib(liblzma_la-vli_size.obj)
0001:0089eed0  _lzma_vli_size
Module: U:\extras\lib\lzma.lib(liblzma_la-crc32_fast.obj)
0001:0089ef00  _lzma_crc32
Module: U:\extras\lib\lzma.lib(liblzma_la-vli_decoder.obj)
0001:0089f020  _lzma_vli_decode
Module: U:\extras\lib\lzma.lib(liblzma_la-sha256.obj)
0001:008a002e  _lzma_sha256_finish
0001:008a01a2  _lzma_sha256_update
0001:008a0234  _lzma_sha256_init
Module: U:\extras\lib\lzma.lib(liblzma_la-crc64_fast.obj)
0001:008a0380  _lzma_crc64
Module: U:\extras\lib\lzma.lib(liblzma_la-filter_flags_decoder.obj)
0001:008a04f0  _lzma_filter_flags_decode
Module: U:\extras\lib\libcrypto.lib(ui_openssl.obj)
0001:008a05cf  _UI_OpenSSL
Module: U:\extras\lib\libcrypto.lib(cms_asn1.obj)
0001:008a0db0  _CMS_IssuerAndSerialNumber_it
0001:008a0e40* _CMS_OtherCertificateFormat_it
0001:008a0f30  _CMS_CertificateChoices_it
0001:008a0fc0* _CMS_SignerIdentifier_it
0001:008a1050* _CMS_EncapsulatedContentInfo_it
0001:008a11d0  _CMS_SignerInfo_it
0001:008a1260* _CMS_OtherRevocationInfoFormat_it
0001:008a12e0  _CMS_RevocationInfoChoice_it
0001:008a13d0  _CMS_SignedData_it
0001:008a1430* _CMS_OriginatorInfo_it
0001:008a14f0* _CMS_EncryptedContentInfo_it
0001:008a15b0  _CMS_KeyTransRecipientInfo_it
0001:008a1620  _CMS_OtherKeyAttribute_it
0001:008a16c0* _CMS_RecipientKeyIdentifier_it
0001:008a1740* _CMS_KeyAgreeRecipientIdentifier_it
0001:008a17b0* _CMS_RecipientEncryptedKey_it
0001:008a1820* _CMS_OriginatorPublicKey_it
0001:008a18b0* _CMS_OriginatorIdentifierOrKey_it
0001:008a1980* _CMS_KeyAgreeRecipientInfo_it
0001:008a1a00* _CMS_KEKIdentifier_it
0001:008a1aa0  _CMS_KEKRecipientInfo_it
0001:008a1b50* _CMS_PasswordRecipientInfo_it
0001:008a1bc0* _CMS_OtherRecipientInfo_it
0001:008a1d50  _CMS_RecipientInfo_it
0001:008a1e30  _CMS_EnvelopedData_it
0001:008a1ed0  _CMS_DigestedData_it
0001:008a1f40  _CMS_EncryptedData_it
0001:008a2060* _CMS_AuthenticatedData_it
0001:008a20f0* _CMS_CompressedData_it
0001:008a2380  _CMS_ContentInfo_it
0001:008a23e0  _CMS_Attributes_Sign_it
0001:008a2430  _CMS_Attributes_Verify_it
0001:008a24b0* _CMS_ReceiptsFrom_it
0001:008a2550* _CMS_ReceiptRequest_it
0001:008a25f0* _CMS_Receipt_it
Module: U:\extras\lib\libcrypto.lib(cms_att.obj)
0001:008a2610  _CMS_signed_get_attr_count
0001:008a2626  _CMS_signed_get_attr_by_NID
0001:008a264a* _CMS_signed_get_attr_by_OBJ
0001:008a266e* _CMS_signed_get_attr
0001:008a268b* _CMS_signed_delete_attr
0001:008a26a8* _CMS_signed_add1_attr
0001:008a26d5* _CMS_signed_add1_attr_by_OBJ
0001:008a2717  _CMS_signed_add1_attr_by_NID
0001:008a2759* _CMS_signed_add1_attr_by_txt
0001:008a279b  _CMS_signed_get0_data_by_OBJ
0001:008a27c6* _CMS_unsigned_get_attr_count
0001:008a27dc* _CMS_unsigned_get_attr_by_NID
0001:008a2800* _CMS_unsigned_get_attr_by_OBJ
0001:008a2824* _CMS_unsigned_get_attr
0001:008a2841* _CMS_unsigned_delete_attr
0001:008a285e* _CMS_unsigned_add1_attr
0001:008a288b* _CMS_unsigned_add1_attr_by_OBJ
0001:008a28cd* _CMS_unsigned_add1_attr_by_NID
0001:008a290f* _CMS_unsigned_add1_attr_by_txt
0001:008a2951* _CMS_unsigned_get0_data_by_OBJ
Module: U:\extras\lib\libcrypto.lib(cms_lib.obj)
0001:008a2980  _d2i_CMS_ContentInfo
0001:008a29a9  _i2d_CMS_ContentInfo
0001:008a29cb  _CMS_ContentInfo_new
0001:008a29df  _CMS_ContentInfo_free
0001:008a29fa* _CMS_ContentInfo_print_ctx
0001:008a2a2a* _CMS_get0_type
0001:008a2a34* _priv_cms_Data_create
0001:008a3063* _CMS_set_detached
0001:008a2a71* _cms_content_bio
0001:008a2df8  _CMS_get0_content
0001:008a2af6  _CMS_dataInit
0001:008a2c39  _CMS_dataFinal
0001:008a2f9e  _CMS_get0_eContentType
0001:008a2fc6* _CMS_set1_eContentType
0001:008a302b* _CMS_is_detached
0001:008a311c  _cms_DigestAlgorithm_set
0001:008a3172  _cms_DigestAlgorithm_init_bio
0001:008a327a  _cms_DigestAlgorithm_find_ctx
0001:008a33e7* _CMS_add0_CertificateChoices
0001:008a3480* _CMS_add0_cert
0001:008a3576  _CMS_add1_cert
0001:008a3635* _CMS_add0_RevocationInfoChoice
0001:008a36ce* _CMS_add0_crl
0001:008a3708* _CMS_add1_crl
0001:008a375c* _CMS_get1_certs
0001:008a3858* _CMS_get1_crls
Module: U:\extras\lib\libcrypto.lib(cms_enc.obj)
0001:008a396a  _cms_EncryptedContent_init_bio
0001:008a3e1d  _cms_EncryptedContent_init
0001:008a3ea9* _CMS_EncryptedData_set1_key
0001:008a3fdd  _cms_EncryptedData_init_bio
Module: U:\extras\lib\libcrypto.lib(aes_wrap.obj)
0001:008a4028  _AES_wrap_key
0001:008a41b8  _AES_unwrap_key
Module: U:\extras\lib\libcrypto.lib(asn_pack.obj)
0001:008a438b* _ASN1_seq_unpack
0001:008a4409* _ASN1_seq_pack
0001:008a452f* _ASN1_unpack_string
0001:008a4594* _ASN1_pack_string
0001:008a46d6  _ASN1_item_pack
0001:008a480b  _ASN1_item_unpack
Module: U:\extras\lib\libcrypto.lib(p12_utl.obj)
0001:008a488a  _OPENSSL_asc2uni
0001:008a4943* _OPENSSL_uni2asc
0001:008a49d3* _i2d_PKCS12_bio
0001:008a49f5* _i2d_PKCS12_fp
0001:008a4a17* _d2i_PKCS12_bio
0001:008a4a39* _d2i_PKCS12_fp
0001:008a4a5b* _PKCS12_x5092certbag
0001:008a4a86* _PKCS12_x509crl2certbag
0001:008a4ab1* _PKCS12_certbag2x509
0001:008a4b0b* _PKCS12_certbag2x509crl
Module: U:\extras\lib\libcrypto.lib(conf_def.obj)
0001:008a4b70* _CONF_def_version
0001:008a4bb2  _NCONF_default
0001:008a4bbc* _NCONF_WIN32
Module: U:\extras\lib\libcrypto.lib(conf_api.obj)
0001:008a616f  __CONF_get_section
0001:008a61b2  __CONF_get_section_values
0001:008a61e2  __CONF_add_string
0001:008a6289  __CONF_get_string
0001:008a6463  __CONF_new_data
0001:008a64b4  __CONF_free_data
0001:008a65fe  __CONF_new_section
Module: U:\extras\lib\libcrypto.lib(x509rset.obj)
0001:008a6740* _X509_REQ_set_version
0001:008a676c  _X509_REQ_set_subject_name
0001:008a67a1  _X509_REQ_set_pubkey
Module: U:\extras\lib\libcrypto.lib(dso_lib.obj)
0001:008a67e0* _DSO_new
0001:008a683a* _DSO_new_method
0001:008a67f4* _DSO_set_default_method
0001:008a6801* _DSO_get_default_method
0001:008a680b* _DSO_get_method
0001:008a6815* _DSO_set_method
0001:008a697a  _DSO_free
0001:008a6af6* _DSO_flags
0001:008a6b0e* _DSO_up_ref
0001:008a6b82  _DSO_load
0001:008a6f6f* _DSO_ctrl
0001:008a710f* _DSO_set_filename
0001:008a6da3* _DSO_bind_var
0001:008a6e89  _DSO_bind_func
0001:008a7068* _DSO_set_name_converter
0001:008a70c8* _DSO_get_filename
0001:008a7241* _DSO_merge
0001:008a72f7* _DSO_convert_filename
0001:008a7473* _DSO_get_loaded_filename
0001:008a74ba* _DSO_pathbyaddr
0001:008a7531* _DSO_global_lookup
Module: U:\extras\lib\libcrypto.lib(f_int.obj)
0001:008a75a8  _i2a_ASN1_INTEGER
0001:008a7716* _a2i_ASN1_INTEGER
Module: U:\extras\lib\libcrypto.lib(f_string.obj)
0001:008a7b25  _i2a_ASN1_STRING
0001:008a7c5c* _a2i_ASN1_STRING
Module: U:\extras\lib\libcrypto.lib(bio_md.obj)
0001:008a804f  _BIO_f_md
Module: U:\extras\lib\libcrypto.lib(bio_enc.obj)
0001:008a84e7  _BIO_f_cipher
0001:008a8e2a* _BIO_set_cipher
Module: U:\extras\lib\libcrypto.lib(bss_null.obj)
0001:008a8f15  _BIO_s_null
Module: U:\extras\lib\libcrypto.lib(pk7_attr.obj)
0001:008a901b* _PKCS7_add_attrib_smimecap
0001:008a90a8* _PKCS7_get_smimecap
0001:008a9110* _PKCS7_simple_smimecap
0001:008a9287* _PKCS7_add_attrib_content_type
0001:008a92e4  _PKCS7_add0_attrib_signing_time
0001:008a9364  _PKCS7_add1_attrib_digest
Module: U:\extras\lib\libcrypto.lib(bn_gf2m.obj)
0001:008a96a1  _BN_GF2m_add
0001:008a97e6  _BN_GF2m_mod_arr
0001:008a9c50* _BN_GF2m_mod
0001:008ab0b4  _BN_GF2m_poly2arr
0001:008a9d27  _BN_GF2m_mod_mul_arr
0001:008aa093  _BN_GF2m_mod_sqr_arr
0001:008a9faa* _BN_GF2m_mod_mul
0001:008aa2d7* _BN_GF2m_mod_sqr
0001:008aa3b5* _BN_GF2m_mod_inv
0001:008aa606* _BN_GF2m_mod_inv_arr
0001:008ab170* _BN_GF2m_arr2poly
0001:008aa681  _BN_GF2m_mod_div
0001:008aa723* _BN_GF2m_mod_div_arr
0001:008aa7a5* _BN_GF2m_mod_exp_arr
0001:008aa910* _BN_GF2m_mod_exp
0001:008aa9f9  _BN_GF2m_mod_sqrt_arr
0001:008aaaa1* _BN_GF2m_mod_sqrt
0001:008aab7f  _BN_GF2m_mod_solve_quad_arr
0001:008aafd6* _BN_GF2m_mod_solve_quad
Module: U:\extras\lib\libcrypto.lib(ec2_mult.obj)
0001:008abe00  _ec_GF2m_simple_mul
0001:008ac0c5  _ec_GF2m_precompute_mult
0001:008ac0df  _ec_GF2m_have_precompute_mult
Module: U:\extras\lib\libcrypto.lib(p12_decr.obj)
0001:008ac10b* _PKCS12_pbe_crypt
0001:008ac2bd  _PKCS12_item_decrypt_d2i
0001:008ac3c5  _PKCS12_item_i2d_encrypt
Module: U:\extras\lib\libcrypto.lib(p12_p8e.obj)
0001:008ac52a  _PKCS8_encrypt
Module: U:\extras\lib\libcrypto.lib(ecp_smpl.obj)
0001:008ac6b0* _EC_GFp_simple_method
0001:008ac6ba  _ec_GFp_simple_group_init
0001:008ac700  _ec_GFp_simple_group_finish
0001:008ac734  _ec_GFp_simple_group_clear_finish
0001:008ac768  _ec_GFp_simple_group_copy
0001:008ac800  _ec_GFp_simple_group_set_curve
0001:008aca68  _ec_GFp_simple_group_get_curve
0001:008acbc5  _ec_GFp_simple_group_get_degree
0001:008acbdb  _ec_GFp_simple_group_check_discriminant
0001:008aceb6  _ec_GFp_simple_point_init
0001:008acef7  _ec_GFp_simple_point_finish
0001:008acf29  _ec_GFp_simple_point_clear_finish
0001:008acf65  _ec_GFp_simple_point_copy
0001:008acfe7  _ec_GFp_simple_point_set_to_infinity
0001:008ad014  _ec_GFp_simple_set_Jprojective_coordinates_GFp
0001:008ad267  _ec_GFp_simple_get_Jprojective_coordinates_GFp
0001:008ad3e8  _ec_GFp_simple_point_set_affine_coordinates
0001:008ad45f  _ec_GFp_simple_point_get_affine_coordinates
0001:008ad88d  _ec_GFp_simple_set_compressed_coordinates
0001:008adea4  _ec_GFp_simple_point2oct
0001:008ae2a6  _ec_GFp_simple_oct2point
0001:008ae6e4  _ec_GFp_simple_add
0001:008aeee5  _ec_GFp_simple_dbl
0001:008af58d  _ec_GFp_simple_invert
0001:008af5de  _ec_GFp_simple_is_at_infinity
0001:008af5f1  _ec_GFp_simple_is_on_curve
0001:008afa39  _ec_GFp_simple_cmp
0001:008afde3  _ec_GFp_simple_make_affine
0001:008aff35  _ec_GFp_simple_points_make_affine
0001:008b062e* _ec_GFp_simple_field_mul
0001:008b0660* _ec_GFp_simple_field_sqr
Module: U:\extras\lib\libcrypto.lib(bn_nist.obj)
0001:008b0bd4  _BN_get0_nist_prime_192
0001:008b0bde  _BN_get0_nist_prime_224
0001:008b0be8  _BN_get0_nist_prime_256
0001:008b0bf2  _BN_get0_nist_prime_384
0001:008b0bfc  _BN_get0_nist_prime_521
0001:008b0c9b  _BN_nist_mod_192
0001:008b0faa  _BN_nist_mod_224
0001:008b13d4  _BN_nist_mod_256
0001:008b196c  _BN_nist_mod_384
0001:008b200a  _BN_nist_mod_521
Module: U:\extras\lib\lzma.lib(liblzma_la-crc32_table.obj)
0001:008b2350  _lzma_crc32_table
Module: U:\extras\lib\lzma.lib(liblzma_la-crc64_table.obj)
0001:008b4350  _lzma_crc64_table
Module: U:\extras\lib\libcrypto.lib(cms_io.obj)
0001:008b6359  _CMS_stream
0001:008b6406* _d2i_CMS_bio
0001:008b6428* _i2d_CMS_bio
0001:008b644e* _PEM_read_bio_CMS
0001:008b6487* _PEM_read_CMS
0001:008b64c0* _PEM_write_bio_CMS
0001:008b6513* _PEM_write_CMS
0001:008b6566* _BIO_new_CMS
0001:008b6588* _i2d_CMS_bio_stream
0001:008b65b8* _PEM_write_bio_CMS_stream
0001:008b65f0* _SMIME_write_CMS
0001:008b6676* _SMIME_read_CMS
Module: U:\extras\lib\libcrypto.lib(cms_dd.obj)
0001:008b66a0* _cms_DigestedData_create
0001:008b673f  _cms_DigestedData_init_bio
0001:008b6767  _cms_DigestedData_do_final
Module: U:\extras\lib\libcrypto.lib(a_set.obj)
0001:008b692c  _i2d_ASN1_SET
0001:008b6c57  _d2i_ASN1_SET
Module: U:\extras\lib\libcrypto.lib(p12_asn.obj)
0001:008b70b0* _PKCS12_MAC_DATA_it
0001:008b6fb0  _PKCS12_it
0001:008b6fcc* _d2i_PKCS12
0001:008b6ff5* _i2d_PKCS12
0001:008b7017* _PKCS12_new
0001:008b702b* _PKCS12_free
0001:008b70cc* _d2i_PKCS12_MAC_DATA
0001:008b70f5* _i2d_PKCS12_MAC_DATA
0001:008b7117* _PKCS12_MAC_DATA_new
0001:008b712b* _PKCS12_MAC_DATA_free
0001:008b7250* _PKCS12_BAGS_it
0001:008b726c* _d2i_PKCS12_BAGS
0001:008b7295* _i2d_PKCS12_BAGS
0001:008b72b7  _PKCS12_BAGS_new
0001:008b72cb* _PKCS12_BAGS_free
0001:008b7450* _PKCS12_SAFEBAG_it
0001:008b746c* _d2i_PKCS12_SAFEBAG
0001:008b7495* _i2d_PKCS12_SAFEBAG
0001:008b74b7  _PKCS12_SAFEBAG_new
0001:008b74cb* _PKCS12_SAFEBAG_free
0001:008b7520  _PKCS12_SAFEBAGS_it
0001:008b7570  _PKCS12_AUTHSAFES_it
Module: U:\extras\lib\libcrypto.lib(p12_add.obj)
0001:008b759a  _PKCS12_item_pack_safebag
0001:008b76a6* _PKCS12_MAKE_KEYBAG
0001:008b770c* _PKCS12_MAKE_SHKEYBAG
0001:008b780e* _PKCS12_pack_p7data
0001:008b7912* _PKCS12_unpack_p7data
0001:008b7976* _PKCS12_pack_p7encdata
0001:008b7b64* _PKCS12_unpack_p7encdata
0001:008b7bc8* _PKCS12_decrypt_skey
0001:008b7bec* _PKCS12_pack_authsafes
0001:008b7c24* _PKCS12_unpack_authsafes
Module: U:\extras\lib\libcrypto.lib(dso_openssl.obj)
0001:008b7c90  _DSO_METHOD_openssl
Module: U:\extras\lib\libcrypto.lib(bn_sqrt.obj)
0001:008b7caa  _BN_mod_sqrt
Module: U:\extras\lib\libcrypto.lib(bn_kron.obj)
0001:008b8800  _BN_kronecker
Module: U:\extras\lib\libcrypto.lib(bio_ndef.obj)
0001:008b8b8b  _BIO_new_NDEF
Module: U:\extras\lib\libcrypto.lib(asn_mime.obj)
0001:008b9083  _i2d_ASN1_bio_stream
0001:008ba3e8* _SMIME_crlf_copy
0001:008b9268  _PEM_write_bio_ASN1_stream
0001:008b9841  _SMIME_write_ASN1
0001:008b9e68  _SMIME_read_ASN1
0001:008ba570* _SMIME_text
Module: U:\extras\lib\libcrypto.lib(dso_null.obj)
0001:008bb1cb  _DSO_METHOD_null
Module: U:\extras\lib\libcrypto.lib(bio_asn1.obj)
0001:008bb1e5  _BIO_f_asn1
0001:008bbb2b  _BIO_asn1_set_prefix
0001:008bbb54* _BIO_asn1_get_prefix
0001:008bbb7d  _BIO_asn1_set_suffix
0001:008bbba6* _BIO_asn1_get_suffix
Module: U:\extras\lib\libcrypto.lib(bio_b64.obj)
0001:008bbbe0  _BIO_f_base64


                        +----------------------+
                        |   Imported Symbols   |
                        +----------------------+

Symbol                              Module
======                              ======

___libc_ForkRegisterModule          libc065
___init_dll                         libc065
___libc_Back_termDll                libc065
___libc_ForkDeregisterModule        libc065
__atfork_callback                   libc065
___libc_GLocaleCtype                libc065
__assert                            libc065
_strlcat                            libc065
DosReleaseMutexSem                  doscalls
DosRequestMutexSem                  doscalls
DosCloseMutexSem                    doscalls
DosSleep                            doscalls
UniFreeUconvObject                  uconv
DosGetDateTime                      doscalls
DosQuerySysInfo                     doscalls
DosGetInfoBlocks                    doscalls
DosFreeModule                       doscalls
DosQueryProcAddr                    doscalls
DosSetFileLocks                     doscalls
DosFreeMem                          doscalls
DosClose                            doscalls
DosQueryFileInfo                    doscalls
DosResetBuffer                      doscalls
DosSetFileSize                      doscalls
DosSetFilePtr                       doscalls
DosWrite                            doscalls
DosRead                             doscalls
DosForceDelete                      doscalls
UniCreateUconvObject                uconv
DosCreateMutexSem                   doscalls
DosGetNamedSharedMem                doscalls
DosAllocSharedMem                   doscalls
DosDupHandle                        doscalls
UniStrToUcs                         uconv
UniStrFromUcs                       uconv
DosLoadModule                       doscalls
DosQueryPathInfo                    doscalls
DosDelete                           doscalls
DosOpen                             doscalls
DosScanEnv                          doscalls
DosQueryCurrentDisk                 doscalls
___stderrp                          libc065
__errno                             libc065
_strlcpy                            libc065
___isfinite                         libc065
_initgroups                         libc065
_getpwuid_r                         libc065
_getpwnam_r                         libc065
_getgrgid_r                         libc065
_getgrnam_r                         libc065
_hstrerror                          tcpip32
_inet_aton                          tcpip32
_gethostbyname                      tcpip32
_tcp_h_errno1                       tcpip32
_getprotobyname                     tcpip32
_inet_ntoa                          tcpip32
_getprotobynumber                   tcpip32
_getservbyport                      tcpip32
_getservbyname                      tcpip32
_inet_ntop                          tcpip32
_inet_pton                          tcpip32
_inet_addr                          tcpip32
_gethostbyaddr                      tcpip32
_gethostname                        tcpip32
DosQueryFSInfo                      doscalls
___stdinp                           libc065
___stdoutp                          libc065
__exit                              libc065
___threadid                         libc065
DosFreeThreadLocalMemory            doscalls
DosAllocThreadLocalMemory           doscalls
_isspace                            libc065
___flt_rounds                       libc065
__CRT_init                          libc065
__std_strnicmp                      libc065
__std_strdup                        libc065
__std_memcpy                        libc065
__std_floor                         libc065
__std_malloc                        libc065
__std_time                          libc065
__std_getenv                        libc065
__std_strftime                      libc065
__std_free                          libc065
__std_sin                           libc065
__std_cos                           libc065
__std_sqrt                          libc065
__std_atan2                         libc065
__std_acos                          libc065
__std_stricmp                       libc065
__std_strchr                        libc065
__std_calloc                        libc065
__std_strtoll                       libc065
__std_strtol                        libc065
__std_realloc                       libc065
__std_pow                           libc065
__std_strtod                        libc065
__std_memset                        libc065
__std_setlocale                     libc065
__std_printf                        libc065
__std_putchar                       libc065
__std_strcmp                        libc065
__std_strncat                       libc065
__std_strncpy                       libc065
__std_strncmp                       libc065
__std_strcpy                        libc065
__std_memmove                       libc065
__std_memcmp                        libc065
__std_localtime                     libc065
__std_sprintf                       libc065
__std_qsort                         libc065
__std_memchr                        libc065
__std_dup                           libc065
__std_fwrite                        libc065
__std_exit                          libc065
__std_fprintf                       libc065
__std_localtime_r                   libc065
__std_mktime                        libc065
___signbit                          libc065
__std_abort                         libc065
__std_fputc                         libc065
__std_strtoull                      libc065
__std_stat                          libc065
__std_strstr                        libc065
__std_puts                          libc065
__std_lseek                         libc065
__std_read                          libc065
__std_ctime                         libc065
__std_write                         libc065
__std_mkstemp                       libc065
__std_unlink                        libc065
__std_dup2                          libc065
__std_close                         libc065
__std_strerror                      libc065
__std_utimes                        libc065
__std_access                        libc065
__std_gmtime                        libc065
__std_asctime                       libc065
__std_strcspn                       libc065
__std_vasprintf                     libc065
__std_atoi                          libc065
__std_strpbrk                       libc065
___libc_FH                          libc065
__libsocket_set_errno               tcpip32
__libsocket_accept                  tcpip32
___libc_TcpipAllocFH44              libc065
__libsocket_soclose                 tcpip32
__libsocket_sock_errno              tcpip32
__libsocket_send                    tcpip32
__libsocket_recv                    tcpip32
__std_sscanf                        libc065
__std_gmtime_r                      libc065
__libsocket_socket                  tcpip32
__libsocket_bind                    tcpip32
__libsocket_getsockname             tcpip32
__libsocket_listen                  tcpip32
__std_strrchr                       libc065
__std_getuid                        libc065
__std_getgid                        libc065
__std_getgroups                     libc065
__std_setjmp                        libc065
__std_strtok_r                      libc065
__std_strtok                        libc065
__std_getrlimit                     libc065
__std_sysconf                       libc065
__std_mknod                         libc065
__std_mkfifo                        libc065
__std_isatty                        libc065
__std_ttyname                       libc065
__std_times                         libc065
__std_uname                         libc065
__std_getsid                        libc065
__std_getpgid                       libc065
__std_setpgid                       libc065
__std_setsid                        libc065
__std_getpgrp                       libc065
__std_getlogin                      libc065
__std_setegid                       libc065
__std_seteuid                       libc065
__std_setgid                        libc065
__std_setuid                        libc065
__std_getegid                       libc065
__std_geteuid                       libc065
__std_getppid                       libc065
__std_getpid                        libc065
__std_kill                          libc065
__std_gettimeofday                  libc065
__std_opendir                       libc065
__std_readdir_r                     libc065
__std_closedir                      libc065
__std_fstat                         libc065
__std_flock                         libc065
__std_fcntl                         libc065
__std_pwrite                        libc065
__std_ftruncate                     libc065
__std_pread                         libc065
__std_timezone                      libc065
__std_strcat                        libc065
__std_open                          libc065
__libsocket_shutdown                tcpip32
__libsocket_getsockopt              tcpip32
__libsocket_sendto                  tcpip32
__libsocket_connect                 tcpip32
__std_select                        libc065
__libsocket_socketpair              tcpip32
___libc_FHClose                     libc065
__libsocket_getpeername             tcpip32
__libsocket_recvfrom                tcpip32
__libsocket_setsockopt              tcpip32
__std_readlink                      libc065
__std_strtoul                       libc065
__std_getloadavg                    libc065
__std_umask                         libc065
__std_nanosleep                     libc065
__std_usleep                        libc065
__std_sleep                         libc065
__std_environ                       libc065
__std_putenv                        libc065
__std_tzset                         libc065
__std_unsetenv                      libc065
__std_strptime                      libc065
__std_glob                          libc065
__std_globfree                      libc065
__std_dlopen                        libc065
__std_dlsym                         libc065
__std_dlclose                       libc065
__std_dlerror                       libc065
__std_nice                          libc065
__std_mblen                         libc065
__std_fnmatch                       libc065
__std_fclose                        libc065
__std_localeconv                    libc065
__std_nl_langinfo                   libc065
__std_getc                          libc065
__std_fileno                        libc065
__std_link                          libc065
__std_symlink                       libc065
__std_popen                         libc065
__std_pclose                        libc065
__std_fmod                          libc065
__std_hypot                         libc065
__std_log10                         libc065
__std_log                           libc065
__std_log1p                         libc065
__std_expm1                         libc065
__std_exp                           libc065
__std_atanh                         libc065
__std_acosh                         libc065
__std_asinh                         libc065
__std_tanh                          libc065
__std_cosh                          libc065
__std_sinh                          libc065
__std_atan                          libc065
__std_asin                          libc065
__std_tan                           libc065
__std_ceil                          libc065
__std_rand_r                        libc065
__std_strcoll                       libc065
__std_ctime_r                       libc065
__getprogname                       libc065
__std_vsnprintf                     libc065
__std_writev                        libc065
__std_getdtablesize                 libc065
__std_strspn                        libc065
__std_ftok                          libc065
__std_waitpid                       libc065
__std_fork                          libc065
__std_chdir                         libc065
__std_execle                        libc065
__std_perror                        libc065
__std_execl                         libc065
__std_fseek                         libc065
__std_ftell                         libc065
__std_clearerr                      libc065
__std_fread                         libc065
__std_ferror                        libc065
__std_fopen                         libc065
__std_remove                        libc065
__std_fdopen                        libc065
__std_rename                        libc065
__std_chmod                         libc065
__std_putc                          libc065
__std_atol                          libc065
__std_atof                          libc065
__std_lstat                         libc065
__std_rmdir                         libc065
__std_mkdir                         libc065
__std_creat                         libc065
__std_chown                         libc065
__std_lchown                        libc065
__std_utime                         libc065
__std_getcwd                        libc065
__std_asctime_r                     libc065
__std_fputs                         libc065
___strnlen                          libc065
__std_vsprintf                      libc065
__std_setmode                       libc065
__std_fflush                        libc065
__std_rewind                        libc065
__std_rewinddir                     libc065
__std_setvbuf                       libc065
__std_feof                          libc065
__std_setitimer                     libc065
__std_signal                        libc065
__std_sigemptyset                   libc065
__std_sigaddset                     libc065
__std_sigprocmask                   libc065
__std_snprintf                      libc065
__std_longjmp                       libc065
DosTrueGetMessage                   msg
___ctordtorTerm1                    libc065
___ctordtorInit1                    libc065
__std_vfprintf                      libc065
__std_iconv                         libc065
__std_iconv_close                   libc065
__std_iconv_open                    libc065
__std_strlen                        libc065
__fmutex_create                     libc065
___libc_Back_threadSleep            libc065
___libc_GpFIBLIS                    libc065
___fmutex_request_internal          libc065
___fmutex_request_internal_must_complete libc065
___fmutex_release_internal_must_complete libc065
___fmutex_release_internal          libc065
DosEnterCritSec                     doscalls
DosExitCritSec                      doscalls
__beginthread                       libc065
__endthread                         libc065
DosSetPriority                      doscalls
__gettid                            libc065
DosWaitThread                       doscalls
DosCreateEventSem                   doscalls
DosCloseEventSem                    doscalls
DosPostEventSem                     doscalls
DosWaitEventSem                     doscalls
__std_ftime                         libc065
__std_fgets                         libc065
DosTmrQueryTime                     doscalls
DosPerfSysCall                      doscalls
DosAllocMem                         doscalls
DosQuerySysState                    doscalls
__std_srand                         libc065
__std_rand                          libc065
__std_random                        libc065
__std_tcgetattr                     libc065
__std_tcsetattr                     libc065
__std_sigaction                     libc065


                        +--------------------+
                        |   Libraries Used   |
                        +--------------------+

U:\extras\lib\libz.lib
U:\extras\lib\xmlrpc.lib
U:\extras\lib\libcrypto.lib
U:\extras\lib\libssl.lib
U:\extras\lib\pthread.lib
U:\extras\lib\expat.lib
U:\extras\lib\poll.lib
U:\extras\lib\lzma.lib
U:\extras\lib\xml2.lib
U:\usr\local446\lib\gcc\i386-pc-os2-emx\4.4.6\libgcc_eh.lib
U:\usr\local446\lib\gcc\i386-pc-os2-emx\4.4.6\libgcc.lib
U:\usr\lib\libc_alias.lib
U:\usr\lib\libc_dll.lib
U:\usr\lib\libos2.lib
U:\usr\lib\libend.lib


                        +-----------------------+
                        |   Linker Statistics   |
                        +-----------------------+

Stack size:  0000 (0.)
Memory size:  008df180 (9302400.)
Link time: 00:00.10
